 jli

 Timestamp is 6710e04f (Thu Oct 17 10:00:47 2024)

 Preferred load address is 10000000

 Start         Length     Name                   Class
 0001:00000000 00027455H .text$mn                CODE
 0001:00027455 000000bbH .text$x                 CODE
 0002:00000000 000001a8H .idata$5                DATA
 0002:000001a8 00000008H .00cfg                  DATA
 0002:000001b0 00000004H .CRT$XCA                DATA
 0002:000001b4 00000004H .CRT$XCZ                DATA
 0002:000001b8 00000004H .CRT$XIA                DATA
 0002:000001bc 00000014H .CRT$XIC                DATA
 0002:000001d0 00000004H .CRT$XIZ                DATA
 0002:000001d4 00000004H .CRT$XPA                DATA
 0002:000001d8 00000008H .CRT$XPX                DATA
 0002:000001e0 00000004H .CRT$XPXA               DATA
 0002:000001e4 00000004H .CRT$XPZ                DATA
 0002:000001e8 00000004H .CRT$XTA                DATA
 0002:000001ec 00000004H .CRT$XTZ                DATA
 0002:000001f0 00000000H .gfids$y                DATA
 0002:000001f0 0000b350H .rdata                  DATA
 0002:0000b540 00000000H .rdata$CastGuardVftablesA DATA
 0002:0000b540 00000000H .rdata$CastGuardVftablesC DATA
 0002:0000b540 000000dcH .rdata$r                DATA
 0002:0000b61c 00000028H .rdata$sxdata           DATA
 0002:0000b644 00000228H .rdata$voltmd           DATA
 0002:0000b86c 00000368H .rdata$zzzdbg           DATA
 0002:0000bbd4 00000004H .rtc$IAA                DATA
 0002:0000bbd8 00000004H .rtc$IZZ                DATA
 0002:0000bbdc 00000004H .rtc$TAA                DATA
 0002:0000bbe0 00000008H .rtc$TZZ                DATA
 0002:0000bbe8 000007f8H .xdata$x                DATA
 0002:0000c3e0 00000170H .edata                  DATA
 0002:0000c550 00000050H .idata$2                DATA
 0002:0000c5a0 00000014H .idata$3                DATA
 0002:0000c5b4 000001a8H .idata$4                DATA
 0002:0000c75c 000007c0H .idata$6                DATA
 0003:00000000 00000aa0H .data                   DATA
 0003:00000aa0 0000003cH .data$r                 DATA
 0003:00000adc 0000001cH .data$rs                DATA
 0003:00000af8 00000d08H .bss                    DATA
 0004:00000000 00000060H .rsrc$01                DATA
 0004:00000060 00000308H .rsrc$02                DATA

  Address         Publics by Value              Rva+Base       Lib:Object

 0000:00000000       ___AbsoluteZero            00000000     <absolute>
 0000:00000000       ___arm64x_extra_rfe_table  00000000     <absolute>
 0000:00000000       ___arm64x_extra_rfe_table_size 00000000     <absolute>
 0000:00000000       ___arm64x_native_entrypoint 00000000     <absolute>
 0000:00000000       ___arm64x_redirection_metadata 00000000     <absolute>
 0000:00000000       ___arm64x_redirection_metadata_count 00000000     <absolute>
 0000:00000000       ___dynamic_value_reloc_table 00000000     <absolute>
 0000:00000000       ___enclave_config          00000000     <absolute>
 0000:00000000       ___guard_check_icall_a64n_fptr 00000000     <absolute>
 0000:00000000       ___guard_eh_cont_count     00000000     <absolute>
 0000:00000000       ___guard_eh_cont_table     00000000     <absolute>
 0000:00000000       ___guard_fids_count        00000000     <absolute>
 0000:00000000       ___guard_fids_table        00000000     <absolute>
 0000:00000000       ___guard_iat_count         00000000     <absolute>
 0000:00000000       ___guard_iat_table         00000000     <absolute>
 0000:00000000       ___guard_longjmp_count     00000000     <absolute>
 0000:00000000       ___guard_longjmp_table     00000000     <absolute>
 0000:00000000       ___hybrid_auxiliary_delayload_iat 00000000     <absolute>
 0000:00000000       ___hybrid_auxiliary_delayload_iat_copy 00000000     <absolute>
 0000:00000000       ___hybrid_auxiliary_iat    00000000     <absolute>
 0000:00000000       ___hybrid_auxiliary_iat_copy 00000000     <absolute>
 0000:00000000       ___hybrid_code_map         00000000     <absolute>
 0000:00000000       ___hybrid_code_map_count   00000000     <absolute>
 0000:00000000       ___hybrid_image_info_bitfield 00000000     <absolute>
 0000:00000000       ___x64_code_ranges_to_entry_points 00000000     <absolute>
 0000:00000000       ___x64_code_ranges_to_entry_points_count 00000000     <absolute>
 0000:00000000       __except_list              00000000     <absolute>
 0000:0000000a       ___safe_se_handler_count   0000000a     <absolute>
 0000:00000100       ___guard_flags             00000100     <absolute>
 0000:00000000       ___ImageBase               10000000     <linker-defined>
 0001:00000000       _JLI_CmdToArgs             10001000 f   cmdtoargs.obj
 0001:00000068       _JLI_GetStdArgc            10001068 f   cmdtoargs.obj
 0001:0000006e       _JLI_GetStdArgs            1000106e f   cmdtoargs.obj
 0001:000002ec       _inflate_fast              100012ec f   inffast.obj
 0001:000006f4       _inflate                   100016f4 f   inflate.obj
 0001:00001c20       _inflateEnd                10002c20 f   inflate.obj
 0001:00001c60       _inflateInit2_             10002c60 f   inflate.obj
 0001:00001d06       _inflateReset              10002d06 f   inflate.obj
 0001:00001d2f       _inflateReset2             10002d2f f   inflate.obj
 0001:00001da7       _inflateResetKeep          10002da7 f   inflate.obj
 0001:00001f20       _inflate_table             10002f20 f   inftrees.obj
 0001:000024dd       _AddOption                 100034dd f   java.obj
 0001:00002612       _CheckJvmType              10003612 f   java.obj
 0001:000028d6       _ContinueInNewThread       100038d6 f   java.obj
 0001:00002aa5       _GetDotVersion             10003aa5 f   java.obj
 0001:00002aab       _GetErgoPolicy             10003aab f   java.obj
 0001:00002ab1       _GetLauncherHelperClass    10003ab1 f   java.obj
 0001:00002ae1       _GetProgramName            10003ae1 f   java.obj
 0001:00002bb0       _IsJavaArgs                10003bb0 f   java.obj
 0001:00002bb6       _JLI_Launch                10003bb6 f   java.obj
 0001:00002f82       _JLI_ReportMessage         10003f82 f   java.obj
 0001:00002fb6       _JavaMain@4                10003fb6 f   java.obj
 0001:0000351b       _NewPlatformStringArray    1000451b f   java.obj
 0001:00003d7a       _ReadKnownVMs              10004d7a f   java.obj
 0001:0000484a       _ShowSplashScreen          1000584a f   java.obj
 0001:00004ac3       ___local_stdio_printf_options 10005ac3 f i java.obj
 0001:00004ac9       ___local_stdio_scanf_options 10005ac9 f i java.obj
 0001:00004acf       __vfprintf_l               10005acf f i java.obj
 0001:00004af2       __vsnprintf_l              10005af2 f i java.obj
 0001:00004b24       __vsscanf_l                10005b24 f i java.obj
 0001:00004b49       _fprintf                   10005b49 f i java.obj
 0001:00004c3a       _printf                    10005c3a f i java.obj
 0001:00004c57       _sprintf                   10005c57 f i java.obj
 0001:00004c71       _sscanf                    10005c71 f i java.obj
 0001:00004c89       _AWTPreload                10005c89 f   java_md.obj
 0001:00004dd1       _ContinueInNewThread0      10005dd1 f   java_md.obj
 0001:00004f05       _Counter2Micros            10005f05 f   java_md.obj
 0001:00004f44       _CounterGet                10005f44 f   java_md.obj
 0001:00004f8c       _CreateApplicationArgs     10005f8c f   java_md.obj
 0001:000051f3       _CreateExecutionEnvironment 100061f3 f   java_md.obj
 0001:000053ec       _ExecJRE                   100063ec f   java_md.obj
 0001:0000577a       _FindBootStrapClass        1000677a f   java_md.obj
 0001:000057c8       _GetApplicationHome        100067c8 f   java_md.obj
 0001:00005802       _GetBoolParamValue         10006802 f   java_md.obj
 0001:000059c0       _GetParamValue             100069c0 f   java_md.obj
 0001:00005bef       _InitLauncher              10006bef f   java_md.obj
 0001:00005c24       _IsJavaw                   10006c24 f   java_md.obj
 0001:00005c2a       _JLI_ReportErrorMessage    10006c2a f   java_md.obj
 0001:00005cb4       _JLI_ReportErrorMessageSys 10006cb4 f   java_md.obj
 0001:00005de4       _JLI_ReportExceptionDescription 10006de4 f   java_md.obj
 0001:00005e0d       _JLI_Snprintf              10006e0d f   java_md.obj
 0001:00005e53       _JVMInit                   10006e53 f   java_md.obj
 0001:00005e7d       _LoadJavaVM                10006e7d f   java_md.obj
 0001:00006061       _LocateJRE                 10007061 f   java_md.obj
 0001:000060dc       @_guard_check_icall_nop@4  100070dc f   LIBCMT:guard_support.obj
 0001:000060dc       _PostJVMInit               100070dc f   java_md.obj
 0001:000060dc       _RegisterThread            100070dc f   java_md.obj
 0001:000060dc       _SetJavaLauncherPlatformProps 100070dc f   java_md.obj
 0001:00006209       _ProcessPlatformOption     10007209 f   java_md.obj
 0001:0000620c       _ServerClassMachine        1000720c f   java_md.obj
 0001:00006218       _SplashProcAddress         10007218 f   java_md.obj
 0001:000062b8       _UnsetEnv                  100072b8 f   java_md.obj
 0001:000062fd       __vscprintf_l              100072fd f i java_md.obj
 0001:0000632c       __vsnprintf                1000732c f i java_md.obj
 0001:00006347       _filterArgs                10007347 f   java_md.obj
 0001:000063a7       _jlong_format_specifier    100073a7 f   java_md.obj
 0001:000064a4       _vsnprintf                 100074a4 f i java_md.obj
 0001:000064d5       _JLI_IsTraceLauncher       100074d5 f   jli_util.obj
 0001:000064db       _JLI_MemAlloc              100074db f   jli_util.obj
 0001:000064fd       ??3@YAXPAX@Z               100074fd f   LIBCMT:delete_scalar.obj
 0001:000064fd       _JLI_MemFree               100074fd f   jli_util.obj
 0001:00006502       _JLI_MemRealloc            10007502 f   jli_util.obj
 0001:00006529       _JLI_SetTraceLauncher      10007529 f   jli_util.obj
 0001:00006550       _JLI_StrCCmp               10007550 f   jli_util.obj
 0001:0000656b       _JLI_StringDup             1000756b f   jli_util.obj
 0001:0000658d       _JLI_TraceLauncher         1000758d f   jli_util.obj
 0001:000065a7       _vprintf                   100075a7 f i jli_util.obj
 0001:000065c3       _JLI_FreeManifest          100075c3 f   parse_manifest.obj
 0001:000065d4       _JLI_JarUnpackFile         100075d4 f   parse_manifest.obj
 0001:0000662b       _JLI_ManifestIterate       1000762b f   parse_manifest.obj
 0001:000066e2       _JLI_ParseManifest         100076e2 f   parse_manifest.obj
 0001:000073c7       _DoSplashGetScaledImageName 100083c7 f   splashscreen_stubs.obj
 0001:000073e7       _DoSplashInit              100083e7 f   splashscreen_stubs.obj
 0001:00007407       _DoSplashLoadFile          10008407 f   splashscreen_stubs.obj
 0001:00007427       _DoSplashLoadMemory        10008427 f   splashscreen_stubs.obj
 0001:00007447       _DoSplashSetFileJarName    10008447 f   splashscreen_stubs.obj
 0001:00007467       _DoSplashSetScaleFactor    10008467 f   splashscreen_stubs.obj
 0001:00007494       _JLI_AcceptableRelease     10008494 f   version_comp.obj
 0001:00007507       _JLI_ExactVersionId        10008507 f   version_comp.obj
 0001:000075e5       _JLI_PrefixVersionId       100085e5 f   version_comp.obj
 0001:00007694       _JLI_ValidVersionString    10008694 f   version_comp.obj
 0001:00007b95       _JLI_WildcardExpandClasspath 10008b95 f   wildcard.obj
 0001:00007d41       _adler32                   10008d41 f   zadler32.obj
 0001:00007d46       _adler32_z                 10008d46 f   zadler32.obj
 0001:00007f83       _crc32                     10008f83 f   zcrc32.obj
 0001:00007f88       _crc32_z                   10008f88 f   zcrc32.obj
 0001:00008271       _zcalloc                   10009271 f   zutil.obj
 0001:00008282       _zcfree                    10009282 f   zutil.obj
 0001:0000828d       @__security_check_cookie@4 1000928d f   LIBCMT:secchk.obj
 0001:0000829b       ___raise_securityfailure   1000929b f   LIBCMT:gs_report.obj
 0001:000082c3       ___report_gsfailure        100092c3 f   LIBCMT:gs_report.obj
 0001:000083bd       ___report_rangecheckfailure 100093bd f   LIBCMT:gs_report.obj
 0001:000083c9       ___report_securityfailure  100093c9 f   LIBCMT:gs_report.obj
 0001:000084a0       __alldiv                   100094a0 f   LIBCMT:lldiv.obj
 0001:00008550       __allmul                   10009550 f   LIBCMT:llmul.obj
 0001:00008590       __allrem                   10009590 f   LIBCMT:llrem.obj
 0001:00008982       __DllMainCRTStartup@12     10009982 f   LIBCMT:dll_dllmain.obj
 0001:000089f2       ___security_init_cookie    100099f2 f   LIBCMT:gs_support.obj
 0001:00008a3d       _DllMain@12                10009a3d f   LIBCMT:dll_dllmain_stub.obj
 0001:00008a43       ?__scrt_initialize_type_info@@YAXXZ 10009a43 f   LIBCMT:tncleanup.obj
 0001:00008a4f       ?__scrt_uninitialize_type_info@@YAXXZ 10009a4f f   LIBCMT:tncleanup.obj
 0001:00008a5b       ___scrt_initialize_default_local_stdio_options 10009a5b f   LIBCMT:default_local_stdio_options.obj
 0001:00008abc       ___scrt_acquire_startup_lock 10009abc f   LIBCMT:utility.obj
 0001:00008aee       ___scrt_dllmain_after_initialize_c 10009aee f   LIBCMT:utility.obj
 0001:00008b19       ___scrt_dllmain_before_initialize_c 10009b19 f   LIBCMT:utility.obj
 0001:00008b27       ___scrt_dllmain_crt_thread_attach 10009b27 f   LIBCMT:utility.obj
 0001:00008b46       ___scrt_dllmain_crt_thread_detach 10009b46 f   LIBCMT:utility.obj
 0001:00008b53       ___scrt_dllmain_exception_filter 10009b53 f   LIBCMT:utility.obj
 0001:00008b87       ___scrt_dllmain_uninitialize_c 10009b87 f   LIBCMT:utility.obj
 0001:00008baa       ___scrt_dllmain_uninitialize_critical 10009baa f   LIBCMT:utility.obj
 0001:00008bb7       ___scrt_initialize_crt     10009bb7 f   LIBCMT:utility.obj
 0001:00008bf0       ___scrt_initialize_onexit_tables 10009bf0 f   LIBCMT:utility.obj
 0001:00008c77       ___scrt_is_nonwritable_in_current_image 10009c77 f   LIBCMT:utility.obj
 0001:00008d0b       ___scrt_release_startup_lock 10009d0b f   LIBCMT:utility.obj
 0001:00008d28       ___scrt_uninitialize_crt   10009d28 f   LIBCMT:utility.obj
 0001:00008d50       ___scrt_get_dyn_tls_init_callback 10009d50 f   LIBCMT:dyn_tls_init.obj
 0001:00008d56       ___scrt_fastfail           10009d56 f   LIBCMT:utility_desktop.obj
 0001:00008e71       __crt_debugger_hook        10009e71 f   LIBCMT:utility_desktop.obj
 0001:00008e79       __RTC_Initialize           10009e79 f   LIBCMT:initsect.obj
 0001:00008ea5       __RTC_Terminate            10009ea5 f   LIBCMT:initsect.obj
 0001:00008ee0       __SEH_prolog4              10009ee0 f   LIBCMT:sehprolg4.obj
 0001:00008f25       ___isa_available_init      10009f25 f   LIBCMT:cpu_disp.obj
 0001:000090f9       __get_startup_argv_mode    1000a0f9 f   LIBCMT:argv_mode.obj
 0001:000090fd       ___scrt_is_ucrt_dll_in_use 1000a0fd f   LIBCMT:ucrt_detection.obj
 0001:00009110       _memcpy                    1000a110 f   libvcruntime:memcpy.obj
 0001:00009110       _memmove                   1000a110 f   libvcruntime:memmove.obj
 0001:00009690       _memset                    1000a690 f   libvcruntime:memset.obj
 0001:000097f0       _strchr                    1000a7f0 f   libvcruntime:strchr.obj
 0001:0000985e       ___from_strstr_to_strchr   1000a85e     libvcruntime:strchr.obj
 0001:00009920       _strrchr                   1000a920 f   libvcruntime:strrchr.obj
 0001:00009a57       _memcmp                    1000aa57 f   libvcruntime:memcmp.obj
 0001:0000b120       __except_handler4          1000c120 f   libvcruntime:chandler4.obj
 0001:0000b27e       ___std_type_info_compare   1000c27e f   libvcruntime:std_type_info.obj
 0001:0000b2ba       ___std_type_info_destroy_list 1000c2ba f   libvcruntime:std_type_info.obj
 0001:0000b2dd       ___vcrt_initialize         1000c2dd f   libvcruntime:initialization.obj
 0001:0000b2fc       ___vcrt_thread_attach      1000c2fc f   libvcruntime:initialization.obj
 0001:0000b307       ___vcrt_thread_detach      1000c307 f   libvcruntime:initialization.obj
 0001:0000b30f       ___vcrt_uninitialize       1000c30f f   libvcruntime:initialization.obj
 0001:0000b326       ___vcrt_uninitialize_critical 1000c326 f   libvcruntime:initialization.obj
 0001:0000b32e       ___DestructExceptionObject 1000c32e f   libvcruntime:ehhelpers.obj
 0001:0000b3cf       ?_CallMemberFunction0@@YGXQAX0@Z 1000c3cf f i libvcruntime:ehhelpers.obj
 0001:0000b434       __IsExceptionObjectToBeDestroyed 1000c434 f   libvcruntime:ehhelpers.obj
 0001:0000b45a       ___AdjustPointer           1000c45a f   libvcruntime:ehhelpers.obj
 0001:0000b47f       ___FrameUnwindFilter       1000c47f f   libvcruntime:ehhelpers.obj
 0001:0000b4d5       ___std_terminate           1000c4d5 f   libvcruntime:ehhelpers.obj
 0001:0000b4e0       __local_unwind4            1000c4e0 f   libvcruntime:exsup4.obj
 0001:0000b5d0       @_EH4_CallFilterFunc@8     1000c5d0 f   libvcruntime:exsup4.obj
 0001:0000b5f0       @_EH4_TransferToHandler@8  1000c5f0 f   libvcruntime:exsup4.obj
 0001:0000b610       @_EH4_GlobalUnwind2@8      1000c610 f   libvcruntime:exsup4.obj
 0001:0000b630       @_EH4_LocalUnwind@16       1000c630 f   libvcruntime:exsup4.obj
 0001:0000b647       ___except_validate_context_record 1000c647 f   libvcruntime:jbcxrval.obj
 0001:0000b677       ___vcrt_freefls@4          1000c677 f   libvcruntime:per_thread_data.obj
 0001:0000b693       ___vcrt_freeptd_for_this_thread 1000c693 f   libvcruntime:per_thread_data.obj
 0001:0000b6be       ___vcrt_getptd             1000c6be f   libvcruntime:per_thread_data.obj
 0001:0000b6cc       ___vcrt_getptd_noexit      1000c6cc f   libvcruntime:per_thread_data.obj
 0001:0000b75e       ___vcrt_initialize_ptd     1000c75e f   libvcruntime:per_thread_data.obj
 0001:0000b791       ___vcrt_uninitialize_ptd   1000c791 f   libvcruntime:per_thread_data.obj
 0001:0000b7ac       ___vcrt_initialize_locks   1000c7ac f   libvcruntime:locks.obj
 0001:0000b7e8       ___vcrt_uninitialize_locks 1000c7e8 f   libvcruntime:locks.obj
 0001:0000b820       __NLG_Notify1              1000c820 f   libvcruntime:exsup.obj
 0001:0000b830       __NLG_Notify               1000c830 f   libvcruntime:exsup.obj
 0001:0000b847       __NLG_Dispatch             1000c847     libvcruntime:exsup.obj
 0001:0000b847       __NLG_Dispatch2            1000c847     libvcruntime:exsup.obj
 0001:0000b850       __NLG_Call                 1000c850 f   libvcruntime:exsup.obj
 0001:0000b852       __NLG_Return2              1000c852     libvcruntime:exsup.obj
 0001:0000b853       ?GetRangeOfTrysToCheck@__FrameHandler3@@SA?AU?$pair@Viterator@TryBlockMap@__FrameHandler3@@V123@@std@@AAVTryBlockMap@1@HPAXPBU_s_FuncInfo@@H@Z 1000c853 f   libvcruntime:trnsctrl.obj
 0001:0000b8c3       ?_CallCatchBlock2@@YAPAXPAUEHRegistrationNode@@PBU_s_FuncInfo@@PAXHK@Z 1000c8c3 f   libvcruntime:trnsctrl.obj
 0001:0000b920       ?_CallSETranslator@@YAHPAUEHExceptionRecord@@PAUEHRegistrationNode@@PAX2PBU_s_FuncInfo@@H1@Z 1000c920 f   libvcruntime:trnsctrl.obj
 0001:0000ba16       ?_JumpToContinuation@@YGXPAXPAUEHRegistrationNode@@@Z 1000ca16 f   libvcruntime:trnsctrl.obj
 0001:0000ba46       ?_UnwindNestedFrames@@YGXPAUEHRegistrationNode@@PAUEHExceptionRecord@@@Z 1000ca46 f   libvcruntime:trnsctrl.obj
 0001:0000ba99       __CatchGuardHandler        1000ca99 f   libvcruntime:trnsctrl.obj
 0001:0000baca       __CreateFrameInfo          1000caca f   libvcruntime:trnsctrl.obj
 0001:0000baee       __FindAndUnlinkFrame       1000caee f   libvcruntime:trnsctrl.obj
 0001:0000bb36       __TranslatorGuardHandler   1000cb36 f   libvcruntime:trnsctrl.obj
 0001:0000bbd3       ___CxxFrameHandler3        1000cbd3 f   libvcruntime:trnsctrl.obj
 0001:0000bcf4       ___vcrt_FlsAlloc           1000ccf4 f   libvcruntime:winapi_downlevel.obj
 0001:0000bd2f       ___vcrt_FlsFree            1000cd2f f   libvcruntime:winapi_downlevel.obj
 0001:0000bd6a       ___vcrt_FlsGetValue        1000cd6a f   libvcruntime:winapi_downlevel.obj
 0001:0000bda5       ___vcrt_FlsSetValue        1000cda5 f   libvcruntime:winapi_downlevel.obj
 0001:0000bde3       ___vcrt_InitializeCriticalSectionEx 1000cde3 f   libvcruntime:winapi_downlevel.obj
 0001:0000c55c       ??$TypeMatchHelper@V__FrameHandler3@@@@YAHPBU_s_HandlerType@@PBU_s_CatchableType@@PBU_s_ThrowInfo@@@Z 1000d55c f i libvcruntime:frame.obj
 0001:0000c5ea       ??$__InternalCxxFrameHandler@V__FrameHandler3@@@@YA?AW4_EXCEPTION_DISPOSITION@@PAUEHExceptionRecord@@PAUEHRegistrationNode@@PAU_CONTEXT@@PAXPBU_s_FuncInfo@@H1E@Z 1000d5ea f i libvcruntime:frame.obj
 0001:0000c6ec       ??$__InternalCxxFrameHandlerWrapper@V__FrameHandler3@@@@YA?AW4_EXCEPTION_DISPOSITION@@PAUEHExceptionRecord@@PAUEHRegistrationNode@@PAU_CONTEXT@@PAXPBU_s_FuncInfo@@H1E@Z 1000d6ec f i libvcruntime:frame.obj
 0001:0000c6f5       ??0bad_exception@std@@QAE@ABV01@@Z 1000d6f5 f i libvcruntime:frame.obj
 0001:0000c710       ??0bad_exception@std@@QAE@XZ 1000d710 f i libvcruntime:frame.obj
 0001:0000c728       ??0exception@std@@QAE@ABV01@@Z 1000d728 f i libvcruntime:frame.obj
 0001:0000c754       ??1bad_exception@std@@UAE@XZ 1000d754 f i libvcruntime:frame.obj
 0001:0000c765       ??8type_info@@QBE_NABV0@@Z 1000d765 f i libvcruntime:frame.obj
 0001:0000c784       ??_Ebad_exception@std@@UAEPAXI@Z 1000d784 f i libvcruntime:frame.obj
 0001:0000c784       ??_Eexception@std@@UAEPAXI@Z 1000d784 f i libvcruntime:frame.obj
 0001:0000c784       ??_Gbad_exception@std@@UAEPAXI@Z 1000d784 f i libvcruntime:frame.obj
 0001:0000c784       ??_Gexception@std@@UAEPAXI@Z 1000d784 f i libvcruntime:frame.obj
 0001:0000ca09       ?FrameUnwindToEmptyState@__FrameHandler3@@SAXPAUEHRegistrationNode@@PAXPBU_s_FuncInfo@@@Z 1000da09 f   libvcruntime:frame.obj
 0001:0000ca21       ?FrameUnwindToState@__FrameHandler3@@SAXPAUEHRegistrationNode@@PAXPBU_s_FuncInfo@@H@Z 1000da21 f   libvcruntime:frame.obj
 0001:0000cba3       ?_CallMemberFunction1@@YGXQAX00@Z 1000dba3 f i libvcruntime:frame.obj
 0001:0000cbb3       ?_CallMemberFunction2@@YGXQAX00H@Z 1000dbb3 f i libvcruntime:frame.obj
 0001:0000cbc6       ?getESTypes@__FrameHandler3@@SAPBU_s_ESTypeList@@PBU_s_FuncInfo@@@Z 1000dbc6 f i libvcruntime:frame.obj
 0001:0000cbd1       ?what@exception@std@@UBEPBDXZ 1000dbd1 f i libvcruntime:frame.obj
 0001:0000cbe0       __CallSettingFrame@12      1000dbe0 f   libvcruntime:lowhelpr.obj
 0001:0000cc07       __NLG_Return               1000dc07     libvcruntime:lowhelpr.obj
 0001:0000cc2c       _unexpected                1000dc2c f   libvcruntime:unexpected.obj
 0001:0000cc49       ?GetCurrentState@__FrameHandler3@@SAHPAUEHRegistrationNode@@PAXPBU_s_FuncInfo@@@Z 1000dc49 f   libvcruntime:ehstate.obj
 0001:0000cc66       ?SetState@__FrameHandler3@@SAXPAUEHRegistrationNode@@PBU_s_FuncInfo@@H@Z 1000dc66 f   libvcruntime:ehstate.obj
 0001:0000cc74       ___std_exception_copy      1000dc74 f   libvcruntime:std_exception.obj
 0001:0000ccd7       ___std_exception_destroy   1000dcd7 f   libvcruntime:std_exception.obj
 0001:0000ccf6       __CxxThrowException@8      1000dcf6 f   libvcruntime:throw.obj
 0001:0000cd62       ___acrt_initialize_stdio   1000dd62 f   libucrt:_file.obj
 0001:0000ce2a       ___acrt_iob_func           1000de2a f   libucrt:_file.obj
 0001:0000ce3a       ___acrt_uninitialize_stdio 1000de3a f   libucrt:_file.obj
 0001:0000ce86       __lock_file                1000de86 f   libucrt:_file.obj
 0001:0000ce9a       __unlock_file              1000de9a f   libucrt:_file.obj
 0001:0000ceae       ??0__crt_cached_ptd_host@@QAE@QAU__crt_locale_pointers@@@Z 1000deae f i libucrt:fclose.obj
 0001:0000cef6       ??1__crt_cached_ptd_host@@QAE@XZ 1000def6 f i libucrt:fclose.obj
 0001:0000d057       ?force_synchronize_per_thread_data@__crt_cached_ptd_host@@AAEPAU__acrt_ptd@@XZ 1000e057 f i libucrt:fclose.obj
 0001:0000d09d       ?get_raw_ptd@__crt_cached_ptd_host@@QAEPAU__acrt_ptd@@XZ 1000e09d f i libucrt:fclose.obj
 0001:0000d0ba       _fclose                    1000e0ba f   libucrt:fclose.obj
 0001:0000d1bc       ?validate_stream_is_ansi_if_required@?$__acrt_stdio_char_traits@D@@SA_NQAU_iobuf@@@Z 1000e1bc f i libucrt:fgets.obj
 0001:0000d243       _fgets                     1000e243 f   libucrt:fgets.obj
 0001:0000d305       _fopen                     1000e305 f   libucrt:fopen.obj
 0001:0000d4eb       ??$count@D@formatting_buffer@__crt_stdio_output@@QBEIXZ 1000e4eb f i libucrt:output.obj
 0001:0000d503       ??$ensure_buffer_is_big_enough@D@formatting_buffer@__crt_stdio_output@@QAE_NIAAV__crt_cached_ptd_host@@@Z 1000e503 f i libucrt:output.obj
 0001:0000d584       ??$is_overflow_condition@K@__crt_strtox@@YA_NIK@Z 1000e584 f i libucrt:output.obj
 0001:0000d5b8       ??$is_wide_character_specifier@D@__crt_stdio_output@@YA_N_KDW4length_modifier@0@@Z 1000e5b8 f i libucrt:output.obj
 0001:0000d5e9       ??$make_c_string_character_source@DPAPAD@__crt_strtox@@YA?AV?$c_string_character_source@D@0@QBDQAPAD@Z 1000e5e9 f i libucrt:output.obj
 0001:0000d5e9       ??$make_c_string_character_source@_WPAPA_W@__crt_strtox@@YA?AV?$c_string_character_source@_W@0@QB_WQAPA_W@Z 1000e5e9 f i libucrt:output.obj
 0001:0000d604       ??$parse_integer@KV?$c_string_character_source@D@__crt_strtox@@$0A@@__crt_strtox@@YAKAAV__crt_cached_ptd_host@@V?$c_string_character_source@D@0@H_N@Z 1000e604 f i libucrt:output.obj
 0001:0000d813       ??$scratch_data@D@formatting_buffer@__crt_stdio_output@@QAEPADXZ 1000e813 f i libucrt:output.obj
 0001:0000d831       ??$type_case_integer@$07@?$output_processor@DV?$stream_output_adapter@D@__crt_stdio_output@@V?$standard_base@DV?$stream_output_adapter@D@__crt_stdio_output@@@2@@__crt_stdio_output@@AAE_N_N@Z 1000e831 f i libucrt:output.obj
 0001:0000d831       ??$type_case_integer@$07@?$output_processor@DV?$string_output_adapter@D@__crt_stdio_output@@V?$standard_base@DV?$string_output_adapter@D@__crt_stdio_output@@@2@@__crt_stdio_output@@AAE_N_N@Z 1000e831 f i libucrt:output.obj
 0001:0000d9be       ??$type_case_integer@$09@?$output_processor@DV?$stream_output_adapter@D@__crt_stdio_output@@V?$standard_base@DV?$stream_output_adapter@D@__crt_stdio_output@@@2@@__crt_stdio_output@@AAE_N_N@Z 1000e9be f i libucrt:output.obj
 0001:0000d9be       ??$type_case_integer@$09@?$output_processor@DV?$string_output_adapter@D@__crt_stdio_output@@V?$standard_base@DV?$string_output_adapter@D@__crt_stdio_output@@@2@@__crt_stdio_output@@AAE_N_N@Z 1000e9be f i libucrt:output.obj
 0001:0000db4b       ??$type_case_integer@$0BA@@?$output_processor@DV?$stream_output_adapter@D@__crt_stdio_output@@V?$standard_base@DV?$stream_output_adapter@D@__crt_stdio_output@@@2@@__crt_stdio_output@@AAE_N_N@Z 1000eb4b f i libucrt:output.obj
 0001:0000db4b       ??$type_case_integer@$0BA@@?$output_processor@DV?$string_output_adapter@D@__crt_stdio_output@@V?$standard_base@DV?$string_output_adapter@D@__crt_stdio_output@@@2@@__crt_stdio_output@@AAE_N_N@Z 1000eb4b f i libucrt:output.obj
 0001:0000dcd8       ??$type_case_integer_parse_into_buffer@I$07@?$output_processor@DV?$stream_output_adapter@D@__crt_stdio_output@@V?$standard_base@DV?$stream_output_adapter@D@__crt_stdio_output@@@2@@__crt_stdio_output@@AAEXI_N@Z 1000ecd8 f i libucrt:output.obj
 0001:0000dcd8       ??$type_case_integer_parse_into_buffer@I$07@?$output_processor@DV?$string_output_adapter@D@__crt_stdio_output@@V?$standard_base@DV?$string_output_adapter@D@__crt_stdio_output@@@2@@__crt_stdio_output@@AAEXI_N@Z 1000ecd8 f i libucrt:output.obj
 0001:0000dd3b       ??$type_case_integer_parse_into_buffer@I$09@?$output_processor@DV?$stream_output_adapter@D@__crt_stdio_output@@V?$standard_base@DV?$stream_output_adapter@D@__crt_stdio_output@@@2@@__crt_stdio_output@@AAEXI_N@Z 1000ed3b f i libucrt:output.obj
 0001:0000dd3b       ??$type_case_integer_parse_into_buffer@I$09@?$output_processor@DV?$string_output_adapter@D@__crt_stdio_output@@V?$standard_base@DV?$string_output_adapter@D@__crt_stdio_output@@@2@@__crt_stdio_output@@AAEXI_N@Z 1000ed3b f i libucrt:output.obj
 0001:0000ddc2       ??$type_case_integer_parse_into_buffer@I$0BA@@?$output_processor@DV?$stream_output_adapter@D@__crt_stdio_output@@V?$standard_base@DV?$stream_output_adapter@D@__crt_stdio_output@@@2@@__crt_stdio_output@@AAEXI_N@Z 1000edc2 f i libucrt:output.obj
 0001:0000ddc2       ??$type_case_integer_parse_into_buffer@I$0BA@@?$output_processor@DV?$string_output_adapter@D@__crt_stdio_output@@V?$standard_base@DV?$string_output_adapter@D@__crt_stdio_output@@@2@@__crt_stdio_output@@AAEXI_N@Z 1000edc2 f i libucrt:output.obj
 0001:0000de3f       ??$type_case_integer_parse_into_buffer@_K$07@?$output_processor@DV?$stream_output_adapter@D@__crt_stdio_output@@V?$standard_base@DV?$stream_output_adapter@D@__crt_stdio_output@@@2@@__crt_stdio_output@@AAEX_K_N@Z 1000ee3f f i libucrt:output.obj
 0001:0000de3f       ??$type_case_integer_parse_into_buffer@_K$07@?$output_processor@DV?$string_output_adapter@D@__crt_stdio_output@@V?$standard_base@DV?$string_output_adapter@D@__crt_stdio_output@@@2@@__crt_stdio_output@@AAEX_K_N@Z 1000ee3f f i libucrt:output.obj
 0001:0000deb7       ??$type_case_integer_parse_into_buffer@_K$09@?$output_processor@DV?$stream_output_adapter@D@__crt_stdio_output@@V?$standard_base@DV?$stream_output_adapter@D@__crt_stdio_output@@@2@@__crt_stdio_output@@AAEX_K_N@Z 1000eeb7 f i libucrt:output.obj
 0001:0000deb7       ??$type_case_integer_parse_into_buffer@_K$09@?$output_processor@DV?$string_output_adapter@D@__crt_stdio_output@@V?$standard_base@DV?$string_output_adapter@D@__crt_stdio_output@@@2@@__crt_stdio_output@@AAEX_K_N@Z 1000eeb7 f i libucrt:output.obj
 0001:0000df5e       ??$type_case_integer_parse_into_buffer@_K$0BA@@?$output_processor@DV?$stream_output_adapter@D@__crt_stdio_output@@V?$standard_base@DV?$stream_output_adapter@D@__crt_stdio_output@@@2@@__crt_stdio_output@@AAEX_K_N@Z 1000ef5e f i libucrt:output.obj
 0001:0000df5e       ??$type_case_integer_parse_into_buffer@_K$0BA@@?$output_processor@DV?$string_output_adapter@D@__crt_stdio_output@@V?$standard_base@DV?$string_output_adapter@D@__crt_stdio_output@@@2@@__crt_stdio_output@@AAEX_K_N@Z 1000ef5e f i libucrt:output.obj
 0001:0000dfe8       ??0?$output_adapter_data@DV?$stream_output_adapter@D@__crt_stdio_output@@@__crt_stdio_output@@IAE@ABV?$stream_output_adapter@D@1@_KQBDAAV__crt_cached_ptd_host@@QAD@Z 1000efe8 f i libucrt:output.obj
 0001:0000dfe8       ??0?$output_adapter_data@DV?$string_output_adapter@D@__crt_stdio_output@@@__crt_stdio_output@@IAE@ABV?$string_output_adapter@D@1@_KQBDAAV__crt_cached_ptd_host@@QAD@Z 1000efe8 f i libucrt:output.obj
 0001:0000e04f       ??1formatting_buffer@__crt_stdio_output@@QAE@XZ 1000f04f f i libucrt:output.obj
 0001:0000e069       ??4?$__crt_unique_heap_ptr@DU__crt_internal_free_policy@@@@QAEAAV0@$$QAV0@@Z 1000f069 f i libucrt:output.obj
 0001:0000e129       ?crop_zeroes@__crt_stdio_output@@YAXPADQAU__crt_locale_pointers@@@Z 1000f129 f i libucrt:output.obj
 0001:0000e189       ?find_next_state@?$output_processor@DV?$stream_output_adapter@D@__crt_stdio_output@@V?$standard_base@DV?$stream_output_adapter@D@__crt_stdio_output@@@2@@__crt_stdio_output@@ABE?AW4state@2@DW432@@Z 1000f189 f i libucrt:output.obj
 0001:0000e189       ?find_next_state@?$output_processor@DV?$string_output_adapter@D@__crt_stdio_output@@V?$standard_base@DV?$string_output_adapter@D@__crt_stdio_output@@@2@@__crt_stdio_output@@ABE?AW4state@2@DW432@@Z 1000f189 f i libucrt:output.obj
 0001:0000e1c4       ?force_decimal_point@__crt_stdio_output@@YAXPADQAU__crt_locale_pointers@@@Z 1000f1c4 f i libucrt:output.obj
 0001:0000e220       ?parse_int_from_format_string@?$output_processor@DV?$stream_output_adapter@D@__crt_stdio_output@@V?$standard_base@DV?$stream_output_adapter@D@__crt_stdio_output@@@2@@__crt_stdio_output@@AAE_NQAH@Z 1000f220 f i libucrt:output.obj
 0001:0000e220       ?parse_int_from_format_string@?$output_processor@DV?$string_output_adapter@D@__crt_stdio_output@@V?$standard_base@DV?$string_output_adapter@D@__crt_stdio_output@@@2@@__crt_stdio_output@@AAE_NQAH@Z 1000f220 f i libucrt:output.obj
 0001:0000e298       ?process@?$output_processor@DV?$stream_output_adapter@D@__crt_stdio_output@@V?$standard_base@DV?$stream_output_adapter@D@__crt_stdio_output@@@2@@__crt_stdio_output@@QAEHXZ 1000f298 f i libucrt:output.obj
 0001:0000e548       ?process@?$output_processor@DV?$string_output_adapter@D@__crt_stdio_output@@V?$standard_base@DV?$string_output_adapter@D@__crt_stdio_output@@@2@@__crt_stdio_output@@QAEHXZ 1000f548 f i libucrt:output.obj
 0001:0000e81c       ?state_case_size@?$output_processor@DV?$stream_output_adapter@D@__crt_stdio_output@@V?$standard_base@DV?$stream_output_adapter@D@__crt_stdio_output@@@2@@__crt_stdio_output@@AAE_NXZ 1000f81c f i libucrt:output.obj
 0001:0000e975       ?state_case_size@?$output_processor@DV?$string_output_adapter@D@__crt_stdio_output@@V?$standard_base@DV?$string_output_adapter@D@__crt_stdio_output@@@2@@__crt_stdio_output@@AAE_NXZ 1000f975 f i libucrt:output.obj
 0001:0000eace       ?state_case_type@?$output_processor@DV?$stream_output_adapter@D@__crt_stdio_output@@V?$standard_base@DV?$stream_output_adapter@D@__crt_stdio_output@@@2@@__crt_stdio_output@@AAE_NXZ 1000face f i libucrt:output.obj
 0001:0000ee10       ?state_case_type@?$output_processor@DV?$string_output_adapter@D@__crt_stdio_output@@V?$standard_base@DV?$string_output_adapter@D@__crt_stdio_output@@@2@@__crt_stdio_output@@AAE_NXZ 1000fe10 f i libucrt:output.obj
 0001:0000f16f       ?to_integer_size@__crt_stdio_output@@YAIW4length_modifier@1@@Z 1001016f f i libucrt:output.obj
 0001:0000f1c3       ?type_case_Z@?$output_processor@DV?$stream_output_adapter@D@__crt_stdio_output@@V?$standard_base@DV?$stream_output_adapter@D@__crt_stdio_output@@@2@@__crt_stdio_output@@AAE_NXZ 100101c3 f i libucrt:output.obj
 0001:0000f1c3       ?type_case_Z@?$output_processor@DV?$string_output_adapter@D@__crt_stdio_output@@V?$standard_base@DV?$string_output_adapter@D@__crt_stdio_output@@@2@@__crt_stdio_output@@AAE_NXZ 100101c3 f i libucrt:output.obj
 0001:0000f226       ?type_case_a@?$output_processor@DV?$stream_output_adapter@D@__crt_stdio_output@@V?$standard_base@DV?$stream_output_adapter@D@__crt_stdio_output@@@2@@__crt_stdio_output@@AAE_NXZ 10010226 f i libucrt:output.obj
 0001:0000f226       ?type_case_a@?$output_processor@DV?$string_output_adapter@D@__crt_stdio_output@@V?$standard_base@DV?$string_output_adapter@D@__crt_stdio_output@@@2@@__crt_stdio_output@@AAE_NXZ 10010226 f i libucrt:output.obj
 0001:0000f3b7       ?type_case_c_tchar@?$output_processor@DV?$stream_output_adapter@D@__crt_stdio_output@@V?$standard_base@DV?$stream_output_adapter@D@__crt_stdio_output@@@2@@__crt_stdio_output@@AAE_ND@Z 100103b7 f i libucrt:output.obj
 0001:0000f3b7       ?type_case_c_tchar@?$output_processor@DV?$string_output_adapter@D@__crt_stdio_output@@V?$standard_base@DV?$string_output_adapter@D@__crt_stdio_output@@@2@@__crt_stdio_output@@AAE_ND@Z 100103b7 f i libucrt:output.obj
 0001:0000f44c       ?type_case_n@?$output_processor@DV?$stream_output_adapter@D@__crt_stdio_output@@V?$standard_base@DV?$stream_output_adapter@D@__crt_stdio_output@@@2@@__crt_stdio_output@@AAE_NXZ 1001044c f i libucrt:output.obj
 0001:0000f44c       ?type_case_n@?$output_processor@DV?$string_output_adapter@D@__crt_stdio_output@@V?$standard_base@DV?$string_output_adapter@D@__crt_stdio_output@@@2@@__crt_stdio_output@@AAE_NXZ 1001044c f i libucrt:output.obj
 0001:0000f4d1       ?type_case_o@?$output_processor@DV?$stream_output_adapter@D@__crt_stdio_output@@V?$standard_base@DV?$stream_output_adapter@D@__crt_stdio_output@@@2@@__crt_stdio_output@@AAE_NXZ 100104d1 f i libucrt:output.obj
 0001:0000f4d1       ?type_case_o@?$output_processor@DV?$string_output_adapter@D@__crt_stdio_output@@V?$standard_base@DV?$string_output_adapter@D@__crt_stdio_output@@@2@@__crt_stdio_output@@AAE_NXZ 100104d1 f i libucrt:output.obj
 0001:0000f4ee       ?type_case_p@?$output_processor@DV?$stream_output_adapter@D@__crt_stdio_output@@V?$standard_base@DV?$stream_output_adapter@D@__crt_stdio_output@@@2@@__crt_stdio_output@@AAE_NXZ 100104ee f i libucrt:output.obj
 0001:0000f4ee       ?type_case_p@?$output_processor@DV?$string_output_adapter@D@__crt_stdio_output@@V?$standard_base@DV?$string_output_adapter@D@__crt_stdio_output@@@2@@__crt_stdio_output@@AAE_NXZ 100104ee f i libucrt:output.obj
 0001:0000f504       ?type_case_s@?$output_processor@DV?$stream_output_adapter@D@__crt_stdio_output@@V?$standard_base@DV?$stream_output_adapter@D@__crt_stdio_output@@@2@@__crt_stdio_output@@AAE_NXZ 10010504 f i libucrt:output.obj
 0001:0000f504       ?type_case_s@?$output_processor@DV?$string_output_adapter@D@__crt_stdio_output@@V?$standard_base@DV?$string_output_adapter@D@__crt_stdio_output@@@2@@__crt_stdio_output@@AAE_NXZ 10010504 f i libucrt:output.obj
 0001:0000f576       ?unget@?$c_string_character_source@D@__crt_strtox@@QAEXD@Z 10010576 f i libucrt:output.obj
 0001:0000f59f       ?unget@?$c_string_character_source@_W@__crt_strtox@@QAEX_W@Z 1001059f f i libucrt:output.obj
 0001:0000f5d0       ?update_locale_slow@__crt_cached_ptd_host@@AAEXXZ 100105d0 f i libucrt:output.obj
 0001:0000f62b       ?validate@?$c_string_character_source@D@__crt_strtox@@QBE_NXZ 1001062b f i libucrt:output.obj
 0001:0000f62b       ?validate@?$c_string_character_source@_W@__crt_strtox@@QBE_NXZ 1001062b f i libucrt:output.obj
 0001:0000f646       ?validate@?$stream_output_adapter@D@__crt_stdio_output@@QBE_NAAV__crt_cached_ptd_host@@@Z 10010646 f i libucrt:output.obj
 0001:0000f67e       ?validate@?$string_output_adapter@D@__crt_stdio_output@@QBE_NAAV__crt_cached_ptd_host@@@Z 1001067e f i libucrt:output.obj
 0001:0000f6af       ?write_character@?$output_adapter_common@DV?$stream_output_adapter@D@__crt_stdio_output@@@__crt_stdio_output@@QBEXDQAHAAV__crt_cached_ptd_host@@@Z 100106af f i libucrt:output.obj
 0001:0000f6d1       ?write_character_without_count_update@?$stream_output_adapter@D@__crt_stdio_output@@QBE_NDAAV__crt_cached_ptd_host@@@Z 100106d1 f i libucrt:output.obj
 0001:0000f70b       ?write_string@?$stream_output_adapter@D@__crt_stdio_output@@QBEXQBDHQAHAAV__crt_cached_ptd_host@@@Z 1001070b f i libucrt:output.obj
 0001:0000f737       ?write_string@?$string_output_adapter@D@__crt_stdio_output@@QBEXQBDHQAHAAV__crt_cached_ptd_host@@@Z 10010737 f i libucrt:output.obj
 0001:0000f79e       ?write_string_impl@?$output_adapter_common@DV?$stream_output_adapter@D@__crt_stdio_output@@@__crt_stdio_output@@IBEXQBDHQAHAAV__crt_cached_ptd_host@@@Z 1001079e f i libucrt:output.obj
 0001:0000f81d       ___acrt_locale_get_ctype_array_value 1001081d f i libucrt:output.obj
 0001:0000f83f       ___stdio_common_vfprintf   1001083f f   libucrt:output.obj
 0001:0000f8e3       ___stdio_common_vsprintf   100108e3 f   libucrt:output.obj
 0001:0000f924       ??$assemble_floating_point_snan@N@__crt_strtox@@YAX_NAAN@Z 10010924 f i libucrt:input.obj
 0001:0000f945       ??$assemble_floating_point_value_t@M@__crt_strtox@@YA?AW4SLD_STATUS@@_NH_KAAM@Z 10010945 f i libucrt:input.obj
 0001:0000f975       ??$assemble_floating_point_value_t@N@__crt_strtox@@YA?AW4SLD_STATUS@@_NH_KAAN@Z 10010975 f i libucrt:input.obj
 0001:0000fa6b       ??$convert_decimal_string_to_floating_type@M@__crt_strtox@@YA?AW4SLD_STATUS@@ABUfloating_point_string@0@AAM@Z 10010a6b f i libucrt:input.obj
 0001:0000fa8c       ??$convert_decimal_string_to_floating_type@N@__crt_strtox@@YA?AW4SLD_STATUS@@ABUfloating_point_string@0@AAN@Z 10010a8c f i libucrt:input.obj
 0001:0000faad       ??$convert_hexadecimal_string_to_floating_type@M@__crt_strtox@@YA?AW4SLD_STATUS@@ABUfloating_point_string@0@AAM@Z 10010aad f i libucrt:input.obj
 0001:0000face       ??$convert_hexadecimal_string_to_floating_type@N@__crt_strtox@@YA?AW4SLD_STATUS@@ABUfloating_point_string@0@AAN@Z 10010ace f i libucrt:input.obj
 0001:0000faef       ??$is_overflow_condition@_K@__crt_strtox@@YA_NI_K@Z 10010aef f i libucrt:input.obj
 0001:0000fb30       ??$make_input_adapter_character_source@V?$string_input_adapter@D@__crt_stdio_input@@@__crt_strtox@@YA?AV?$input_adapter_character_source@V?$string_input_adapter@D@__crt_stdio_input@@@0@QAV?$string_input_adapter@D@__crt_stdio_input@@_KQA_N@Z 10010b30 f i libucrt:input.obj
 0001:0000fb4e       ??$parse_floating_point@V?$input_adapter_character_source@V?$string_input_adapter@D@__crt_stdio_input@@@__crt_strtox@@M@__crt_strtox@@YA?AW4SLD_STATUS@@QAU__crt_locale_pointers@@V?$input_adapter_character_source@V?$string_input_adapter@D@__crt_stdio_input@@@0@QAM@Z 10010b4e f i libucrt:input.obj
 0001:0000fbd8       ??$parse_floating_point@V?$input_adapter_character_source@V?$string_input_adapter@D@__crt_stdio_input@@@__crt_strtox@@N@__crt_strtox@@YA?AW4SLD_STATUS@@QAU__crt_locale_pointers@@V?$input_adapter_character_source@V?$string_input_adapter@D@__crt_stdio_input@@@0@QAN@Z 10010bd8 f i libucrt:input.obj
 0001:0000fc62       ??$parse_floating_point_from_source@V?$input_adapter_character_source@V?$string_input_adapter@D@__crt_stdio_input@@@__crt_strtox@@@__crt_strtox@@YA?AW4floating_point_parse_result@0@QAU__crt_locale_pointers@@AAV?$input_adapter_character_source@V?$string_input_adapter@D@__crt_stdio_input@@@0@AAUfloating_point_string@0@@Z 10010c62 f i libucrt:input.obj
 0001:000100c4       ??$parse_floating_point_possible_infinity@DV?$input_adapter_character_source@V?$string_input_adapter@D@__crt_stdio_input@@@__crt_strtox@@_K@__crt_strtox@@YA?AW4floating_point_parse_result@0@AADAAV?$input_adapter_character_source@V?$string_input_adapter@D@__crt_stdio_input@@@0@_K@Z 100110c4 f i libucrt:input.obj
 0001:00010183       ??$parse_floating_point_possible_nan@DV?$input_adapter_character_source@V?$string_input_adapter@D@__crt_stdio_input@@@__crt_strtox@@_K@__crt_strtox@@YA?AW4floating_point_parse_result@0@AADAAV?$input_adapter_character_source@V?$string_input_adapter@D@__crt_stdio_input@@@0@_K@Z 10011183 f i libucrt:input.obj
 0001:0001028b       ??$parse_floating_point_possible_nan_is_ind@DV?$input_adapter_character_source@V?$string_input_adapter@D@__crt_stdio_input@@@__crt_strtox@@@__crt_strtox@@YA_NAADAAV?$input_adapter_character_source@V?$string_input_adapter@D@__crt_stdio_input@@@0@@Z 1001128b f i libucrt:input.obj
 0001:000102c5       ??$parse_floating_point_possible_nan_is_snan@DV?$input_adapter_character_source@V?$string_input_adapter@D@__crt_stdio_input@@@__crt_strtox@@@__crt_strtox@@YA_NAADAAV?$input_adapter_character_source@V?$string_input_adapter@D@__crt_stdio_input@@@0@@Z 100112c5 f i libucrt:input.obj
 0001:000102ff       ??$parse_floating_point_write_result@M@__crt_strtox@@YA?AW4SLD_STATUS@@W4floating_point_parse_result@0@ABUfloating_point_string@0@QAM@Z 100112ff f i libucrt:input.obj
 0001:0001046b       ??$parse_floating_point_write_result@N@__crt_strtox@@YA?AW4SLD_STATUS@@W4floating_point_parse_result@0@ABUfloating_point_string@0@QAN@Z 1001146b f i libucrt:input.obj
 0001:0001058f       ??$parse_integer@_KV?$input_adapter_character_source@V?$string_input_adapter@D@__crt_stdio_input@@@__crt_strtox@@$00@__crt_strtox@@YA_KAAV__crt_cached_ptd_host@@V?$input_adapter_character_source@V?$string_input_adapter@D@__crt_stdio_input@@@0@H_N@Z 1001158f f i libucrt:input.obj
 0001:00010893       ??$parse_integer@_KV?$input_adapter_character_source@V?$string_input_adapter@D@__crt_stdio_input@@@__crt_strtox@@@__crt_strtox@@YA_KQAU__crt_locale_pointers@@V?$input_adapter_character_source@V?$string_input_adapter@D@__crt_stdio_input@@@0@H_N@Z 10011893 f i libucrt:input.obj
 0001:000108ef       ??$process_floating_point_specifier_t@M@?$input_processor@DV?$string_input_adapter@D@__crt_stdio_input@@@__crt_stdio_input@@AAE_NXZ 100118ef f i libucrt:input.obj
 0001:00010958       ??$process_floating_point_specifier_t@N@?$input_processor@DV?$string_input_adapter@D@__crt_stdio_input@@@__crt_stdio_input@@AAE_NXZ 10011958 f i libucrt:input.obj
 0001:000109c1       ??$process_string_specifier_tchar@D@?$input_processor@DV?$string_input_adapter@D@__crt_stdio_input@@@__crt_stdio_input@@AAE_NW4conversion_mode@1@D@Z 100119c1 f i libucrt:input.obj
 0001:00010b23       ??$process_string_specifier_tchar@_W@?$input_processor@DV?$string_input_adapter@D@__crt_stdio_input@@@__crt_stdio_input@@AAE_NW4conversion_mode@1@_W@Z 10011b23 f i libucrt:input.obj
 0001:00010c91       ??$skip_whitespace@Vstring_input_adapter@__crt_stdio_input@@D@__crt_stdio_input@@YAHAAV?$string_input_adapter@D@0@QAU__crt_locale_pointers@@@Z 10011c91 f i libucrt:input.obj
 0001:00010cc0       ??$write_floating_point@M@?$input_processor@DV?$string_input_adapter@D@__crt_stdio_input@@@__crt_stdio_input@@AAE_NABM@Z 10011cc0 f i libucrt:input.obj
 0001:00010cf5       ??$write_floating_point@N@?$input_processor@DV?$string_input_adapter@D@__crt_stdio_input@@@__crt_stdio_input@@AAE_NABN@Z 10011cf5 f i libucrt:input.obj
 0001:00010d30       ??0?$format_string_parser@D@__crt_stdio_input@@QAE@_KQBE@Z 10011d30 f i libucrt:input.obj
 0001:00010d7a       ??0?$input_adapter_character_source@V?$string_input_adapter@D@__crt_stdio_input@@@__crt_strtox@@QAE@$$QAV01@@Z 10011d7a f i libucrt:input.obj
 0001:00010db7       ??0?$input_adapter_character_source@V?$string_input_adapter@D@__crt_stdio_input@@@__crt_strtox@@QAE@QAV?$string_input_adapter@D@__crt_stdio_input@@_KQA_N@Z 10011db7 f i libucrt:input.obj
 0001:00010de8       ??0?$input_processor@DV?$string_input_adapter@D@__crt_stdio_input@@@__crt_stdio_input@@QAE@ABV?$string_input_adapter@D@1@_KQBDQAU__crt_locale_pointers@@QAD@Z 10011de8 f i libucrt:input.obj
 0001:00010e2c       ??0_LocaleUpdate@@QAE@QAU__crt_locale_pointers@@@Z 10011e2c f i libucrt:input.obj
 0001:00010eae       ??R<lambda_644f8ab42ed3fd1d660977a2364b3a7d>@@QBE@XZ 10011eae f i libucrt:input.obj
 0001:00010eae       ??R<lambda_f1fa4c266c18b246f3ed9c36247dab4f>@@QBE@XZ 10011eae f i libucrt:input.obj
 0001:00010eae       ??R<lambda_f765c90ab33e8386abf09c0f079d37e9>@@QBE@XZ 10011eae f i libucrt:input.obj
 0001:00010ed8       ?advance@?$format_string_parser@D@__crt_stdio_input@@QAE_NXZ 10011ed8 f i libucrt:input.obj
 0001:00010ff0       ?as_double@floating_point_value@__crt_strtox@@QBEAANXZ 10011ff0 f i libucrt:input.obj
 0001:00011015       ?as_float@floating_point_value@__crt_strtox@@QBEAAMXZ 10012015 f i libucrt:input.obj
 0001:0001103a       ?assemble_floating_point_infinity@__crt_strtox@@YAX_NABVfloating_point_value@1@@Z 1001203a f i libucrt:input.obj
 0001:0001107a       ?assemble_floating_point_value@__crt_strtox@@YA?AW4SLD_STATUS@@_KH_N1ABVfloating_point_value@1@@Z 1001207a f i libucrt:input.obj
 0001:000113d3       ?assemble_floating_point_value_from_big_integer@__crt_strtox@@YA?AW4SLD_STATUS@@ABUbig_integer@1@I_N1ABVfloating_point_value@1@@Z 100123d3 f i libucrt:input.obj
 0001:00011565       ?assemble_floating_point_zero@__crt_strtox@@YAX_NABVfloating_point_value@1@@Z 10012565 f i libucrt:input.obj
 0001:0001159a       ?convert_decimal_string_to_floating_type_common@__crt_strtox@@YA?AW4SLD_STATUS@@ABUfloating_point_string@1@ABVfloating_point_value@1@@Z 1001259a f i libucrt:input.obj
 0001:00013340       ?convert_hexadecimal_string_to_floating_type_common@__crt_strtox@@YA?AW4SLD_STATUS@@ABUfloating_point_string@1@ABVfloating_point_value@1@@Z 10014340 f i libucrt:input.obj
 0001:000133e6       ?denormal_mantissa_mask@floating_point_value@__crt_strtox@@QBE_KXZ 100143e6 f i libucrt:input.obj
 0001:00013400       ?divide@__crt_strtox@@YA_KAAUbig_integer@1@ABU21@@Z 10014400 f i libucrt:input.obj
 0001:000138ab       ?get@?$input_adapter_character_source@V?$string_input_adapter@D@__crt_stdio_input@@@__crt_strtox@@QAEDXZ 100148ab f i libucrt:input.obj
 0001:000138e2       ?get@?$string_input_adapter@D@__crt_stdio_input@@QAEHXZ 100148e2 f i libucrt:input.obj
 0001:000138f8       ?is_character_allowed_in_string@?$input_processor@DV?$string_input_adapter@D@__crt_stdio_input@@@__crt_stdio_input@@ABE_NW4conversion_mode@2@H@Z 100148f8 f i libucrt:input.obj
 0001:00013948       ?length@?$format_string_parser@D@__crt_stdio_input@@QBEIXZ 10014948 f i libucrt:input.obj
 0001:00013996       ?normal_mantissa_mask@floating_point_value@__crt_strtox@@QBE_KXZ 10014996 f i libucrt:input.obj
 0001:000139ad       ?process@?$input_processor@DV?$string_input_adapter@D@__crt_stdio_input@@@__crt_stdio_input@@QAEHXZ 100149ad f i libucrt:input.obj
 0001:00013a31       ?process_character_count_specifier@?$input_processor@DV?$string_input_adapter@D@__crt_stdio_input@@@__crt_stdio_input@@AAE_NXZ 10014a31 f i libucrt:input.obj
 0001:00013a49       ?process_conversion_specifier@?$input_processor@DV?$string_input_adapter@D@__crt_stdio_input@@@__crt_stdio_input@@AAE_NXZ 10014a49 f i libucrt:input.obj
 0001:00013abd       ?process_floating_point_specifier@?$input_processor@DV?$string_input_adapter@D@__crt_stdio_input@@@__crt_stdio_input@@AAE_NXZ 10014abd f i libucrt:input.obj
 0001:00013aed       ?process_integer_specifier@?$input_processor@DV?$string_input_adapter@D@__crt_stdio_input@@@__crt_stdio_input@@AAE_NI_N@Z 10014aed f i libucrt:input.obj
 0001:00013b52       ?process_literal_character@?$input_processor@DV?$string_input_adapter@D@__crt_stdio_input@@@__crt_stdio_input@@AAE_NXZ 10014b52 f i libucrt:input.obj
 0001:00013b88       ?process_literal_character_tchar@?$input_processor@DV?$string_input_adapter@D@__crt_stdio_input@@@__crt_stdio_input@@AAE_ND@Z 10014b88 f i libucrt:input.obj
 0001:00013bd6       ?process_state@?$input_processor@DV?$string_input_adapter@D@__crt_stdio_input@@@__crt_stdio_input@@AAE_NXZ 10014bd6 f i libucrt:input.obj
 0001:00013c18       ?process_string_specifier@?$input_processor@DV?$string_input_adapter@D@__crt_stdio_input@@@__crt_stdio_input@@AAE_NW4conversion_mode@2@@Z 10014c18 f i libucrt:input.obj
 0001:00013c60       ?process_whitespace@?$input_processor@DV?$string_input_adapter@D@__crt_stdio_input@@@__crt_stdio_input@@AAE_NXZ 10014c60 f i libucrt:input.obj
 0001:00013c7d       ?restore_state@?$input_adapter_character_source@V?$string_input_adapter@D@__crt_stdio_input@@@__crt_strtox@@QAE_N_K@Z 10014c7d f i libucrt:input.obj
 0001:00013ca2       ?scan_conversion_specifier@?$format_string_parser@D@__crt_stdio_input@@AAE_NXZ 10014ca2 f i libucrt:input.obj
 0001:00013e1e       ?scan_optional_field_width@?$format_string_parser@D@__crt_stdio_input@@AAE_NXZ 10014e1e f i libucrt:input.obj
 0001:00013eb2       ?scan_optional_length_modifier@?$format_string_parser@D@__crt_stdio_input@@AAEXXZ 10014eb2 f i libucrt:input.obj
 0001:00013fd2       ?scan_optional_literal_character_trail_bytes_tchar@?$format_string_parser@D@__crt_stdio_input@@AAE_ND@Z 10014fd2 f i libucrt:input.obj
 0001:00014024       ?scan_optional_wide_modifier@?$format_string_parser@D@__crt_stdio_input@@AAEXXZ 10015024 f i libucrt:input.obj
 0001:00014042       ?scan_scanset_range@?$format_string_parser@D@__crt_stdio_input@@AAE_NXZ 10015042 f i libucrt:input.obj
 0001:0001417b       ?set@?$scanset_buffer@E@__crt_stdio_input@@QAEXE@Z 1001517b f i libucrt:input.obj
 0001:000141a6       ?set_wide_for_c_s_or_scanset@?$format_string_parser@D@__crt_stdio_input@@AAEXXZ 100151a6 f i libucrt:input.obj
 0001:000141c7       ?to_floating_point_length@__crt_stdio_input@@YAIW4length_modifier@1@@Z 100151c7 f i libucrt:input.obj
 0001:000141ea       ?to_integer_length@__crt_stdio_input@@YAIW4length_modifier@1@@Z 100151ea f i libucrt:input.obj
 0001:0001423d       ?unget@?$input_adapter_character_source@V?$string_input_adapter@D@__crt_stdio_input@@@__crt_strtox@@QAEXD@Z 1001523d f i libucrt:input.obj
 0001:00014284       ?unget@?$string_input_adapter@D@__crt_stdio_input@@QAEXH@Z 10015284 f i libucrt:input.obj
 0001:000142a3       ?validate@?$format_string_parser@D@__crt_stdio_input@@QBE_NXZ 100152a3 f i libucrt:input.obj
 0001:000142bf       ?validate@?$input_adapter_character_source@V?$string_input_adapter@D@__crt_stdio_input@@@__crt_strtox@@QBE_NXZ 100152bf f i libucrt:input.obj
 0001:000142e0       ?validate@?$string_input_adapter@D@__crt_stdio_input@@QAE_NXZ 100152e0 f i libucrt:input.obj
 0001:00014302       ?write_character@?$input_processor@DV?$string_input_adapter@D@__crt_stdio_input@@@__crt_stdio_input@@AAE_NQA_WIAAPA_WAAID@Z 10015302 f i libucrt:input.obj
 0001:0001436f       ?write_integer@?$input_processor@DV?$string_input_adapter@D@__crt_stdio_input@@@__crt_stdio_input@@AAE_N_K@Z 1001536f f i libucrt:input.obj
 0001:000143de       ___stdio_common_vsscanf    100153de f   libucrt:input.obj
 0001:00014402       __ischartype_l             10015402 f i libucrt:input.obj
 0001:000144da       _free                      100154da f   libucrt:free.obj
 0001:00014542       ??$__crt_fast_decode_pointer@P6AHI@Z@@YAP6AHI@ZQ6AHI@Z@Z 10015542 f i libucrt:new_handler.obj
 0001:00014542       ??$__crt_fast_decode_pointer@P6AXH@Z@@YAP6AXH@ZQ6AXH@Z@Z 10015542 f i libucrt:signal.obj
 0001:00014542       ??$__crt_fast_decode_pointer@P6GXPAXK0@Z@@YAP6GXPAXK0@ZQ6GX0K0@Z@Z 10015542 f i libucrt:exit.obj
 0001:000147ea       ___acrt_initialize_thread_local_exit_callback 100157ea f   libucrt:exit.obj
 0001:000147f9       __cexit                    100157f9 f   libucrt:exit.obj
 0001:00014808       __exit                     10015808 f   libucrt:exit.obj
 0001:0001481e       __is_c_termination_complete 1001581e f   libucrt:exit.obj
 0001:00014825       _exit                      10015825 f   libucrt:exit.obj
 0001:00014ab8       __wgetenv_s                10015ab8 f   libucrt:getenv.obj
 0001:00014ac3       _getenv                    10015ac3 f   libucrt:getenv.obj
 0001:00014d72       __putenv                   10015d72 f   libucrt:putenv.obj
 0001:00014d72       _putenv                    10015d72 f   libucrt:putenv.obj
 0001:00014d90       _strcpy                    10015d90 f   libucrt:strcat.obj
 0001:00014da0       _strcat                    10015da0 f   libucrt:strcat.obj
 0001:00014e90       _strcmp                    10015e90 f   libucrt:strcmp.obj
 0001:00014f20       _strcspn                   10015f20 f   libucrt:strcspn.obj
 0001:00014f70       _strlen                    10015f70 f   libucrt:strlen.obj
 0001:00015000       _strspn                    10016000 f   libucrt:strspn.obj
 0001:00015046       __getpid                   10016046 f   libucrt:getpid.obj
 0001:0001504c       ___acrt_errno_from_os_error 1001604c f   libucrt:errno.obj
 0001:0001508f       ___acrt_errno_map_os_error 1001608f f   libucrt:errno.obj
 0001:000150b2       ___acrt_errno_map_os_error_ptd 100160b2 f   libucrt:errno.obj
 0001:000150d6       ___doserrno                100160d6 f   libucrt:errno.obj
 0001:000150e9       __errno                    100160e9 f   libucrt:errno.obj
 0001:0001516f       __get_sys_err_msg          1001616f f i libucrt:strerror.obj
 0001:000151c7       _strerror                  100161c7 f   libucrt:strerror.obj
 0001:000151e0       _strncmp                   100161e0 f   libucrt:strncmp.obj
 0001:00015258       ??$__acrt_convert_wcs_mbs_cp@D_WV<lambda_62f6974d9771e494a5ea317cc32e971c>@@U__crt_win32_buffer_internal_dynamic_resizing@@@@YAHQBDAAV?$__crt_win32_buffer@_WU__crt_win32_buffer_internal_dynamic_resizing@@@@ABV<lambda_62f6974d9771e494a5ea317cc32e971c>@@I@Z 10016258 f i libucrt:access.obj
 0001:0001530a       ??$__acrt_mbs_to_wcs_cp@U__crt_win32_buffer_internal_dynamic_resizing@@@@YAHQBDAAV?$__crt_win32_buffer@_WU__crt_win32_buffer_internal_dynamic_resizing@@@@I@Z 1001630a f i libucrt:access.obj
 0001:00015327       ?__acrt_get_utf8_acp_compatibility_codepage@@YAIXZ 10016327 f i libucrt:access.obj
 0001:00015366       ?_deallocate@?$__crt_win32_buffer@DU__crt_win32_buffer_internal_dynamic_resizing@@@@AAEXXZ 10016366 f i libucrt:argv_wildcards.obj
 0001:00015366       ?_deallocate@?$__crt_win32_buffer@_WU__crt_win32_buffer_internal_dynamic_resizing@@@@AAEXXZ 10016366 f i libucrt:access.obj
 0001:00015380       ?allocate@?$__crt_win32_buffer@_WU__crt_win32_buffer_internal_dynamic_resizing@@@@QAEHI@Z 10016380 f i libucrt:access.obj
 0001:000153bf       ?allocate@__crt_win32_buffer_internal_dynamic_resizing@@SAHQAPAXIABV__crt_win32_buffer_empty_debug_info@@@Z 100163bf f i libucrt:access.obj
 0001:000153de       __access                   100163de f   libucrt:access.obj
 0001:000153f6       __access_s                 100163f6 f   libucrt:access.obj
 0001:000155c4       __beginthreadex            100165c4 f   libucrt:thread.obj
 0001:00015647       __endthreadex              10016647 f   libucrt:thread.obj
 0001:0001588e       ___acrt_stdio_flush_nolock 1001688e f   libucrt:fflush.obj
 0001:000158f7       __fflush_nolock            100168f7 f   libucrt:fflush.obj
 0001:0001595c       __flushall                 1001695c f   libucrt:fflush.obj
 0001:00015965       _fflush                    10016965 f   libucrt:fflush.obj
 0001:00015dba       ??$loctotime@AAGAAGAAGAAGAAGAAGH@?$__crt_integer_traits@_J@@SA_JAAG00000$$QAH@Z 10016dba f i libucrt:stat.obj
 0001:0001616f       __stat64i32                1001716f f   libucrt:stat.obj
 0001:0001622e       _perror                    1001722e f   libucrt:perror.obj
 0001:00016258       _malloc                    10017258 f   libucrt:malloc.obj
 0001:00016263       _realloc                   10017263 f   libucrt:realloc.obj
 0001:00016270       _strpbrk                   10017270 f   libucrt:strpbrk.obj
 0001:00016458       __lseeki64                 10017458 f   libucrt:lseek.obj
 0001:00016498       __lseeki64_nolock          10017498 f   libucrt:lseek.obj
 0001:000164d8       __lseeki64_nolock_internal 100174d8 f   libucrt:lseek.obj
 0001:00016500       _isdigit                   10017500 f   libucrt:_ctype.obj
 0001:00016590       _isspace                   10017590 f   libucrt:_ctype.obj
 0001:00016614       __initterm                 10017614 f   libucrt:initterm.obj
 0001:0001663f       __initterm_e               1001763f f   libucrt:initterm.obj
 0001:0001666d       __seh_filter_dll           1001766d f   libucrt:exception_filter.obj
 0001:0001668d       __seh_filter_exe           1001768d f   libucrt:exception_filter.obj
 0001:00016a84       ___acrt_allocate_buffer_for_argv 10017a84 f   libucrt:argv_parsing.obj
 0001:00016ad3       __configure_narrow_argv    10017ad3 f   libucrt:argv_parsing.obj
 0001:00016f4e       ___dcrt_get_or_create_narrow_environment_nolock 10017f4e f   libucrt:environment_initialization.obj
 0001:00016f53       ___dcrt_get_or_create_wide_environment_nolock 10017f53 f   libucrt:environment_initialization.obj
 0001:00016f58       ___dcrt_uninitialize_environments_nolock 10017f58 f   libucrt:environment_initialization.obj
 0001:00016fa9       __initialize_narrow_environment 10017fa9 f   libucrt:environment_initialization.obj
 0001:000170e3       __execute_onexit_table     100180e3 f   libucrt:onexit.obj
 0001:00017121       __initialize_onexit_table  10018121 f   libucrt:onexit.obj
 0001:00017171       ___acrt_uninitialize_command_line 10018171 f   libucrt:argv_data.obj
 0001:0001721a       ??$__crt_fast_encode_pointer@PAX@@YAPAXQAX@Z 1001821a f i libucrt:initialization.obj
 0001:00017267       ___acrt_initialize         10018267 f   libucrt:initialization.obj
 0001:00017279       ___acrt_thread_attach      10018279 f   libucrt:initialization.obj
 0001:00017284       ___acrt_thread_detach      10018284 f   libucrt:initialization.obj
 0001:0001728c       ___acrt_uninitialize       1001828c f   libucrt:initialization.obj
 0001:000172bc       ___acrt_uninitialize_critical 100182bc f   libucrt:initialization.obj
 0001:000172ce       _terminate                 100182ce f   libucrt:terminate.obj
 0001:0001730a       ___ascii_stricmp           1001830a f   libucrt:stricmp.obj
 0001:00017343       __stricmp                  10018343 f   libucrt:stricmp.obj
 0001:00017343       _stricmp                   10018343 f   libucrt:stricmp.obj
 0001:0001738c       __stricmp_l                1001838c f   libucrt:stricmp.obj
 0001:0001741c       __strnicmp                 1001841c f   libucrt:strnicmp.obj
 0001:0001741c       _strnicmp                  1001841c f   libucrt:strnicmp.obj
 0001:00017489       __strnicmp_l               10018489 f   libucrt:strnicmp.obj
 0001:00017554       __strdup                   10018554 f   libucrt:strdup.obj
 0001:00017554       _strdup                    10018554 f   libucrt:strdup.obj
 0001:00017639       __close                    10018639 f   libucrt:close.obj
 0001:00017639       _close                     10018639 f   libucrt:close.obj
 0001:00017669       __close_internal           10018669 f   libucrt:close.obj
 0001:0001770c       __close_nolock             1001870c f   libucrt:close.obj
 0001:0001773c       __close_nolock_internal    1001873c f   libucrt:close.obj
 0001:00017e97       __open                     10018e97 f   libucrt:open.obj
 0001:00017e97       _open                      10018e97 f   libucrt:open.obj
 0001:00017eaf       __sopen_nolock             10018eaf f   libucrt:open.obj
 0001:00017f1d       __sopen_s                  10018f1d f   libucrt:open.obj
 0001:00017f3d       __wsopen_nolock            10018f3d f   libucrt:open.obj
 0001:00018743       __read                     10019743 f   libucrt:read.obj
 0001:00018743       _read                      10019743 f   libucrt:read.obj
 0001:0001885c       __read_nolock              1001985c f   libucrt:read.obj
 0001:00018be7       _strcpy_s                  10019be7 f   libucrt:strcpy_s.obj
 0001:00018c41       _abort                     10019c41 f   libucrt:abort.obj
 0001:00018c85       ??$parse_integer@KV?$c_string_character_source@_W@__crt_strtox@@$00@__crt_strtox@@YAKAAV__crt_cached_ptd_host@@V?$c_string_character_source@_W@0@H_N@Z 10019c85 f i libucrt:atox.obj
 0001:00019293       ??$parse_integer@_KV?$c_string_character_source@D@__crt_strtox@@$00@__crt_strtox@@YA_KAAV__crt_cached_ptd_host@@V?$c_string_character_source@D@0@H_N@Z 1001a293 f i libucrt:atox.obj
 0001:0001955b       _calloc                    1001a55b f   libucrt:calloc.obj
 0001:00019566       _wcsncmp                   1001a566 f   libucrt:wcsncmp.obj
 0001:000195a0       ?check_synchronize_global_state_index@__crt_cached_ptd_host@@AAEIXZ 1001a5a0 f i libucrt:invalid_parameter.obj
 0001:000195c9       ___acrt_call_reportfault   1001a5c9 f   libucrt:invalid_parameter.obj
 0001:00019702       ___acrt_initialize_invalid_parameter_handler 1001a702 f   libucrt:invalid_parameter.obj
 0001:00019711       __invalid_parameter        1001a711 f   libucrt:invalid_parameter.obj
 0001:00019748       __invalid_parameter_internal 1001a748 f   libucrt:invalid_parameter.obj
 0001:000197c5       __invalid_parameter_noinfo 1001a7c5 f   libucrt:invalid_parameter.obj
 0001:000197d5       __invoke_watson            1001a7d5 f   libucrt:invalid_parameter.obj
 0001:00019809       __calloc_base              1001a809 f   libucrt:calloc_base.obj
 0001:00019866       __free_base                1001a866 f   libucrt:free_base.obj
 0001:00019a58       ___acrt_AppPolicyGetProcessTerminationMethodInternal@4 1001aa58 f   libucrt:winapi_thunks.obj
 0001:00019a98       ___acrt_AppPolicyGetThreadInitializationTypeInternal@4 1001aa98 f   libucrt:winapi_thunks.obj
 0001:00019ad8       ___acrt_AreFileApisANSI@0  1001aad8 f   libucrt:winapi_thunks.obj
 0001:00019af7       ___acrt_CompareStringEx@36 1001aaf7 f   libucrt:winapi_thunks.obj
 0001:00019b54       ___acrt_FlsAlloc@4         1001ab54 f   libucrt:winapi_thunks.obj
 0001:00019b93       ___acrt_FlsFree@4          1001ab93 f   libucrt:winapi_thunks.obj
 0001:00019bd2       ___acrt_FlsGetValue@4      1001abd2 f   libucrt:winapi_thunks.obj
 0001:00019c11       ___acrt_FlsSetValue@8      1001ac11 f   libucrt:winapi_thunks.obj
 0001:00019c53       ___acrt_InitializeCriticalSectionEx@12 1001ac53 f   libucrt:winapi_thunks.obj
 0001:00019c9e       ___acrt_LCMapStringEx@36   1001ac9e f   libucrt:winapi_thunks.obj
 0001:00019cfb       ___acrt_LocaleNameToLCID@8 1001acfb f   libucrt:winapi_thunks.obj
 0001:00019d2c       ___acrt_RoInitialize@4     1001ad2c f   libucrt:winapi_thunks.obj
 0001:00019d67       ___acrt_RoUninitialize@0   1001ad67 f   libucrt:winapi_thunks.obj
 0001:00019d95       ___acrt_initialize_winapi_thunks 1001ad95 f   libucrt:winapi_thunks.obj
 0001:00019da9       ___acrt_uninitialize_winapi_thunks 1001ada9 f   libucrt:winapi_thunks.obj
 0001:00019ddf       __fcloseall                1001addf f   libucrt:closeall.obj
 0001:00019e8a       ___acrt_stdio_free_buffer_nolock 1001ae8a f   libucrt:_freebuf.obj
 0001:0001a030       ___acrt_initialize_lowio   1001b030 f   libucrt:ioinit.obj
 0001:0001a090       ___acrt_uninitialize_lowio 1001b090 f   libucrt:ioinit.obj
 0001:0001a0bc       __fileno                   1001b0bc f   libucrt:fileno.obj
 0001:0001a0e3       ?__acrt_stdio_allocate_stream@@YA?AV__crt_stdio_stream@@XZ 1001b0e3 f   libucrt:stream.obj
 0001:0001a14c       ?__acrt_stdio_free_stream@@YAXV__crt_stdio_stream@@@Z 1001b14c f   libucrt:stream.obj
 0001:0001a587       ___acrt_freeptd            1001b587 f   libucrt:per_thread_data.obj
 0001:0001a5b3       ___acrt_getptd             1001b5b3 f   libucrt:per_thread_data.obj
 0001:0001a66e       ___acrt_getptd_head        1001b66e f   libucrt:per_thread_data.obj
 0001:0001a704       ___acrt_getptd_noexit      1001b704 f   libucrt:per_thread_data.obj
 0001:0001a7b5       ___acrt_getptd_noexit_explicit 1001b7b5 f   libucrt:per_thread_data.obj
 0001:0001a858       ___acrt_initialize_ptd     1001b858 f   libucrt:per_thread_data.obj
 0001:0001a884       ___acrt_uninitialize_ptd   1001b884 f   libucrt:per_thread_data.obj
 0001:0001a90c       ___acrt_set_locale_changed 1001b90c f   libucrt:wsetlocale.obj
 0001:0001a917       ___acrt_uninitialize_locale 1001b917 f   libucrt:wsetlocale.obj
 0001:0001a93e       __fgetc_nolock             1001b93e f   libucrt:fgetc.obj
 0001:0001a97a       __getc_nolock              1001b97a f   libucrt:fgetc.obj
 0001:0001a985       ??$__acrt_stdio_parse_mode@D@@YA?AU__acrt_stdio_stream_mode@@QBD@Z 1001b985 f i libucrt:openfile.obj
 0001:0001ac32       ?__acrt_stdio_parse_mode_D@@YA_NAAU__acrt_stdio_stream_mode@@@Z 1001bc32 f i libucrt:openfile.obj
 0001:0001ac4d       ?__acrt_stdio_parse_mode_T@@YA_NAAU__acrt_stdio_stream_mode@@@Z 1001bc4d f i libucrt:openfile.obj
 0001:0001ac6c       ?__acrt_stdio_parse_mode_b@@YA_NAAU__acrt_stdio_stream_mode@@@Z 1001bc6c f i libucrt:openfile.obj
 0001:0001ac8c       ?__acrt_stdio_parse_mode_c@@YA_NAAU__acrt_stdio_stream_mode@@AA_N@Z 1001bc8c f i libucrt:openfile.obj
 0001:0001acae       ?__acrt_stdio_parse_mode_n@@YA_NAAU__acrt_stdio_stream_mode@@AA_N@Z 1001bcae f i libucrt:openfile.obj
 0001:0001acd0       ?__acrt_stdio_parse_mode_plus@@YA_NAAU__acrt_stdio_stream_mode@@AA_N@Z 1001bcd0 f i libucrt:openfile.obj
 0001:0001ad06       ?__acrt_stdio_parse_mode_t@@YA_NAAU__acrt_stdio_stream_mode@@@Z 1001bd06 f i libucrt:openfile.obj
 0001:0001ad26       ?__acrt_stdio_parse_mode_x@@YA_NAAU__acrt_stdio_stream_mode@@@Z 1001bd26 f i libucrt:openfile.obj
 0001:0001ad46       __openfile                 1001bd46 f   libucrt:openfile.obj
 0001:0001ad51       __malloc_base              1001bd51 f   libucrt:malloc_base.obj
 0001:0001ad9f       _strnlen                   1001bd9f f   libucrt:strnlen.obj
 0001:0001aec1       _wcsnlen                   1001bec1 f   libucrt:strnlen.obj
 0001:0001b071       ___acrt_update_locale_info 1001c071 f   libucrt:locale_update.obj
 0001:0001b09e       ___acrt_update_locale_info_explicit 1001c09e f   libucrt:locale_update.obj
 0001:0001b0cf       ___acrt_update_multibyte_info 1001c0cf f   libucrt:locale_update.obj
 0001:0001b0fc       ___acrt_update_multibyte_info_explicit 1001c0fc f   libucrt:locale_update.obj
 0001:0001b12d       ?__acrt_fp_classify@@YA?AW4__acrt_fp_class@@ABN@Z 1001c12d f i libucrt:cvt.obj
 0001:0001bb05       ___acrt_fp_format          1001cb05 f   libucrt:cvt.obj
 0001:0001bc86       __wctomb_internal          1001cc86 f   libucrt:wctomb.obj
 0001:0001bdf0       __mbtowc_internal          1001cdf0 f   libucrt:mbtowc.obj
 0001:0001bf23       __mbtowc_l                 1001cf23 f   libucrt:mbtowc.obj
 0001:0001bf5b       __get_printf_count_output  1001cf5b f   libucrt:printf_count_output.obj
 0001:0001bf70       __fputc_nolock_internal    1001cf70 f   libucrt:fputc.obj
 0001:0001bf9d       ___acrt_should_use_temporary_buffer 1001cf9d f   libucrt:_sftbuf.obj
 0001:0001bfdb       ___acrt_stdio_begin_temporary_buffering_nolock 1001cfdb f   libucrt:_sftbuf.obj
 0001:0001c086       ___acrt_stdio_end_temporary_buffering_nolock 1001d086 f   libucrt:_sftbuf.obj
 0001:0001c0c4       ___pctype_func             1001d0c4 f   libucrt:ctype.obj
 0001:0001c0e8       _iswctype                  1001d0e8 f   libucrt:iswctype.obj
 0001:0001c151       __isctype_l                1001d151 f   libucrt:isctype.obj
 0001:0001c21c       _strtoull                  1001d21c f   libucrt:strtox.obj
 0001:0001c268       _wcstol                    1001d268 f   libucrt:strtox.obj
 0001:0001c2ae       _fegetround                1001d2ae f   libucrt:fegetround.obj
 0001:0001c2bb       ___acrt_initialize_locks   1001d2bb f   libucrt:locks.obj
 0001:0001c2fc       ___acrt_lock               1001d2fc f   libucrt:locks.obj
 0001:0001c313       ___acrt_uninitialize_locks 1001d313 f   libucrt:locks.obj
 0001:0001c344       ___acrt_unlock             1001d344 f   libucrt:locks.obj
 0001:0001c35b       ___acrt_app_verifier_enabled 1001d35b f   libucrt:peb_access.obj
 0001:0001c36d       ___acrt_is_secure_process  1001d36d f   libucrt:peb_access.obj
 0001:0001c380       ___acrt_get_begin_thread_init_policy 1001d380 f   libucrt:win_policies.obj
 0001:0001c3ba       ___acrt_get_process_end_policy 1001d3ba f   libucrt:win_policies.obj
 0001:0001c3e1       _wcscpy_s                  1001d3e1 f   libucrt:wcscpy_s.obj
 0001:0001c445       __wcsnicoll                1001d445 f   libucrt:wcsnicol.obj
 0001:0001c4b2       __wcsnicoll_l              1001d4b2 f   libucrt:wcsnicol.obj
 0001:0001c572       __strnicoll                1001d572 f   libucrt:strnicol.obj
 0001:0001c59b       __strnicoll_l              1001d59b f   libucrt:strnicol.obj
 0001:0001c6fb       ___acrt_MultiByteToWideChar 1001d6fb f   libucrt:multibytetowidechar.obj
 0001:0001c7b5       ___acrt_WideCharToMultiByte 1001d7b5 f   libucrt:widechartomultibyte.obj
 0001:0001cf5b       ___dcrt_set_variable_in_narrow_environment_nolock 1001df5b f   libucrt:setenv.obj
 0001:0001cf66       ___dcrt_set_variable_in_wide_environment_nolock 1001df66 f   libucrt:setenv.obj
 0001:0001cf71       ___sys_errlist             1001df71 f   libucrt:syserr.obj
 0001:0001cf77       ___sys_nerr                1001df77 f   libucrt:syserr.obj
 0001:0001d034       _strncpy_s                 1001e034 f   libucrt:strncpy_s.obj
 0001:0001d03f       __waccess_s                1001e03f f   libucrt:waccess.obj
 0001:0001d19f       __commit                   1001e19f f   libucrt:commit.obj
 0001:0001d9be       __write                    1001e9be f   libucrt:write.obj
 0001:0001d9f5       __write_internal           1001e9f5 f   libucrt:write.obj
 0001:0001db06       __write_nolock             1001eb06 f   libucrt:write.obj
 0001:0001dd4d       __getdrive                 1001ed4d f   libucrt:drive.obj
 0001:0001ddf1       ??$__acrt_convert_wcs_mbs_cp@_WDV<lambda_0fec1a7b3f42a53036604e18c2d5e07e>@@U__crt_win32_buffer_no_resizing@@@@YAHQB_WAAV?$__crt_win32_buffer@DU__crt_win32_buffer_no_resizing@@@@ABV<lambda_0fec1a7b3f42a53036604e18c2d5e07e>@@I@Z 1001edf1 f i libucrt:fullpath.obj
 0001:0001deb3       ??$__acrt_get_full_path_name_wide@U__crt_win32_buffer_no_resizing@@@@YAHQB_WAAV?$__crt_win32_buffer@_WU__crt_win32_buffer_no_resizing@@@@@Z 1001eeb3 f i libucrt:fullpath.obj
 0001:0001decd       ??$__acrt_get_full_path_name_wide@U__crt_win32_buffer_public_dynamic_resizing@@@@YAHQB_WAAV?$__crt_win32_buffer@_WU__crt_win32_buffer_public_dynamic_resizing@@@@@Z 1001eecd f i libucrt:fullpath.obj
 0001:0001dee7       ??$call_win32_function@V<lambda_0d87af4cf61654f651d26e3c6a4f13fc>@@@?$__crt_win32_buffer@_WU__crt_win32_buffer_public_dynamic_resizing@@@@QAEHABV<lambda_0d87af4cf61654f651d26e3c6a4f13fc>@@@Z 1001eee7 f i libucrt:fullpath.obj
 0001:0001df4d       ??$call_win32_function@V<lambda_33d632c04396b3de813369f94278cf6d>@@@?$__crt_win32_buffer@_WU__crt_win32_buffer_no_resizing@@@@QAEHABV<lambda_33d632c04396b3de813369f94278cf6d>@@@Z 1001ef4d f i libucrt:fullpath.obj
 0001:0001e04b       ??R<lambda_0fec1a7b3f42a53036604e18c2d5e07e>@@QBE@IQB_WQADI@Z 1001f04b f i libucrt:fullpath.obj
 0001:0001e04b       ??R<lambda_28bda7af82a03b66c1cb3803a755f95d>@@QBE@IQB_WQADI@Z 1001f04b f i libucrt:argv_wildcards.obj
 0001:0001e06f       ?_deallocate@?$__crt_win32_buffer@_WU__crt_win32_buffer_public_dynamic_resizing@@@@AAEXXZ 1001f06f f i libucrt:fullpath.obj
 0001:0001e089       ?allocate@?$__crt_win32_buffer@DU__crt_win32_buffer_no_resizing@@@@QAEHI@Z 1001f089 f i libucrt:fullpath.obj
 0001:0001e089       ?allocate@?$__crt_win32_buffer@_WU__crt_win32_buffer_no_resizing@@@@QAEHI@Z 1001f089 f i libucrt:fullpath.obj
 0001:0001e0b0       ?allocate@?$__crt_win32_buffer@_WU__crt_win32_buffer_public_dynamic_resizing@@@@QAEHI@Z 1001f0b0 f i libucrt:fullpath.obj
 0001:0001e0ef       ?allocate@__crt_win32_buffer_public_dynamic_resizing@@SAHQAPAXIABV__crt_win32_buffer_debug_info@@@Z 1001f0ef f i libucrt:fullpath.obj
 0001:0001e10e       ?detach@?$__crt_win32_buffer@_WU__crt_win32_buffer_public_dynamic_resizing@@@@QAEPA_WXZ 1001f10e f i libucrt:fullpath.obj
 0001:0001e15c       ?set_to_nullptr@?$__crt_win32_buffer@DU__crt_win32_buffer_no_resizing@@@@QAEXXZ 1001f15c f i libucrt:fullpath.obj
 0001:0001e170       __wfullpath                1001f170 f   libucrt:fullpath.obj
 0001:0001e18e       _wcspbrk                   1001f18e f   libucrt:wcspbrk.obj
 0001:0001e1dc       ___ascii_wcsicmp           1001f1dc f   libucrt:wcsicmp.obj
 0001:0001e219       __towlower_internal        1001f219 f i libucrt:wcsicmp.obj
 0001:0001e258       __wcsicmp                  1001f258 f   libucrt:wcsicmp.obj
 0001:0001e2a1       __wcsicmp_l                1001f2a1 f   libucrt:wcsicmp.obj
 0001:0001e359       ___acrt_lowio_create_handle_array 1001f359 f   libucrt:osfinfo.obj
 0001:0001e3d4       ___acrt_lowio_destroy_handle_array 1001f3d4 f   libucrt:osfinfo.obj
 0001:0001e409       ___acrt_lowio_ensure_fh_exists 1001f409 f   libucrt:osfinfo.obj
 0001:0001e4a7       ___acrt_lowio_lock_fh      1001f4a7 f   libucrt:osfinfo.obj
 0001:0001e4ca       ___acrt_lowio_set_os_handle 1001f4ca f   libucrt:osfinfo.obj
 0001:0001e55c       ___acrt_lowio_unlock_fh    1001f55c f   libucrt:osfinfo.obj
 0001:0001e57f       __alloc_osfhnd             1001f57f f   libucrt:osfinfo.obj
 0001:0001e692       __free_osfhnd              1001f692 f   libucrt:osfinfo.obj
 0001:0001e723       __get_osfhandle            1001f723 f   libucrt:osfinfo.obj
 0001:0001e78d       ??$__crt_time_elapsed_leap_years@H@@YAHH@Z 1001f78d f i libucrt:loctotime.obj
 0001:0001e7c7       ??$__crt_time_is_leap_year@H@@YA_NH@Z 1001f7c7 f i libucrt:loctotime.obj
 0001:0001e9d9       ?__crt_time_is_day_valid@@YA_NHHH@Z 1001f9d9 f i libucrt:loctotime.obj
 0001:0001ea1f       ___loctotime64_t           1001fa1f f   libucrt:loctotime.obj
 0001:0001ea2a       __realloc_base             1001fa2a f   libucrt:realloc_base.obj
 0001:0001eaab       ??$__acrt_convert_wcs_mbs_cp@_WDV<lambda_28bda7af82a03b66c1cb3803a755f95d>@@U__crt_win32_buffer_internal_dynamic_resizing@@@@YAHQB_WAAV?$__crt_win32_buffer@DU__crt_win32_buffer_internal_dynamic_resizing@@@@ABV<lambda_28bda7af82a03b66c1cb3803a755f95d>@@I@Z 1001faab f i libucrt:argv_wildcards.obj
 0001:0001f049       ?allocate@?$__crt_win32_buffer@DU__crt_win32_buffer_internal_dynamic_resizing@@@@QAEHI@Z 10020049 f i libucrt:argv_wildcards.obj
 0001:0001f10c       ___acrt_expand_narrow_argv_wildcards 1002010c f   libucrt:argv_wildcards.obj
 0001:0001f117       ___acrt_GetModuleFileNameA 10020117 f   libucrt:getmodulefilenamea.obj
 0001:0001f734       ___acrt_initialize_multibyte 10020734 f   libucrt:mbctype.obj
 0001:0001f77c       ___acrt_update_thread_multibyte_data 1002077c f   libucrt:mbctype.obj
 0001:0001f78f       __setmbcp_nolock           1002078f f   libucrt:mbctype.obj
 0001:0001f9e4       __ismbblead                100209e4 f   libucrt:ismbbyte.obj
 0001:0001f9fc       ___acrt_initialize_command_line 100209fc f   libucrt:argv_data.obj
 0001:0001fa4c       ___dcrt_get_narrow_environment_from_os 10020a4c f   libucrt:get_environment_from_os.obj
 0001:0001faec       ___dcrt_get_wide_environment_from_os 10020aec f   libucrt:get_environment_from_os.obj
 0001:0001fb3a       __recalloc_base            10020b3a f   libucrt:recalloc.obj
 0001:0001fba7       ___acrt_initialize_heap    10020ba7 f   libucrt:heap_handle.obj
 0001:0001fbb8       ___acrt_uninitialize_heap  10020bb8 f   libucrt:heap_handle.obj
 0001:0001fbc2       ___acrt_execute_initializers 10020bc2 f   libucrt:shared_initialization.obj
 0001:0001fc2a       ___acrt_execute_uninitializers 10020c2a f   libucrt:shared_initialization.obj
 0001:0001fc5b       ___acrt_initialize_new_handler 10020c5b f   libucrt:new_handler.obj
 0001:0001fc6a       __callnewh                 10020c6a f   libucrt:new_handler.obj
 0001:0001fc96       __query_new_handler        10020c96 f   libucrt:new_handler.obj
 0001:0001fdbf       ___acrt_get_sigabrt_handler 10020dbf f   libucrt:signal.obj
 0001:0001fde6       ___acrt_initialize_signal_handlers 10020de6 f   libucrt:signal.obj
 0001:0001fe04       _raise                     10020e04 f   libucrt:signal.obj
 0001:0001fff8       ___acrt_has_user_matherr   10020ff8 f   libucrt:matherr.obj
 0001:00020015       ___acrt_initialize_user_matherr 10021015 f   libucrt:matherr.obj
 0001:00020024       ___acrt_invoke_user_matherr 10021024 f   libucrt:matherr.obj
 0001:00020060       ___ascii_strnicmp          10021060 f   libucrt:_strnicm.obj
 0001:000200c1       __get_fmode                100210c1 f   libucrt:setmode.obj
 0001:000200ee       __setmode_nolock           100210ee f   libucrt:setmode.obj
 0001:000201bd       ??0__crt_seek_guard@@QAE@H_J@Z 100211bd f i libucrt:chsize.obj
 0001:0002020a       __chsize_nolock            1002120a f   libucrt:chsize.obj
 0001:00020241       __chsize_nolock_internal   10021241 f   libucrt:chsize.obj
 0001:000203d8       __isatty                   100213d8 f   libucrt:isatty.obj
 0001:0002042e       __query_new_mode           1002142e f   libucrt:new_mode.obj
 0001:00020485       ___acrt_DownlevelLocaleNameToLCID 10021485 f   libucrt:lcidtoname_downlevel.obj
 0001:000204b1       ___acrt_add_locale_ref     100214b1 f   libucrt:locale_refcounting.obj
 0001:0002052e       ___acrt_free_locale        1002152e f   libucrt:locale_refcounting.obj
 0001:00020676       ___acrt_locale_add_lc_time_reference 10021676 f   libucrt:locale_refcounting.obj
 0001:0002069f       ___acrt_locale_free_lc_time_if_unreferenced 1002169f f   libucrt:locale_refcounting.obj
 0001:000206d0       ___acrt_locale_release_lc_time_reference 100216d0 f   libucrt:locale_refcounting.obj
 0001:000206f9       ___acrt_release_locale_ref 100216f9 f   libucrt:locale_refcounting.obj
 0001:0002077a       ___acrt_update_thread_locale_data 1002177a f   libucrt:locale_refcounting.obj
 0001:000207fb       __updatetlocinfoEx_nolock  100217fb f   libucrt:locale_refcounting.obj
 0001:0002084b       ____lc_codepage_func       1002184b f   libucrt:initctype.obj
 0001:00020870       ___acrt_locale_free_monetary 10021870 f   libucrt:initmon.obj
 0001:0002096e       ___acrt_locale_free_numeric 1002196e f   libucrt:initnum.obj
 0001:000209fc       ___acrt_locale_free_time   100219fc f   libucrt:inittime.obj
 0001:00020bae       _wcsncpy_s                 10021bae f   libucrt:wcsncpy_s.obj
 0001:00020bb9       ___acrt_GetStringTypeA     10021bb9 f   libucrt:getstringtypea.obj
 0001:00020cba       __freea_crt                10021cba f i libucrt:getstringtypea.obj
 0001:00020e69       ___acrt_stdio_refill_and_read_narrow_nolock 10021e69 f   libucrt:_filbuf.obj
 0001:00020e74       ___ascii_wcsnicmp          10021e74 f   libucrt:wcsnicmp.obj
 0001:00020f74       ___acrt_fp_strflt_to_string 10021f74 f   libucrt:_fptostr.obj
 0001:0002106e       ___acrt_fltout             1002206e f   libucrt:cfout.obj
 0001:00022656       ?__c32rtomb_utf8@__crt_mbstring@@YAIPAD_UPAU_Mbstatet@@AAV__crt_cached_ptd_host@@@Z 10023656 f   libucrt:c32rtomb.obj
 0001:00022732       ?__mbrtowc_utf8@__crt_mbstring@@YAIPA_WPBDIPAU_Mbstatet@@AAV__crt_cached_ptd_host@@@Z 10023732 f   libucrt:mbrtowc.obj
 0001:00022775       ?__mbsrtowcs_utf8@__crt_mbstring@@YAIPA_WPAPBDIPAU_Mbstatet@@AAV__crt_cached_ptd_host@@@Z 10023775 f   libucrt:mbrtowc.obj
 0001:00022aca       ___acrt_stdio_flush_and_write_narrow_nolock 10023aca f   libucrt:_flsbuf.obj
 0001:00022ad5       ___acrt_GetStringTypeW     10023ad5 f   libucrt:getstringtypew.obj
 0001:00022aee       ___acrt_stdio_allocate_buffer_nolock 10023aee f   libucrt:_getbuf.obj
 0001:00022e13       ___acrt_fenv_get_common_round_control 10023e13 f   libucrt:_fenvutils.obj
 0001:00022e35       ___acrt_fenv_get_control   10023e35 f   libucrt:_fenvutils.obj
 0001:00022eb5       ___acrt_fenv_get_status    10023eb5 f   libucrt:_fenvutils.obj
 0001:00022f5f       ___acrt_fenv_set_control   10023f5f f   libucrt:_fenvutils.obj
 0001:00022fda       ___acrt_fenv_set_status    10023fda f   libucrt:_fenvutils.obj
 0001:000230d6       ___acrt_CompareStringW     100240d6 f   libucrt:comparestringw.obj
 0001:000233da       ___acrt_CompareStringA     100243da f   libucrt:comparestringa.obj
 0001:00023420       ___acrt_SetEnvironmentVariableA 10024420 f   libucrt:setenvironmentvariablea.obj
 0001:000234b5       __putwch_nolock            100244b5 f   libucrt:putwch.obj
 0001:000236ba       __wgetcwd                  100246ba f   libucrt:getcwd.obj
 0001:000236d6       __towlower_l               100246d6 f   libucrt:towlower.obj
 0001:000237aa       __query_app_type           100247aa f   libucrt:report_runtime_error.obj
 0001:000237b0       ___acrt_initialize_timeset 100247b0 f   libucrt:timeset.obj
 0001:000237e5       ___daylight                100247e5 f   libucrt:timeset.obj
 0001:000237eb       ___dstbias                 100247eb f   libucrt:timeset.obj
 0001:000237f1       ___timezone                100247f1 f   libucrt:timeset.obj
 0001:000237f7       ___tzname                  100247f7 f   libucrt:timeset.obj
 0001:000237fd       ___wide_tzname             100247fd f   libucrt:timeset.obj
 0001:00023803       __get_daylight             10024803 f   libucrt:timeset.obj
 0001:0002382f       __get_dstbias              1002482f f   libucrt:timeset.obj
 0001:0002385b       __get_timezone             1002485b f   libucrt:timeset.obj
 0001:00024146       ___tzset                   10025146 f   libucrt:tzset.obj
 0001:000241a3       __isindst                  100251a3 f   libucrt:tzset.obj
 0001:00024200       _qsort                     10025200 f   libucrt:qsort.obj
 0001:000246ee       __mbsdec                   100256ee f   libucrt:mbsdec.obj
 0001:00024705       __mbsdec_l                 10025705 f   libucrt:mbsdec.obj
 0001:00024981       ___acrt_LCMapStringA       10025981 f   libucrt:lcmapstringa.obj
 0001:000249d9       __msize_base               100259d9 f   libucrt:msize.obj
 0001:00024a0c       ___acrt_initialize_fmode   10025a0c f   libucrt:txtmode.obj
 0001:00024a22       __controlfp_s              10025a22 f   libucrt:contrlfp.obj
 0001:00024a81       _fegetenv                  10025a81 f   libucrt:fegetenv.obj
 0001:00024a9e       _fesetenv                  10025a9e f   libucrt:fesetenv.obj
 0001:00024aea       _feholdexcept              10025aea f   libucrt:feholdexcept.obj
 0001:00024b40       __CIlog10                  10025b40 f   libucrt:log10_impl.obj
 0001:00024b7b       __CIlog10_default          10025b7b f   libucrt:log10_impl.obj
 0001:00024b8f       __log10_default            10025b8f     libucrt:log10_impl.obj
 0001:00024c50       _ceil                      10025c50 f   libucrt:ceil_pentium4.obj
 0001:00024c90       __ceil_pentium4            10025c90 f   libucrt:ceil_pentium4.obj
 0001:00024d6d       ?reset_and_return@__crt_mbstring@@YAIIPAU_Mbstatet@@@Z 10025d6d f   libucrt:common_utf8.obj
 0001:00024d81       ?return_illegal_sequence@__crt_mbstring@@YAIPAU_Mbstatet@@AAV__crt_cached_ptd_host@@@Z 10025d81 f   libucrt:common_utf8.obj
 0001:00024da3       ?__mbrtoc32_utf8@__crt_mbstring@@YAIPA_UPBDIPAU_Mbstatet@@AAV__crt_cached_ptd_host@@@Z 10025da3 f   libucrt:mbrtoc32.obj
 0001:00024f54       ___strncnt                 10025f54 f   libucrt:strncnt.obj
 0001:00024f8f       ___dcrt_lowio_ensure_console_output_initialized 10025f8f f   libucrt:initcon.obj
 0001:00024fae       ___dcrt_terminate_console_output 10025fae f   libucrt:initcon.obj
 0001:00024fc5       ___dcrt_write_console      10025fc5 f   libucrt:initcon.obj
 0001:0002501a       ___acrt_LCMapStringW       1002601a f   libucrt:lcmapstringw.obj
 0001:000250ff       __clearfp                  100260ff f   libucrt:ieee87.obj
 0001:000251dd       __control87                100261dd f   libucrt:ieee87.obj
 0001:0002557c       ___acrt_initialize_sse2    1002657c f   libucrt:mathfcns.obj
 0001:00025590       __CIlog10_pentium4         10026590 f   libucrt:log10_pentium4.obj
 0001:000255a8       __log10_pentium4           100265a8     libucrt:log10_pentium4.obj
 0001:00025840       __fFEXP                    10026840 f   libucrt:87tran.obj
 0001:00025897       __rtinfpopse               10026897     libucrt:87tran.obj
 0001:00025899       __rtinfnpopse              10026899     libucrt:87tran.obj
 0001:000258a9       __fFLN                     100268a9     libucrt:87tran.obj
 0001:0002595e       __rtinfpop                 1002695e     libucrt:87tran.obj
 0001:00025960       __rtinfnpop                10026960     libucrt:87tran.obj
 0001:00025970       __rtforexpinf              10026970 f   libucrt:87tran.obj
 0001:0002597d       __ffexpm1                  1002697d     libucrt:87tran.obj
 0001:00025a30       __trandisp1                10026a30 f   libucrt:87disp.obj
 0001:00025aa5       __trandisp2                10026aa5 f   libucrt:87disp.obj
 0001:00025b3f       __rttospopde               10026b3f     libucrt:87disp.obj
 0001:00025b44       __rttospop                 10026b44     libucrt:87disp.obj
 0001:00025b50       __rtnospop                 10026b50 f   libucrt:87disp.obj
 0001:00025b60       __rttosnpop                10026b60 f   libucrt:87disp.obj
 0001:00025b61       __rtnospopde               10026b61     libucrt:87disp.obj
 0001:00025b68       __rtzeropop                10026b68     libucrt:87disp.obj
 0001:00025b6a       __rtzeronpop               10026b6a     libucrt:87disp.obj
 0001:00025b70       __rtzerospop               10026b70 f   libucrt:87disp.obj
 0001:00025b7d       __rtonepop                 10026b7d     libucrt:87disp.obj
 0001:00025b80       __rtonenpop                10026b80 f   libucrt:87disp.obj
 0001:00025b90       __tosnan1                  10026b90 f   libucrt:87disp.obj
 0001:00025bc0       __nosnan2                  10026bc0 f   libucrt:87disp.obj
 0001:00025bd0       __tosnan2                  10026bd0 f   libucrt:87disp.obj
 0001:00025c00       __nan2                     10026c00 f   libucrt:87disp.obj
 0001:00025c40       __rtindfpop                10026c40 f   libucrt:87disp.obj
 0001:00025c42       __rtindfnpop               10026c42     libucrt:87disp.obj
 0001:00025c53       __rttosnpopde              10026c53     libucrt:87disp.obj
 0001:00025c60       __rtatan2inf               10026c60 f   libucrt:87disp.obj
 0001:00025c7d       __rtchsifneg               10026c7d     libucrt:87disp.obj
 0001:00025c90       __twoToTOS                 10026c90 f   libucrt:common.obj
 0001:00025ca5       __load_CW                  10026ca5 f   libucrt:common.obj
 0001:00025cbc       __convertTOStoQNaN         10026cbc f   libucrt:common.obj
 0001:00025cd5       __fload_withFB             10026cd5 f   libucrt:common.obj
 0001:00025d18       __checkTOS_withFB          10026d18 f   libucrt:common.obj
 0001:00025d2e       __fast_exit                10026d2e f   libucrt:common.obj
 0001:00025d3b       __math_exit                10026d3b f   libucrt:common.obj
 0001:00025d65       __check_overflow_exit      10026d65 f   libucrt:common.obj
 0001:00025d79       __check_range_exit         10026d79 f   libucrt:common.obj
 0001:00025e20       __startTwoArgErrorHandling 10026e20 f   libucrt:genexcep.obj
 0001:00025e37       __startOneArgErrorHandling 10026e37 f   libucrt:genexcep.obj
 0001:00025e73       ___libm_error_support      10026e73 f   libucrt:libm_error.obj
 0001:00026067       __ceil_default             10027067 f   libucrt:ceil.obj
 0001:00026125       ___set_fpsr_sse2           10027125 f   libucrt:fpctrl.obj
 0001:000261a5       __clrfp                    100271a5 f   libucrt:fpctrl.obj
 0001:000261b6       __ctrlfp                   100271b6 f   libucrt:fpctrl.obj
 0001:000261e0       __set_statfp               100271e0 f   libucrt:fpctrl.obj
 0001:00026239       __statfp                   10027239 f   libucrt:fpctrl.obj
 0001:00026249       __d_inttype                10027249 f   libucrt:powhlp.obj
 0001:000262b1       __powhlp                   100272b1 f   libucrt:powhlp.obj
 0001:000263dc       __87except                 100273dc f   libucrt:87except.obj
 0001:000264ec       __frnd                     100274ec f   libucrt:frnd.obj
 0001:00026500       __errcode                  10027500 f   libucrt:fpexcept.obj
 0001:00026534       __except1                  10027534 f   libucrt:fpexcept.obj
 0001:00026602       __handle_exc               10027602 f   libucrt:fpexcept.obj
 0001:00026882       __raise_exc                10027882 f   libucrt:fpexcept.obj
 0001:000268a5       __raise_exc_ex             100278a5 f   libucrt:fpexcept.obj
 0001:00026b96       __set_errno_from_matherr   10027b96 f   libucrt:fpexcept.obj
 0001:00026bc7       __umatherr                 10027bc7 f   libucrt:fpexcept.obj
 0001:00026c67       __decomp                   10027c67 f   libucrt:util.obj
 0001:00026d39       __set_exp                  10027d39 f   libucrt:util.obj
 0001:00026d66       __sptype                   10027d66 f   libucrt:util.obj
 0001:00026dc9       __fpclass                  10027dc9 f   libucrt:ieeemisc.obj
 0001:00026e70       __FindPESection            10027e70 f   LIBCMT:pesect.obj
 0001:00026ec0       __IsNonwritableInCurrentImage 10027ec0 f   LIBCMT:pesect.obj
 0001:00026f80       __ValidateImageBase        10027f80 f   LIBCMT:pesect.obj
 0001:00026fb1       ??_Etype_info@@UAEPAXI@Z   10027fb1 f i LIBCMT:std_type_info_static.obj
 0001:00026fb1       ??_Gtype_info@@UAEPAXI@Z   10027fb1 f i LIBCMT:std_type_info_static.obj
 0001:00026fd4       __EH_epilog3               10027fd4 f   LIBCMT:ehprolg3.obj
 0001:00026fe8       __EH_prolog3               10027fe8 f   LIBCMT:ehprolg3.obj
 0001:0002701b       __EH_prolog3_catch         1002801b f   LIBCMT:ehprolg3.obj
 0001:00027060       ??3@YAXPAXI@Z              10028060 f   LIBCMT:delete_scalar_size.obj
 0001:00027070       __aulldiv                  10028070 f   LIBCMT:ulldiv.obj
 0001:000270e0       __aullrem                  100280e0 f   LIBCMT:ullrem.obj
 0001:00027160       __allshl                   10028160 f   LIBCMT:llshl.obj
 0001:00027180       __aullshr                  10028180 f   LIBCMT:ullshr.obj
 0001:000271a0       __alloca_probe             100281a0 f   LIBCMT:chkstk.obj
 0001:000271a0       __chkstk                   100281a0 f   LIBCMT:chkstk.obj
 0001:000271d0       __alloca_probe_16          100281d0 f   LIBCMT:alloca16.obj
 0001:000271e6       __alloca_probe_8           100281e6     LIBCMT:alloca16.obj
 0001:00027200       __ftol2_sse                10028200 f   LIBCMT:ftol2.obj
 0001:00027210       __ftoi2                    10028210 f   LIBCMT:ftol2.obj
 0001:0002728c       _wcschr                    1002828c f   libvcruntime:wcschr.obj
 0001:0002733c       _wcsrchr                   1002833c f   libvcruntime:wcsrchr.obj
 0001:000273dd       __filter_x86_sse2_floating_point_exception 100283dd f   LIBCMT:x86_exception_filter.obj
 0001:000273dd       __filter_x86_sse2_floating_point_exception_default 100283dd f   LIBCMT:x86_exception_filter.obj
 0002:00000000       __imp__RegEnumKeyA@16      10029000     advapi32:ADVAPI32.dll
 0002:00000004       __imp__RegOpenKeyExA@20    10029004     advapi32:ADVAPI32.dll
 0002:00000008       __imp__RegQueryValueExA@24 10029008     advapi32:ADVAPI32.dll
 0002:0000000c       __imp__RegCloseKey@4       1002900c     advapi32:ADVAPI32.dll
 0002:00000010       \177ADVAPI32_NULL_THUNK_DATA 10029010     advapi32:ADVAPI32.dll
 0002:00000014       __imp__InitCommonControlsEx@4 10029014     comctl32:COMCTL32.dll
 0002:00000018       \177COMCTL32_NULL_THUNK_DATA 10029018     comctl32:COMCTL32.dll
 0002:0000001c       __imp__WriteConsoleW@20    1002901c     kernel32:KERNEL32.dll
 0002:00000020       __imp__HeapSize@12         10029020     kernel32:KERNEL32.dll
 0002:00000024       __imp__GetCommandLineA@0   10029024     kernel32:KERNEL32.dll
 0002:00000028       __imp__CloseHandle@4       10029028     kernel32:KERNEL32.dll
 0002:0000002c       __imp__GetLastError@0      1002902c     kernel32:KERNEL32.dll
 0002:00000030       __imp__QueryPerformanceCounter@4 10029030     kernel32:KERNEL32.dll
 0002:00000034       __imp__QueryPerformanceFrequency@4 10029034     kernel32:KERNEL32.dll
 0002:00000038       __imp__WaitForSingleObject@8 10029038     kernel32:KERNEL32.dll
 0002:0000003c       __imp__GetExitCodeProcess@8 1002903c     kernel32:KERNEL32.dll
 0002:00000040       __imp__GetExitCodeThread@8 10029040     kernel32:KERNEL32.dll
 0002:00000044       __imp__CreateProcessA@40   10029044     kernel32:KERNEL32.dll
 0002:00000048       __imp__FreeLibrary@4       10029048     kernel32:KERNEL32.dll
 0002:0000004c       __imp__GetModuleFileNameA@12 1002904c     kernel32:KERNEL32.dll
 0002:00000050       __imp__GetModuleHandleA@4  10029050     kernel32:KERNEL32.dll
 0002:00000054       __imp__GetProcAddress@8    10029054     kernel32:KERNEL32.dll
 0002:00000058       __imp__LoadLibraryA@4      10029058     kernel32:KERNEL32.dll
 0002:0000005c       __imp__LocalFree@4         1002905c     kernel32:KERNEL32.dll
 0002:00000060       __imp__FormatMessageA@28   10029060     kernel32:KERNEL32.dll
 0002:00000064       __imp__FindClose@4         10029064     kernel32:KERNEL32.dll
 0002:00000068       __imp__FindFirstFileA@8    10029068     kernel32:KERNEL32.dll
 0002:0000006c       __imp__FindNextFileA@8     1002906c     kernel32:KERNEL32.dll
 0002:00000070       __imp__UnhandledExceptionFilter@4 10029070     kernel32:KERNEL32.dll
 0002:00000074       __imp__SetUnhandledExceptionFilter@4 10029074     kernel32:KERNEL32.dll
 0002:00000078       __imp__GetCurrentProcess@0 10029078     kernel32:KERNEL32.dll
 0002:0000007c       __imp__TerminateProcess@8  1002907c     kernel32:KERNEL32.dll
 0002:00000080       __imp__IsProcessorFeaturePresent@4 10029080     kernel32:KERNEL32.dll
 0002:00000084       __imp__GetCurrentProcessId@0 10029084     kernel32:KERNEL32.dll
 0002:00000088       __imp__GetCurrentThreadId@0 10029088     kernel32:KERNEL32.dll
 0002:0000008c       __imp__GetSystemTimeAsFileTime@4 1002908c     kernel32:KERNEL32.dll
 0002:00000090       __imp__InitializeSListHead@4 10029090     kernel32:KERNEL32.dll
 0002:00000094       __imp__IsDebuggerPresent@0 10029094     kernel32:KERNEL32.dll
 0002:00000098       __imp__GetStartupInfoW@4   10029098     kernel32:KERNEL32.dll
 0002:0000009c       __imp__GetModuleHandleW@4  1002909c     kernel32:KERNEL32.dll
 0002:000000a0       __imp__GetTimeZoneInformation@4 100290a0     kernel32:KERNEL32.dll
 0002:000000a4       __imp__InterlockedFlushSList@4 100290a4     kernel32:KERNEL32.dll
 0002:000000a8       __imp__RtlUnwind@16        100290a8     kernel32:KERNEL32.dll
 0002:000000ac       __imp__SetLastError@4      100290ac     kernel32:KERNEL32.dll
 0002:000000b0       __imp__EnterCriticalSection@4 100290b0     kernel32:KERNEL32.dll
 0002:000000b4       __imp__LeaveCriticalSection@4 100290b4     kernel32:KERNEL32.dll
 0002:000000b8       __imp__DeleteCriticalSection@4 100290b8     kernel32:KERNEL32.dll
 0002:000000bc       __imp__InitializeCriticalSectionAndSpinCount@8 100290bc     kernel32:KERNEL32.dll
 0002:000000c0       __imp__TlsAlloc@0          100290c0     kernel32:KERNEL32.dll
 0002:000000c4       __imp__TlsGetValue@4       100290c4     kernel32:KERNEL32.dll
 0002:000000c8       __imp__TlsSetValue@8       100290c8     kernel32:KERNEL32.dll
 0002:000000cc       __imp__TlsFree@4           100290cc     kernel32:KERNEL32.dll
 0002:000000d0       __imp__LoadLibraryExW@12   100290d0     kernel32:KERNEL32.dll
 0002:000000d4       __imp__EncodePointer@4     100290d4     kernel32:KERNEL32.dll
 0002:000000d8       __imp__RaiseException@16   100290d8     kernel32:KERNEL32.dll
 0002:000000dc       __imp__ExitProcess@4       100290dc     kernel32:KERNEL32.dll
 0002:000000e0       __imp__GetModuleHandleExW@12 100290e0     kernel32:KERNEL32.dll
 0002:000000e4       __imp__CreateThread@24     100290e4     kernel32:KERNEL32.dll
 0002:000000e8       __imp__ExitThread@4        100290e8     kernel32:KERNEL32.dll
 0002:000000ec       __imp__FreeLibraryAndExitThread@8 100290ec     kernel32:KERNEL32.dll
 0002:000000f0       __imp__CreateFileW@28      100290f0     kernel32:KERNEL32.dll
 0002:000000f4       __imp__GetDriveTypeW@4     100290f4     kernel32:KERNEL32.dll
 0002:000000f8       __imp__GetFileInformationByHandle@8 100290f8     kernel32:KERNEL32.dll
 0002:000000fc       __imp__GetFileType@4       100290fc     kernel32:KERNEL32.dll
 0002:00000100       __imp__PeekNamedPipe@24    10029100     kernel32:KERNEL32.dll
 0002:00000104       __imp__SystemTimeToTzSpecificLocalTime@12 10029104     kernel32:KERNEL32.dll
 0002:00000108       __imp__FileTimeToSystemTime@8 10029108     kernel32:KERNEL32.dll
 0002:0000010c       __imp__SetFilePointerEx@20 1002910c     kernel32:KERNEL32.dll
 0002:00000110       __imp__GetModuleFileNameW@12 10029110     kernel32:KERNEL32.dll
 0002:00000114       __imp__ReadFile@20         10029114     kernel32:KERNEL32.dll
 0002:00000118       __imp__GetConsoleMode@8    10029118     kernel32:KERNEL32.dll
 0002:0000011c       __imp__ReadConsoleW@20     1002911c     kernel32:KERNEL32.dll
 0002:00000120       __imp__HeapAlloc@12        10029120     kernel32:KERNEL32.dll
 0002:00000124       __imp__HeapFree@12         10029124     kernel32:KERNEL32.dll
 0002:00000128       __imp__CompareStringW@24   10029128     kernel32:KERNEL32.dll
 0002:0000012c       __imp__LCMapStringW@24     1002912c     kernel32:KERNEL32.dll
 0002:00000130       __imp__GetStdHandle@4      10029130     kernel32:KERNEL32.dll
 0002:00000134       __imp__MultiByteToWideChar@24 10029134     kernel32:KERNEL32.dll
 0002:00000138       __imp__WideCharToMultiByte@32 10029138     kernel32:KERNEL32.dll
 0002:0000013c       __imp__SetEnvironmentVariableW@8 1002913c     kernel32:KERNEL32.dll
 0002:00000140       __imp__GetFileAttributesExW@12 10029140     kernel32:KERNEL32.dll
 0002:00000144       __imp__FlushFileBuffers@4  10029144     kernel32:KERNEL32.dll
 0002:00000148       __imp__WriteFile@20        10029148     kernel32:KERNEL32.dll
 0002:0000014c       __imp__GetConsoleOutputCP@0 1002914c     kernel32:KERNEL32.dll
 0002:00000150       __imp__GetCurrentDirectoryW@8 10029150     kernel32:KERNEL32.dll
 0002:00000154       __imp__GetFullPathNameW@16 10029154     kernel32:KERNEL32.dll
 0002:00000158       __imp__SetStdHandle@8      10029158     kernel32:KERNEL32.dll
 0002:0000015c       __imp__HeapReAlloc@16      1002915c     kernel32:KERNEL32.dll
 0002:00000160       __imp__FindFirstFileExW@24 10029160     kernel32:KERNEL32.dll
 0002:00000164       __imp__FindNextFileW@8     10029164     kernel32:KERNEL32.dll
 0002:00000168       __imp__IsValidCodePage@4   10029168     kernel32:KERNEL32.dll
 0002:0000016c       __imp__GetACP@0            1002916c     kernel32:KERNEL32.dll
 0002:00000170       __imp__GetOEMCP@0          10029170     kernel32:KERNEL32.dll
 0002:00000174       __imp__GetCPInfo@8         10029174     kernel32:KERNEL32.dll
 0002:00000178       __imp__GetCommandLineW@0   10029178     kernel32:KERNEL32.dll
 0002:0000017c       __imp__GetEnvironmentStringsW@0 1002917c     kernel32:KERNEL32.dll
 0002:00000180       __imp__FreeEnvironmentStringsW@4 10029180     kernel32:KERNEL32.dll
 0002:00000184       __imp__GetProcessHeap@0    10029184     kernel32:KERNEL32.dll
 0002:00000188       __imp__SetEndOfFile@4      10029188     kernel32:KERNEL32.dll
 0002:0000018c       __imp__GetStringTypeW@16   1002918c     kernel32:KERNEL32.dll
 0002:00000190       __imp__GetFileSizeEx@8     10029190     kernel32:KERNEL32.dll
 0002:00000194       __imp__DecodePointer@4     10029194     kernel32:KERNEL32.dll
 0002:00000198       \177KERNEL32_NULL_THUNK_DATA 10029198     kernel32:KERNEL32.dll
 0002:0000019c       __imp__CharNextExA@12      1002919c     user32:USER32.dll
 0002:000001a0       __imp__MessageBoxA@16      100291a0     user32:USER32.dll
 0002:000001a4       \177USER32_NULL_THUNK_DATA 100291a4     user32:USER32.dll
 0002:000001a8       ___guard_check_icall_fptr  100291a8     LIBCMT:guard_support.obj
 0002:000001ac       ___castguard_check_failure_os_handled_fptr 100291ac     LIBCMT:guard_support.obj
 0002:000001b0       ___xc_a                    100291b0     LIBCMT:initializers.obj
 0002:000001b4       ___xc_z                    100291b4     LIBCMT:initializers.obj
 0002:000001b8       ___xi_a                    100291b8     LIBCMT:initializers.obj
 0002:000001bc       ___acrt_stdio_initializer  100291bc     libucrt:stdio_initializer.obj
 0002:000001c0       ___acrt_multibyte_initializer 100291c0     libucrt:multibyte_initializer.obj
 0002:000001c4       ___acrt_timeset_initializer 100291c4     libucrt:timeset_initializer.obj
 0002:000001c8       ___acrt_fmode_initializer  100291c8     libucrt:fmode_initializer.obj
 0002:000001cc       ___acrt_tran_sse2_initializer 100291cc     libucrt:sse2_initializer.obj
 0002:000001d0       ___xi_z                    100291d0     LIBCMT:initializers.obj
 0002:000001d4       ___xp_a                    100291d4     LIBCMT:initializers.obj
 0002:000001d8       ___acrt_locale_terminator  100291d8     libucrt:locale_initializer.obj
 0002:000001dc       ___dcrt_console_output_terminator 100291dc     libucrt:console_output_initializer.obj
 0002:000001e0       ___acrt_stdio_terminator   100291e0     libucrt:stdio_initializer.obj
 0002:000001e4       ___xp_z                    100291e4     LIBCMT:initializers.obj
 0002:000001e8       ___xt_a                    100291e8     LIBCMT:initializers.obj
 0002:000001ec       ___xt_z                    100291ec     LIBCMT:initializers.obj
 0002:000001f0       ??_C@_07NBCGADJA@Unknown@  100291f0     cmdtoargs.obj
 0002:000001f8       ??_C@_0L@EOAAECLN@Main?5class@ 100291f8     cmdtoargs.obj
 0002:00000204       ??_C@_08NIAMKNB@JAR?5file@ 10029204     cmdtoargs.obj
 0002:00000210       ??_C@_0BO@ECPMAOGG@invalid?5distance?5too?5far?5back@ 10029210     inffast.obj
 0002:00000230       ??_C@_0BG@LBKINIKP@invalid?5distance?5code@ 10029230     inffast.obj
 0002:00000248       ??_C@_0BM@FFFLPBBC@invalid?5literal?1length?5code@ 10029248     inffast.obj
 0002:00000b10       ??_C@_0BH@LIBMMIGA@incorrect?5header?5check@ 10029b10     inflate.obj
 0002:00000b28       ??_C@_0BL@IHKGDAEE@unknown?5compression?5method@ 10029b28     inflate.obj
 0002:00000b44       ??_C@_0BE@EMOGCLGO@invalid?5window?5size@ 10029b44     inflate.obj
 0002:00000b58       ??_C@_0BJ@BLBBCOMO@unknown?5header?5flags?5set@ 10029b58     inflate.obj
 0002:00000b74       ??_C@_0BE@GONKLEPM@header?5crc?5mismatch@ 10029b74     inflate.obj
 0002:00000b88       ??_C@_0BD@PJCBIDD@invalid?5block?5type@ 10029b88     inflate.obj
 0002:00000b9c       ??_C@_0BN@LGAADGOK@invalid?5stored?5block?5lengths@ 10029b9c     inflate.obj
 0002:00000bbc       ??_C@_0CE@GMIGFPBB@too?5many?5length?5or?5distance?5sym@ 10029bbc     inflate.obj
 0002:00000be0       ??_C@_0BJ@HDEPPGOH@invalid?5code?5lengths?5set@ 10029be0     inflate.obj
 0002:00000bfc       ??_C@_0BK@BMMPFBBH@invalid?5bit?5length?5repeat@ 10029bfc     inflate.obj
 0002:00000c18       ??_C@_0CF@DGDMADCD@invalid?5code?5?9?9?5missing?5end?9of?9@ 10029c18     inflate.obj
 0002:00000c40       ??_C@_0BM@IIMGAINC@invalid?5literal?1lengths?5set@ 10029c40     inflate.obj
 0002:00000c5c       ??_C@_0BG@GMDFCBGP@invalid?5distances?5set@ 10029c5c     inflate.obj
 0002:00000c74       ??_C@_0BF@MEIGEHBE@incorrect?5data?5check@ 10029c74     inflate.obj
 0002:00000c8c       ??_C@_0BH@FGKKJGOC@incorrect?5length?5check@ 10029c8c     inflate.obj
 0002:00000ca8       _inflate_copyright         10029ca8     inftrees.obj
 0002:00000dd8       ??_C@_0L@FLLOCCHD@NMT_LEVEL_@ 10029dd8     java.obj
 0002:00000dfc       ??_C@_02OJDBNLEE@?5?7@     10029dfc     java.obj
 0002:00000e00       ??_C@_0BE@OFPFKAIO@Command?5line?5args?3?6@ 10029e00     java.obj
 0002:00000e14       ??_C@_0P@NAHECKMG@argv?$FL?$CFd?$FN?5?$DN?5?$CFs?6@ 10029e14     java.obj
 0002:00000e24       ??_C@_0BO@JELEMDBE@?9Dsun?4java?4launcher?4diag?$DNtrue@ 10029e24     java.obj
 0002:00000e44       ??_C@_0CB@IBPGMCMH@?$CFld?5micro?5seconds?5to?5LoadJavaVM@ 10029e44     java.obj
 0002:00000e68       ??_C@_09GEOACDML@CLASSPATH@ 10029e68     java.obj
 0002:00000e74       ??_C@_01LFCBOECM@?4@       10029e74     java.obj
 0002:00000e78       ??_C@_0GM@ELCKKLGK@Error?3?5Could?5not?5create?5the?5Jav@ 10029e78     java.obj
 0002:00000ee8       ??_C@_0HD@PPKHMHGL@Error?3?5Could?5not?5detach?5main?5th@ 10029ee8     java.obj
 0002:00000f5c       ??_C@_0CE@ODMOBDNM@?$CFld?5micro?5seconds?5to?5Initialize@ 10029f5c     java.obj
 0002:00000f80       ??_C@_0M@JMGIBICN@?$CFs?5is?5?8?$CFs?8?6@ 10029f80     java.obj
 0002:00000f8c       ??_C@_0BC@IKMDOBPK@App?8s?5argc?5is?5?$CFd?6@ 10029f8c     java.obj
 0002:00000fa0       ??_C@_0BG@EAAKBDAJ@?5?5?5?5argv?$FL?$CF2d?$FN?5?$DN?5?8?$CFs?8?6@ 10029fa0     java.obj
 0002:00000fb8       ??_C@_0EO@KGGGJHNP@Error?3?5A?5JNI?5error?5has?5occurred@ 10029fb8     java.obj
 0002:00001008       ??_C@_0BH@IALIHDHM@?$CI?$FLLjava?1lang?1String?$DL?$CJV@ 1002a008     java.obj
 0002:00001020       ??_C@_04GHJNJNPO@main@     1002a020     java.obj
 0002:00001028       ??_C@_0BB@BIGIFKOD@JDK_ALTERNATE_VM@ 1002a028     java.obj
 0002:0000103c       ??_C@_0L@JBBEAFHG@?9classpath@ 1002a03c     java.obj
 0002:00001048       ??_C@_03OJENFLIP@?9cp@     1002a048     java.obj
 0002:0000104c       ??_C@_0L@MNOMOABD@?9XXaltjvm?$DN@ 1002a04c     java.obj
 0002:00001058       ??_C@_0N@IHBJGDGH@?9J?9XXaltjvm?$DN@ 1002a058     java.obj
 0002:00001068       ??_C@_0BA@ENLNODBJ@Default?5VM?3?5?$CFs?6@ 1002a068     java.obj
 0002:00001078       ??_C@_0DC@GMKJBLDL@Error?3?5Corrupt?5jvm?4cfg?5file?$DL?5cy@ 1002a078     java.obj
 0002:000010ac       ??_C@_05MBDEGLCK@ERROR@    1002a0ac     java.obj
 0002:000010b4       ??_C@_0CF@EHKDFPIN@Error?3?5Unable?5to?5resolve?5VM?5ali@ 1002a0b4     java.obj
 0002:000010dc       ??_C@_0DB@ICJLIDMC@Warning?3?5?$CFs?5VM?5not?5supported?$DL?5?$CF@ 1002a0dc     java.obj
 0002:00001110       ??_C@_0BL@ICJEGBLP@Error?3?5?$CFs?5VM?5not?5supported@ 1002a110     java.obj
 0002:0000112c       ??_C@_08NPLKDBJI@?9version@ 1002a12c     java.obj
 0002:00001138       ??_C@_0N@IILNIMNM@?9fullversion@ 1002a138     java.obj
 0002:00001148       ??_C@_05DOEHDILL@?9help@   1002a148     java.obj
 0002:00001150       ??_C@_02GIPFNJGC@?9?$DP@   1002a150     java.obj
 0002:00001154       ??_C@_04LEOFD@?9jar@       1002a154     java.obj
 0002:0000115c       ??_C@_02ECEJCEAC@?9X@      1002a15c     java.obj
 0002:00001160       ??_C@_0BK@KPPPPIMG@?9XX?3NativeMemoryTracking?$DN@ 1002a160     java.obj
 0002:0000117c       ??_C@_07PFMNENFI@?$CFs?$CFd?$DN?$CFs@ 1002a17c     java.obj
 0002:00001184       ??_C@_04HGGBINEM@?$CFs?$CFd@ 1002a184     java.obj
 0002:0000118c       ??_C@_0DE@KEMGKHHI@TRACER_MARKER?3?5NativeMemoryTrac@ 1002a18c     java.obj
 0002:000011c0       ??_C@_0DE@KHHPGILD@TRACER_MARKER?3?5NativeMemoryTrac@ 1002a1c0     java.obj
 0002:000011f4       ??_C@_0DD@JGMKIPCJ@TRACER_MARKER?3?5NativeMemoryTrac@ 1002a1f4     java.obj
 0002:00001228       ??_C@_04FMJADICG@?9Xss@    1002a228     java.obj
 0002:00001230       ??_C@_04KJNMGPJH@?9Xmx@    1002a230     java.obj
 0002:00001238       ??_C@_04EKCILGFM@?9Xms@    1002a238     java.obj
 0002:00001240       ??_C@_0BD@BJIHGBGF@_JAVA_VERSION_SET?$DN@ 1002a240     java.obj
 0002:00001254       ??_C@_0BC@LDDPFIIH@_JAVA_VERSION_SET@ 1002a254     java.obj
 0002:00001268       ??_C@_09NLKCHPDO@?9version?3@ 1002a268     java.obj
 0002:00001274       ??_C@_0BF@BOPFKIEC@?9jre?9restrict?9search@ 1002a274     java.obj
 0002:0000128c       ??_C@_0BI@EMNPBDOF@?9no?9jre?9restrict?9search@ 1002a28c     java.obj
 0002:000012a4       ??_C@_0BJ@MCNGENOM@?9Djava?4awt?4headless?$DNtrue@ 1002a2a4     java.obj
 0002:000012c0       ??_C@_0BF@CMFGICHD@?9Djava?4awt?4headless?$DN@ 1002a2c0     java.obj
 0002:000012d8       ??_C@_08GFHMBCLC@?9splash?3@ 1002a2d8     java.obj
 0002:000012e4       ??_C@_0CD@DBKPDEJE@Error?3?5Unable?5to?5access?5jarfile@ 1002a2e4     java.obj
 0002:00001308       ??_C@_0CF@JOEJCGOC@Error?3?5Invalid?5or?5corrupt?5jarfi@ 1002a308     java.obj
 0002:00001330       ??_C@_0BD@NDCPPKLD@_JAVA_SPLASH_FILE?$DN@ 1002a330     java.obj
 0002:00001344       ??_C@_0BC@FAHMLMBM@_JAVA_SPLASH_JAR?$DN@ 1002a344     java.obj
 0002:00001358       ??_C@_0DC@CMGFJGAO@Error?3?5Syntax?5error?5in?5version?5@ 1002a358     java.obj
 0002:0000138c       ??_C@_04MLLLIHIP@null@     1002a38c     java.obj
 0002:00001394       ??_C@_04LOAJBDKD@true@     1002a394     java.obj
 0002:0000139c       ??_C@_05LAPONLG@false@     1002a39c     java.obj
 0002:000013a4       ??_C@_0DK@JKAIOFLC@JRE?9Version?5?$DN?5?$CFs?0?5JRE?9Restrict?9@ 1002a3a4     java.obj
 0002:000013e0       ??_C@_0DH@FJKKHGPC@Error?3?5Unable?5to?5locate?5JRE?5mee@ 1002a3e0     java.obj
 0002:00001418       ??_C@_0HJ@JOAGODKD@Error?3?5main?9class?3?5attribute?5ex@ 1002a418     java.obj
 0002:00001494       ??_C@_0CM@DPCHNCBN@Error?3?5?$CFs?5requires?5class?5path?5s@ 1002a494     java.obj
 0002:000014c0       ??_C@_0CK@JHECGGGO@Error?3?5?$CFs?5requires?5jar?5file?5spe@ 1002a4c0     java.obj
 0002:000014ec       ??_C@_02JNAPBCPB@?9h@      1002a4ec     java.obj
 0002:000014f0       ??_C@_0N@LMMGPIFD@?9showversion@ 1002a4f0     java.obj
 0002:00001500       ??_C@_0P@OLHNJJJN@?9XshowSettings@ 1002a500     java.obj
 0002:00001510       ??_C@_0BA@KLPMEMBJ@?9XshowSettings?3@ 1002a510     java.obj
 0002:00001520       ??_C@_06GFBBMHDE@?9Xdiag@  1002a520     java.obj
 0002:00001528       ??_C@_0BF@CGIIANBK@?$CFs?5full?5version?5?$CC?$CFs?$CC@ 1002a528     java.obj
 0002:00001540       ??_C@_0L@IOOPLDLG@?9verbosegc@ 1002a540     java.obj
 0002:0000154c       ??_C@_0M@FCDCLOMN@?9verbose?3gc@ 1002a54c     java.obj
 0002:00001558       ??_C@_02HLHIEPKM@?9t@      1002a558     java.obj
 0002:0000155c       ??_C@_03KFBPJEPK@?9Xt@     1002a55c     java.obj
 0002:00001560       ??_C@_03PEIICGG@?9tm@      1002a560     java.obj
 0002:00001564       ??_C@_04INJOBBHM@?9Xtm@    1002a564     java.obj
 0002:0000156c       ??_C@_06OHOHKFPP@?9debug@  1002a56c     java.obj
 0002:00001574       ??_C@_07MDIKCNOD@?9Xdebug@ 1002a574     java.obj
 0002:0000157c       ??_C@_0L@IAOONLOP@?9noclassgc@ 1002a57c     java.obj
 0002:00001588       ??_C@_0M@JJFHIIML@?9Xnoclassgc@ 1002a588     java.obj
 0002:00001594       ??_C@_08EAEOLGAG@?9Xfuture@ 1002a594     java.obj
 0002:000015a0       ??_C@_0N@CKMDLKDL@?9Xverify?3all@ 1002a5a0     java.obj
 0002:000015b0       ??_C@_07FILEFCOC@?9verify@ 1002a5b0     java.obj
 0002:000015b8       ??_C@_0O@IDLLNEML@?9verifyremote@ 1002a5b8     java.obj
 0002:000015c8       ??_C@_0BA@FABHJJHD@?9Xverify?3remote@ 1002a5c8     java.obj
 0002:000015d8       ??_C@_09JLKGPCDL@?9noverify@ 1002a5d8     java.obj
 0002:000015e4       ??_C@_0O@DKMKFJCN@?9Xverify?3none@ 1002a5e4     java.obj
 0002:000015f4       ??_C@_05LNMHIAFA@?9prof@   1002a5f4     java.obj
 0002:000015fc       ??_C@_0BL@EPNBHIKE@?9Xrunhprof?3cpu?$DNold?0file?$DN?$CFs@ 1002a5fc     java.obj
 0002:00001618       ??_C@_0CC@PMGACDGN@?9Xrunhprof?3cpu?$DNold?0file?$DNjava?4pr@ 1002a618     java.obj
 0002:0000163c       ??_C@_03NOEGKLDM@?9ss@     1002a63c     java.obj
 0002:00001640       ??_C@_04DBGMPIDO@?9oss@    1002a640     java.obj
 0002:00001648       ??_C@_03MIPOCFEG@?9ms@     1002a648     java.obj
 0002:0000164c       ??_C@_03CLAKPMIN@?9mx@     1002a64c     java.obj
 0002:00001650       ??_C@_04DEKBGKCE@?9X?$CFs@ 1002a650     java.obj
 0002:00001658       ??_C@_0N@OIJOAPMB@?9checksource@ 1002a658     java.obj
 0002:00001668       ??_C@_03MCGAAIEM@?9cs@     1002a668     java.obj
 0002:0000166c       ??_C@_0L@HELBLEOP@?9noasyncgc@ 1002a66c     java.obj
 0002:00001678       ??_C@_0CL@CAKBCILK@Warning?3?5?$CFs?5option?5is?5no?5longer@ 1002a678     java.obj
 0002:000016a4       ??_C@_0BC@JGENKKKB@JavaVM?5args?3?6?5?5?5?5@ 1002a6a4     java.obj
 0002:000016b8       ??_C@_0BC@FPGFOMNN@version?50x?$CF08lx?0?5@ 1002a6b8     java.obj
 0002:000016cc       ??_C@_08JPIMBKG@JNI_TRUE@  1002a6cc     java.obj
 0002:000016d8       ??_C@_09OOFGMMEJ@JNI_FALSE@ 1002a6d8     java.obj
 0002:000016e4       ??_C@_0BL@KOPLOMOC@ignoreUnrecognized?5is?5?$CFs?0?5@ 1002a6e4     java.obj
 0002:00001700       ??_C@_0BB@MHDPODII@nOptions?5is?5?$CFld?6@ 1002a700     java.obj
 0002:00001714       ??_C@_0BI@DAIGOBCB@?5?5?5?5option?$FL?$CF2d?$FN?5?$DN?5?8?$CFs?8?6@ 1002a714     java.obj
 0002:0000172c       ??_C@_0BM@GGJONNLD@sun?1launcher?1LauncherHelper@ 1002a72c     java.obj
 0002:00001748       ??_C@_0BI@DIGBKJNJ@?$CIZ?$FLB?$CJLjava?1lang?1String?$DL@ 1002a748     java.obj
 0002:00001760       ??_C@_0BD@KFHODOP@makePlatformString@ 1002a760     java.obj
 0002:00001774       ??_C@_0BB@FLFAIHG@java?1lang?1String@ 1002a774     java.obj
 0002:00001788       ??_C@_0CI@BKCMKGDB@?$CIZILjava?1lang?1String?$DL?$CJLjava?1lan@ 1002a788     java.obj
 0002:000017b0       ??_C@_0BB@FFCCDEMN@checkAndLoadMain@ 1002a7b0     java.obj
 0002:000017c4       ??_C@_0CG@FBCAJICK@?$CFld?5micro?5seconds?5to?5load?5main?5@ 1002a7c4     java.obj
 0002:000017ec       ??_C@_0BF@FJHGBKOC@_JAVA_LAUNCHER_DEBUG@ 1002a7ec     java.obj
 0002:00001804       ??_C@_0M@PAPGNNMB@?9?9?9?9?$CFs?9?9?9?9?6@ 1002a804     java.obj
 0002:00001810       ??_C@_0BE@IIFEGCLG@?$CI?$CJLjava?1lang?1Class?$DL@ 1002a810     java.obj
 0002:00001824       ??_C@_0BE@JCLPIBOC@getApplicationClass@ 1002a824     java.obj
 0002:00001838       ??_C@_0DI@DPHDCKMH@Error?3?5The?5?9J?5option?5should?5not@ 1002a838     java.obj
 0002:00001870       ??_C@_0BE@EHGMLIJH@?9Denv?4class?4path?$DN?$CFs@ 1002a870     java.obj
 0002:00001884       ??_C@_0CN@LAMKHMKA@Error?3?5Could?5not?5determine?5appl@ 1002a884     java.obj
 0002:000018b4       ??_C@_0BG@FKBCOFMO@?9Dapplication?4home?$DN?$CFs@ 1002a8b4     java.obj
 0002:000018cc       ??_C@_0BD@HCEIMOC@?9Djava?4class?4path?$DN@ 1002a8cc     java.obj
 0002:000018e0       ??_C@_0BE@NJODCGLC@?9Dsun?4java?4command?$DN@ 1002a8e0     java.obj
 0002:000018f4       ??_C@_01CLKCMJKC@?5@       1002a8f4     java.obj
 0002:000018f8       ??_C@_0CB@JGILPBEK@?9Dsun?4java?4launcher?$DNSUN_STANDAR@ 1002a8f8     java.obj
 0002:0000191c       ??_C@_0BB@CAEEJDCD@sun?1misc?1Version@ 1002a91c     java.obj
 0002:00001930       ??_C@_03GAEACAIP@?$CI?$CJV@ 1002a930     java.obj
 0002:00001934       ??_C@_07BKGNKEBM@println@  1002a934     java.obj
 0002:0000193c       ??_C@_05IJDJACGD@print@    1002a93c     java.obj
 0002:00001944       ??_C@_0BL@PCCDHECB@?$CIZLjava?1lang?1String?$DLJJJZ?$CJV@ 1002a944     java.obj
 0002:00001960       ??_C@_0N@FDEDEFMB@showSettings@ 1002a960     java.obj
 0002:00001970       ??_C@_04LHKBAEFM@?$CIZ?$CJV@ 1002a970     java.obj
 0002:00001978       ??_C@_0BD@HPNJGMKF@printXUsageMessage@ 1002a978     java.obj
 0002:0000198c       ??_C@_0BG@IKDDPPGD@?$CILjava?1lang?1String?$DL?$CJV@ 1002a98c     java.obj
 0002:000019a4       ??_C@_0BA@KCDLFDGO@initHelpMessage@ 1002a9a4     java.obj
 0002:000019b4       ??_C@_0CI@HEGLGDKJ@?$CILjava?1lang?1String?$DLLjava?1lang?1S@ 1002a9b4     java.obj
 0002:000019dc       ??_C@_0BG@DGHNKDKK@appendVmSelectMessage@ 1002a9dc     java.obj
 0002:000019f4       ??_C@_0BH@EGFKIDIP@appendVmSynonymMessage@ 1002a9f4     java.obj
 0002:00001a0c       ??_C@_0BH@JHJABHLM@?$CIZLjava?1lang?1String?$DL?$CJV@ 1002aa0c     java.obj
 0002:00001a24       ??_C@_0BE@PLAGLJPD@appendVmErgoMessage@ 1002aa24     java.obj
 0002:00001a38       ??_C@_0BB@KBOLJHAM@printHelpMessage@ 1002aa38     java.obj
 0002:00001a4c       ??_C@_01KDCPPGHE@r@        1002aa4c     java.obj
 0002:00001a50       ??_C@_0BL@FBFFBAJO@Error?3?5could?5not?5open?5?$GA?$CFs?8@ 1002aa50     java.obj
 0002:00001a6c       ??_C@_0CJ@IIPHEFLM@Warning?3?5No?5leading?5?9?5on?5line?5?$CF@ 1002aa6c     java.obj
 0002:00001a98       ??_C@_0CM@HIKCBBNP@Warning?3?5Missing?5VM?5type?5on?5lin@ 1002aa98     java.obj
 0002:00001ac4       ??_C@_05IBPFAAO@KNOWN@     1002aac4     java.obj
 0002:00001acc       ??_C@_0L@PPNPEEBD@ALIASED_TO@ 1002aacc     java.obj
 0002:00001ad8       ??_C@_04JBIELMDE@WARN@     1002aad8     java.obj
 0002:00001ae0       ??_C@_06GHNPMFCC@IGNORE@   1002aae0     java.obj
 0002:00001ae8       ??_C@_0BA@GPBHNCNO@IF_SERVER_CLASS@ 1002aae8     java.obj
 0002:00001af8       ??_C@_0DE@NGDEDBBF@Warning?3?5Missing?5server?5class?5V@ 1002aaf8     java.obj
 0002:00001b2c       ??_C@_0CM@FGNACLCO@Warning?3?5Unknown?5VM?5type?5on?5lin@ 1002ab2c     java.obj
 0002:00001b58       ??_C@_0BG@IFIDBPPB@jvm?4cfg?$FL?$CFd?$FN?5?$DN?5?9?$DO?$CFs?$DM?9?6@ 1002ab58     java.obj
 0002:00001b70       ??_C@_0O@COGEDILL@VM_ALIASED_TO@ 1002ab70     java.obj
 0002:00001b80       ??_C@_0CF@IFGPMOPD@?5?5?5?5name?3?5?$CFs?5?5vmType?3?5?$CFs?5?5alias@ 1002ab80     java.obj
 0002:00001ba8       ??_C@_0BD@FPIBPMAC@VM_IF_SERVER_CLASS@ 1002aba8     java.obj
 0002:00001bbc       ??_C@_0CM@CPEKMEIJ@?5?5?5?5name?3?5?$CFs?5?5vmType?3?5?$CFs?5?5serve@ 1002abbc     java.obj
 0002:00001be8       ??_C@_0CE@ELPMGLDL@?$CFld?5micro?5seconds?5to?5parse?5jvm?4@ 1002abe8     java.obj
 0002:00001c0c       ??_C@_02DKLNFENB@?9J@      1002ac0c     java.obj
 0002:00001c10       ??_C@_0BB@CBKFGMGB@_JAVA_SPLASH_JAR@ 1002ac10     java.obj
 0002:00001c24       ??_C@_0BC@KBGGAEHG@_JAVA_SPLASH_FILE@ 1002ac24     java.obj
 0002:00001c38       ??_C@_0BB@PNLKJHCD@Launcher?5state?3?6@ 1002ac38     java.obj
 0002:00001c4c       ??_C@_02LIELOMNJ@on@       1002ac4c     java.obj
 0002:00001c50       ??_C@_03MCADLMAF@off@      1002ac50     java.obj
 0002:00001c54       ??_C@_0L@MIIHLGHH@?7debug?3?$CFs?6@ 1002ac54     java.obj
 0002:00001c60       ??_C@_0N@GJJJEEHN@?7javargs?3?$CFs?6@ 1002ac60     java.obj
 0002:00001c70       ??_C@_0BC@PEOMGKPB@?7program?5name?3?$CFs?6@ 1002ac70     java.obj
 0002:00001c84       ??_C@_0BD@OJIEGNIP@?7launcher?5name?3?$CFs?6@ 1002ac84     java.obj
 0002:00001c98       ??_C@_0L@ODBEFCFP@?7javaw?3?$CFs?6@ 1002ac98     java.obj
 0002:00001ca4       ??_C@_0BB@LLCLOLLP@?7fullversion?3?$CFs?6@ 1002aca4     java.obj
 0002:00001cb8       ??_C@_0BA@CHJOCLPM@?7dotversion?3?$CFs?6@ 1002acb8     java.obj
 0002:00001cc8       ??_C@_0O@MCPHPPHF@?7ergo_policy?3@ 1002acc8     java.obj
 0002:00001cd8       ??_C@_0CF@NLABEOAG@NEVER_ACT_AS_A_SERVER_CLASS_MAC@ 1002acd8     java.obj
 0002:00001d00       ??_C@_0CG@KJCEBOIF@ALWAYS_ACT_AS_A_SERVER_CLASS_MA@ 1002ad00     java.obj
 0002:00001d28       ??_C@_0BL@NOPGACED@DEFAULT_ERGONOMICS_POLICY?6@ 1002ad28     java.obj
 0002:00001d44       ??_C@_04HPJFIMLL@?9d32@    1002ad44     java.obj
 0002:00001d4c       ??_C@_04CPAEOJNG@?9d64@    1002ad4c     java.obj
 0002:00001d54       ??_C@_01EEMJAFIK@?6@       1002ad54     java.obj
 0002:00001d58       ??_C@_0BG@JDMBLFEN@?2bin?2splashscreen?4dll@ 1002ad58     java_md.obj
 0002:00001d70       ??_C@_04OMAFGPMM@i386@     1002ad70     java_md.obj
 0002:00001d78       ??_C@_06HEODLAOD@?9J?9d64@ 1002ad78     java_md.obj
 0002:00001d80       ??_C@_06CEHCNFIO@?9J?9d32@ 1002ad80     java_md.obj
 0002:00001d88       ??_C@_0FN@OKDNEENA@Error?3?5This?5Java?5instance?5does?5@ 1002ad88     java_md.obj
 0002:00001de8       ??_C@_0DD@KOHGIEIN@Error?3?5Could?5not?5find?5Java?5SE?5R@ 1002ade8     java_md.obj
 0002:00001e1c       ??_C@_01KICIPPFI@?2@       1002ae1c     java_md.obj
 0002:00001e20       ??_C@_0BF@JFGIBLHG@?$CFs?$CFslib?$CFs?$CFs?$CFsjvm?4cfg@ 1002ae20     java_md.obj
 0002:00001e38       ??_C@_0DG@EBKNCNED@Error?3?5no?5known?5VMs?4?5?$CIcheck?5for@ 1002ae38     java_md.obj
 0002:00001e70       ??_C@_0CF@EOPDIDEN@Error?3?5could?5not?5determine?5JVM?5@ 1002ae70     java_md.obj
 0002:00001e98       ??_C@_0GO@EHNKANIL@Error?3?5missing?5?$GA?$CFs?8?5JVM?5at?5?$GA?$CFs?8@ 1002ae98     java_md.obj
 0002:00001f08       ??_C@_0BB@JFPKNOOA@?9Dsun?4awt?4warmup@ 1002af08     java_md.obj
 0002:00001f1c       ??_C@_0BF@NJKIMEMJ@?9Dsun?4java2d?4noddraw@ 1002af1c     java_md.obj
 0002:00001f34       ??_C@_0BB@NOIMNAMG@?9Dsun?4java2d?4d3d@ 1002af34     java_md.obj
 0002:00001f48       ??_C@_0BE@BJJGJMIO@?9Dsun?4java2d?4opengl@ 1002af48     java_md.obj
 0002:00001f5c       ??_C@_05MEOKPOAG@?2bin?2@  1002af5c     java_md.obj
 0002:00001f64       ??_C@_0BB@LMCDEFHL@vcruntime140?4dll@ 1002af64     java_md.obj
 0002:00001f78       ??_C@_0DF@CLDFKAFM@Error?3?5Path?5length?5exceeds?5maxi@ 1002af78     java_md.obj
 0002:00001fb0       ??_C@_0BG@HMMNHEMF@?2bin?2vcruntime140?4dll@ 1002afb0     java_md.obj
 0002:00001fc8       ??_C@_0BA@ICKGDIKE@CRT?5path?5is?5?$CFs?6@ 1002afc8     java_md.obj
 0002:00001fd8       ??_C@_0BD@FIJKEMFL@Error?3?5loading?3?5?$CFs@ 1002afd8     java_md.obj
 0002:00001fec       ??_C@_0N@GFGFIGJO@msvcp140?4dll@ 1002afec     java_md.obj
 0002:00001ffc       ??_C@_0BC@GEINBJJF@?2bin?2msvcp140?4dll@ 1002affc     java_md.obj
 0002:00002010       ??_C@_0BA@ENEJLCMI@PRT?5path?5is?5?$CFs?6@ 1002b010     java_md.obj
 0002:00002020       ??_C@_0BA@MFAPGPPP@?$CFs?2bin?2java?4dll@ 1002b020     java_md.obj
 0002:00002030       ??_C@_0BA@KEGAOLGA@JRE?5path?5is?5?$CFs?6@ 1002b030     java_md.obj
 0002:00002040       ??_C@_0CG@KCIKNEAK@Insufficient?5space?5to?5store?5JRE@ 1002b040     java_md.obj
 0002:00002068       ??_C@_0BE@FGKJLOCF@?$CFs?2jre?2bin?2java?4dll@ 1002b068     java_md.obj
 0002:0000207c       ??_C@_04NPFKBOJD@?2jre@    1002b07c     java_md.obj
 0002:00002084       ??_C@_0BP@GFBADFON@Error?3?5could?5not?5find?5java?4dll@ 1002b084     java_md.obj
 0002:000020a4       ??_C@_0L@NCGCEDEH@?$CFs?2jvm?4dll@ 1002b0a4     java_md.obj
 0002:000020b0       ??_C@_0BC@DKEACPBC@?$CFs?2bin?2?$CFs?2jvm?4dll@ 1002b0b0     java_md.obj
 0002:000020c4       ??_C@_0BA@BNEFJADF@JVM?5path?5is?5?$CFs?6@ 1002b0c4     java_md.obj
 0002:000020d4       ??_C@_0BB@IDHJDMHA@JNI_CreateJavaVM@ 1002b0d4     java_md.obj
 0002:000020e8       ??_C@_0BN@LEMGLGLC@JNI_GetDefaultJavaVMInitArgs@ 1002b0e8     java_md.obj
 0002:00002108       ??_C@_0CI@NEHNFCJI@Error?3?5can?8t?5find?5JNI?5interface@ 1002b108     java_md.obj
 0002:00002130       ??_C@_0CL@FJGCCGIP@Software?2JavaSoft?2Java?5Runtime?5@ 1002b130     java_md.obj
 0002:0000215c       ??_C@_0CB@NNAMBOJM@Error?3?5opening?5registry?5key?5?8?$CFs@ 1002b15c     java_md.obj
 0002:00002180       ??_C@_0P@IANJKHJL@CurrentVersion@ 1002b180     java_md.obj
 0002:00002190       ??_C@_0EA@EDAOGLOA@Error?3?5Failed?5reading?5value?5of?5@ 1002b190     java_md.obj
 0002:000021d0       ??_C@_0EP@CIHJIPHL@Error?3?5Registry?5key?5?8?$CFs?8?2Curren@ 1002b1d0     java_md.obj
 0002:00002220       ??_C@_08FBFIMIEP@JavaHome@ 1002b220     java_md.obj
 0002:0000222c       ??_C@_0DG@OIEIPEHI@Failed?5reading?5value?5of?5registr@ 1002b22c     java_md.obj
 0002:00002264       ??_C@_0N@ELAFCILD@MicroVersion@ 1002b264     java_md.obj
 0002:00002274       ??_C@_0CC@OJPECNPK@Warning?3?5Can?8t?5read?5MicroVersio@ 1002b274     java_md.obj
 0002:00002298       ??_C@_0CD@PGAFLHMF@Version?5major?4minor?4micro?5?$DN?5?$CFs?4@ 1002b298     java_md.obj
 0002:000022bc       ??_C@_0BO@HBHLOLEF@Java?5Virtual?5Machine?5Launcher@ 1002b2bc     java_md.obj
 0002:000022da       ??_C@_00CNPNBAHC@@         1002b2da     java_md.obj
 0002:000022dc       ??_C@_02DKCKIIND@?$CFs@    1002b2dc     java_md.obj
 0002:000022e0       ??_C@_0BP@HLKODNMI@A?5Java?5Exception?5has?5occurred?4@ 1002b2e0     java_md.obj
 0002:00002300       ??_C@_0BM@DDAANPNE@Error?3?5Unable?5to?5resolve?5?$CFs@ 1002b300     java_md.obj
 0002:0000231c       ??_C@_0BC@KHJPFJBM@ExecJRE?3?5old?3?5?$CFs?6@ 1002b31c     java_md.obj
 0002:00002330       ??_C@_0BC@PJJNNACH@ExecJRE?3?5new?3?5?$CFs?6@ 1002b330     java_md.obj
 0002:00002344       ??_C@_0O@MKPMHCLM@?$CFs?2bin?2?$CFs?4exe@ 1002b344     java_md.obj
 0002:00002354       ??_C@_01BJJEKLCA@?$CC@     1002b354     java_md.obj
 0002:00002358       ??_C@_0BJ@ICJJCECN@ReExec?5Command?3?5?$CFs?5?$CI?$CFs?$CJ?6@ 1002b358     java_md.obj
 0002:00002374       ??_C@_0BB@PGPCIMOD@ReExec?5Args?3?5?$CFs?6@ 1002b374     java_md.obj
 0002:00002388       ??_C@_0CG@MFHJILDH@Error?3?5CreateProcess?$CI?$CFs?0?5?4?4?4?$CJ?5f@ 1002b388     java_md.obj
 0002:000023b0       ??_C@_0CF@PKJBBIAG@Error?3?5WaitForSingleObject?$CI?$CJ?5fa@ 1002b3b0     java_md.obj
 0002:000023d8       ??_C@_01NEMOKFLO@?$DN@     1002b3d8     java_md.obj
 0002:000023dc       ??_C@_05LLAMLEHD@?$CFI64d@ 1002b3dc     java_md.obj
 0002:000023e4       ??_C@_07JFLIEEAK@J2D_D3D@  1002b3e4     java_md.obj
 0002:000023ec       ??_C@_0BA@GGNAPKCP@J2D_D3D_PRELOAD@ 1002b3ec     java_md.obj
 0002:000023fc       ??_C@_0L@HNPMBHIG@preloadD3D@ 1002b3fc     java_md.obj
 0002:00002408       ??_C@_07KCBEICKO@jvm?4dll@ 1002b408     java_md.obj
 0002:00002410       ??_C@_0BM@GLGHANGM@JVM_FindClassFromBootLoader@ 1002b410     java_md.obj
 0002:0000242c       ??_C@_0BA@MPLLCPDB@?2bin?2verify?4dll@ 1002b42c     java_md.obj
 0002:0000243c       ??_C@_0O@ICEIELND@?2bin?2java?4dll@ 1002b43c     java_md.obj
 0002:0000244c       ??_C@_0N@DAAOANPF@?2bin?2awt?4dll@ 1002b44c     java_md.obj
 0002:0000245c       ??_C@_0M@MLICCBOD@preloadStop@ 1002b45c     java_md.obj
 0002:00002468       ??_C@_0DG@HDGLDAO@Warning?3?5app?5args?5is?5larger?5tha@ 1002b468     java_md.obj
 0002:000024a0       ??_C@_0BK@KGACHCN@passing?5arguments?5as?9is?4?6@ 1002b4a0     java_md.obj
 0002:000024bc       ??_C@_0CB@NLLCMEJ@Warning?3?5app?5args?5parsing?5error@ 1002b4bc     java_md.obj
 0002:000024e0       ??_C@_0BJ@HBLEACDG@passing?5arguments?5as?9is?6@ 1002b4e0     java_md.obj
 0002:000024fc       ??_C@_04CDPLFOEF@?$CFc?$CFs@ 1002b4fc     java_md.obj
 0002:00002504       ??_C@_03OFAPEBGM@?$CFs?6@  1002b504     java_md.obj
 0002:00002508       ??_C@_0CJ@HEGLPLDP@?$CI?$FLLjava?1lang?1String?$DL?$CJ?$FLLjava?1lan@ 1002b508     java_md.obj
 0002:00002534       ??_C@_0L@BJEEEGHP@expandArgs@ 1002b534     java_md.obj
 0002:00002540       ??_C@_06GLDDLHNF@malloc@   1002b540     jli_util.obj
 0002:00002548       ??_C@_07EOOHGPEI@realloc@  1002b548     jli_util.obj
 0002:00002550       ??_C@_06GFPDKFFG@strdup@   1002b550     jli_util.obj
 0002:00002558       ??_C@_0BF@LACNODFI@META?9INF?1MANIFEST?4MF@ 1002b558     parse_manifest.obj
 0002:00002570       ??_C@_05OJPKCACG@1?43?41@  1002b570     parse_manifest.obj
 0002:00002578       ??_C@_02LIIHNNHG@?6?$AN@   1002b578     parse_manifest.obj
 0002:0000257c       ??_C@_0BB@NKLIEOFJ@Manifest?9Version@ 1002b57c     parse_manifest.obj
 0002:00002590       ??_C@_0L@CIHLCGEL@Main?9Class@ 1002b590     parse_manifest.obj
 0002:0000259c       ??_C@_0M@DJAFHGJP@JRE?9Version@ 1002b59c     parse_manifest.obj
 0002:000025a8       ??_C@_0BE@NGIBIBAB@JRE?9Restrict?9Search@ 1002b5a8     parse_manifest.obj
 0002:000025bc       ??_C@_0BD@ODACGPCD@Splashscreen?9Image@ 1002b5bc     parse_manifest.obj
 0002:000025d0       ??_C@_0BB@PKAPNNLJ@SplashLoadMemory@ 1002b5d0     splashscreen_stubs.obj
 0002:000025e4       ??_C@_0P@JIPKACHN@SplashLoadFile@ 1002b5e4     splashscreen_stubs.obj
 0002:000025f4       ??_C@_0L@JOBDBDOP@SplashInit@ 1002b5f4     splashscreen_stubs.obj
 0002:00002600       ??_C@_0BF@GABHKIKD@SplashSetFileJarName@ 1002b600     splashscreen_stubs.obj
 0002:00002618       ??_C@_0BF@LIMBEMBN@SplashSetScaleFactor@ 1002b618     splashscreen_stubs.obj
 0002:00002630       ??_C@_0BJ@FJIBEMML@SplashGetScaledImageName@ 1002b630     splashscreen_stubs.obj
 0002:0000264c       ??_C@_03JDOAGMMG@?4?9_@    1002b64c     version_comp.obj
 0002:00002650       ??_C@_01GBGANLPD@0@        1002b650     version_comp.obj
 0002:00002654       ??_C@_04CGDGLCCN@?5?$CG?$CL?$CK@ 1002b654     version_comp.obj
 0002:0000265c       ??_C@_03NODMINOH@jar@      1002b65c     wildcard.obj
 0002:00002660       ??_C@_03NDMHEAJL@JAR@      1002b660     wildcard.obj
 0002:00002664       ??_C@_0DH@KEOBCGCG@Expanded?5wildcards?3?6?5?5?5?5before?3@ 1002b664     wildcard.obj
 0002:00004f20       _z_errmsg                  1002df20     zutil.obj
 0002:00004f48       ??_C@_0BA@MOKMMFOD@need?5dictionary@ 1002df48     zutil.obj
 0002:00004f58       ??_C@_0L@FNAOCBOG@stream?5end@ 1002df58     zutil.obj
 0002:00004f64       ??_C@_0L@KIJFAKBJ@file?5error@ 1002df64     zutil.obj
 0002:00004f70       ??_C@_0N@MKKNPMJD@stream?5error@ 1002df70     zutil.obj
 0002:00004f80       ??_C@_0L@HAHMBNLP@data?5error@ 1002df80     zutil.obj
 0002:00004f8c       ??_C@_0BE@OGGJBMCE@insufficient?5memory@ 1002df8c     zutil.obj
 0002:00004fa0       ??_C@_0N@DFPGLBGC@buffer?5error@ 1002dfa0     zutil.obj
 0002:00004fb0       ??_C@_0BF@CJFPCCEG@incompatible?5version@ 1002dfb0     zutil.obj
 0002:00004fd0       __pDefaultRawDllMain       1002dfd0     LIBCMT:dll_dllmain.obj
 0002:00004fd0       __pRawDllMain              1002dfd0     LIBCMT:dll_dllmain.obj
 0002:00004fd4       __pDestructExceptionObject 1002dfd4     libvcruntime:ehhelpers.obj
 0002:00005360       ??_C@_08EHJDFFNH@__based?$CI@ 1002e360     libvcruntime:undname.obj
 0002:0000536c       ??_C@_07KOLFKCDI@__cdecl@  1002e36c     libvcruntime:undname.obj
 0002:00005374       ??_C@_08GHMPAG@__pascal@   1002e374     libvcruntime:undname.obj
 0002:00005380       ??_C@_09IFJBGAPI@__stdcall@ 1002e380     libvcruntime:undname.obj
 0002:0000538c       ??_C@_0L@NPHFGOKO@__thiscall@ 1002e38c     libvcruntime:undname.obj
 0002:00005398       ??_C@_0L@JMKHOMEK@__fastcall@ 1002e398     libvcruntime:undname.obj
 0002:000053a4       ??_C@_0N@BCKKPABJ@__vectorcall@ 1002e3a4     libvcruntime:undname.obj
 0002:000053b4       ??_C@_09HIJEGCPM@__clrcall@ 1002e3b4     libvcruntime:undname.obj
 0002:000053c0       ??_C@_06GHPCKEAG@__eabi@   1002e3c0     libvcruntime:undname.obj
 0002:000053c8       ??_C@_09IOPIDJLG@__swift_1@ 1002e3c8     libvcruntime:undname.obj
 0002:000053d4       ??_C@_09KFNFGKHF@__swift_2@ 1002e3d4     libvcruntime:undname.obj
 0002:000053e0       ??_C@_09LMMOFLDE@__swift_3@ 1002e3e0     libvcruntime:undname.obj
 0002:000053ec       ??_C@_07JOMMBBKO@__ptr64@  1002e3ec     libvcruntime:undname.obj
 0002:000053f4       ??_C@_0L@PILCLIHE@__restrict@ 1002e3f4     libvcruntime:undname.obj
 0002:00005400       ??_C@_0M@GFIIJFMG@__unaligned@ 1002e400     libvcruntime:undname.obj
 0002:0000540c       ??_C@_09DHDLOLLB@restrict?$CI@ 1002e40c     libvcruntime:undname.obj
 0002:00005418       ??_C@_04NIHEBCM@?5new@     1002e418     libvcruntime:undname.obj
 0002:00005420       ??_C@_07FPCDHGMM@?5delete@ 1002e420     libvcruntime:undname.obj
 0002:00005428       ??_C@_02GPIOPFAK@?$DO?$DO@ 1002e428     libvcruntime:undname.obj
 0002:0000542c       ??_C@_02FODMEDOG@?$DM?$DM@ 1002e42c     libvcruntime:undname.obj
 0002:00005430       ??_C@_01DCLJPIOD@?$CB@     1002e430     libvcruntime:undname.obj
 0002:00005434       ??_C@_02EGOFBIJA@?$DN?$DN@ 1002e434     libvcruntime:undname.obj
 0002:00005438       ??_C@_02FDNJECIE@?$CB?$DN@ 1002e438     libvcruntime:undname.obj
 0002:0000543c       ??_C@_02GPECMEKF@?$FL?$FN@ 1002e43c     libvcruntime:undname.obj
 0002:00005440       ??_C@_08LHJFAFGD@operator@ 1002e440     libvcruntime:undname.obj
 0002:0000544c       ??_C@_02HBOOOICD@?9?$DO@   1002e44c     libvcruntime:undname.obj
 0002:00005450       ??_C@_01NBENCBCI@?$CK@     1002e450     libvcruntime:undname.obj
 0002:00005454       ??_C@_02ECNGHCIF@?$CL?$CL@ 1002e454     libvcruntime:undname.obj
 0002:00005458       ??_C@_02BAABKJLB@?9?9@     1002e458     libvcruntime:undname.obj
 0002:0000545c       ??_C@_01JOAMLHOP@?9@       1002e45c     libvcruntime:undname.obj
 0002:00005460       ??_C@_01MIFGBAGJ@?$CL@     1002e460     libvcruntime:undname.obj
 0002:00005464       ??_C@_01HNPIGOCE@?$CG@     1002e464     libvcruntime:undname.obj
 0002:00005468       ??_C@_03MNHNFDLC@?9?$DO?$CK@ 1002e468     libvcruntime:undname.obj
 0002:0000546c       ??_C@_01KMDKNFGN@?1@       1002e46c     libvcruntime:undname.obj
 0002:00005470       ??_C@_01FGNFDNOH@?$CF@     1002e470     libvcruntime:undname.obj
 0002:00005474       ??_C@_01MNNFJEPP@?$DM@     1002e474     libvcruntime:undname.obj
 0002:00005478       ??_C@_02EHCHHCKH@?$DM?$DN@ 1002e478     libvcruntime:undname.obj
 0002:0000547c       ??_C@_01PPODPGHN@?$DO@     1002e47c     libvcruntime:undname.obj
 0002:00005480       ??_C@_02EEKDKGMJ@?$DO?$DN@ 1002e480     libvcruntime:undname.obj
 0002:00005484       ??_C@_01IHBHIGKO@?0@       1002e484     libvcruntime:undname.obj
 0002:00005488       ??_C@_02HCKGKOFO@?$CI?$CJ@ 1002e488     libvcruntime:undname.obj
 0002:0000548c       ??_C@_01PJKLJHI@?$HO@      1002e48c     libvcruntime:undname.obj
 0002:00005490       ??_C@_01JKBOJNNK@?$FO@     1002e490     libvcruntime:undname.obj
 0002:00005494       ??_C@_01DNKMNLPK@?$HM@     1002e494     libvcruntime:undname.obj
 0002:00005498       ??_C@_02PPKAJPJL@?$CG?$CG@ 1002e498     libvcruntime:undname.obj
 0002:0000549c       ??_C@_02NONPIBCD@?$HM?$HM@ 1002e49c     libvcruntime:undname.obj
 0002:000054a0       ??_C@_02FPIMKNGF@?$CK?$DN@ 1002e4a0     libvcruntime:undname.obj
 0002:000054a4       ??_C@_02FOEOMHFC@?$CL?$DN@ 1002e4a4     libvcruntime:undname.obj
 0002:000054a8       ??_C@_02FKMDLLOA@?9?$DN@   1002e4a8     libvcruntime:undname.obj
 0002:000054ac       ??_C@_02FJEHGPIO@?1?$DN@   1002e4ac     libvcruntime:undname.obj
 0002:000054b0       ??_C@_02FENAOKFI@?$CF?$DN@ 1002e4b0     libvcruntime:undname.obj
 0002:000054b4       ??_C@_03IKFCCPFF@?$DO?$DO?$DN@ 1002e4b4     libvcruntime:undname.obj
 0002:000054b8       ??_C@_03CDNPDDLA@?$DM?$DM?$DN@ 1002e4b8     libvcruntime:undname.obj
 0002:000054bc       ??_C@_02FGJGFEAB@?$CG?$DN@ 1002e4bc     libvcruntime:undname.obj
 0002:000054c0       ??_C@_02DHLNPPGH@?$HM?$DN@ 1002e4c0     libvcruntime:undname.obj
 0002:000054c4       ??_C@_02MHEGNOJ@?$FO?$DN@  1002e4c4     libvcruntime:undname.obj
 0002:000054c8       ??_C@_09IFPLHPGF@?$GAvftable?8@ 1002e4c8     libvcruntime:undname.obj
 0002:000054d4       ??_C@_09BLBHBJP@?$GAvbtable?8@ 1002e4d4     libvcruntime:undname.obj
 0002:000054e0       ??_C@_07FEEIOKP@?$GAvcall?8@ 1002e4e0     libvcruntime:undname.obj
 0002:000054e8       ??_C@_08LLFFHHDJ@?$GAtypeof?8@ 1002e4e8     libvcruntime:undname.obj
 0002:000054f4       ??_C@_0BF@KDPPACIK@?$GAlocal?5static?5guard?8@ 1002e4f4     libvcruntime:undname.obj
 0002:0000550c       ??_C@_08OBABFOLI@?$GAstring?8@ 1002e50c     libvcruntime:undname.obj
 0002:00005518       ??_C@_0BD@JDLKDPAB@?$GAvbase?5destructor?8@ 1002e518     libvcruntime:undname.obj
 0002:0000552c       ??_C@_0BN@DEGPLNFK@?$GAvector?5deleting?5destructor?8@ 1002e52c     libvcruntime:undname.obj
 0002:0000554c       ??_C@_0BO@OBMKPJIG@?$GAdefault?5constructor?5closure?8@ 1002e54c     libvcruntime:undname.obj
 0002:0000556c       ??_C@_0BN@IMDCHIKM@?$GAscalar?5deleting?5destructor?8@ 1002e56c     libvcruntime:undname.obj
 0002:0000558c       ??_C@_0BO@PFGOCPJJ@?$GAvector?5constructor?5iterator?8@ 1002e58c     libvcruntime:undname.obj
 0002:000055ac       ??_C@_0BN@LFPFMEDL@?$GAvector?5destructor?5iterator?8@ 1002e5ac     libvcruntime:undname.obj
 0002:000055cc       ??_C@_0CE@IKBNEHA@?$GAvector?5vbase?5constructor?5itera@ 1002e5cc     libvcruntime:undname.obj
 0002:000055f0       ??_C@_0BL@NILFHHPC@?$GAvirtual?5displacement?5map?8@ 1002e5f0     libvcruntime:undname.obj
 0002:0000560c       ??_C@_0CB@JONCMFFK@?$GAeh?5vector?5constructor?5iterator@ 1002e60c     libvcruntime:undname.obj
 0002:00005630       ??_C@_0CA@GCEOPDGL@?$GAeh?5vector?5destructor?5iterator?8@ 1002e630     libvcruntime:undname.obj
 0002:00005650       ??_C@_0CH@OOJPLCPH@?$GAeh?5vector?5vbase?5constructor?5it@ 1002e650     libvcruntime:undname.obj
 0002:00005678       ??_C@_0BL@LLKPOHJI@?$GAcopy?5constructor?5closure?8@ 1002e678     libvcruntime:undname.obj
 0002:00005694       ??_C@_0BA@KBCDOMBN@?$GAudt?5returning?8@ 1002e694     libvcruntime:undname.obj
 0002:000056a4       ??_C@_03KLGMFNMG@?$GAEH@   1002e6a4     libvcruntime:undname.obj
 0002:000056a8       ??_C@_05KHLCHHI@?$GARTTI@  1002e6a8     libvcruntime:undname.obj
 0002:000056b0       ??_C@_0BA@KKLDJDLB@?$GAlocal?5vftable?8@ 1002e6b0     libvcruntime:undname.obj
 0002:000056c0       ??_C@_0CE@IIHCMGGL@?$GAlocal?5vftable?5constructor?5clos@ 1002e6c0     libvcruntime:undname.obj
 0002:000056e4       ??_C@_06FHBGPFGH@?5new?$FL?$FN@ 1002e6e4     libvcruntime:undname.obj
 0002:000056ec       ??_C@_09LBNFPBCA@?5delete?$FL?$FN@ 1002e6ec     libvcruntime:undname.obj
 0002:000056f8       ??_C@_0P@HJKNJFNN@?$GAomni?5callsig?8@ 1002e6f8     libvcruntime:undname.obj
 0002:00005708       ??_C@_0BL@CNOONJFP@?$GAplacement?5delete?5closure?8@ 1002e708     libvcruntime:undname.obj
 0002:00005724       ??_C@_0BN@CKNJLHMB@?$GAplacement?5delete?$FL?$FN?5closure?8@ 1002e724     libvcruntime:undname.obj
 0002:00005744       ??_C@_0CG@CFDHKGGD@?$GAmanaged?5vector?5constructor?5ite@ 1002e744     libvcruntime:undname.obj
 0002:0000576c       ??_C@_0CF@IMGKMJNO@?$GAmanaged?5vector?5destructor?5iter@ 1002e76c     libvcruntime:undname.obj
 0002:00005794       ??_C@_0CG@HLDDJMAG@?$GAeh?5vector?5copy?5constructor?5ite@ 1002e794     libvcruntime:undname.obj
 0002:000057bc       ??_C@_0CM@FCBBDIGB@?$GAeh?5vector?5vbase?5copy?5construct@ 1002e7bc     libvcruntime:undname.obj
 0002:000057e8       ??_C@_0BL@CLIPGLGB@?$GAdynamic?5initializer?5for?5?8@ 1002e7e8     libvcruntime:undname.obj
 0002:00005804       ??_C@_0CB@PDBIFEP@?$GAdynamic?5atexit?5destructor?5for?5@ 1002e804     libvcruntime:undname.obj
 0002:00005828       ??_C@_0CD@CGAJBKEJ@?$GAvector?5copy?5constructor?5iterat@ 1002e828     libvcruntime:undname.obj
 0002:0000584c       ??_C@_0CJ@GJELGAMM@?$GAvector?5vbase?5copy?5constructor?5@ 1002e84c     libvcruntime:undname.obj
 0002:00005878       ??_C@_0CL@FGIJHLCE@?$GAmanaged?5vector?5copy?5constructo@ 1002e878     libvcruntime:undname.obj
 0002:000058a4       ??_C@_0BM@PMGGMLDN@?$GAlocal?5static?5thread?5guard?8@ 1002e8a4     libvcruntime:undname.obj
 0002:000058c0       ??_C@_0N@BDNMDMOL@operator?5?$CC?$CC?5@ 1002e8c0     libvcruntime:undname.obj
 0002:000058d0       ??_C@_0BC@GGEBGALA@operator?5co_await@ 1002e8d0     libvcruntime:undname.obj
 0002:000058e4       ??_C@_0M@GAAIMMOH@operator?$DM?$DN?$DO@ 1002e8e4     libvcruntime:undname.obj
 0002:000058f0       ??_C@_0BC@DAFEJGAK@?5Type?5Descriptor?8@ 1002e8f0     libvcruntime:undname.obj
 0002:00005904       ??_C@_0BM@LDKODKLH@?5Base?5Class?5Descriptor?5at?5?$CI@ 1002e904     libvcruntime:undname.obj
 0002:00005920       ??_C@_0BD@LGICGFMM@?5Base?5Class?5Array?8@ 1002e920     libvcruntime:undname.obj
 0002:00005934       ??_C@_0BN@MECKDCOJ@?5Class?5Hierarchy?5Descriptor?8@ 1002e934     libvcruntime:undname.obj
 0002:00005954       ??_C@_0BK@CFCOFLF@?5Complete?5Object?5Locator?8@ 1002e954     libvcruntime:undname.obj
 0002:00005970       ??_C@_0BG@JNJLAMPM@?$GAanonymous?5namespace?8@ 1002e970     libvcruntime:undname.obj
 0002:00005994       ??_C@_1DM@KHCHBNEB@?$AAa?$AAp?$AAi?$AA?9?$AAm?$AAs?$AA?9?$AAw?$AAi?$AAn?$AA?9?$AAc?$AAo?$AAr?$AAe@ 1002e994     libvcruntime:winapi_downlevel.obj
 0002:000059d0       ??_C@_1DK@LPPGFMPP@?$AAa?$AAp?$AAi?$AA?9?$AAm?$AAs?$AA?9?$AAw?$AAi?$AAn?$AA?9?$AAc?$AAo?$AAr?$AAe@ 1002e9d0     libvcruntime:winapi_downlevel.obj
 0002:00005a0c       ??_C@_1BC@GDMECMAK@?$AAk?$AAe?$AAr?$AAn?$AAe?$AAl?$AA3?$AA2@ 1002ea0c     libvcruntime:winapi_downlevel.obj
 0002:00005a20       ??_C@_1BA@PFFKHIOG@?$AAa?$AAp?$AAi?$AA?9?$AAm?$AAs?$AA?9@ 1002ea20     libvcruntime:winapi_downlevel.obj
 0002:00005a38       ??_C@_08KNHFBNJ@FlsAlloc@  1002ea38     libvcruntime:winapi_downlevel.obj
 0002:00005a4c       ??_C@_07PEJMOBNF@FlsFree@  1002ea4c     libvcruntime:winapi_downlevel.obj
 0002:00005a5c       ??_C@_0M@GDNOONDI@FlsGetValue@ 1002ea5c     libvcruntime:winapi_downlevel.obj
 0002:00005a70       ??_C@_0M@JCPCPOEF@FlsSetValue@ 1002ea70     libvcruntime:winapi_downlevel.obj
 0002:00005a84       ??_C@_0BM@HCFOFFN@InitializeCriticalSectionEx@ 1002ea84     libvcruntime:winapi_downlevel.obj
 0002:00005aa4       ??_7exception@std@@6B@     1002eaa4     libvcruntime:frame.obj
 0002:00005aac       ??_C@_0BC@EOODALEL@Unknown?5exception@ 1002eaac     libvcruntime:frame.obj
 0002:00005ac4       ??_7bad_exception@std@@6B@ 1002eac4     libvcruntime:frame.obj
 0002:00005acc       ??_C@_0O@DPKOEFFH@bad?5exception@ 1002eacc     libvcruntime:frame.obj
 0002:00005ae0       ?standard_lookup_table_spectre@__crt_stdio_output@@3V?$spectre_mitigated_lookup_table@Ustate_transition_pair@__crt_stdio_output@@$0IA@@1@B 1002eae0     libucrt:output.obj
 0002:00005be0       ??_C@_1O@CEDCILHN@?$AA?$CI?$AAn?$AAu?$AAl?$AAl?$AA?$CJ@ 1002ebe0     libucrt:output.obj
 0002:00005bf0       ??_C@_06OJHGLDPL@?$CInull?$CJ@ 1002ebf0     libucrt:output.obj
 0002:00005bf8       ?large_power_data@?1??multiply_by_power_of_ten@__crt_strtox@@YA_NAAUbig_integer@2@I@Z@4QBIB 1002ebf8     libucrt:input.obj
 0002:00006500       ?large_power_indices@?1??multiply_by_power_of_ten@__crt_strtox@@YA_NAAUbig_integer@2@I@Z@4QBUunpack_index@?1??12@YA_N0I@Z@B 1002f500     libucrt:input.obj
 0002:00006598       ?small_powers_of_ten@?1??multiply_by_power_of_ten@__crt_strtox@@YA_NAAUbig_integer@2@I@Z@4QBIB 1002f598     libucrt:input.obj
 0002:000065c0       ??_C@_1GE@DPGDJKLM@?$AAm?$AAi?$AAn?$AAk?$AAe?$AAr?$AAn?$AAe?$AAl?$AA?2?$AAc?$AAr?$AAt?$AAs?$AA?2@ 1002f5c0     libucrt:input.obj
 0002:00006628       ??_C@_1FM@FELNCOBF@?$AA_?$AA_?$AAc?$AAr?$AAt?$AA_?$AAs?$AAt?$AAr?$AAt?$AAo?$AAx?$AA?3?$AA?3?$AAf@ 1002f628     libucrt:input.obj
 0002:00006684       ??_C@_1BG@GEMHBGAF@?$AA_?$AAi?$AAs?$AA_?$AAd?$AAo?$AAu?$AAb?$AAl?$AAe@ 1002f684     libucrt:input.obj
 0002:000066a0       ??_C@_1FK@JOJELFFO@?$AA_?$AA_?$AAc?$AAr?$AAt?$AA_?$AAs?$AAt?$AAr?$AAt?$AAo?$AAx?$AA?3?$AA?3?$AAf@ 1002f6a0     libucrt:input.obj
 0002:000066fc       ??_C@_1BI@BANMPGJI@?$AA?$CB?$AA_?$AAi?$AAs?$AA_?$AAd?$AAo?$AAu?$AAb?$AAl?$AAe@ 1002f6fc     libucrt:input.obj
 0002:00006718       ?constraints@?1??is_length_valid@__crt_stdio_input@@YA_NW4conversion_mode@2@W4length_modifier@2@@Z@4QAY0M@$$CBEA 1002f718     libucrt:input.obj
 0002:00006790       ?inf_uppercase@?1???$parse_floating_point_possible_infinity@DV?$input_adapter_character_source@V?$string_input_adapter@D@__crt_stdio_input@@@__crt_strtox@@_K@__crt_strtox@@YA?AW4floating_point_parse_result@1@AADAAV?$input_adapter_character_source@V?$string_input_adapter@D@__crt_stdio_input@@@1@_K@Z@4QBDB 1002f790     libucrt:input.obj
 0002:00006794       ?inf_lowercase@?1???$parse_floating_point_possible_infinity@DV?$input_adapter_character_source@V?$string_input_adapter@D@__crt_stdio_input@@@__crt_strtox@@_K@__crt_strtox@@YA?AW4floating_point_parse_result@1@AADAAV?$input_adapter_character_source@V?$string_input_adapter@D@__crt_stdio_input@@@1@_K@Z@4QBDB 1002f794     libucrt:input.obj
 0002:00006798       ?inity_uppercase@?1???$parse_floating_point_possible_infinity@DV?$input_adapter_character_source@V?$string_input_adapter@D@__crt_stdio_input@@@__crt_strtox@@_K@__crt_strtox@@YA?AW4floating_point_parse_result@1@AADAAV?$input_adapter_character_source@V?$string_input_adapter@D@__crt_stdio_input@@@1@_K@Z@4QBDB 1002f798     libucrt:input.obj
 0002:000067a0       ?inity_lowercase@?1???$parse_floating_point_possible_infinity@DV?$input_adapter_character_source@V?$string_input_adapter@D@__crt_stdio_input@@@__crt_strtox@@_K@__crt_strtox@@YA?AW4floating_point_parse_result@1@AADAAV?$input_adapter_character_source@V?$string_input_adapter@D@__crt_stdio_input@@@1@_K@Z@4QBDB 1002f7a0     libucrt:input.obj
 0002:000067a8       ?uppercase@?1???$parse_floating_point_possible_nan@DV?$input_adapter_character_source@V?$string_input_adapter@D@__crt_stdio_input@@@__crt_strtox@@_K@__crt_strtox@@YA?AW4floating_point_parse_result@1@AADAAV?$input_adapter_character_source@V?$string_input_adapter@D@__crt_stdio_input@@@1@_K@Z@4QBDB 1002f7a8     libucrt:input.obj
 0002:000067ac       ?lowercase@?1???$parse_floating_point_possible_nan@DV?$input_adapter_character_source@V?$string_input_adapter@D@__crt_stdio_input@@@__crt_strtox@@_K@__crt_strtox@@YA?AW4floating_point_parse_result@1@AADAAV?$input_adapter_character_source@V?$string_input_adapter@D@__crt_stdio_input@@@1@_K@Z@4QBDB 1002f7ac     libucrt:input.obj
 0002:000067b0       ?uppercase@?1???$parse_floating_point_possible_nan_is_snan@DV?$input_adapter_character_source@V?$string_input_adapter@D@__crt_stdio_input@@@__crt_strtox@@@__crt_strtox@@YA_NAADAAV?$input_adapter_character_source@V?$string_input_adapter@D@__crt_stdio_input@@@1@@Z@4QBDB 1002f7b0     libucrt:input.obj
 0002:000067b8       ?lowercase@?1???$parse_floating_point_possible_nan_is_snan@DV?$input_adapter_character_source@V?$string_input_adapter@D@__crt_stdio_input@@@__crt_strtox@@@__crt_strtox@@YA_NAADAAV?$input_adapter_character_source@V?$string_input_adapter@D@__crt_stdio_input@@@1@@Z@4QBDB 1002f7b8     libucrt:input.obj
 0002:000067c0       ?uppercase@?1???$parse_floating_point_possible_nan_is_ind@DV?$input_adapter_character_source@V?$string_input_adapter@D@__crt_stdio_input@@@__crt_strtox@@@__crt_strtox@@YA_NAADAAV?$input_adapter_character_source@V?$string_input_adapter@D@__crt_stdio_input@@@1@@Z@4QBDB 1002f7c0     libucrt:input.obj
 0002:000067c4       ?lowercase@?1???$parse_floating_point_possible_nan_is_ind@DV?$input_adapter_character_source@V?$string_input_adapter@D@__crt_stdio_input@@@__crt_strtox@@@__crt_strtox@@YA_NAADAAV?$input_adapter_character_source@V?$string_input_adapter@D@__crt_stdio_input@@@1@@Z@4QBDB 1002f7c4     libucrt:input.obj
 0002:000067c8       ??_C@_1BI@BGOHAHKC@?$AAm?$AAs?$AAc?$AAo?$AAr?$AAe?$AAe?$AA?4?$AAd?$AAl?$AAl@ 1002f7c8     libucrt:exit.obj
 0002:000067e0       ??_C@_0P@MIGLKIOC@CorExitProcess@ 1002f7e0     libucrt:exit.obj
 0002:00006958       ??_C@_0EA@FCLIIPNN@Visual?5C?$CL?$CL?5CRT?3?5Not?5enough?5memo@ 1002f958     libucrt:strerror.obj
 0002:00006998       ??_C@_19DOGDICKI@?$AA?4?$AAe?$AAx?$AAe@ 1002f998     libucrt:stat.obj
 0002:000069a4       ??_C@_19BDKLHPGC@?$AA?4?$AAc?$AAm?$AAd@ 1002f9a4     libucrt:stat.obj
 0002:000069b0       ??_C@_19PINKOIBI@?$AA?4?$AAb?$AAa?$AAt@ 1002f9b0     libucrt:stat.obj
 0002:000069bc       ??_C@_19CDGLJBOD@?$AA?4?$AAc?$AAo?$AAm@ 1002f9bc     libucrt:stat.obj
 0002:000069c8       ??_C@_17BAAFHAL@?$AA?4?$AA?1?$AA?2@ 1002f9c8     libucrt:stat.obj
 0002:000069d0       ??_C@_02LMMGGCAJ@?3?5@     1002f9d0     libucrt:perror.obj
 0002:000069d8       ___acrt_exception_action_table 1002f9d8     libucrt:exception_filter.obj
 0002:00006a68       ___acrt_signal_action_table_count 1002fa68     libucrt:exception_filter.obj
 0002:00006a6c       ___acrt_signal_action_first_fpe_index 1002fa6c     libucrt:exception_filter.obj
 0002:00006a70       ___acrt_signal_action_fpe_count 1002fa70     libucrt:exception_filter.obj
 0002:00006b50       ??_C@_1EA@JGEFHKEI@?$AAa?$AAp?$AAi?$AA?9?$AAm?$AAs?$AA?9?$AAw?$AAi?$AAn?$AA?9?$AAc?$AAo?$AAr?$AAe@ 1002fb50     libucrt:winapi_thunks.obj
 0002:00006b90       ??_C@_1DI@KMEPCBPN@?$AAa?$AAp?$AAi?$AA?9?$AAm?$AAs?$AA?9?$AAw?$AAi?$AAn?$AA?9?$AAc?$AAo?$AAr?$AAe@ 1002fb90     libucrt:winapi_thunks.obj
 0002:00006bc8       ??_C@_1DI@IJCEHOCB@?$AAa?$AAp?$AAi?$AA?9?$AAm?$AAs?$AA?9?$AAw?$AAi?$AAn?$AA?9?$AAc?$AAo?$AAr?$AAe@ 1002fbc8     libucrt:winapi_thunks.obj
 0002:00006c00       ??_C@_1EI@MPIAOHOC@?$AAa?$AAp?$AAi?$AA?9?$AAm?$AAs?$AA?9?$AAw?$AAi?$AAn?$AA?9?$AAc?$AAo?$AAr?$AAe@ 1002fc00     libucrt:winapi_thunks.obj
 0002:00006c48       ??_C@_1FK@FPHCKFIE@?$AAa?$AAp?$AAi?$AA?9?$AAm?$AAs?$AA?9?$AAw?$AAi?$AAn?$AA?9?$AAc?$AAo?$AAr?$AAe@ 1002fc48     libucrt:winapi_thunks.obj
 0002:00006ca8       ??_C@_1EM@DILCGIIO@?$AAa?$AAp?$AAi?$AA?9?$AAm?$AAs?$AA?9?$AAw?$AAi?$AAn?$AA?9?$AAc?$AAo?$AAr?$AAe@ 1002fca8     libucrt:winapi_thunks.obj
 0002:00006cf4       ??_C@_1DM@LNCGDDPN@?$AAa?$AAp?$AAi?$AA?9?$AAm?$AAs?$AA?9?$AAw?$AAi?$AAn?$AA?9?$AAc?$AAo?$AAr?$AAe@ 1002fcf4     libucrt:winapi_thunks.obj
 0002:00006d30       ??_C@_1DO@FPAPJEMD@?$AAa?$AAp?$AAi?$AA?9?$AAm?$AAs?$AA?9?$AAw?$AAi?$AAn?$AA?9?$AAc?$AAo?$AAr?$AAe@ 1002fd30     libucrt:winapi_thunks.obj
 0002:00006d70       ??_C@_1DK@NDHNAHIO@?$AAa?$AAp?$AAi?$AA?9?$AAm?$AAs?$AA?9?$AAw?$AAi?$AAn?$AA?9?$AAc?$AAo?$AAr?$AAe@ 1002fd70     libucrt:winapi_thunks.obj
 0002:00006dac       ??_C@_1DM@KGHDGBCM@?$AAa?$AAp?$AAi?$AA?9?$AAm?$AAs?$AA?9?$AAw?$AAi?$AAn?$AA?9?$AAc?$AAo?$AAr?$AAe@ 1002fdac     libucrt:winapi_thunks.obj
 0002:00006de8       ??_C@_1EO@IJIOEFOH@?$AAa?$AAp?$AAi?$AA?9?$AAm?$AAs?$AA?9?$AAw?$AAi?$AAn?$AA?9?$AAr?$AAt?$AAc?$AAo@ 1002fde8     libucrt:winapi_thunks.obj
 0002:00006e38       ??_C@_1FG@HHGEKANL@?$AAa?$AAp?$AAi?$AA?9?$AAm?$AAs?$AA?9?$AAw?$AAi?$AAn?$AA?9?$AAs?$AAe?$AAc?$AAu@ 1002fe38     libucrt:winapi_thunks.obj
 0002:00006e90       ??_C@_1EG@DBIOJECG@?$AAe?$AAx?$AAt?$AA?9?$AAm?$AAs?$AA?9?$AAw?$AAi?$AAn?$AA?9?$AAn?$AAt?$AAu?$AAs@ 1002fe90     libucrt:winapi_thunks.obj
 0002:00006ed8       ??_C@_1EO@FIHMJCLF@?$AAe?$AAx?$AAt?$AA?9?$AAm?$AAs?$AA?9?$AAw?$AAi?$AAn?$AA?9?$AAn?$AAt?$AAu?$AAs@ 1002fed8     libucrt:winapi_thunks.obj
 0002:00006f28       ??_C@_1BC@DNHGCMLG@?$AAa?$AAd?$AAv?$AAa?$AAp?$AAi?$AA3?$AA2@ 1002ff28     libucrt:winapi_thunks.obj
 0002:00006f3c       ??_C@_1BG@CJPGBMEF@?$AAk?$AAe?$AAr?$AAn?$AAe?$AAl?$AAb?$AAa?$AAs?$AAe@ 1002ff3c     libucrt:winapi_thunks.obj
 0002:00006f54       ??_C@_1M@OAIMIKLP@?$AAn?$AAt?$AAd?$AAl?$AAl@ 1002ff54     libucrt:winapi_thunks.obj
 0002:00006f60       ??_C@_1EG@DPGNFKGC@?$AAa?$AAp?$AAi?$AA?9?$AAm?$AAs?$AA?9?$AAw?$AAi?$AAn?$AA?9?$AAa?$AAp?$AAp?$AAm@ 1002ff60     libucrt:winapi_thunks.obj
 0002:00006fa8       ??_C@_1O@BCCLBEOE@?$AAu?$AAs?$AAe?$AAr?$AA3?$AA2@ 1002ffa8     libucrt:winapi_thunks.obj
 0002:00006fb8       ??_C@_1DM@BPJLHKCE@?$AAa?$AAp?$AAi?$AA?9?$AAm?$AAs?$AA?9?$AAw?$AAi?$AAn?$AA?9?$AAc?$AAo?$AAr?$AAe@ 1002ffb8     libucrt:winapi_thunks.obj
 0002:00006ff4       ??_C@_1BA@IAIFMGEF@?$AAe?$AAx?$AAt?$AA?9?$AAm?$AAs?$AA?9@ 1002fff4     libucrt:winapi_thunks.obj
 0002:00007008       ??_C@_0BA@FHFNEAED@AreFileApisANSI@ 10030008     libucrt:winapi_thunks.obj
 0002:00007020       ??_C@_0BA@IHGNDAEB@CompareStringEx@ 10030020     libucrt:winapi_thunks.obj
 0002:00007040       ??_C@_0O@KKBNKAPF@LCMapStringEx@ 10030040     libucrt:winapi_thunks.obj
 0002:00007058       ??_C@_0BB@HBDEELFH@LocaleNameToLCID@ 10030058     libucrt:winapi_thunks.obj
 0002:00007070       ??_C@_0N@PPOMPGGK@RoInitialize@ 10030070     libucrt:winapi_thunks.obj
 0002:00007084       ??_C@_0P@LLFHBIJD@RoUninitialize@ 10030084     libucrt:winapi_thunks.obj
 0002:00007098       ??_C@_0CF@OJOFEIGO@AppPolicyGetProcessTerminationM@ 10030098     libucrt:winapi_thunks.obj
 0002:000070c4       ??_C@_0CF@NNDFDCOC@AppPolicyGetThreadInitializatio@ 100300c4     libucrt:winapi_thunks.obj
 0002:00007110       ___lc_time_c               10030110     libucrt:nlsdata.obj
 0002:00007274       ??_C@_03KOEHGMDN@Sun@      10030274     libucrt:nlsdata.obj
 0002:00007278       ??_C@_03PDAGKDH@Mon@       10030278     libucrt:nlsdata.obj
 0002:0000727c       ??_C@_03NAGEINEP@Tue@      1003027c     libucrt:nlsdata.obj
 0002:00007280       ??_C@_03MHOMLAJA@Wed@      10030280     libucrt:nlsdata.obj
 0002:00007284       ??_C@_03IOFIKPDN@Thu@      10030284     libucrt:nlsdata.obj
 0002:00007288       ??_C@_03IDIOELNC@Fri@      10030288     libucrt:nlsdata.obj
 0002:0000728c       ??_C@_03FEFJNEK@Sat@       1003028c     libucrt:nlsdata.obj
 0002:00007290       ??_C@_06OOPIFAJ@Sunday@    10030290     libucrt:nlsdata.obj
 0002:00007298       ??_C@_06JLEDEDGH@Monday@   10030298     libucrt:nlsdata.obj
 0002:000072a0       ??_C@_07BAAGCFCM@Tuesday@  100302a0     libucrt:nlsdata.obj
 0002:000072a8       ??_C@_09DLIGFAKA@Wednesday@ 100302a8     libucrt:nlsdata.obj
 0002:000072b4       ??_C@_08HACCIKIA@Thursday@ 100302b4     libucrt:nlsdata.obj
 0002:000072c0       ??_C@_06JECMNKMI@Friday@   100302c0     libucrt:nlsdata.obj
 0002:000072c8       ??_C@_08INBOOONO@Saturday@ 100302c8     libucrt:nlsdata.obj
 0002:000072d4       ??_C@_03JIHJHPIE@Jan@      100302d4     libucrt:nlsdata.obj
 0002:000072d8       ??_C@_03HJBDCHOM@Feb@      100302d8     libucrt:nlsdata.obj
 0002:000072dc       ??_C@_03ODNJBKGA@Mar@      100302dc     libucrt:nlsdata.obj
 0002:000072e0       ??_C@_03LEOLGMJP@Apr@      100302e0     libucrt:nlsdata.obj
 0002:000072e4       ??_C@_03CNMDKL@May@        100302e4     libucrt:nlsdata.obj
 0002:000072e8       ??_C@_03IDFGHECI@Jun@      100302e8     libucrt:nlsdata.obj
 0002:000072ec       ??_C@_03LBGABGKK@Jul@      100302ec     libucrt:nlsdata.obj
 0002:000072f0       ??_C@_03IFJFEIGA@Aug@      100302f0     libucrt:nlsdata.obj
 0002:000072f4       ??_C@_03GGCAPAJC@Sep@      100302f4     libucrt:nlsdata.obj
 0002:000072f8       ??_C@_03BMAOKBAD@Oct@      100302f8     libucrt:nlsdata.obj
 0002:000072fc       ??_C@_03JPJOFNIA@Nov@      100302fc     libucrt:nlsdata.obj
 0002:00007300       ??_C@_03MKABNOCG@Dec@      10030300     libucrt:nlsdata.obj
 0002:00007304       ??_C@_07CGJPFGJA@January@  10030304     libucrt:nlsdata.obj
 0002:0000730c       ??_C@_08GNJGEPFN@February@ 1003030c     libucrt:nlsdata.obj
 0002:00007318       ??_C@_05HPCKOFNC@March@    10030318     libucrt:nlsdata.obj
 0002:00007320       ??_C@_05DMJDNLEJ@April@    10030320     libucrt:nlsdata.obj
 0002:00007328       ??_C@_04CNLMGBGM@June@     10030328     libucrt:nlsdata.obj
 0002:00007330       ??_C@_04MIEPOIFP@July@     10030330     libucrt:nlsdata.obj
 0002:00007338       ??_C@_06LBBHFDDG@August@   10030338     libucrt:nlsdata.obj
 0002:00007340       ??_C@_09BHHEALKD@September@ 10030340     libucrt:nlsdata.obj
 0002:0000734c       ??_C@_07JJNFCEND@October@  1003034c     libucrt:nlsdata.obj
 0002:00007354       ??_C@_08HCHEGEOA@November@ 10030354     libucrt:nlsdata.obj
 0002:00007360       ??_C@_08EDHMEBNP@December@ 10030360     libucrt:nlsdata.obj
 0002:0000736c       ??_C@_02DEDBPAFC@AM@       1003036c     libucrt:nlsdata.obj
 0002:00007370       ??_C@_02CJNFDJBF@PM@       10030370     libucrt:nlsdata.obj
 0002:00007374       ??_C@_08BPBNCDIB@MM?1dd?1yy@ 10030374     libucrt:nlsdata.obj
 0002:00007380       ??_C@_0BE@CKGJFCPC@dddd?0?5MMMM?5dd?0?5yyyy@ 10030380     libucrt:nlsdata.obj
 0002:00007394       ??_C@_08JCCMCCIL@HH?3mm?3ss@ 10030394     libucrt:nlsdata.obj
 0002:000073a0       ??_C@_17MBGCMIPB@?$AAS?$AAu?$AAn@ 100303a0     libucrt:nlsdata.obj
 0002:000073a8       ??_C@_17KBOMKBF@?$AAM?$AAo?$AAn@ 100303a8     libucrt:nlsdata.obj
 0002:000073b0       ??_C@_17BMKGEGOJ@?$AAT?$AAu?$AAe@ 100303b0     libucrt:nlsdata.obj
 0002:000073b8       ??_C@_17CJEDCEPE@?$AAW?$AAe?$AAd@ 100303b8     libucrt:nlsdata.obj
 0002:000073c0       ??_C@_17PDPHAADD@?$AAT?$AAh?$AAu@ 100303c0     libucrt:nlsdata.obj
 0002:000073c8       ??_C@_17HFOLPPLP@?$AAF?$AAr?$AAi@ 100303c8     libucrt:nlsdata.obj
 0002:000073d0       ??_C@_17GGIBDPIH@?$AAS?$AAa?$AAt@ 100303d0     libucrt:nlsdata.obj
 0002:000073d8       ??_C@_1O@IHNHDHPB@?$AAS?$AAu?$AAn?$AAd?$AAa?$AAy@ 100303d8     libucrt:nlsdata.obj
 0002:000073e8       ??_C@_1O@MMNBFLIA@?$AAM?$AAo?$AAn?$AAd?$AAa?$AAy@ 100303e8     libucrt:nlsdata.obj
 0002:000073f8       ??_C@_1BA@ENFBFFEK@?$AAT?$AAu?$AAe?$AAs?$AAd?$AAa?$AAy@ 100303f8     libucrt:nlsdata.obj
 0002:00007408       ??_C@_1BE@EBOGMDOH@?$AAW?$AAe?$AAd?$AAn?$AAe?$AAs?$AAd?$AAa?$AAy@ 10030408     libucrt:nlsdata.obj
 0002:0000741c       ??_C@_1BC@HHMNLIHE@?$AAT?$AAh?$AAu?$AAr?$AAs?$AAd?$AAa?$AAy@ 1003041c     libucrt:nlsdata.obj
 0002:00007430       ??_C@_1O@PDICJHAG@?$AAF?$AAr?$AAi?$AAd?$AAa?$AAy@ 10030430     libucrt:nlsdata.obj
 0002:00007440       ??_C@_1BC@ENMNNPAJ@?$AAS?$AAa?$AAt?$AAu?$AAr?$AAd?$AAa?$AAy@ 10030440     libucrt:nlsdata.obj
 0002:00007454       ??_C@_17DKNBKCHM@?$AAJ?$AAa?$AAn@ 10030454     libucrt:nlsdata.obj
 0002:0000745c       ??_C@_17LMDJEKJN@?$AAF?$AAe?$AAb@ 1003045c     libucrt:nlsdata.obj
 0002:00007464       ??_C@_17CKNLEDEC@?$AAM?$AAa?$AAr@ 10030464     libucrt:nlsdata.obj
 0002:0000746c       ??_C@_17LFPOIHDD@?$AAA?$AAp?$AAr@ 1003046c     libucrt:nlsdata.obj
 0002:00007474       ??_C@_17PNNKMEED@?$AAM?$AAa?$AAy@ 10030474     libucrt:nlsdata.obj
 0002:0000747c       ??_C@_17KCJGOCPB@?$AAJ?$AAu?$AAn@ 1003047c     libucrt:nlsdata.obj
 0002:00007484       ??_C@_17IJPCKHK@?$AAJ?$AAu?$AAl@ 10030484     libucrt:nlsdata.obj
 0002:0000748c       ??_C@_17ICPELBCN@?$AAA?$AAu?$AAg@ 1003048c     libucrt:nlsdata.obj
 0002:00007494       ??_C@_17HCHCOKMG@?$AAS?$AAe?$AAp@ 10030494     libucrt:nlsdata.obj
 0002:0000749c       ??_C@_17FNLKOI@?$AAO?$AAc?$AAt@ 1003049c     libucrt:nlsdata.obj
 0002:000074a4       ??_C@_17BBDMLCIG@?$AAN?$AAo?$AAv@ 100304a4     libucrt:nlsdata.obj
 0002:000074ac       ??_C@_17EGKACKIF@?$AAD?$AAe?$AAc@ 100304ac     libucrt:nlsdata.obj
 0002:000074b4       ??_C@_1BA@EFMEIEBA@?$AAJ?$AAa?$AAn?$AAu?$AAa?$AAr?$AAy@ 100304b4     libucrt:nlsdata.obj
 0002:000074c4       ??_C@_1BC@JGDDFFAM@?$AAF?$AAe?$AAb?$AAr?$AAu?$AAa?$AAr?$AAy@ 100304c4     libucrt:nlsdata.obj
 0002:000074d8       ??_C@_1M@IKEENEDF@?$AAM?$AAa?$AAr?$AAc?$AAh@ 100304d8     libucrt:nlsdata.obj
 0002:000074e4       ??_C@_1M@GJNLMHFD@?$AAA?$AAp?$AAr?$AAi?$AAl@ 100304e4     libucrt:nlsdata.obj
 0002:000074f0       ??_C@_19EPFLPGAP@?$AAJ?$AAu?$AAn?$AAe@ 100304f0     libucrt:nlsdata.obj
 0002:000074fc       ??_C@_19BIFMLPCD@?$AAJ?$AAu?$AAl?$AAy@ 100304fc     libucrt:nlsdata.obj
 0002:00007508       ??_C@_1O@PAHLKOAC@?$AAA?$AAu?$AAg?$AAu?$AAs?$AAt@ 10030508     libucrt:nlsdata.obj
 0002:00007518       ??_C@_1BE@DKAAMBJL@?$AAS?$AAe?$AAp?$AAt?$AAe?$AAm?$AAb?$AAe?$AAr@ 10030518     libucrt:nlsdata.obj
 0002:0000752c       ??_C@_1BA@EPANDLNG@?$AAO?$AAc?$AAt?$AAo?$AAb?$AAe?$AAr@ 1003052c     libucrt:nlsdata.obj
 0002:0000753c       ??_C@_1BC@BGLIFPF@?$AAN?$AAo?$AAv?$AAe?$AAm?$AAb?$AAe?$AAr@ 1003053c     libucrt:nlsdata.obj
 0002:00007550       ??_C@_1BC@FEMKIFH@?$AAD?$AAe?$AAc?$AAe?$AAm?$AAb?$AAe?$AAr@ 10030550     libucrt:nlsdata.obj
 0002:00007564       ??_C@_15ODEHAHHF@?$AAA?$AAM@ 10030564     libucrt:nlsdata.obj
 0002:0000756c       ??_C@_15CLMNNGEL@?$AAP?$AAM@ 1003056c     libucrt:nlsdata.obj
 0002:00007574       ??_C@_1BC@IEBCMHCM@?$AAM?$AAM?$AA?1?$AAd?$AAd?$AA?1?$AAy?$AAy@ 10030574     libucrt:nlsdata.obj
 0002:00007588       ??_C@_1CI@KNAKOEBC@?$AAd?$AAd?$AAd?$AAd?$AA?0?$AA?5?$AAM?$AAM?$AAM?$AAM?$AA?5?$AAd?$AAd?$AA?0?$AA?5@ 10030588     libucrt:nlsdata.obj
 0002:000075b0       ??_C@_1BC@GDGBMEMK@?$AAH?$AAH?$AA?3?$AAm?$AAm?$AA?3?$AAs?$AAs@ 100305b0     libucrt:nlsdata.obj
 0002:000075c4       ??_C@_1M@BMHNFIME@?$AAe?$AAn?$AA?9?$AAU?$AAS@ 100305c4     libucrt:nlsdata.obj
 0002:000075d0       ?ccs@?1???$__acrt_stdio_parse_mode@D@@YA?AU__acrt_stdio_stream_mode@@QBD@Z@4QBDB 100305d0     libucrt:openfile.obj
 0002:000075d4       ?utf8_encoding@?1???$__acrt_stdio_parse_mode@D@@YA?AU__acrt_stdio_stream_mode@@QBD@Z@4QBDB 100305d4     libucrt:openfile.obj
 0002:000075dc       ?utf16_encoding@?1???$__acrt_stdio_parse_mode@D@@YA?AU__acrt_stdio_stream_mode@@QBD@Z@4QBDB 100305dc     libucrt:openfile.obj
 0002:000075e4       ?unicode_encoding@?1???$__acrt_stdio_parse_mode@D@@YA?AU__acrt_stdio_stream_mode@@QBD@Z@4QBDB 100305e4     libucrt:openfile.obj
 0002:00007630       ??_C@_03OEIAHPBN@INF@      10030630     libucrt:cvt.obj
 0002:00007634       ??_C@_03OJHLLCGB@inf@      10030634     libucrt:cvt.obj
 0002:00007638       ??_C@_03LKNCIKJB@NAN@      10030638     libucrt:cvt.obj
 0002:0000763c       ??_C@_03LHCJEHON@nan@      1003063c     libucrt:cvt.obj
 0002:00007640       ??_C@_09OFJJIMPC@NAN?$CISNAN?$CJ@ 10030640     libucrt:cvt.obj
 0002:0000764c       ??_C@_09IPFBKMDL@nan?$CIsnan?$CJ@ 1003064c     libucrt:cvt.obj
 0002:00007658       ??_C@_08IKHNHAJ@NAN?$CIIND?$CJ@ 10030658     libucrt:cvt.obj
 0002:00007664       ??_C@_08OFCDMILK@nan?$CIind?$CJ@ 10030664     libucrt:cvt.obj
 0002:00007670       ??_C@_05KLBDPFGC@e?$CL000@ 10030670     libucrt:cvt.obj
 0002:00007678       ___newctype                10030678     libucrt:ctype.obj
 0002:00007978       ___newclmap                10030978     libucrt:ctype.obj
 0002:00007af8       ___newcumap                10030af8     libucrt:ctype.obj
 0002:00007c78       __wctype                   10030c78     libucrt:ctype.obj
 0002:00007e7c       __sys_first_posix_error    10030e7c     libucrt:syserr.obj
 0002:00007e80       __sys_last_posix_error     10030e80     libucrt:syserr.obj
 0002:00007e88       __sys_posix_errlist        10030e88     libucrt:syserr.obj
 0002:00007f30       __sys_errlist              10030f30     libucrt:syserr.obj
 0002:00007fe0       ??_C@_08INEPGKHH@No?5error@ 10030fe0     libucrt:syserr.obj
 0002:00007fec       ??_C@_0BI@BJFCGOHL@Operation?5not?5permitted@ 10030fec     libucrt:syserr.obj
 0002:00008004       ??_C@_0BK@FMDHKPNF@No?5such?5file?5or?5directory@ 10031004     libucrt:syserr.obj
 0002:00008020       ??_C@_0BA@FKIAIBGA@No?5such?5process@ 10031020     libucrt:syserr.obj
 0002:00008030       ??_C@_0BK@FJBOAFDK@Interrupted?5function?5call@ 10031030     libucrt:syserr.obj
 0002:0000804c       ??_C@_0BD@KKNFOBBD@Input?1output?5error@ 1003104c     libucrt:syserr.obj
 0002:00008060       ??_C@_0BK@DPKMCKJ@No?5such?5device?5or?5address@ 10031060     libucrt:syserr.obj
 0002:0000807c       ??_C@_0BC@MFFGCDFL@Arg?5list?5too?5long@ 1003107c     libucrt:syserr.obj
 0002:00008090       ??_C@_0BC@HKPNECK@Exec?5format?5error@ 10031090     libucrt:syserr.obj
 0002:000080a4       ??_C@_0BE@NFGDDCEF@Bad?5file?5descriptor@ 100310a4     libucrt:syserr.obj
 0002:000080b8       ??_C@_0BD@LOHELEP@No?5child?5processes@ 100310b8     libucrt:syserr.obj
 0002:000080cc       ??_C@_0CB@EPFKGNAK@Resource?5temporarily?5unavailabl@ 100310cc     libucrt:syserr.obj
 0002:000080f0       ??_C@_0BB@IMDKMPFB@Not?5enough?5space@ 100310f0     libucrt:syserr.obj
 0002:00008104       ??_C@_0BC@HFNFNKAI@Permission?5denied@ 10031104     libucrt:syserr.obj
 0002:00008118       ??_C@_0M@LOEHLCJD@Bad?5address@ 10031118     libucrt:syserr.obj
 0002:00008124       ??_C@_0O@NIPGCINC@Unknown?5error@ 10031124     libucrt:syserr.obj
 0002:00008134       ??_C@_0BA@BIBLIOEK@Resource?5device@ 10031134     libucrt:syserr.obj
 0002:00008144       ??_C@_0M@NAAJNNGH@File?5exists@ 10031144     libucrt:syserr.obj
 0002:00008150       ??_C@_0O@OAMDNOCP@Improper?5link@ 10031150     libucrt:syserr.obj
 0002:00008160       ??_C@_0P@NLEIANHE@No?5such?5device@ 10031160     libucrt:syserr.obj
 0002:00008170       ??_C@_0BA@CJBACOOL@Not?5a?5directory@ 10031170     libucrt:syserr.obj
 0002:00008180       ??_C@_0P@NDHGCGKE@Is?5a?5directory@ 10031180     libucrt:syserr.obj
 0002:00008190       ??_C@_0BB@HMGGCEBG@Invalid?5argument@ 10031190     libucrt:syserr.obj
 0002:000081a4       ??_C@_0BO@IIFBODJE@Too?5many?5open?5files?5in?5system@ 100311a4     libucrt:syserr.obj
 0002:000081c4       ??_C@_0BE@INBJMKGG@Too?5many?5open?5files@ 100311c4     libucrt:syserr.obj
 0002:000081d8       ??_C@_0CE@ONOKNLPF@Inappropriate?5I?1O?5control?5opera@ 100311d8     libucrt:syserr.obj
 0002:000081fc       ??_C@_0P@LFMMIPAE@File?5too?5large@ 100311fc     libucrt:syserr.obj
 0002:0000820c       ??_C@_0BI@FEALHKLD@No?5space?5left?5on?5device@ 1003120c     libucrt:syserr.obj
 0002:00008224       ??_C@_0N@FEHLOILP@Invalid?5seek@ 10031224     libucrt:syserr.obj
 0002:00008234       ??_C@_0BG@DDBFNKBH@Read?9only?5file?5system@ 10031234     libucrt:syserr.obj
 0002:0000824c       ??_C@_0P@PKCJJLLM@Too?5many?5links@ 1003124c     libucrt:syserr.obj
 0002:0000825c       ??_C@_0M@LHEPIIOM@Broken?5pipe@ 1003125c     libucrt:syserr.obj
 0002:00008268       ??_C@_0N@MMJPGLJK@Domain?5error@ 10031268     libucrt:syserr.obj
 0002:00008278       ??_C@_0BB@FCBJFCAJ@Result?5too?5large@ 10031278     libucrt:syserr.obj
 0002:0000828c       ??_C@_0BK@JAEBMJJM@Resource?5deadlock?5avoided@ 1003128c     libucrt:syserr.obj
 0002:000082a8       ??_C@_0BC@BEDIHIDK@Filename?5too?5long@ 100312a8     libucrt:syserr.obj
 0002:000082bc       ??_C@_0BD@CLHBCGPB@No?5locks?5available@ 100312bc     libucrt:syserr.obj
 0002:000082d0       ??_C@_0BJ@IHEHINLI@Function?5not?5implemented@ 100312d0     libucrt:syserr.obj
 0002:000082ec       ??_C@_0BE@ICMCHPHH@Directory?5not?5empty@ 100312ec     libucrt:syserr.obj
 0002:00008300       ??_C@_0BG@KLEAJEFJ@Illegal?5byte?5sequence@ 10031300     libucrt:syserr.obj
 0002:00008318       ??_C@_0P@LDMLAFHI@address?5in?5use@ 10031318     libucrt:syserr.obj
 0002:00008328       ??_C@_0BG@DHPCNBJB@address?5not?5available@ 10031328     libucrt:syserr.obj
 0002:00008340       ??_C@_0BN@LKKBCCDB@address?5family?5not?5supported@ 10031340     libucrt:syserr.obj
 0002:00008360       ??_C@_0BP@KAIHPOGN@connection?5already?5in?5progress@ 10031360     libucrt:syserr.obj
 0002:00008380       ??_C@_0M@PMMIEFCP@bad?5message@ 10031380     libucrt:syserr.obj
 0002:0000838c       ??_C@_0BD@MOLBPMEA@operation?5canceled@ 1003138c     libucrt:syserr.obj
 0002:000083a0       ??_C@_0BD@MGNDDEGM@connection?5aborted@ 100313a0     libucrt:syserr.obj
 0002:000083b4       ??_C@_0BD@PJLIIJEL@connection?5refused@ 100313b4     libucrt:syserr.obj
 0002:000083c8       ??_C@_0BB@IECNJNOI@connection?5reset@ 100313c8     libucrt:syserr.obj
 0002:000083dc       ??_C@_0BN@KDMIFEIP@destination?5address?5required@ 100313dc     libucrt:syserr.obj
 0002:000083fc       ??_C@_0BB@DHFDFGDM@host?5unreachable@ 100313fc     libucrt:syserr.obj
 0002:00008410       ??_C@_0BD@JPHBMONG@identifier?5removed@ 10031410     libucrt:syserr.obj
 0002:00008424       ??_C@_0BG@KDKHOPCO@operation?5in?5progress@ 10031424     libucrt:syserr.obj
 0002:0000843c       ??_C@_0BC@DFIBIBIL@already?5connected@ 1003143c     libucrt:syserr.obj
 0002:00008450       ??_C@_0BO@EFGOJEF@too?5many?5symbolic?5link?5levels@ 10031450     libucrt:syserr.obj
 0002:00008470       ??_C@_0N@IFLPBIOP@message?5size@ 10031470     libucrt:syserr.obj
 0002:00008480       ??_C@_0N@KIIEAAIO@network?5down@ 10031480     libucrt:syserr.obj
 0002:00008490       ??_C@_0O@FNPDBHEE@network?5reset@ 10031490     libucrt:syserr.obj
 0002:000084a0       ??_C@_0BE@IFNCKGE@network?5unreachable@ 100314a0     libucrt:syserr.obj
 0002:000084b4       ??_C@_0BA@PFFCAOFK@no?5buffer?5space@ 100314b4     libucrt:syserr.obj
 0002:000084c4       ??_C@_0BF@PBGGPKKE@no?5message?5available@ 100314c4     libucrt:syserr.obj
 0002:000084dc       ??_C@_07PLECNNKG@no?5link@ 100314dc     libucrt:syserr.obj
 0002:000084e4       ??_C@_0L@EDOLMPAK@no?5message@ 100314e4     libucrt:syserr.obj
 0002:000084f0       ??_C@_0BD@EAMBFIDF@no?5protocol?5option@ 100314f0     libucrt:syserr.obj
 0002:00008504       ??_C@_0BE@MKFDAFMP@no?5stream?5resources@ 10031504     libucrt:syserr.obj
 0002:00008518       ??_C@_0N@LGAPMMPI@not?5a?5stream@ 10031518     libucrt:syserr.obj
 0002:00008528       ??_C@_0O@GLMIBBEG@not?5connected@ 10031528     libucrt:syserr.obj
 0002:00008538       ??_C@_0BG@MPLKFPAE@state?5not?5recoverable@ 10031538     libucrt:syserr.obj
 0002:00008550       ??_C@_0N@POEIPGGF@not?5a?5socket@ 10031550     libucrt:syserr.obj
 0002:00008560       ??_C@_0O@NHEDABJP@not?5supported@ 10031560     libucrt:syserr.obj
 0002:00008570       ??_C@_0BI@LNEGIFLN@operation?5not?5supported@ 10031570     libucrt:syserr.obj
 0002:00008588       ??_C@_0BA@KGKGOOJA@value?5too?5large@ 10031588     libucrt:syserr.obj
 0002:00008598       ??_C@_0L@BLPOFLNJ@owner?5dead@ 10031598     libucrt:syserr.obj
 0002:000085a4       ??_C@_0P@FNPOCJBE@protocol?5error@ 100315a4     libucrt:syserr.obj
 0002:000085b4       ??_C@_0BH@JPPPLHJB@protocol?5not?5supported@ 100315b4     libucrt:syserr.obj
 0002:000085cc       ??_C@_0BE@MIEJDDNH@wrong?5protocol?5type@ 100315cc     libucrt:syserr.obj
 0002:000085e0       ??_C@_0P@DIIFGFCG@stream?5timeout@ 100315e0     libucrt:syserr.obj
 0002:000085f0       ??_C@_09KJPPMAOI@timed?5out@ 100315f0     libucrt:syserr.obj
 0002:000085fc       ??_C@_0P@IPFDMIFL@text?5file?5busy@ 100315fc     libucrt:syserr.obj
 0002:0000860c       ??_C@_0BG@OEMDKMEE@operation?5would?5block@ 1003160c     libucrt:syserr.obj
 0002:00008624       __sys_nerr                 10031624     libucrt:syserr.obj
 0002:00008638       ??_C@_1M@HPNHIDJI@?$AAj?$AAa?$AA?9?$AAJ?$AAP@ 10031638     libucrt:mbctype.obj
 0002:00008644       ??_C@_1M@BIBDDEMK@?$AAz?$AAh?$AA?9?$AAC?$AAN@ 10031644     libucrt:mbctype.obj
 0002:00008650       ??_C@_1M@JLOOOEGK@?$AAk?$AAo?$AA?9?$AAK?$AAR@ 10031650     libucrt:mbctype.obj
 0002:0000865c       ??_C@_1M@CLNBBOPM@?$AAz?$AAh?$AA?9?$AAT?$AAW@ 1003165c     libucrt:mbctype.obj
 0002:00008d88       ??_C@_15EMKDOKLE@?$AAa?$AAr@ 10031d88     libucrt:lcidtoname_downlevel.obj
 0002:00008d90       ??_C@_15KNPADPLH@?$AAb?$AAg@ 10031d90     libucrt:lcidtoname_downlevel.obj
 0002:00008d98       ??_C@_15EDMHLDMO@?$AAc?$AAa@ 10031d98     libucrt:lcidtoname_downlevel.obj
 0002:00008da0       ??_C@_1O@BPEAJADD@?$AAz?$AAh?$AA?9?$AAC?$AAH?$AAS@ 10031da0     libucrt:lcidtoname_downlevel.obj
 0002:00008db0       ??_C@_15LJNHCMNK@?$AAc?$AAs@ 10031db0     libucrt:lcidtoname_downlevel.obj
 0002:00008db8       ??_C@_15FOMCIDHG@?$AAd?$AAa@ 10031db8     libucrt:lcidtoname_downlevel.obj
 0002:00008dc0       ??_C@_15NBKABECB@?$AAd?$AAe@ 10031dc0     libucrt:lcidtoname_downlevel.obj
 0002:00008dc8       ??_C@_15GHPEIIAO@?$AAe?$AAl@ 10031dc8     libucrt:lcidtoname_downlevel.obj
 0002:00008dd0       ??_C@_15MNPNEAIF@?$AAe?$AAn@ 10031dd0     libucrt:lcidtoname_downlevel.obj
 0002:00008dd8       ??_C@_15GPIOMPMH@?$AAe?$AAs@ 10031dd8     libucrt:lcidtoname_downlevel.obj
 0002:00008de0       ??_C@_15NGLOAKJC@?$AAf?$AAi@ 10031de0     libucrt:lcidtoname_downlevel.obj
 0002:00008de8       ??_C@_15FBKGNKAM@?$AAf?$AAr@ 10031de8     libucrt:lcidtoname_downlevel.obj
 0002:00008df0       ??_C@_15KGGCNEFK@?$AAh?$AAe@ 10031df0     libucrt:lcidtoname_downlevel.obj
 0002:00008df8       ??_C@_15PGHLIDMF@?$AAh?$AAu@ 10031df8     libucrt:lcidtoname_downlevel.obj
 0002:00008e00       ??_C@_15BIEMAPLM@?$AAi?$AAs@ 10031e00     libucrt:lcidtoname_downlevel.obj
 0002:00008e08       ??_C@_15IFJLDHAF@?$AAi?$AAt@ 10031e08     libucrt:lcidtoname_downlevel.obj
 0002:00008e10       ??_C@_15GEMIOCAG@?$AAj?$AAa@ 10031e10     libucrt:lcidtoname_downlevel.obj
 0002:00008e18       ??_C@_15EPELEGJA@?$AAk?$AAo@ 10031e18     libucrt:lcidtoname_downlevel.obj
 0002:00008e20       ??_C@_15NDDHIMN@?$AAn?$AAl@ 10031e20     libucrt:lcidtoname_downlevel.obj
 0002:00008e28       ??_C@_15BPIGNHCD@?$AAn?$AAo@ 10031e28     libucrt:lcidtoname_downlevel.obj
 0002:00008e30       ??_C@_15DEOPBLCG@?$AAp?$AAl@ 10031e30     libucrt:lcidtoname_downlevel.obj
 0002:00008e38       ??_C@_15KBECGEFG@?$AAp?$AAt@ 10031e38     libucrt:lcidtoname_downlevel.obj
 0002:00008e40       ??_C@_15GLJCBFMD@?$AAr?$AAo@ 10031e40     libucrt:lcidtoname_downlevel.obj
 0002:00008e48       ??_C@_15FEDGKCDI@?$AAr?$AAu@ 10031e48     libucrt:lcidtoname_downlevel.obj
 0002:00008e50       ??_C@_15GLKMLLHM@?$AAh?$AAr@ 10031e50     libucrt:lcidtoname_downlevel.obj
 0002:00008e58       ??_C@_15CPKMFBDB@?$AAs?$AAk@ 10031e58     libucrt:lcidtoname_downlevel.obj
 0002:00008e60       ??_C@_15BAAIOGMK@?$AAs?$AAq@ 10031e60     libucrt:lcidtoname_downlevel.obj
 0002:00008e68       ??_C@_15INNPNOHD@?$AAs?$AAv@ 10031e68     libucrt:lcidtoname_downlevel.obj
 0002:00008e70       ??_C@_15CABMMOGH@?$AAt?$AAh@ 10031e70     libucrt:lcidtoname_downlevel.obj
 0002:00008e78       ??_C@_15BPLIHJJM@?$AAt?$AAr@ 10031e78     libucrt:lcidtoname_downlevel.obj
 0002:00008e80       ??_C@_15NEOEKKDJ@?$AAu?$AAr@ 10031e80     libucrt:lcidtoname_downlevel.obj
 0002:00008e88       ??_C@_15NFICGAJK@?$AAi?$AAd@ 10031e88     libucrt:lcidtoname_downlevel.obj
 0002:00008e90       ??_C@_15PJPFLCCM@?$AAu?$AAk@ 10031e90     libucrt:lcidtoname_downlevel.obj
 0002:00008e98       ??_C@_15HPJPHDM@?$AAb?$AAe@ 10031e98     libucrt:lcidtoname_downlevel.obj
 0002:00008ea0       ??_C@_15LCHLGJII@?$AAs?$AAl@ 10031ea0     libucrt:lcidtoname_downlevel.obj
 0002:00008ea8       ??_C@_15PCFJPHHO@?$AAe?$AAt@ 10031ea8     libucrt:lcidtoname_downlevel.obj
 0002:00008eb0       ??_C@_15HPFPGODN@?$AAl?$AAv@ 10031eb0     libucrt:lcidtoname_downlevel.obj
 0002:00008eb8       ??_C@_15NFFGKGLG@?$AAl?$AAt@ 10031eb8     libucrt:lcidtoname_downlevel.obj
 0002:00008ec0       ??_C@_15BDAKCCHN@?$AAf?$AAa@ 10031ec0     libucrt:lcidtoname_downlevel.obj
 0002:00008ec8       ??_C@_15NFGIAIAJ@?$AAv?$AAi@ 10031ec8     libucrt:lcidtoname_downlevel.obj
 0002:00008ed0       ??_C@_15LMKNDMHN@?$AAh?$AAy@ 10031ed0     libucrt:lcidtoname_downlevel.obj
 0002:00008ed8       ??_C@_15IJBHMCFL@?$AAa?$AAz@ 10031ed8     libucrt:lcidtoname_downlevel.obj
 0002:00008ee0       ??_C@_15EKOFJABL@?$AAe?$AAu@ 10031ee0     libucrt:lcidtoname_downlevel.obj
 0002:00008ee8       ??_C@_15BGHADCNK@?$AAm?$AAk@ 10031ee8     libucrt:lcidtoname_downlevel.obj
 0002:00008ef0       ??_C@_15JDNICKHM@?$AAa?$AAf@ 10031ef0     libucrt:lcidtoname_downlevel.obj
 0002:00008ef8       ??_C@_15KPJEDBKD@?$AAk?$AAa@ 10031ef8     libucrt:lcidtoname_downlevel.obj
 0002:00008f00       ??_C@_15PDNFFFEO@?$AAf?$AAo@ 10031f00     libucrt:lcidtoname_downlevel.obj
 0002:00008f08       ??_C@_15OMLEGLOC@?$AAh?$AAi@ 10031f08     libucrt:lcidtoname_downlevel.obj
 0002:00008f10       ??_C@_15IDNNENKK@?$AAm?$AAs@ 10031f10     libucrt:lcidtoname_downlevel.obj
 0002:00008f18       ??_C@_15MACJNBMH@?$AAk?$AAk@ 10031f18     libucrt:lcidtoname_downlevel.obj
 0002:00008f20       ??_C@_15DKDJEOND@?$AAk?$AAy@ 10031f20     libucrt:lcidtoname_downlevel.obj
 0002:00008f28       ??_C@_15DFGDLJBG@?$AAs?$AAw@ 10031f28     libucrt:lcidtoname_downlevel.obj
 0002:00008f30       ??_C@_15BBFAICNG@?$AAu?$AAz@ 10031f30     libucrt:lcidtoname_downlevel.obj
 0002:00008f38       ??_C@_15DKNDCGEA@?$AAt?$AAt@ 10031f38     libucrt:lcidtoname_downlevel.obj
 0002:00008f40       ??_C@_15MGIFMDPL@?$AAp?$AAa@ 10031f40     libucrt:lcidtoname_downlevel.obj
 0002:00008f48       ??_C@_15HCNDBBA@?$AAg?$AAu@ 10031f48     libucrt:lcidtoname_downlevel.obj
 0002:00008f50       ??_C@_15FNBEIBON@?$AAt?$AAa@ 10031f50     libucrt:lcidtoname_downlevel.obj
 0002:00008f58       ??_C@_15NCHGBGLK@?$AAt?$AAe@ 10031f58     libucrt:lcidtoname_downlevel.obj
 0002:00008f60       ??_C@_15PHPHCBPF@?$AAk?$AAn@ 10031f60     libucrt:lcidtoname_downlevel.obj
 0002:00008f68       ??_C@_15DLGBCKMP@?$AAm?$AAr@ 10031f68     libucrt:lcidtoname_downlevel.obj
 0002:00008f70       ??_C@_15EABBLBFF@?$AAs?$AAa@ 10031f70     libucrt:lcidtoname_downlevel.obj
 0002:00008f78       ??_C@_15CBKOMCOI@?$AAm?$AAn@ 10031f78     libucrt:lcidtoname_downlevel.obj
 0002:00008f80       ??_C@_15CKDMCJAF@?$AAg?$AAl@ 10031f80     libucrt:lcidtoname_downlevel.obj
 0002:00008f88       ??_C@_17CNJFBPG@?$AAk?$AAo?$AAk@ 10031f88     libucrt:lcidtoname_downlevel.obj
 0002:00008f90       ??_C@_17FFBJICPL@?$AAs?$AAy?$AAr@ 10031f90     libucrt:lcidtoname_downlevel.obj
 0002:00008f98       ??_C@_17KPNDCPAF@?$AAd?$AAi?$AAv@ 10031f98     libucrt:lcidtoname_downlevel.obj
 0002:00008fa0       ??_C@_11LOCGONAA@@         10031fa0     libucrt:lcidtoname_downlevel.obj
 0002:00008fa4       ??_C@_1M@OKAHONE@?$AAa?$AAr?$AA?9?$AAS?$AAA@ 10031fa4     libucrt:lcidtoname_downlevel.obj
 0002:00008fb0       ??_C@_1M@FFFIGIGK@?$AAb?$AAg?$AA?9?$AAB?$AAG@ 10031fb0     libucrt:lcidtoname_downlevel.obj
 0002:00008fbc       ??_C@_1M@BJNKEDC@?$AAc?$AAa?$AA?9?$AAE?$AAS@ 10031fbc     libucrt:lcidtoname_downlevel.obj
 0002:00008fc8       ??_C@_1M@IJJHFJHA@?$AAc?$AAs?$AA?9?$AAC?$AAZ@ 10031fc8     libucrt:lcidtoname_downlevel.obj
 0002:00008fd4       ??_C@_1M@CLPEOBGI@?$AAd?$AAa?$AA?9?$AAD?$AAK@ 10031fd4     libucrt:lcidtoname_downlevel.obj
 0002:00008fe0       ??_C@_1M@MCMADGCB@?$AAd?$AAe?$AA?9?$AAD?$AAE@ 10031fe0     libucrt:lcidtoname_downlevel.obj
 0002:00008fec       ??_C@_1M@OOCKEMAM@?$AAe?$AAl?$AA?9?$AAG?$AAR@ 10031fec     libucrt:lcidtoname_downlevel.obj
 0002:00008ff8       ??_C@_1M@DDNJFGID@?$AAf?$AAi?$AA?9?$AAF?$AAI@ 10031ff8     libucrt:lcidtoname_downlevel.obj
 0002:00009004       ??_C@_1M@GLIPPMAC@?$AAf?$AAr?$AA?9?$AAF?$AAR@ 10032004     libucrt:lcidtoname_downlevel.obj
 0002:00009010       ??_C@_1M@GFMCHPE@?$AAh?$AAe?$AA?9?$AAI?$AAL@ 10032010     libucrt:lcidtoname_downlevel.obj
 0002:0000901c       ??_C@_1M@MHLPGNKM@?$AAh?$AAu?$AA?9?$AAH?$AAU@ 1003201c     libucrt:lcidtoname_downlevel.obj
 0002:00009028       ??_C@_1M@LPDDNNPN@?$AAi?$AAs?$AA?9?$AAI?$AAS@ 10032028     libucrt:lcidtoname_downlevel.obj
 0002:00009034       ??_C@_1M@MADIPODN@?$AAi?$AAt?$AA?9?$AAI?$AAT@ 10032034     libucrt:lcidtoname_downlevel.obj
 0002:00009040       ??_C@_1M@IHBJJGG@?$AAn?$AAl?$AA?9?$AAN?$AAL@ 10032040     libucrt:lcidtoname_downlevel.obj
 0002:0000904c       ??_C@_1M@EANAGDL@?$AAn?$AAb?$AA?9?$AAN?$AAO@ 1003204c     libucrt:lcidtoname_downlevel.obj
 0002:00009058       ??_C@_1M@NEIEMEGP@?$AAp?$AAl?$AA?9?$AAP?$AAL@ 10032058     libucrt:lcidtoname_downlevel.obj
 0002:00009064       ??_C@_1M@BOCFIGEP@?$AAp?$AAt?$AA?9?$AAB?$AAR@ 10032064     libucrt:lcidtoname_downlevel.obj
 0002:00009070       ??_C@_1M@IMPFOPBG@?$AAr?$AAo?$AA?9?$AAR?$AAO@ 10032070     libucrt:lcidtoname_downlevel.obj
 0002:0000907c       ??_C@_1M@IDNNEJMM@?$AAr?$AAu?$AA?9?$AAR?$AAU@ 1003207c     libucrt:lcidtoname_downlevel.obj
 0002:00009088       ??_C@_1M@LILEEOGM@?$AAh?$AAr?$AA?9?$AAH?$AAR@ 10032088     libucrt:lcidtoname_downlevel.obj
 0002:00009094       ??_C@_1M@FKIFEHPB@?$AAs?$AAk?$AA?9?$AAS?$AAK@ 10032094     libucrt:lcidtoname_downlevel.obj
 0002:000090a0       ??_C@_1M@LJMAMNPJ@?$AAs?$AAq?$AA?9?$AAA?$AAL@ 100320a0     libucrt:lcidtoname_downlevel.obj
 0002:000090ac       ??_C@_1M@GIAKDKJK@?$AAs?$AAv?$AA?9?$AAS?$AAE@ 100320ac     libucrt:lcidtoname_downlevel.obj
 0002:000090b8       ??_C@_1M@MKJKIKCL@?$AAt?$AAh?$AA?9?$AAT?$AAH@ 100320b8     libucrt:lcidtoname_downlevel.obj
 0002:000090c4       ??_C@_1M@MFLCCMPB@?$AAt?$AAr?$AA?9?$AAT?$AAR@ 100320c4     libucrt:lcidtoname_downlevel.obj
 0002:000090d0       ??_C@_1M@OIJHDKJN@?$AAu?$AAr?$AA?9?$AAP?$AAK@ 100320d0     libucrt:lcidtoname_downlevel.obj
 0002:000090dc       ??_C@_1M@LHIPCIEK@?$AAi?$AAd?$AA?9?$AAI?$AAD@ 100320dc     libucrt:lcidtoname_downlevel.obj
 0002:000090e8       ??_C@_1M@MFMOBGI@?$AAu?$AAk?$AA?9?$AAU?$AAA@ 100320e8     libucrt:lcidtoname_downlevel.obj
 0002:000090f4       ??_C@_1M@OBGLJIPL@?$AAb?$AAe?$AA?9?$AAB?$AAY@ 100320f4     libucrt:lcidtoname_downlevel.obj
 0002:00009100       ??_C@_1M@BCFAJEAD@?$AAs?$AAl?$AA?9?$AAS?$AAI@ 10032100     libucrt:lcidtoname_downlevel.obj
 0002:0000910c       ??_C@_1M@FKFFEDDN@?$AAe?$AAt?$AA?9?$AAE?$AAE@ 1003210c     libucrt:lcidtoname_downlevel.obj
 0002:00009118       ??_C@_1M@KGKKAACI@?$AAl?$AAv?$AA?9?$AAL?$AAV@ 10032118     libucrt:lcidtoname_downlevel.obj
 0002:00009124       ??_C@_1M@IFGBIJO@?$AAl?$AAt?$AA?9?$AAL?$AAT@ 10032124     libucrt:lcidtoname_downlevel.obj
 0002:00009130       ??_C@_1M@FGEAHEDM@?$AAf?$AAa?$AA?9?$AAI?$AAR@ 10032130     libucrt:lcidtoname_downlevel.obj
 0002:0000913c       ??_C@_1M@KBMAIBFN@?$AAv?$AAi?$AA?9?$AAV?$AAN@ 1003213c     libucrt:lcidtoname_downlevel.obj
 0002:00009148       ??_C@_1M@GPCBKDJK@?$AAh?$AAy?$AA?9?$AAA?$AAM@ 10032148     libucrt:lcidtoname_downlevel.obj
 0002:00009154       ??_C@_1BG@BECMDDJB@?$AAa?$AAz?$AA?9?$AAA?$AAZ?$AA?9?$AAL?$AAa?$AAt?$AAn@ 10032154     libucrt:lcidtoname_downlevel.obj
 0002:0000916c       ??_C@_1M@MAOFCAEA@?$AAe?$AAu?$AA?9?$AAE?$AAS@ 1003216c     libucrt:lcidtoname_downlevel.obj
 0002:00009178       ??_C@_1M@IGHABKPI@?$AAm?$AAk?$AA?9?$AAM?$AAK@ 10032178     libucrt:lcidtoname_downlevel.obj
 0002:00009184       ??_C@_1M@IAIGNEJG@?$AAt?$AAn?$AA?9?$AAZ?$AAA@ 10032184     libucrt:lcidtoname_downlevel.obj
 0002:00009190       ??_C@_1M@IIJCOJFA@?$AAx?$AAh?$AA?9?$AAZ?$AAA@ 10032190     libucrt:lcidtoname_downlevel.obj
 0002:0000919c       ??_C@_1M@LGPJHNJH@?$AAz?$AAu?$AA?9?$AAZ?$AAA@ 1003219c     libucrt:lcidtoname_downlevel.obj
 0002:000091a8       ??_C@_1M@HOKAOIO@?$AAa?$AAf?$AA?9?$AAZ?$AAA@ 100321a8     libucrt:lcidtoname_downlevel.obj
 0002:000091b4       ??_C@_1M@DPCLHLIE@?$AAk?$AAa?$AA?9?$AAG?$AAE@ 100321b4     libucrt:lcidtoname_downlevel.obj
 0002:000091c0       ??_C@_1M@BLKMHJBI@?$AAf?$AAo?$AA?9?$AAF?$AAO@ 100321c0     libucrt:lcidtoname_downlevel.obj
 0002:000091cc       ??_C@_1M@LGGJAPPB@?$AAh?$AAi?$AA?9?$AAI?$AAN@ 100321cc     libucrt:lcidtoname_downlevel.obj
 0002:000091d8       ??_C@_1M@FIKPIHFE@?$AAm?$AAt?$AA?9?$AAM?$AAT@ 100321d8     libucrt:lcidtoname_downlevel.obj
 0002:000091e4       ??_C@_1M@HEGGPBFA@?$AAs?$AAe?$AA?9?$AAN?$AAO@ 100321e4     libucrt:lcidtoname_downlevel.obj
 0002:000091f0       ??_C@_1M@EIBJEEPA@?$AAm?$AAs?$AA?9?$AAM?$AAY@ 100321f0     libucrt:lcidtoname_downlevel.obj
 0002:000091fc       ??_C@_1M@FHLBGMPP@?$AAk?$AAk?$AA?9?$AAK?$AAZ@ 100321fc     libucrt:lcidtoname_downlevel.obj
 0002:00009208       ??_C@_1M@NGJJLCGI@?$AAk?$AAy?$AA?9?$AAK?$AAG@ 10032208     libucrt:lcidtoname_downlevel.obj
 0002:00009214       ??_C@_1M@GIENNBFC@?$AAs?$AAw?$AA?9?$AAK?$AAE@ 10032214     libucrt:lcidtoname_downlevel.obj
 0002:00009220       ??_C@_1BG@NDGMJIMJ@?$AAu?$AAz?$AA?9?$AAU?$AAZ?$AA?9?$AAL?$AAa?$AAt?$AAn@ 10032220     libucrt:lcidtoname_downlevel.obj
 0002:00009238       ??_C@_1M@IDCCIHBC@?$AAt?$AAt?$AA?9?$AAR?$AAU@ 10032238     libucrt:lcidtoname_downlevel.obj
 0002:00009244       ??_C@_1M@LOICPMOJ@?$AAb?$AAn?$AA?9?$AAI?$AAN@ 10032244     libucrt:lcidtoname_downlevel.obj
 0002:00009250       ??_C@_1M@KPKKNEAH@?$AAp?$AAa?$AA?9?$AAI?$AAN@ 10032250     libucrt:lcidtoname_downlevel.obj
 0002:0000925c       ??_C@_1M@PJGPPBOG@?$AAg?$AAu?$AA?9?$AAI?$AAN@ 1003225c     libucrt:lcidtoname_downlevel.obj
 0002:00009268       ??_C@_1M@KMKMOPHI@?$AAt?$AAa?$AA?9?$AAI?$AAN@ 10032268     libucrt:lcidtoname_downlevel.obj
 0002:00009274       ??_C@_1M@KFEHEPAC@?$AAt?$AAe?$AA?9?$AAI?$AAN@ 10032274     libucrt:lcidtoname_downlevel.obj
 0002:00009280       ??_C@_1M@CDCLMGHI@?$AAk?$AAn?$AA?9?$AAI?$AAN@ 10032280     libucrt:lcidtoname_downlevel.obj
 0002:0000928c       ??_C@_1M@MIODLDKF@?$AAm?$AAl?$AA?9?$AAI?$AAN@ 1003228c     libucrt:lcidtoname_downlevel.obj
 0002:00009298       ??_C@_1M@PBIEACPO@?$AAm?$AAr?$AA?9?$AAI?$AAN@ 10032298     libucrt:lcidtoname_downlevel.obj
 0002:000092a4       ??_C@_1M@NIDEAGPH@?$AAs?$AAa?$AA?9?$AAI?$AAN@ 100322a4     libucrt:lcidtoname_downlevel.obj
 0002:000092b0       ??_C@_1M@FHIHCBIO@?$AAm?$AAn?$AA?9?$AAM?$AAN@ 100322b0     libucrt:lcidtoname_downlevel.obj
 0002:000092bc       ??_C@_1M@JAIJPENP@?$AAc?$AAy?$AA?9?$AAG?$AAB@ 100322bc     libucrt:lcidtoname_downlevel.obj
 0002:000092c8       ??_C@_1M@PHGFBEPN@?$AAg?$AAl?$AA?9?$AAE?$AAS@ 100322c8     libucrt:lcidtoname_downlevel.obj
 0002:000092d4       ??_C@_1O@KPIPDNCP@?$AAk?$AAo?$AAk?$AA?9?$AAI?$AAN@ 100322d4     libucrt:lcidtoname_downlevel.obj
 0002:000092e4       ??_C@_1O@KNHJLDJA@?$AAs?$AAy?$AAr?$AA?9?$AAS?$AAY@ 100322e4     libucrt:lcidtoname_downlevel.obj
 0002:000092f4       ??_C@_1O@MKEKBLAH@?$AAd?$AAi?$AAv?$AA?9?$AAM?$AAV@ 100322f4     libucrt:lcidtoname_downlevel.obj
 0002:00009304       ??_C@_1O@OHDCKDDF@?$AAq?$AAu?$AAz?$AA?9?$AAB?$AAO@ 10032304     libucrt:lcidtoname_downlevel.obj
 0002:00009314       ??_C@_1M@LEPJNLFD@?$AAn?$AAs?$AA?9?$AAZ?$AAA@ 10032314     libucrt:lcidtoname_downlevel.obj
 0002:00009320       ??_C@_1M@OMLEIIJB@?$AAm?$AAi?$AA?9?$AAN?$AAZ@ 10032320     libucrt:lcidtoname_downlevel.obj
 0002:0000932c       ??_C@_1M@PMPEAILG@?$AAa?$AAr?$AA?9?$AAI?$AAQ@ 1003232c     libucrt:lcidtoname_downlevel.obj
 0002:00009338       ??_C@_1M@CNKPNOEE@?$AAd?$AAe?$AA?9?$AAC?$AAH@ 10032338     libucrt:lcidtoname_downlevel.obj
 0002:00009344       ??_C@_1M@LKMGMLKO@?$AAe?$AAn?$AA?9?$AAG?$AAB@ 10032344     libucrt:lcidtoname_downlevel.obj
 0002:00009350       ??_C@_1M@PGKJFFGL@?$AAe?$AAs?$AA?9?$AAM?$AAX@ 10032350     libucrt:lcidtoname_downlevel.obj
 0002:0000935c       ??_C@_1M@DNNANBDC@?$AAf?$AAr?$AA?9?$AAB?$AAE@ 1003235c     libucrt:lcidtoname_downlevel.obj
 0002:00009368       ??_C@_1M@HLGMDFHM@?$AAi?$AAt?$AA?9?$AAC?$AAH@ 10032368     libucrt:lcidtoname_downlevel.obj
 0002:00009374       ??_C@_1M@CLLBGJH@?$AAn?$AAl?$AA?9?$AAB?$AAE@ 10032374     libucrt:lcidtoname_downlevel.obj
 0002:00009380       ??_C@_1M@BODBOGLF@?$AAn?$AAn?$AA?9?$AAN?$AAO@ 10032380     libucrt:lcidtoname_downlevel.obj
 0002:0000938c       ??_C@_1M@HFFAHKAD@?$AAp?$AAt?$AA?9?$AAP?$AAT@ 1003238c     libucrt:lcidtoname_downlevel.obj
 0002:00009398       ??_C@_1BG@LNOAKHIE@?$AAs?$AAr?$AA?9?$AAS?$AAP?$AA?9?$AAL?$AAa?$AAt?$AAn@ 10032398     libucrt:lcidtoname_downlevel.obj
 0002:000093b0       ??_C@_1M@HBMHBGAK@?$AAs?$AAv?$AA?9?$AAF?$AAI@ 100323b0     libucrt:lcidtoname_downlevel.obj
 0002:000093bc       ??_C@_1BG@DGCJGJBE@?$AAa?$AAz?$AA?9?$AAA?$AAZ?$AA?9?$AAC?$AAy?$AAr?$AAl@ 100323bc     libucrt:lcidtoname_downlevel.obj
 0002:000093d4       ??_C@_1M@KEJDAAHB@?$AAs?$AAe?$AA?9?$AAS?$AAE@ 100323d4     libucrt:lcidtoname_downlevel.obj
 0002:000093e0       ??_C@_1M@HEIBJJAD@?$AAm?$AAs?$AA?9?$AAB?$AAN@ 100323e0     libucrt:lcidtoname_downlevel.obj
 0002:000093ec       ??_C@_1BG@PBGJMCEM@?$AAu?$AAz?$AA?9?$AAU?$AAZ?$AA?9?$AAC?$AAy?$AAr?$AAl@ 100323ec     libucrt:lcidtoname_downlevel.obj
 0002:00009404       ??_C@_1O@LAOBCMDF@?$AAq?$AAu?$AAz?$AA?9?$AAE?$AAC@ 10032404     libucrt:lcidtoname_downlevel.obj
 0002:00009414       ??_C@_1M@POEEMAIO@?$AAa?$AAr?$AA?9?$AAE?$AAG@ 10032414     libucrt:lcidtoname_downlevel.obj
 0002:00009420       ??_C@_1M@EFAKDEDL@?$AAz?$AAh?$AA?9?$AAH?$AAK@ 10032420     libucrt:lcidtoname_downlevel.obj
 0002:0000942c       ??_C@_1M@HKKIJHGI@?$AAd?$AAe?$AA?9?$AAA?$AAT@ 1003242c     libucrt:lcidtoname_downlevel.obj
 0002:00009438       ??_C@_1M@KBFBEHJF@?$AAe?$AAn?$AA?9?$AAA?$AAU@ 10032438     libucrt:lcidtoname_downlevel.obj
 0002:00009444       ??_C@_1M@MNPLFAAH@?$AAe?$AAs?$AA?9?$AAE?$AAS@ 10032444     libucrt:lcidtoname_downlevel.obj
 0002:00009450       ??_C@_1M@HJOOJFMA@?$AAf?$AAr?$AA?9?$AAC?$AAA@ 10032450     libucrt:lcidtoname_downlevel.obj
 0002:0000945c       ??_C@_1BG@JPOFPNAB@?$AAs?$AAr?$AA?9?$AAS?$AAP?$AA?9?$AAC?$AAy?$AAr?$AAl@ 1003245c     libucrt:lcidtoname_downlevel.obj
 0002:00009474       ??_C@_1M@LNFOCMOB@?$AAs?$AAe?$AA?9?$AAF?$AAI@ 10032474     libucrt:lcidtoname_downlevel.obj
 0002:00009480       ??_C@_1O@MGJBOAMB@?$AAq?$AAu?$AAz?$AA?9?$AAP?$AAE@ 10032480     libucrt:lcidtoname_downlevel.obj
 0002:00009490       ??_C@_1M@GJINLBOK@?$AAa?$AAr?$AA?9?$AAL?$AAY@ 10032490     libucrt:lcidtoname_downlevel.obj
 0002:0000949c       ??_C@_1M@GGMNHJNL@?$AAz?$AAh?$AA?9?$AAS?$AAG@ 1003249c     libucrt:lcidtoname_downlevel.obj
 0002:000094a8       ??_C@_1M@HOIKODND@?$AAd?$AAe?$AA?9?$AAL?$AAU@ 100324a8     libucrt:lcidtoname_downlevel.obj
 0002:000094b4       ??_C@_1M@DDOCCGFG@?$AAe?$AAn?$AA?9?$AAC?$AAA@ 100324b4     libucrt:lcidtoname_downlevel.obj
 0002:000094c0       ??_C@_1M@BNOEMJLF@?$AAe?$AAs?$AA?9?$AAG?$AAT@ 100324c0     libucrt:lcidtoname_downlevel.obj
 0002:000094cc       ??_C@_1M@EOGNKEK@?$AAf?$AAr?$AA?9?$AAC?$AAH@ 100324cc     libucrt:lcidtoname_downlevel.obj
 0002:000094d8       ??_C@_1M@FLIDJFHL@?$AAh?$AAr?$AA?9?$AAB?$AAA@ 100324d8     libucrt:lcidtoname_downlevel.obj
 0002:000094e4       ??_C@_1O@FMCELNAJ@?$AAs?$AAm?$AAj?$AA?9?$AAN?$AAO@ 100324e4     libucrt:lcidtoname_downlevel.obj
 0002:000094f4       ??_C@_1M@JHGLJMGJ@?$AAa?$AAr?$AA?9?$AAD?$AAZ@ 100324f4     libucrt:lcidtoname_downlevel.obj
 0002:00009500       ??_C@_1M@JKKFDCNP@?$AAz?$AAh?$AA?9?$AAM?$AAO@ 10032500     libucrt:lcidtoname_downlevel.obj
 0002:0000950c       ??_C@_1M@GEEFALPE@?$AAd?$AAe?$AA?9?$AAL?$AAI@ 1003250c     libucrt:lcidtoname_downlevel.obj
 0002:00009518       ??_C@_1M@IGEOFBG@?$AAe?$AAn?$AA?9?$AAN?$AAZ@ 10032518     libucrt:lcidtoname_downlevel.obj
 0002:00009524       ??_C@_1M@KDBONEHP@?$AAe?$AAs?$AA?9?$AAC?$AAR@ 10032524     libucrt:lcidtoname_downlevel.obj
 0002:00009530       ??_C@_1M@FHMDOHNN@?$AAf?$AAr?$AA?9?$AAL?$AAU@ 10032530     libucrt:lcidtoname_downlevel.obj
 0002:0000953c       ??_C@_1BG@NFKKMAFG@?$AAb?$AAs?$AA?9?$AAB?$AAA?$AA?9?$AAL?$AAa?$AAt?$AAn@ 1003253c     libucrt:lcidtoname_downlevel.obj
 0002:00009554       ??_C@_1O@IMNBEMCI@?$AAs?$AAm?$AAj?$AA?9?$AAS?$AAE@ 10032554     libucrt:lcidtoname_downlevel.obj
 0002:00009564       ??_C@_1M@DHHMBNDP@?$AAa?$AAr?$AA?9?$AAM?$AAA@ 10032564     libucrt:lcidtoname_downlevel.obj
 0002:00009570       ??_C@_1M@BNBLJCGH@?$AAe?$AAn?$AA?9?$AAI?$AAE@ 10032570     libucrt:lcidtoname_downlevel.obj
 0002:0000957c       ??_C@_1M@GEPAFMDL@?$AAe?$AAs?$AA?9?$AAP?$AAA@ 1003257c     libucrt:lcidtoname_downlevel.obj
 0002:00009588       ??_C@_1M@OJONDMDL@?$AAf?$AAr?$AA?9?$AAM?$AAC@ 10032588     libucrt:lcidtoname_downlevel.obj
 0002:00009594       ??_C@_1BG@OBCNFJB@?$AAs?$AAr?$AA?9?$AAB?$AAA?$AA?9?$AAL?$AAa?$AAt?$AAn@ 10032594     libucrt:lcidtoname_downlevel.obj
 0002:000095ac       ??_C@_1O@KEMEEGPO@?$AAs?$AAm?$AAa?$AA?9?$AAN?$AAO@ 100325ac     libucrt:lcidtoname_downlevel.obj
 0002:000095bc       ??_C@_1M@ELMGFODK@?$AAa?$AAr?$AA?9?$AAT?$AAN@ 100325bc     libucrt:lcidtoname_downlevel.obj
 0002:000095c8       ??_C@_1M@BHDLHFAF@?$AAe?$AAn?$AA?9?$AAZ?$AAA@ 100325c8     libucrt:lcidtoname_downlevel.obj
 0002:000095d4       ??_C@_1M@BMGIGLIF@?$AAe?$AAs?$AA?9?$AAD?$AAO@ 100325d4     libucrt:lcidtoname_downlevel.obj
 0002:000095e0       ??_C@_1BG@CMBHIPBE@?$AAs?$AAr?$AA?9?$AAB?$AAA?$AA?9?$AAC?$AAy?$AAr?$AAl@ 100325e0     libucrt:lcidtoname_downlevel.obj
 0002:000095f8       ??_C@_1O@HEDBLHNP@?$AAs?$AAm?$AAa?$AA?9?$AAS?$AAE@ 100325f8     libucrt:lcidtoname_downlevel.obj
 0002:00009608       ??_C@_1M@DAGCADIM@?$AAa?$AAr?$AA?9?$AAO?$AAM@ 10032608     libucrt:lcidtoname_downlevel.obj
 0002:00009614       ??_C@_1M@FODLMICG@?$AAe?$AAn?$AA?9?$AAJ?$AAM@ 10032614     libucrt:lcidtoname_downlevel.obj
 0002:00009620       ??_C@_1M@DNMLCIHB@?$AAe?$AAs?$AA?9?$AAV?$AAE@ 10032620     libucrt:lcidtoname_downlevel.obj
 0002:0000962c       ??_C@_1O@EOKHMKJK@?$AAs?$AAm?$AAs?$AA?9?$AAF?$AAI@ 1003262c     libucrt:lcidtoname_downlevel.obj
 0002:0000963c       ??_C@_1M@CAFJMKOF@?$AAa?$AAr?$AA?9?$AAY?$AAE@ 1003263c     libucrt:lcidtoname_downlevel.obj
 0002:00009648       ??_C@_1M@CBFHIJLI@?$AAe?$AAn?$AA?9?$AAC?$AAB@ 10032648     libucrt:lcidtoname_downlevel.obj
 0002:00009654       ??_C@_1M@BGNFLDN@?$AAe?$AAs?$AA?9?$AAC?$AAO@ 10032654     libucrt:lcidtoname_downlevel.obj
 0002:00009660       ??_C@_1O@JMPHMAMC@?$AAs?$AAm?$AAn?$AA?9?$AAF?$AAI@ 10032660     libucrt:lcidtoname_downlevel.obj
 0002:00009670       ??_C@_1M@JLANABKE@?$AAa?$AAr?$AA?9?$AAS?$AAY@ 10032670     libucrt:lcidtoname_downlevel.obj
 0002:0000967c       ??_C@_1M@HPKGCFGN@?$AAe?$AAn?$AA?9?$AAB?$AAZ@ 1003267c     libucrt:lcidtoname_downlevel.obj
 0002:00009688       ??_C@_1M@OLJCMLGM@?$AAe?$AAs?$AA?9?$AAP?$AAE@ 10032688     libucrt:lcidtoname_downlevel.obj
 0002:00009694       ??_C@_1M@MKKGFKLE@?$AAa?$AAr?$AA?9?$AAJ?$AAO@ 10032694     libucrt:lcidtoname_downlevel.obj
 0002:000096a0       ??_C@_1M@EKPGLDNI@?$AAe?$AAn?$AA?9?$AAT?$AAT@ 100326a0     libucrt:lcidtoname_downlevel.obj
 0002:000096ac       ??_C@_1M@OONGHFHE@?$AAe?$AAs?$AA?9?$AAA?$AAR@ 100326ac     libucrt:lcidtoname_downlevel.obj
 0002:000096b8       ??_C@_1M@OOJFGBHE@?$AAa?$AAr?$AA?9?$AAL?$AAB@ 100326b8     libucrt:lcidtoname_downlevel.obj
 0002:000096c4       ??_C@_1M@GCEJHNEG@?$AAe?$AAn?$AA?9?$AAZ?$AAW@ 100326c4     libucrt:lcidtoname_downlevel.obj
 0002:000096d0       ??_C@_1M@JNOCAHJI@?$AAe?$AAs?$AA?9?$AAE?$AAC@ 100326d0     libucrt:lcidtoname_downlevel.obj
 0002:000096dc       ??_C@_1M@JEFHPGGB@?$AAa?$AAr?$AA?9?$AAK?$AAW@ 100326dc     libucrt:lcidtoname_downlevel.obj
 0002:000096e8       ??_C@_1M@MLKIBJOJ@?$AAe?$AAn?$AA?9?$AAP?$AAH@ 100326e8     libucrt:lcidtoname_downlevel.obj
 0002:000096f4       ??_C@_1M@BDNIPEND@?$AAe?$AAs?$AA?9?$AAC?$AAL@ 100326f4     libucrt:lcidtoname_downlevel.obj
 0002:00009700       ??_C@_1M@MPNMEKBD@?$AAa?$AAr?$AA?9?$AAA?$AAE@ 10032700     libucrt:lcidtoname_downlevel.obj
 0002:0000970c       ??_C@_1M@KBJALCPI@?$AAe?$AAs?$AA?9?$AAU?$AAY@ 1003270c     libucrt:lcidtoname_downlevel.obj
 0002:00009718       ??_C@_1M@LLCCOAGA@?$AAa?$AAr?$AA?9?$AAB?$AAH@ 10032718     libucrt:lcidtoname_downlevel.obj
 0002:00009724       ??_C@_1M@PBFNCDEL@?$AAe?$AAs?$AA?9?$AAP?$AAY@ 10032724     libucrt:lcidtoname_downlevel.obj
 0002:00009730       ??_C@_1M@EDGINPNP@?$AAa?$AAr?$AA?9?$AAQ?$AAA@ 10032730     libucrt:lcidtoname_downlevel.obj
 0002:0000973c       ??_C@_1M@MKDBIIJI@?$AAe?$AAs?$AA?9?$AAB?$AAO@ 1003273c     libucrt:lcidtoname_downlevel.obj
 0002:00009748       ??_C@_1M@CPKKEBLD@?$AAe?$AAs?$AA?9?$AAS?$AAV@ 10032748     libucrt:lcidtoname_downlevel.obj
 0002:00009754       ??_C@_1M@NDBGMMJL@?$AAe?$AAs?$AA?9?$AAH?$AAN@ 10032754     libucrt:lcidtoname_downlevel.obj
 0002:00009760       ??_C@_1M@JIJIBHDP@?$AAe?$AAs?$AA?9?$AAN?$AAI@ 10032760     libucrt:lcidtoname_downlevel.obj
 0002:0000976c       ??_C@_1M@CGFMKEEK@?$AAe?$AAs?$AA?9?$AAP?$AAR@ 1003276c     libucrt:lcidtoname_downlevel.obj
 0002:00009778       ??_C@_1O@ICJHKIIK@?$AAz?$AAh?$AA?9?$AAC?$AAH?$AAT@ 10032778     libucrt:lcidtoname_downlevel.obj
 0002:00009788       ??_C@_15CLNEJCE@?$AAs?$AAr@ 10032788     libucrt:lcidtoname_downlevel.obj
 0002:00009eb0       ??_C@_1M@KAHEKEIG@?$AAa?$AAf?$AA?9?$AAz?$AAa@ 10032eb0     libucrt:lcidtoname_downlevel.obj
 0002:00009ebc       ??_C@_1M@GIECOABL@?$AAa?$AAr?$AA?9?$AAa?$AAe@ 10032ebc     libucrt:lcidtoname_downlevel.obj
 0002:00009ec8       ??_C@_1M@BMLMEKGI@?$AAa?$AAr?$AA?9?$AAb?$AAh@ 10032ec8     libucrt:lcidtoname_downlevel.obj
 0002:00009ed4       ??_C@_1M@DAPFDGGB@?$AAa?$AAr?$AA?9?$AAd?$AAz@ 10032ed4     libucrt:lcidtoname_downlevel.obj
 0002:00009ee0       ??_C@_1M@FJNKGKIG@?$AAa?$AAr?$AA?9?$AAe?$AAg@ 10032ee0     libucrt:lcidtoname_downlevel.obj
 0002:00009eec       ??_C@_1M@FLGKKCLO@?$AAa?$AAr?$AA?9?$AAi?$AAq@ 10032eec     libucrt:lcidtoname_downlevel.obj
 0002:00009ef8       ??_C@_1M@GNDIPALM@?$AAa?$AAr?$AA?9?$AAj?$AAo@ 10032ef8     libucrt:lcidtoname_downlevel.obj
 0002:00009f04       ??_C@_1M@DDMJFMGJ@?$AAa?$AAr?$AA?9?$AAk?$AAw@ 10032f04     libucrt:lcidtoname_downlevel.obj
 0002:00009f10       ??_C@_1M@EJALMLHM@?$AAa?$AAr?$AA?9?$AAl?$AAb@ 10032f10     libucrt:lcidtoname_downlevel.obj
 0002:00009f1c       ??_C@_1M@MOBDBLOC@?$AAa?$AAr?$AA?9?$AAl?$AAy@ 10032f1c     libucrt:lcidtoname_downlevel.obj
 0002:00009f28       ??_C@_1M@JAOCLHDH@?$AAa?$AAr?$AA?9?$AAm?$AAa@ 10032f28     libucrt:lcidtoname_downlevel.obj
 0002:00009f34       ??_C@_1M@JHPMKJIE@?$AAa?$AAr?$AA?9?$AAo?$AAm@ 10032f34     libucrt:lcidtoname_downlevel.obj
 0002:00009f40       ??_C@_1M@OEPGHFNH@?$AAa?$AAr?$AA?9?$AAq?$AAa@ 10032f40     libucrt:lcidtoname_downlevel.obj
 0002:00009f4c       ??_C@_1M@KJDONENM@?$AAa?$AAr?$AA?9?$AAs?$AAa@ 10032f4c     libucrt:lcidtoname_downlevel.obj
 0002:00009f58       ??_C@_1M@DMJDKLKM@?$AAa?$AAr?$AA?9?$AAs?$AAy@ 10032f58     libucrt:lcidtoname_downlevel.obj
 0002:00009f64       ??_C@_1M@OMFIPEDC@?$AAa?$AAr?$AA?9?$AAt?$AAn@ 10032f64     libucrt:lcidtoname_downlevel.obj
 0002:00009f70       ??_C@_1M@IHMHGAON@?$AAa?$AAr?$AA?9?$AAy?$AAe@ 10032f70     libucrt:lcidtoname_downlevel.obj
 0002:00009f7c       ??_C@_1BG@KDCPGJGB@?$AAa?$AAz?$AA?9?$AAa?$AAz?$AA?9?$AAc?$AAy?$AAr?$AAl@ 10032f7c     libucrt:lcidtoname_downlevel.obj
 0002:00009f94       ??_C@_1BG@IBCKDDOE@?$AAa?$AAz?$AA?9?$AAa?$AAz?$AA?9?$AAl?$AAa?$AAt?$AAn@ 10032f94     libucrt:lcidtoname_downlevel.obj
 0002:00009fac       ??_C@_1M@EGPFDCPD@?$AAb?$AAe?$AA?9?$AAb?$AAy@ 10032fac     libucrt:lcidtoname_downlevel.obj
 0002:00009fb8       ??_C@_1M@PCMGMCGC@?$AAb?$AAg?$AA?9?$AAb?$AAg@ 10032fb8     libucrt:lcidtoname_downlevel.obj
 0002:00009fc4       ??_C@_1M@BJBMFGOB@?$AAb?$AAn?$AA?9?$AAi?$AAn@ 10032fc4     libucrt:lcidtoname_downlevel.obj
 0002:00009fd0       ??_C@_1BG@EAKMMACD@?$AAb?$AAs?$AA?9?$AAb?$AAa?$AA?9?$AAl?$AAa?$AAt?$AAn@ 10032fd0     libucrt:lcidtoname_downlevel.obj
 0002:00009fe8       ??_C@_1M@KGADAODK@?$AAc?$AAa?$AA?9?$AAe?$AAs@ 10032fe8     libucrt:lcidtoname_downlevel.obj
 0002:00009ff4       ??_C@_1M@COAJPDHI@?$AAc?$AAs?$AA?9?$AAc?$AAz@ 10032ff4     libucrt:lcidtoname_downlevel.obj
 0002:0000a000       ??_C@_1M@DHBHFONH@?$AAc?$AAy?$AA?9?$AAg?$AAb@ 10033000     libucrt:lcidtoname_downlevel.obj
 0002:0000a00c       ??_C@_1M@IMGKELGA@?$AAd?$AAa?$AA?9?$AAd?$AAk@ 1003300c     libucrt:lcidtoname_downlevel.obj
 0002:0000a018       ??_C@_1M@NNDGDNGA@?$AAd?$AAe?$AA?9?$AAa?$AAt@ 10033018     libucrt:lcidtoname_downlevel.obj
 0002:0000a024       ??_C@_1M@IKDBHEEM@?$AAd?$AAe?$AA?9?$AAc?$AAh@ 10033024     libucrt:lcidtoname_downlevel.obj
 0002:0000a030       ??_C@_1M@GFFOJMCJ@?$AAd?$AAe?$AA?9?$AAd?$AAe@ 10033030     libucrt:lcidtoname_downlevel.obj
 0002:0000a03c       ??_C@_1M@MDNLKBPM@?$AAd?$AAe?$AA?9?$AAl?$AAi@ 1003303c     libucrt:lcidtoname_downlevel.obj
 0002:0000a048       ??_C@_1M@NJBEEJNL@?$AAd?$AAe?$AA?9?$AAl?$AAu@ 10033048     libucrt:lcidtoname_downlevel.obj
 0002:0000a054       ??_C@_1O@GNNELBAP@?$AAd?$AAi?$AAv?$AA?9?$AAm?$AAv@ 10033054     libucrt:lcidtoname_downlevel.obj
 0002:0000a064       ??_C@_1M@EJLEOGAE@?$AAe?$AAl?$AA?9?$AAg?$AAr@ 10033064     libucrt:lcidtoname_downlevel.obj
 0002:0000a070       ??_C@_1M@GMPONJN@?$AAe?$AAn?$AA?9?$AAa?$AAu@ 10033070     libucrt:lcidtoname_downlevel.obj
 0002:0000a07c       ??_C@_1M@NIDIIPGF@?$AAe?$AAn?$AA?9?$AAb?$AAz@ 1003307c     libucrt:lcidtoname_downlevel.obj
 0002:0000a088       ??_C@_1M@JEHMIMFO@?$AAe?$AAn?$AA?9?$AAc?$AAa@ 10033088     libucrt:lcidtoname_downlevel.obj
 0002:0000a094       ??_C@_1M@IGMJCDLA@?$AAe?$AAn?$AA?9?$AAc?$AAb@ 10033094     libucrt:lcidtoname_downlevel.obj
 0002:0000a0a0       ??_C@_1M@BNFIGBKG@?$AAe?$AAn?$AA?9?$AAg?$AAb@ 100330a0     libucrt:lcidtoname_downlevel.obj
 0002:0000a0ac       ??_C@_1M@LKIFDIGP@?$AAe?$AAn?$AA?9?$AAi?$AAe@ 100330ac     libucrt:lcidtoname_downlevel.obj
 0002:0000a0b8       ??_C@_1M@PJKFGCCO@?$AAe?$AAn?$AA?9?$AAj?$AAm@ 100330b8     libucrt:lcidtoname_downlevel.obj
 0002:0000a0c4       ??_C@_1M@KPPKEPBO@?$AAe?$AAn?$AA?9?$AAn?$AAz@ 100330c4     libucrt:lcidtoname_downlevel.obj
 0002:0000a0d0       ??_C@_1M@GMDGLDOB@?$AAe?$AAn?$AA?9?$AAp?$AAh@ 100330d0     libucrt:lcidtoname_downlevel.obj
 0002:0000a0dc       ??_C@_1M@ONGIBJNA@?$AAe?$AAn?$AA?9?$AAt?$AAt@ 100330dc     libucrt:lcidtoname_downlevel.obj
 0002:0000a0e8       ??_C@_1M@LLODPCMM@?$AAe?$AAn?$AA?9?$AAu?$AAs@ 100330e8     libucrt:lcidtoname_downlevel.obj
 0002:0000a0f4       ??_C@_1M@LAKFNPAN@?$AAe?$AAn?$AA?9?$AAz?$AAa@ 100330f4     libucrt:lcidtoname_downlevel.obj
 0002:0000a100       ??_C@_1M@MFNHNHEO@?$AAe?$AAn?$AA?9?$AAz?$AAw@ 10033100     libucrt:lcidtoname_downlevel.obj
 0002:0000a10c       ??_C@_1M@EJEINPHM@?$AAe?$AAs?$AA?9?$AAa?$AAr@ 1003310c     libucrt:lcidtoname_downlevel.obj
 0002:0000a118       ??_C@_1M@GNKPCCJA@?$AAe?$AAs?$AA?9?$AAb?$AAo@ 10033118     libucrt:lcidtoname_downlevel.obj
 0002:0000a124       ??_C@_1M@LEEGFONL@?$AAe?$AAs?$AA?9?$AAc?$AAl@ 10033124     libucrt:lcidtoname_downlevel.obj
 0002:0000a130       ??_C@_1M@KGPDPBDF@?$AAe?$AAs?$AA?9?$AAc?$AAo@ 10033130     libucrt:lcidtoname_downlevel.obj
 0002:0000a13c       ??_C@_1M@EIAHOHH@?$AAe?$AAs?$AA?9?$AAc?$AAr@ 1003313c     libucrt:lcidtoname_downlevel.obj
 0002:0000a148       ??_C@_1M@LLPGMBIN@?$AAe?$AAs?$AA?9?$AAd?$AAo@ 10033148     libucrt:lcidtoname_downlevel.obj
 0002:0000a154       ??_C@_1M@DKHMKNJA@?$AAe?$AAs?$AA?9?$AAe?$AAc@ 10033154     libucrt:lcidtoname_downlevel.obj
 0002:0000a160       ??_C@_1M@GKGFPKAP@?$AAe?$AAs?$AA?9?$AAe?$AAs@ 10033160     libucrt:lcidtoname_downlevel.obj
 0002:0000a16c       ??_C@_1M@LKHKGDLN@?$AAe?$AAs?$AA?9?$AAg?$AAt@ 1003316c     libucrt:lcidtoname_downlevel.obj
 0002:0000a178       ??_C@_1M@HEIIGGJD@?$AAe?$AAs?$AA?9?$AAh?$AAn@ 10033178     libucrt:lcidtoname_downlevel.obj
 0002:0000a184       ??_C@_1M@FBDHPPGD@?$AAe?$AAs?$AA?9?$AAm?$AAx@ 10033184     libucrt:lcidtoname_downlevel.obj
 0002:0000a190       ??_C@_1M@DPAGLNDH@?$AAe?$AAs?$AA?9?$AAn?$AAi@ 10033190     libucrt:lcidtoname_downlevel.obj
 0002:0000a19c       ??_C@_1M@MDGOPGDD@?$AAe?$AAs?$AA?9?$AAp?$AAa@ 1003319c     libucrt:lcidtoname_downlevel.obj
 0002:0000a1a8       ??_C@_1M@EMAMGBGE@?$AAe?$AAs?$AA?9?$AAp?$AAe@ 100331a8     libucrt:lcidtoname_downlevel.obj
 0002:0000a1b4       ??_C@_1M@IBMCAOEC@?$AAe?$AAs?$AA?9?$AAp?$AAr@ 100331b4     libucrt:lcidtoname_downlevel.obj
 0002:0000a1c0       ??_C@_1M@FGMDIJED@?$AAe?$AAs?$AA?9?$AAp?$AAy@ 100331c0     libucrt:lcidtoname_downlevel.obj
 0002:0000a1cc       ??_C@_1M@IIDEOLLL@?$AAe?$AAs?$AA?9?$AAs?$AAv@ 100331cc     libucrt:lcidtoname_downlevel.obj
 0002:0000a1d8       ??_C@_1M@GAOBIPA@?$AAe?$AAs?$AA?9?$AAu?$AAy@ 100331d8     libucrt:lcidtoname_downlevel.obj
 0002:0000a1e4       ??_C@_1M@JKFFICHJ@?$AAe?$AAs?$AA?9?$AAv?$AAe@ 100331e4     libucrt:lcidtoname_downlevel.obj
 0002:0000a1f0       ??_C@_1M@PNMLOJDF@?$AAe?$AAt?$AA?9?$AAe?$AAe@ 100331f0     libucrt:lcidtoname_downlevel.obj
 0002:0000a1fc       ??_C@_1M@GHHLIKEI@?$AAe?$AAu?$AA?9?$AAe?$AAs@ 100331fc     libucrt:lcidtoname_downlevel.obj
 0002:0000a208       ??_C@_1M@PBNONODE@?$AAf?$AAa?$AA?9?$AAi?$AAr@ 10033208     libucrt:lcidtoname_downlevel.obj
 0002:0000a214       ??_C@_1M@JEEHPMIL@?$AAf?$AAi?$AA?9?$AAf?$AAi@ 10033214     libucrt:lcidtoname_downlevel.obj
 0002:0000a220       ??_C@_1M@LMDCNDBA@?$AAf?$AAo?$AA?9?$AAf?$AAo@ 10033220     libucrt:lcidtoname_downlevel.obj
 0002:0000a22c       ??_C@_1M@JKEOHLDK@?$AAf?$AAr?$AA?9?$AAb?$AAe@ 1003322c     libucrt:lcidtoname_downlevel.obj
 0002:0000a238       ??_C@_1M@NOHADPMI@?$AAf?$AAr?$AA?9?$AAc?$AAa@ 10033238     libucrt:lcidtoname_downlevel.obj
 0002:0000a244       ??_C@_1M@KDHIHAEC@?$AAf?$AAr?$AA?9?$AAc?$AAh@ 10033244     libucrt:lcidtoname_downlevel.obj
 0002:0000a250       ??_C@_1M@MMBBFGAK@?$AAf?$AAr?$AA?9?$AAf?$AAr@ 10033250     libucrt:lcidtoname_downlevel.obj
 0002:0000a25c       ??_C@_1M@PAFNENNF@?$AAf?$AAr?$AA?9?$AAl?$AAu@ 1003325c     libucrt:lcidtoname_downlevel.obj
 0002:0000a268       ??_C@_1M@EOHDJGDD@?$AAf?$AAr?$AA?9?$AAm?$AAc@ 10033268     libucrt:lcidtoname_downlevel.obj
 0002:0000a274       ??_C@_1M@FAPLLOPF@?$AAg?$AAl?$AA?9?$AAe?$AAs@ 10033274     libucrt:lcidtoname_downlevel.obj
 0002:0000a280       ??_C@_1M@FOPBFLOO@?$AAg?$AAu?$AA?9?$AAi?$AAn@ 10033280     libucrt:lcidtoname_downlevel.obj
 0002:0000a28c       ??_C@_1M@KBMCINPM@?$AAh?$AAe?$AA?9?$AAi?$AAl@ 1003328c     libucrt:lcidtoname_downlevel.obj
 0002:0000a298       ??_C@_1M@BBPHKFPJ@?$AAh?$AAi?$AA?9?$AAi?$AAn@ 10033298     libucrt:lcidtoname_downlevel.obj
 0002:0000a2a4       ??_C@_1M@PMBNDPHD@?$AAh?$AAr?$AA?9?$AAb?$AAa@ 100332a4     libucrt:lcidtoname_downlevel.obj
 0002:0000a2b0       ??_C@_1M@BPCKOEGE@?$AAh?$AAr?$AA?9?$AAh?$AAr@ 100332b0     libucrt:lcidtoname_downlevel.obj
 0002:0000a2bc       ??_C@_1M@GACBMHKE@?$AAh?$AAu?$AA?9?$AAh?$AAu@ 100332bc     libucrt:lcidtoname_downlevel.obj
 0002:0000a2c8       ??_C@_1M@MILPAJJC@?$AAh?$AAy?$AA?9?$AAa?$AAm@ 100332c8     libucrt:lcidtoname_downlevel.obj
 0002:0000a2d4       ??_C@_1M@BABBICEC@?$AAi?$AAd?$AA?9?$AAi?$AAd@ 100332d4     libucrt:lcidtoname_downlevel.obj
 0002:0000a2e0       ??_C@_1M@BIKNHHPF@?$AAi?$AAs?$AA?9?$AAi?$AAs@ 100332e0     libucrt:lcidtoname_downlevel.obj
 0002:0000a2ec       ??_C@_1M@NMPCJPHE@?$AAi?$AAt?$AA?9?$AAc?$AAh@ 100332ec     libucrt:lcidtoname_downlevel.obj
 0002:0000a2f8       ??_C@_1M@GHKGFEDF@?$AAi?$AAt?$AA?9?$AAi?$AAt@ 100332f8     libucrt:lcidtoname_downlevel.obj
 0002:0000a304       ??_C@_1M@NIEJCJJA@?$AAj?$AAa?$AA?9?$AAj?$AAp@ 10033304     libucrt:lcidtoname_downlevel.obj
 0002:0000a310       ??_C@_1M@JILFNBIM@?$AAk?$AAa?$AA?9?$AAg?$AAe@ 10033310     libucrt:lcidtoname_downlevel.obj
 0002:0000a31c       ??_C@_1M@PACPMGPH@?$AAk?$AAk?$AA?9?$AAk?$AAz@ 1003331c     libucrt:lcidtoname_downlevel.obj
 0002:0000a328       ??_C@_1M@IELFGMHA@?$AAk?$AAn?$AA?9?$AAi?$AAn@ 10033328     libucrt:lcidtoname_downlevel.obj
 0002:0000a334       ??_C@_1O@IBBJHCH@?$AAk?$AAo?$AAk?$AA?9?$AAi?$AAn@ 10033334     libucrt:lcidtoname_downlevel.obj
 0002:0000a344       ??_C@_1M@DMHAEOGC@?$AAk?$AAo?$AA?9?$AAk?$AAr@ 10033344     libucrt:lcidtoname_downlevel.obj
 0002:0000a350       ??_C@_1M@HBAHBIGA@?$AAk?$AAy?$AA?9?$AAk?$AAg@ 10033350     libucrt:lcidtoname_downlevel.obj
 0002:0000a35c       ??_C@_1M@KPMILCJG@?$AAl?$AAt?$AA?9?$AAl?$AAt@ 1003335c     libucrt:lcidtoname_downlevel.obj
 0002:0000a368       ??_C@_1M@BDEKKCA@?$AAl?$AAv?$AA?9?$AAl?$AAv@ 10033368     libucrt:lcidtoname_downlevel.obj
 0002:0000a374       ??_C@_1M@ELCKCCJJ@?$AAm?$AAi?$AA?9?$AAn?$AAz@ 10033374     libucrt:lcidtoname_downlevel.obj
 0002:0000a380       ??_C@_1M@CBOOLAPA@?$AAm?$AAk?$AA?9?$AAm?$AAk@ 10033380     libucrt:lcidtoname_downlevel.obj
 0002:0000a38c       ??_C@_1M@GPHNBJKN@?$AAm?$AAl?$AA?9?$AAi?$AAn@ 1003338c     libucrt:lcidtoname_downlevel.obj
 0002:0000a398       ??_C@_1M@PABJILIG@?$AAm?$AAn?$AA?9?$AAm?$AAn@ 10033398     libucrt:lcidtoname_downlevel.obj
 0002:0000a3a4       ??_C@_1M@FGBKKIPG@?$AAm?$AAr?$AA?9?$AAi?$AAn@ 100333a4     libucrt:lcidtoname_downlevel.obj
 0002:0000a3b0       ??_C@_1M@NDBPDDAL@?$AAm?$AAs?$AA?9?$AAb?$AAn@ 100333b0     libucrt:lcidtoname_downlevel.obj
 0002:0000a3bc       ??_C@_1M@OPIHOOPI@?$AAm?$AAs?$AA?9?$AAm?$AAy@ 100333bc     libucrt:lcidtoname_downlevel.obj
 0002:0000a3c8       ??_C@_1M@PPDBCNFM@?$AAm?$AAt?$AA?9?$AAm?$AAt@ 100333c8     libucrt:lcidtoname_downlevel.obj
 0002:0000a3d4       ??_C@_1M@KDJDKMDD@?$AAn?$AAb?$AA?9?$AAn?$AAo@ 100333d4     libucrt:lcidtoname_downlevel.obj
 0002:0000a3e0       ??_C@_1M@KFCFLMJP@?$AAn?$AAl?$AA?9?$AAb?$AAe@ 100333e0     libucrt:lcidtoname_downlevel.obj
 0002:0000a3ec       ??_C@_1M@KPOPDDGO@?$AAn?$AAl?$AA?9?$AAn?$AAl@ 100333ec     libucrt:lcidtoname_downlevel.obj
 0002:0000a3f8       ??_C@_1M@LJKPEMLN@?$AAn?$AAn?$AA?9?$AAn?$AAo@ 100333f8     libucrt:lcidtoname_downlevel.obj
 0002:0000a404       ??_C@_1M@BDGHHBFL@?$AAn?$AAs?$AA?9?$AAz?$AAa@ 10033404     libucrt:lcidtoname_downlevel.obj
 0002:0000a410       ??_C@_1M@IDEHOAP@?$AAp?$AAa?$AA?9?$AAi?$AAn@ 10033410     libucrt:lcidtoname_downlevel.obj
 0002:0000a41c       ??_C@_1M@HDBKGOGH@?$AAp?$AAl?$AA?9?$AAp?$AAl@ 1003341c     libucrt:lcidtoname_downlevel.obj
 0002:0000a428       ??_C@_1M@LJLLCMEH@?$AAp?$AAt?$AA?9?$AAb?$AAr@ 10033428     libucrt:lcidtoname_downlevel.obj
 0002:0000a434       ??_C@_1M@NCMONAAL@?$AAp?$AAt?$AA?9?$AAp?$AAt@ 10033434     libucrt:lcidtoname_downlevel.obj
 0002:0000a440       ??_C@_1O@EAKMAJDN@?$AAq?$AAu?$AAz?$AA?9?$AAb?$AAo@ 10033440     libucrt:lcidtoname_downlevel.obj
 0002:0000a450       ??_C@_1O@BHHPIGDN@?$AAq?$AAu?$AAz?$AA?9?$AAe?$AAc@ 10033450     libucrt:lcidtoname_downlevel.obj
 0002:0000a460       ??_C@_1O@GBAPEKMJ@?$AAq?$AAu?$AAz?$AA?9?$AAp?$AAe@ 10033460     libucrt:lcidtoname_downlevel.obj
 0002:0000a470       ??_C@_1M@CLGLEFBO@?$AAr?$AAo?$AA?9?$AAr?$AAo@ 10033470     libucrt:lcidtoname_downlevel.obj
 0002:0000a47c       ??_C@_1M@CEEDODME@?$AAr?$AAu?$AA?9?$AAr?$AAu@ 1003347c     libucrt:lcidtoname_downlevel.obj
 0002:0000a488       ??_C@_1M@HPKKKMPP@?$AAs?$AAa?$AA?9?$AAi?$AAn@ 10033488     libucrt:lcidtoname_downlevel.obj
 0002:0000a494       ??_C@_1M@BKMAIGOJ@?$AAs?$AAe?$AA?9?$AAf?$AAi@ 10033494     libucrt:lcidtoname_downlevel.obj
 0002:0000a4a0       ??_C@_1M@NDPIFLFI@?$AAs?$AAe?$AA?9?$AAn?$AAo@ 100334a0     libucrt:lcidtoname_downlevel.obj
 0002:0000a4ac       ??_C@_1M@DANKKHJ@?$AAs?$AAe?$AA?9?$AAs?$AAe@ 100334ac     libucrt:lcidtoname_downlevel.obj
 0002:0000a4b8       ??_C@_1M@PNBLONPJ@?$AAs?$AAk?$AA?9?$AAs?$AAk@ 100334b8     libucrt:lcidtoname_downlevel.obj
 0002:0000a4c4       ??_C@_1M@LFMODOAL@?$AAs?$AAl?$AA?9?$AAs?$AAi@ 100334c4     libucrt:lcidtoname_downlevel.obj
 0002:0000a4d0       ??_C@_1O@DFKOMPG@?$AAs?$AAm?$AAa?$AA?9?$AAn?$AAo@ 100334d0     libucrt:lcidtoname_downlevel.obj
 0002:0000a4e0       ??_C@_1O@NDKPBNNH@?$AAs?$AAm?$AAa?$AA?9?$AAs?$AAe@ 100334e0     libucrt:lcidtoname_downlevel.obj
 0002:0000a4f0       ??_C@_1O@PLLKBHAB@?$AAs?$AAm?$AAj?$AA?9?$AAn?$AAo@ 100334f0     libucrt:lcidtoname_downlevel.obj
 0002:0000a500       ??_C@_1O@CLEPOGCA@?$AAs?$AAm?$AAj?$AA?9?$AAs?$AAe@ 10033500     libucrt:lcidtoname_downlevel.obj
 0002:0000a510       ??_C@_1O@DLGJGKMK@?$AAs?$AAm?$AAn?$AA?9?$AAf?$AAi@ 10033510     libucrt:lcidtoname_downlevel.obj
 0002:0000a520       ??_C@_1O@OJDJGAJC@?$AAs?$AAm?$AAs?$AA?9?$AAf?$AAi@ 10033520     libucrt:lcidtoname_downlevel.obj
 0002:0000a530       ??_C@_1M@BOFOGHPB@?$AAs?$AAq?$AA?9?$AAa?$AAl@ 10033530     libucrt:lcidtoname_downlevel.obj
 0002:0000a53c       ??_C@_1BG@LJBBIPGB@?$AAs?$AAr?$AA?9?$AAb?$AAa?$AA?9?$AAc?$AAy?$AAr?$AAl@ 1003353c     libucrt:lcidtoname_downlevel.obj
 0002:0000a554       ??_C@_1BG@JLBENFOE@?$AAs?$AAr?$AA?9?$AAb?$AAa?$AA?9?$AAl?$AAa?$AAt?$AAn@ 10033554     libucrt:lcidtoname_downlevel.obj
 0002:0000a56c       ??_C@_1BG@KODPNHE@?$AAs?$AAr?$AA?9?$AAs?$AAp?$AA?9?$AAc?$AAy?$AAr?$AAl@ 1003356c     libucrt:lcidtoname_downlevel.obj
 0002:0000a584       ??_C@_1BG@CIOGKHPB@?$AAs?$AAr?$AA?9?$AAs?$AAp?$AA?9?$AAl?$AAa?$AAt?$AAn@ 10033584     libucrt:lcidtoname_downlevel.obj
 0002:0000a59c       ??_C@_1M@NGFJLMAC@?$AAs?$AAv?$AA?9?$AAf?$AAi@ 1003359c     libucrt:lcidtoname_downlevel.obj
 0002:0000a5a8       ??_C@_1M@MPJEJAJC@?$AAs?$AAv?$AA?9?$AAs?$AAe@ 100335a8     libucrt:lcidtoname_downlevel.obj
 0002:0000a5b4       ??_C@_1M@MPNDHLFK@?$AAs?$AAw?$AA?9?$AAk?$AAe@ 100335b4     libucrt:lcidtoname_downlevel.obj
 0002:0000a5c0       ??_C@_1O@KOHBJJI@?$AAs?$AAy?$AAr?$AA?9?$AAs?$AAy@ 100335c0     libucrt:lcidtoname_downlevel.obj
 0002:0000a5d0       ??_C@_1M@LDCEFHA@?$AAt?$AAa?$AA?9?$AAi?$AAn@ 100335d0     libucrt:lcidtoname_downlevel.obj
 0002:0000a5dc       ??_C@_1M@CNJOFAK@?$AAt?$AAe?$AA?9?$AAi?$AAn@ 100335dc     libucrt:lcidtoname_downlevel.obj
 0002:0000a5e8       ??_C@_1M@GNAECACD@?$AAt?$AAh?$AA?9?$AAt?$AAh@ 100335e8     libucrt:lcidtoname_downlevel.obj
 0002:0000a5f4       ??_C@_1M@CHBIHOJO@?$AAt?$AAn?$AA?9?$AAz?$AAa@ 100335f4     libucrt:lcidtoname_downlevel.obj
 0002:0000a600       ??_C@_1M@GCCMIGPJ@?$AAt?$AAr?$AA?9?$AAt?$AAr@ 10033600     libucrt:lcidtoname_downlevel.obj
 0002:0000a60c       ??_C@_1M@CELMCNBK@?$AAt?$AAt?$AA?9?$AAr?$AAu@ 1003360c     libucrt:lcidtoname_downlevel.obj
 0002:0000a618       ??_C@_1M@KLMCELGA@?$AAu?$AAk?$AA?9?$AAu?$AAa@ 10033618     libucrt:lcidtoname_downlevel.obj
 0002:0000a624       ??_C@_1M@EPAJJAJF@?$AAu?$AAr?$AA?9?$AAp?$AAk@ 10033624     libucrt:lcidtoname_downlevel.obj
 0002:0000a630       ??_C@_1BG@GEGPMCDJ@?$AAu?$AAz?$AA?9?$AAu?$AAz?$AA?9?$AAc?$AAy?$AAr?$AAl@ 10033630     libucrt:lcidtoname_downlevel.obj
 0002:0000a648       ??_C@_1BG@EGGKJILM@?$AAu?$AAz?$AA?9?$AAu?$AAz?$AA?9?$AAl?$AAa?$AAt?$AAn@ 10033648     libucrt:lcidtoname_downlevel.obj
 0002:0000a660       ??_C@_1M@GFOCLFF@?$AAv?$AAi?$AA?9?$AAv?$AAn@ 10033660     libucrt:lcidtoname_downlevel.obj
 0002:0000a66c       ??_C@_1M@CPAMEDFI@?$AAx?$AAh?$AA?9?$AAz?$AAa@ 1003366c     libucrt:lcidtoname_downlevel.obj
 0002:0000a678       ??_C@_1O@EBKIFIGN@?$AAz?$AAh?$AA?9?$AAc?$AAh?$AAs@ 10033678     libucrt:lcidtoname_downlevel.obj
 0002:0000a688       ??_C@_1O@NMHPGANE@?$AAz?$AAh?$AA?9?$AAc?$AAh?$AAt@ 10033688     libucrt:lcidtoname_downlevel.obj
 0002:0000a698       ??_C@_1M@LPINJOMC@?$AAz?$AAh?$AA?9?$AAc?$AAn@ 10033698     libucrt:lcidtoname_downlevel.obj
 0002:0000a6a4       ??_C@_1M@OCJEJODD@?$AAz?$AAh?$AA?9?$AAh?$AAk@ 100336a4     libucrt:lcidtoname_downlevel.obj
 0002:0000a6b0       ??_C@_1M@DNDLJINH@?$AAz?$AAh?$AA?9?$AAm?$AAo@ 100336b0     libucrt:lcidtoname_downlevel.obj
 0002:0000a6bc       ??_C@_1M@MBFDNDND@?$AAz?$AAh?$AA?9?$AAs?$AAg@ 100336bc     libucrt:lcidtoname_downlevel.obj
 0002:0000a6c8       ??_C@_1M@IMEPLEPE@?$AAz?$AAh?$AA?9?$AAt?$AAw@ 100336c8     libucrt:lcidtoname_downlevel.obj
 0002:0000a6d4       ??_C@_1M@BBGHNHJP@?$AAz?$AAu?$AA?9?$AAz?$AAa@ 100336d4     libucrt:lcidtoname_downlevel.obj
 0002:0000a6e0       ??_C@_05DNEBIAHO@1?$CDINF@ 100336e0     libucrt:cfout.obj
 0002:0000a6e8       ??_C@_06IMKFLFPG@1?$CDQNAN@ 100336e8     libucrt:cfout.obj
 0002:0000a6f0       ??_C@_06PGGFOGJG@1?$CDSNAN@ 100336f0     libucrt:cfout.obj
 0002:0000a6f8       ??_C@_05PHHOCPM@1?$CDIND@  100336f8     libucrt:cfout.obj
 0002:0000a700       ??_C@_15HNJCPLHL@?$AAT?$AAZ@ 10033700     libucrt:tzset.obj
 0002:0000a708       __days                     10033708     libucrt:days.obj
 0002:0000a73c       __lpdays                   1003373c     libucrt:days.obj
 0002:0000a7c8       ??_C@_1BA@BALFACEM@?$AAC?$AAO?$AAN?$AAO?$AAU?$AAT?$AA$@ 100337c8     libucrt:initcon.obj
 0002:0000a8e0       __infinity                 100338e0     libucrt:87tran.obj
 0002:0000a8ea       __minfinity                100338ea     libucrt:87tran.obj
 0002:0000a8f4       __logemax                  100338f4     libucrt:87tran.obj
 0002:0000a91a       __OP_EXPjmptab             1003391a     libucrt:87tran.obj
 0002:0000a940       __indefinite               10033940     libucrt:87disp.obj
 0002:0000a94a       __piby2                    1003394a     libucrt:87disp.obj
 0002:0000a954       __piby4                    10033954     libucrt:87disp.obj
 0002:0000a988       __DEFAULT_CW_in_mem        10033988     libucrt:common.obj
 0002:0000a98a       __pi_by_2_to_61            1003398a     libucrt:common.obj
 0002:0000a9c4       ??_C@_03MGHMBJCF@log@      100339c4     libucrt:libm_error.obj
 0002:0000a9c8       ??_C@_05HGHHAHAP@log10@    100339c8     libucrt:libm_error.obj
 0002:0000a9d0       ??_C@_03KHJOGHMM@exp@      100339d0     libucrt:libm_error.obj
 0002:0000a9d4       ??_C@_03JGHBODFD@pow@      100339d4     libucrt:libm_error.obj
 0002:0000a9d8       ??_C@_04FIHNOPOL@asin@     100339d8     libucrt:libm_error.obj
 0002:0000a9e0       ??_C@_04PDIFKINK@acos@     100339e0     libucrt:libm_error.obj
 0002:0000a9e8       ??_C@_04EIAKFFMI@sqrt@     100339e8     libucrt:libm_error.obj
 0002:0000a9f0       __real@3ff0000000000000    100339f0     libucrt:libm_error.obj
 0002:0000aa10       ___acrt_log10_table_t      10033a10     libucrt:log10_tables.obj
 0002:0000ae20       ___acrt_log10_table_cb     10033e20     libucrt:log10_tables.obj
 0002:0000b230       __real@3fe0000000000000    10034230     libucrt:powhlp.obj
 0002:0000b320       ??_C@_04COOMCNPB@sinh@     10034320     libucrt:fpexcept.obj
 0002:0000b328       ??_C@_04HPJJNFIM@cosh@     10034328     libucrt:fpexcept.obj
 0002:0000b330       ??_C@_04FJHINJAO@tanh@     10034330     libucrt:fpexcept.obj
 0002:0000b338       ??_C@_04MLLJIGOK@atan@     10034338     libucrt:fpexcept.obj
 0002:0000b340       ??_C@_05KNGEOGJB@atan2@    10034340     libucrt:fpexcept.obj
 0002:0000b348       ??_C@_03BLEJJJBH@sin@      10034348     libucrt:fpexcept.obj
 0002:0000b34c       ??_C@_03LALBNOCG@cos@      1003434c     libucrt:fpexcept.obj
 0002:0000b350       ??_C@_03IIINPABG@tan@      10034350     libucrt:fpexcept.obj
 0002:0000b354       ??_C@_04GFPJNGEK@ceil@     10034354     libucrt:fpexcept.obj
 0002:0000b35c       ??_C@_05PBJFFIGL@floor@    1003435c     libucrt:fpexcept.obj
 0002:0000b364       ??_C@_04ODHECPBC@fabs@     10034364     libucrt:fpexcept.obj
 0002:0000b36c       ??_C@_04EHEDPDJG@modf@     1003436c     libucrt:fpexcept.obj
 0002:0000b374       ??_C@_05CEJMAHNP@ldexp@    10034374     libucrt:fpexcept.obj
 0002:0000b37c       ??_C@_05KBKMEMPO@_cabs@    1003437c     libucrt:fpexcept.obj
 0002:0000b384       ??_C@_06MEIMCGCF@_hypot@   10034384     libucrt:fpexcept.obj
 0002:0000b38c       ??_C@_04KEPJIHGP@fmod@     1003438c     libucrt:fpexcept.obj
 0002:0000b394       ??_C@_05GKKHEGJL@frexp@    10034394     libucrt:fpexcept.obj
 0002:0000b39c       ??_C@_03MJLDFKDL@_y0@      1003439c     libucrt:fpexcept.obj
 0002:0000b3a0       ??_C@_03NAKIGLHK@_y1@      100343a0     libucrt:fpexcept.obj
 0002:0000b3a4       ??_C@_03ONILCKOB@_yn@      100343a4     libucrt:fpexcept.obj
 0002:0000b3a8       ??_C@_05JGDBENOH@_logb@    100343a8     libucrt:fpexcept.obj
 0002:0000b3b0       ??_C@_0L@KDOEJCKC@_nextafter@ 100343b0     libucrt:fpexcept.obj
 0002:0000b3c0       __d_inf                    100343c0     libucrt:util.obj
 0002:0000b3c8       __d_max                    100343c8     libucrt:util.obj
 0002:0000b3d0       __d_mzero                  100343d0     libucrt:util.obj
 0002:0000b3dc       ??_7type_info@@6B@         100343dc     LIBCMT:std_type_info_static.obj
 0002:0000b3f0       __xmm@00000000000000000000000000000000 100343f0     libvcruntime:wcschr.obj
 0002:0000b400       __load_config_used         10034400     LIBCMT:loadcfg.obj
 0002:0000b540       ??_R4exception@std@@6B@    10034540     libvcruntime:frame.obj
 0002:0000b554       ??_R3exception@std@@8      10034554     libvcruntime:frame.obj
 0002:0000b564       ??_R2exception@std@@8      10034564     libvcruntime:frame.obj
 0002:0000b56c       ??_R1A@?0A@EA@exception@std@@8 1003456c     libvcruntime:frame.obj
 0002:0000b588       ??_R4bad_exception@std@@6B@ 10034588     libvcruntime:frame.obj
 0002:0000b59c       ??_R3bad_exception@std@@8  1003459c     libvcruntime:frame.obj
 0002:0000b5ac       ??_R2bad_exception@std@@8  100345ac     libvcruntime:frame.obj
 0002:0000b5b8       ??_R1A@?0A@EA@bad_exception@std@@8 100345b8     libvcruntime:frame.obj
 0002:0000b5d4       ??_R4type_info@@6B@        100345d4     LIBCMT:std_type_info_static.obj
 0002:0000b5e8       ??_R3type_info@@8          100345e8     LIBCMT:std_type_info_static.obj
 0002:0000b5f8       ??_R2type_info@@8          100345f8     LIBCMT:std_type_info_static.obj
 0002:0000b600       ??_R1A@?0A@EA@type_info@@8 10034600     LIBCMT:std_type_info_static.obj
 0002:0000b61c       ___safe_se_handler_table   1003461c     <linker-defined>
 0002:0000b644       ___volatile_metadata       10034644     <linker-defined>
 0002:0000bbd4       ___rtc_iaa                 10034bd4     LIBCMT:initsect.obj
 0002:0000bbd8       ___rtc_izz                 10034bd8     LIBCMT:initsect.obj
 0002:0000bbdc       ___rtc_taa                 10034bdc     LIBCMT:initsect.obj
 0002:0000bbe0       ___rtc_tzz                 10034be0     LIBCMT:initsect.obj
 0002:0000bd74       __TI2?AVbad_exception@std@@ 10034d74     libvcruntime:frame.obj
 0002:0000bd84       __CTA2?AVbad_exception@std@@ 10034d84     libvcruntime:frame.obj
 0002:0000bd90       __CT??_R0?AVbad_exception@std@@@8??0bad_exception@std@@QAE@ABV01@@Z12 10034d90     libvcruntime:frame.obj
 0002:0000bdac       __CT??_R0?AVexception@std@@@8??0exception@std@@QAE@ABV01@@Z12 10034dac     libvcruntime:frame.obj
 0002:0000c550       __IMPORT_DESCRIPTOR_ADVAPI32 10035550     advapi32:ADVAPI32.dll
 0002:0000c564       __IMPORT_DESCRIPTOR_COMCTL32 10035564     comctl32:COMCTL32.dll
 0002:0000c578       __IMPORT_DESCRIPTOR_USER32 10035578     user32:USER32.dll
 0002:0000c58c       __IMPORT_DESCRIPTOR_KERNEL32 1003558c     kernel32:KERNEL32.dll
 0002:0000c5a0       __NULL_IMPORT_DESCRIPTOR   100355a0     advapi32:ADVAPI32.dll
 0003:00000014       _awtPreloadD3D             10036014     java_md.obj
 0003:00000028       ___security_cookie_complement 10036028     LIBCMT:gs_cookie.obj
 0003:0000002c       ___security_cookie         1003602c     LIBCMT:gs_cookie.obj
 0003:00000030       __fltused                  10036030     LIBCMT:fltused.obj
 0003:00000040       ___scrt_native_dllmain_reason 10036040     LIBCMT:utility.obj
 0003:00000050       ___isa_enabled             10036050     LIBCMT:cpu_disp.obj
 0003:00000070       __NLG_Destination          10036070     libvcruntime:exsup.obj
 0003:00000080       __iob                      10036080     libucrt:_file.obj
 0003:00000140       __lookuptrailbytes         10036140     libucrt:read.obj
 0003:00000240       ___abort_behavior          10036240     libucrt:abort.obj
 0003:00000248       ___badioinfo               10036248     libucrt:ioinit.obj
 0003:00000288       ___acrt_initial_locale_data 10036288     libucrt:nlsdata.obj
 0003:00000340       ___acrt_initial_locale_pointers 10036340     libucrt:nlsdata.obj
 0003:00000348       ___acrt_wide_c_locale_string 10036348     libucrt:nlsdata.obj
 0003:0000034c       __pwctype                  1003634c     libucrt:ctype.obj
 0003:00000350       ___acrt_initial_multibyte_data 10036350     libucrt:mbctype.obj
 0003:00000870       ___acrt_lconv_c            10036870     libucrt:localeconv.obj
 0003:000008c0       ___acrt_lconv_static_decimal 100368c0     libucrt:localeconv.obj
 0003:000008c4       ___acrt_lconv_static_W_decimal 100368c4     libucrt:localeconv.obj
 0003:000008c8       ___globallocalestatus      100368c8     libucrt:glstatus.obj
 0003:00000aa0       ??_R0?AVbad_exception@std@@@8 10036aa0     libvcruntime:frame.obj
 0003:00000ac0       ??_R0?AVexception@std@@@8  10036ac0     libvcruntime:frame.obj
 0003:00000adc       ??_R0?AVtype_info@@@8      10036adc     LIBCMT:std_type_info_static.obj
 0003:00000b60       _awtPreloaded              10036b60     java_md.obj
 0003:00001010       ?__type_info_root_node@@3U__type_info_node@@A 10037010     LIBCMT:tncleanup.obj
 0003:00001018       ___scrt_current_native_startup_state 10037018     LIBCMT:utility.obj
 0003:0000101c       ___scrt_native_startup_lock 1003701c     LIBCMT:utility.obj
 0003:0000103c       ___scrt_debugger_hook_flag 1003703c     LIBCMT:utility_desktop.obj
 0003:00001040       ___isa_available           10037040     LIBCMT:cpu_disp.obj
 0003:00001044       ___favor                   10037044     LIBCMT:cpu_disp.obj
 0003:00001048       ?__WinRTOutOfMemoryExceptionCallback@@3P6GPAXXZA 10037048     libvcruntime:ehhelpers.obj
 0003:0000104c       ?pArgList@UnDecorator@@0PAVReplicator@@A 1003704c     libvcruntime:undname.obj
 0003:00001050       ?pZNameList@UnDecorator@@0PAVReplicator@@A 10037050     libvcruntime:undname.obj
 0003:00001054       ?pTemplateArgList@UnDecorator@@0PAVReplicator@@A 10037054     libvcruntime:undname.obj
 0003:00001058       ?gName@UnDecorator@@0PBDB  10037058     libvcruntime:undname.obj
 0003:0000105c       ?name@UnDecorator@@0PBDB   1003705c     libvcruntime:undname.obj
 0003:00001060       ?disableFlags@UnDecorator@@0KA 10037060     libvcruntime:undname.obj
 0003:00001064       ?fExplicitTemplateParams@UnDecorator@@0_NA 10037064     libvcruntime:undname.obj
 0003:00001065       ?fGetTemplateArgumentList@UnDecorator@@0_NA 10037065     libvcruntime:undname.obj
 0003:00001068       ?m_pGetParameter@UnDecorator@@0P6APADJ@ZA 10037068     libvcruntime:undname.obj
 0003:0000106c       ?m_CHPENameOffset@UnDecorator@@0KA 1003706c     libvcruntime:undname.obj
 0003:00001070       ?m_recursionLevel@UnDecorator@@0KA 10037070     libvcruntime:undname.obj
 0003:000010ec       ___pPurecall               100370ec     libvcruntime:purevirt_data.obj
 0003:000010f0       __nstream                  100370f0     libucrt:_file.obj
 0003:000010f4       ___piob                    100370f4     libucrt:_file.obj
 0003:000010f8       __cflush                   100370f8     libucrt:_file.obj
 0003:00001210       __environ_table            10037210     libucrt:environment_initialization.obj
 0003:00001214       __wenviron_table           10037214     libucrt:environment_initialization.obj
 0003:00001218       ___dcrt_initial_wide_environment 10037218     libucrt:environment_initialization.obj
 0003:0000121c       ___dcrt_initial_narrow_environment 1003721c     libucrt:environment_initialization.obj
 0003:00001220       ___acrt_atexit_table       10037220     libucrt:onexit.obj
 0003:0000122c       ___acrt_at_quick_exit_table 1003722c     libucrt:onexit.obj
 0003:00001328       ___pioinfo                 10037328     libucrt:ioinit.obj
 0003:00001528       __nhandle                  10037528     libucrt:ioinit.obj
 0003:0000152c       ___acrt_locale_changed_data 1003752c     libucrt:wsetlocale.obj
 0003:00001530       ___acrt_current_locale_data 10037530     libucrt:nlsdata.obj
 0003:00001540       ___acrt_stdout_buffer      10037540     libucrt:_sftbuf.obj
 0003:00001544       ___acrt_stderr_buffer      10037544     libucrt:_sftbuf.obj
 0003:000016a0       __mbctype                  100376a0     libucrt:mbctype.obj
 0003:000016a4       __mbcasemap                100376a4     libucrt:mbctype.obj
 0003:000016a8       ___acrt_current_multibyte_data 100376a8     libucrt:mbctype.obj
 0003:000016b4       __pgmptr                   100376b4     libucrt:argv_data.obj
 0003:000016b8       ___argc                    100376b8     libucrt:argv_data.obj
 0003:000016bc       ___argv                    100376bc     libucrt:argv_data.obj
 0003:000016c0       ___wargv                   100376c0     libucrt:argv_data.obj
 0003:000016c4       __acmdln                   100376c4     libucrt:argv_data.obj
 0003:000016c8       __wcmdln                   100376c8     libucrt:argv_data.obj
 0003:000016cc       ___acrt_heap               100376cc     libucrt:heap_handle.obj
 0003:000016e8       __umaskval                 100376e8     libucrt:umask.obj
 0003:000016f0       ___acrt_lconv_static_null  100376f0     libucrt:localeconv.obj
 0003:000016f4       ___acrt_lconv_static_W_null 100376f4     libucrt:localeconv.obj
 0003:000016f8       __commode                  100376f8     libucrt:ncommode.obj
 0003:00001700       ?_timezone@@3V?$dual_state_global@J@__crt_state_management@@A 10037700     libucrt:timeset.obj
 0003:00001704       ?_daylight@@3V?$dual_state_global@H@__crt_state_management@@A 10037704     libucrt:timeset.obj
 0003:00001708       ?_dstbias@@3V?$dual_state_global@J@__crt_state_management@@A 10037708     libucrt:timeset.obj
 0003:000017cc       __fmode                    100377cc     libucrt:txtmode.obj
 0003:000017d8       ___fastflag                100377d8     libucrt:fp_flags.obj
 0003:000017e0       ?_OptionsStorage@?1??__local_stdio_scanf_options@@9@9 100377e0     <common>
 0003:000017e8       ?_OptionsStorage@?1??__local_stdio_printf_options@@9@9 100377e8     <common>
 0003:000017f0       ___scrt_ucrt_dll_is_in_use 100377f0     <common>
 0003:000017f4       ___dyn_tls_init_callback   100377f4     <common>
 0003:000017f8       __pmatherr                 100377f8     <common>
 0003:000017fc       ___use_sse2_mathfcns       100377fc     <common>

 entry point at        0001:00008982

 Static symbols

 0000:fffc5000       .debug$S                   10000000     jli.exp
 0000:fffc5000       .debug$S                   10000000     advapi32:ADVAPI32.dll
 0000:fffc5000       .debug$S                   10000000     advapi32:ADVAPI32.dll
 0000:fffc5000       .debug$S                   10000000     advapi32:ADVAPI32.dll
 0000:fffc5000       .debug$S                   10000000     advapi32:ADVAPI32.dll
 0000:fffc5000       .debug$S                   10000000     comctl32:COMCTL32.dll
 0000:fffc5000       .debug$S                   10000000     kernel32:KERNEL32.dll
 0000:fffc5000       .debug$S                   10000000     kernel32:KERNEL32.dll
 0000:fffc5000       .debug$S                   10000000     kernel32:KERNEL32.dll
 0000:fffc5000       .debug$S                   10000000     kernel32:KERNEL32.dll
 0000:fffc5000       .debug$S                   10000000     kernel32:KERNEL32.dll
 0000:fffc5000       .debug$S                   10000000     kernel32:KERNEL32.dll
 0000:fffc5000       .debug$S                   10000000     kernel32:KERNEL32.dll
 0000:fffc5000       .debug$S                   10000000     kernel32:KERNEL32.dll
 0000:fffc5000       .debug$S                   10000000     kernel32:KERNEL32.dll
 0000:fffc5000       .debug$S                   10000000     kernel32:KERNEL32.dll
 0000:fffc5000       .debug$S                   10000000     kernel32:KERNEL32.dll
 0000:fffc5000       .debug$S                   10000000     kernel32:KERNEL32.dll
 0000:fffc5000       .debug$S                   10000000     kernel32:KERNEL32.dll
 0000:fffc5000       .debug$S                   10000000     kernel32:KERNEL32.dll
 0000:fffc5000       .debug$S                   10000000     kernel32:KERNEL32.dll
 0000:fffc5000       .debug$S                   10000000     kernel32:KERNEL32.dll
 0000:fffc5000       .debug$S                   10000000     kernel32:KERNEL32.dll
 0000:fffc5000       .debug$S                   10000000     kernel32:KERNEL32.dll
 0000:fffc5000       .debug$S                   10000000     kernel32:KERNEL32.dll
 0000:fffc5000       .debug$S                   10000000     kernel32:KERNEL32.dll
 0000:fffc5000       .debug$S                   10000000     kernel32:KERNEL32.dll
 0000:fffc5000       .debug$S                   10000000     kernel32:KERNEL32.dll
 0000:fffc5000       .debug$S                   10000000     kernel32:KERNEL32.dll
 0000:fffc5000       .debug$S                   10000000     kernel32:KERNEL32.dll
 0000:fffc5000       .debug$S                   10000000     kernel32:KERNEL32.dll
 0000:fffc5000       .debug$S                   10000000     kernel32:KERNEL32.dll
 0000:fffc5000       .debug$S                   10000000     kernel32:KERNEL32.dll
 0000:fffc5000       .debug$S                   10000000     kernel32:KERNEL32.dll
 0000:fffc5000       .debug$S                   10000000     kernel32:KERNEL32.dll
 0000:fffc5000       .debug$S                   10000000     kernel32:KERNEL32.dll
 0000:fffc5000       .debug$S                   10000000     kernel32:KERNEL32.dll
 0000:fffc5000       .debug$S                   10000000     kernel32:KERNEL32.dll
 0000:fffc5000       .debug$S                   10000000     kernel32:KERNEL32.dll
 0000:fffc5000       .debug$S                   10000000     kernel32:KERNEL32.dll
 0000:fffc5000       .debug$S                   10000000     kernel32:KERNEL32.dll
 0000:fffc5000       .debug$S                   10000000     kernel32:KERNEL32.dll
 0000:fffc5000       .debug$S                   10000000     kernel32:KERNEL32.dll
 0000:fffc5000       .debug$S                   10000000     kernel32:KERNEL32.dll
 0000:fffc5000       .debug$S                   10000000     kernel32:KERNEL32.dll
 0000:fffc5000       .debug$S                   10000000     kernel32:KERNEL32.dll
 0000:fffc5000       .debug$S                   10000000     kernel32:KERNEL32.dll
 0000:fffc5000       .debug$S                   10000000     kernel32:KERNEL32.dll
 0000:fffc5000       .debug$S                   10000000     kernel32:KERNEL32.dll
 0000:fffc5000       .debug$S                   10000000     kernel32:KERNEL32.dll
 0000:fffc5000       .debug$S                   10000000     kernel32:KERNEL32.dll
 0000:fffc5000       .debug$S                   10000000     kernel32:KERNEL32.dll
 0000:fffc5000       .debug$S                   10000000     kernel32:KERNEL32.dll
 0000:fffc5000       .debug$S                   10000000     kernel32:KERNEL32.dll
 0000:fffc5000       .debug$S                   10000000     kernel32:KERNEL32.dll
 0000:fffc5000       .debug$S                   10000000     kernel32:KERNEL32.dll
 0000:fffc5000       .debug$S                   10000000     kernel32:KERNEL32.dll
 0000:fffc5000       .debug$S                   10000000     kernel32:KERNEL32.dll
 0000:fffc5000       .debug$S                   10000000     kernel32:KERNEL32.dll
 0000:fffc5000       .debug$S                   10000000     kernel32:KERNEL32.dll
 0000:fffc5000       .debug$S                   10000000     kernel32:KERNEL32.dll
 0000:fffc5000       .debug$S                   10000000     kernel32:KERNEL32.dll
 0000:fffc5000       .debug$S                   10000000     kernel32:KERNEL32.dll
 0000:fffc5000       .debug$S                   10000000     kernel32:KERNEL32.dll
 0000:fffc5000       .debug$S                   10000000     kernel32:KERNEL32.dll
 0000:fffc5000       .debug$S                   10000000     kernel32:KERNEL32.dll
 0000:fffc5000       .debug$S                   10000000     kernel32:KERNEL32.dll
 0000:fffc5000       .debug$S                   10000000     kernel32:KERNEL32.dll
 0000:fffc5000       .debug$S                   10000000     kernel32:KERNEL32.dll
 0000:fffc5000       .debug$S                   10000000     kernel32:KERNEL32.dll
 0000:fffc5000       .debug$S                   10000000     kernel32:KERNEL32.dll
 0000:fffc5000       .debug$S                   10000000     kernel32:KERNEL32.dll
 0000:fffc5000       .debug$S                   10000000     kernel32:KERNEL32.dll
 0000:fffc5000       .debug$S                   10000000     kernel32:KERNEL32.dll
 0000:fffc5000       .debug$S                   10000000     kernel32:KERNEL32.dll
 0000:fffc5000       .debug$S                   10000000     kernel32:KERNEL32.dll
 0000:fffc5000       .debug$S                   10000000     kernel32:KERNEL32.dll
 0000:fffc5000       .debug$S                   10000000     kernel32:KERNEL32.dll
 0000:fffc5000       .debug$S                   10000000     kernel32:KERNEL32.dll
 0000:fffc5000       .debug$S                   10000000     kernel32:KERNEL32.dll
 0000:fffc5000       .debug$S                   10000000     kernel32:KERNEL32.dll
 0000:fffc5000       .debug$S                   10000000     kernel32:KERNEL32.dll
 0000:fffc5000       .debug$S                   10000000     kernel32:KERNEL32.dll
 0000:fffc5000       .debug$S                   10000000     kernel32:KERNEL32.dll
 0000:fffc5000       .debug$S                   10000000     kernel32:KERNEL32.dll
 0000:fffc5000       .debug$S                   10000000     kernel32:KERNEL32.dll
 0000:fffc5000       .debug$S                   10000000     kernel32:KERNEL32.dll
 0000:fffc5000       .debug$S                   10000000     kernel32:KERNEL32.dll
 0000:fffc5000       .debug$S                   10000000     kernel32:KERNEL32.dll
 0000:fffc5000       .debug$S                   10000000     kernel32:KERNEL32.dll
 0000:fffc5000       .debug$S                   10000000     kernel32:KERNEL32.dll
 0000:fffc5000       .debug$S                   10000000     kernel32:KERNEL32.dll
 0000:fffc5000       .debug$S                   10000000     kernel32:KERNEL32.dll
 0000:fffc5000       .debug$S                   10000000     kernel32:KERNEL32.dll
 0000:fffc5000       .debug$S                   10000000     kernel32:KERNEL32.dll
 0000:fffc5000       .debug$S                   10000000     kernel32:KERNEL32.dll
 0000:fffc5000       .debug$S                   10000000     kernel32:KERNEL32.dll
 0000:fffc5000       .debug$S                   10000000     kernel32:KERNEL32.dll
 0000:fffc5000       .debug$S                   10000000     kernel32:KERNEL32.dll
 0000:fffc5000       .debug$S                   10000000     kernel32:KERNEL32.dll
 0000:fffc5000       .debug$S                   10000000     kernel32:KERNEL32.dll
 0000:fffc5000       .debug$S                   10000000     kernel32:KERNEL32.dll
 0000:fffc5000       .debug$S                   10000000     kernel32:KERNEL32.dll
 0000:fffc5000       .debug$S                   10000000     kernel32:KERNEL32.dll
 0000:fffc5000       .debug$S                   10000000     kernel32:KERNEL32.dll
 0000:fffc5000       .debug$S                   10000000     kernel32:KERNEL32.dll
 0000:fffc5000       .debug$S                   10000000     kernel32:KERNEL32.dll
 0000:fffc5000       .debug$S                   10000000     kernel32:KERNEL32.dll
 0000:fffc5000       .debug$S                   10000000     kernel32:KERNEL32.dll
 0000:fffc5000       .debug$S                   10000000     kernel32:KERNEL32.dll
 0000:fffc5000       .debug$S                   10000000     kernel32:KERNEL32.dll
 0000:fffc5000       .debug$S                   10000000     kernel32:KERNEL32.dll
 0000:fffc5000       .debug$S                   10000000     kernel32:KERNEL32.dll
 0000:fffc5000       .debug$S                   10000000     kernel32:KERNEL32.dll
 0000:fffc5000       .debug$S                   10000000     user32:USER32.dll
 0000:fffc5000       .debug$S                   10000000     user32:USER32.dll
 0001:00000074       _copyCh                    10001074 f   cmdtoargs.obj
 0001:00000092       _next_arg                  10001092 f   cmdtoargs.obj
 0001:00001ba0       $LN761                     10002ba0     inflate.obj
 0001:00001e1e       _inflateStateCheck         10002e1e f   inflate.obj
 0001:00001e51       _updatewindow              10002e51 f   inflate.obj
 0001:00002359       _AddApplicationOptions     10003359 f   java.obj
 0001:0000297c       _DumpState                 1000397c f   java.obj
 0001:00002a5a       _GetApplicationClass       10003a5a f   java.obj
 0001:00002ae7       _InitializeJVM             10003ae7 f   java.obj
 0001:0000330c       _KnownVMIndex              1000430c f   java.obj
 0001:0000335f       _LoadMainClass             1000435f f   java.obj
 0001:00003446       _NewPlatformString         10004446 f   java.obj
 0001:0000359a       _ParseArguments            1000459a f   java.obj
 0001:00003a90       _PrintJavaVersion          10004a90 f   java.obj
 0001:00003aed       _PrintUsage                10004aed f   java.obj
 0001:00004159       _SelectVersion             10005159 f   java.obj
 0001:0000459b       _SetClassPath              1000559b f   java.obj
 0001:000045fd       _SetJvmEnvironment         100055fd f   java.obj
 0001:000047b5       _ShowSettings              100057b5 f   java.obj
 0001:0000496b       _TranslateApplicationArgs  1000596b f   java.obj
 0001:00004b61       _parse_size                10005b61 f   java.obj
 0001:00005844       _GetJREPath                10006844 f   java_md.obj
 0001:00005940       _GetJVMPath                10006940 f   java_md.obj
 0001:000059f6       _GetPublicJREHome          100069f6 f   java_md.obj
 0001:00005b9d       _GetStringFromRegistry     10006b9d f   java_md.obj
 0001:00005ef2       _LoadMSVCRT                10006ef2 f   java_md.obj
 0001:000060df       _ProcessDir                100070df f   java_md.obj
 0001:000063ad       _nextarg                   100073ad f   java_md.obj
 0001:00006439       _unquote                   10007439 f   java_md.obj
 0001:00006825       _compute_cen               10007825 f   parse_manifest.obj
 0001:00006bdc       _find_end                  10007bdc f   parse_manifest.obj
 0001:00006da1       _find_end64                10007da1 f   parse_manifest.obj
 0001:00006e1b       _find_file                 10007e1b f   parse_manifest.obj
 0001:0000715e       _haveZIP64                 1000815e f   parse_manifest.obj
 0001:000071ce       _inflate_file              100081ce f   parse_manifest.obj
 0001:00007302       _parse_nv_pair             10008302 f   parse_manifest.obj
 0001:00007722       _acceptable_simple_element 10008722 f   version_comp.obj
 0001:0000779d       _comp_string               1000879d f   version_comp.obj
 0001:000077dd       _isjavaint                 100087dd f   version_comp.obj
 0001:0000784f       _valid_simple_element      1000884f f   version_comp.obj
 0001:000078e0       _FileList_ensureCapacity   100088e0 f   wildcard.obj
 0001:0000790a       _FileList_expandWildcards  1000890a f   wildcard.obj
 0001:00007a14       _FileList_free             10008a14 f   wildcard.obj
 0001:00007a4c       _FileList_join             10008a4c f   wildcard.obj
 0001:00007ac1       _FileList_new              10008ac1 f   wildcard.obj
 0001:00007ae7       _FileList_split            10008ae7 f   wildcard.obj
 0001:00007bf8       _wildcardFileList          10008bf8 f   wildcard.obj
 0001:00008257       _crc_word                  10009257 f   zcrc32.obj
 0001:000084a0       $$000000                   100094a0     LIBCMT:lldiv.obj
 0001:000084c1       L1                         100094c1     LIBCMT:lldiv.obj
 0001:000084dd       L2                         100094dd     LIBCMT:lldiv.obj
 0001:000084f9       L3                         100094f9     LIBCMT:lldiv.obj
 0001:00008507       L5                         10009507     LIBCMT:lldiv.obj
 0001:00008535       L6                         10009535     LIBCMT:lldiv.obj
 0001:00008536       L7                         10009536     LIBCMT:lldiv.obj
 0001:0000853a       L4                         1000953a     LIBCMT:lldiv.obj
 0001:00008544       L8                         10009544     LIBCMT:lldiv.obj
 0001:00008550       $$000000                   10009550     LIBCMT:llmul.obj
 0001:00008569       hard                       10009569     LIBCMT:llmul.obj
 0001:00008590       $$000000                   10009590     LIBCMT:llrem.obj
 0001:000085b0       L1                         100095b0     LIBCMT:llrem.obj
 0001:000085cb       L2                         100095cb     LIBCMT:llrem.obj
 0001:000085ea       L3                         100095ea     LIBCMT:llrem.obj
 0001:000085f8       L5                         100095f8     LIBCMT:llrem.obj
 0001:00008623       L6                         10009623     LIBCMT:llrem.obj
 0001:0000862b       L7                         1000962b     LIBCMT:llrem.obj
 0001:00008636       L4                         10009636     LIBCMT:llrem.obj
 0001:0000863d       L8                         1000963d     LIBCMT:llrem.obj
 0001:00008642       ?dllmain_crt_dispatch@@YGHQAUHINSTANCE__@@KQAX@Z 10009642 f   LIBCMT:dll_dllmain.obj
 0001:00008695       ?dllmain_crt_process_attach@@YAHQAUHINSTANCE__@@QAX@Z 10009695 f   LIBCMT:dll_dllmain.obj
 0001:0000879c       ?dllmain_crt_process_detach@@YAH_N@Z 1000979c f   LIBCMT:dll_dllmain.obj
 0001:0000884c       ?dllmain_dispatch@@YAHQAUHINSTANCE__@@KQAX@Z 1000984c f   LIBCMT:dll_dllmain.obj
 0001:00008957       ?dllmain_raw@@YGHQAUHINSTANCE__@@KQAX@Z 10009957 f   LIBCMT:dll_dllmain.obj
 0001:000089a5       ___get_entropy             100099a5 f   LIBCMT:gs_support.obj
 0001:00008a78       ?find_pe_section@@YAPAU_IMAGE_SECTION_HEADER@@QAEI@Z 10009a78 f   LIBCMT:utility.obj
 0001:00008ee0       $$000000                   10009ee0     LIBCMT:sehprolg4.obj
 0001:00009110       $$000000                   1000a110     libvcruntime:memcpy.obj
 0001:00009110       $$000000                   1000a110     libvcruntime:memmove.obj
 0001:00009130       CopyUp                     1000a130     libvcruntime:memcpy.obj
 0001:00009130       CopyUp                     1000a130     libvcruntime:memmove.obj
 0001:00009154       CopyUpLargeMov             1000a154     libvcruntime:memcpy.obj
 0001:00009154       CopyUpLargeMov             1000a154     libvcruntime:memmove.obj
 0001:00009167       CopyUpSSE2Check            1000a167     libvcruntime:memcpy.obj
 0001:00009167       CopyUpSSE2Check            1000a167     libvcruntime:memmove.obj
 0001:00009180       AtomChk                    1000a180     libvcruntime:memcpy.obj
 0001:00009180       AtomChk                    1000a180     libvcruntime:memmove.obj
 0001:000091a6       PalignHead4                1000a1a6     libvcruntime:memcpy.obj
 0001:000091a6       PalignHead4                1000a1a6     libvcruntime:memmove.obj
 0001:000091b9       PalignHead8                1000a1b9     libvcruntime:memcpy.obj
 0001:000091b9       PalignHead8                1000a1b9     libvcruntime:memmove.obj
 0001:000091d0       PalignLoop                 1000a1d0     libvcruntime:memcpy.obj
 0001:000091d0       PalignLoop                 1000a1d0     libvcruntime:memmove.obj
 0001:000091e2       MovPalign12                1000a1e2     libvcruntime:memcpy.obj
 0001:000091e2       MovPalign12                1000a1e2     libvcruntime:memmove.obj
 0001:000091ec       PalignLoop12               1000a1ec     libvcruntime:memcpy.obj
 0001:000091ec       PalignLoop12               1000a1ec     libvcruntime:memmove.obj
 0001:0000923d       MovPalign8                 1000a23d     libvcruntime:memcpy.obj
 0001:0000923d       MovPalign8                 1000a23d     libvcruntime:memmove.obj
 0001:00009248       PalignLoop8                1000a248     libvcruntime:memcpy.obj
 0001:00009248       PalignLoop8                1000a248     libvcruntime:memmove.obj
 0001:00009296       MovPalign4                 1000a296     libvcruntime:memcpy.obj
 0001:00009296       MovPalign4                 1000a296     libvcruntime:memmove.obj
 0001:000092a0       PalignLoop4                1000a2a0     libvcruntime:memcpy.obj
 0001:000092a0       PalignLoop4                1000a2a0     libvcruntime:memmove.obj
 0001:000092ec       PalignTail                 1000a2ec     libvcruntime:memcpy.obj
 0001:000092ec       PalignTail                 1000a2ec     libvcruntime:memmove.obj
 0001:00009304       PalignTail4                1000a304     libvcruntime:memcpy.obj
 0001:00009304       PalignTail4                1000a304     libvcruntime:memmove.obj
 0001:00009317       PalignTail8                1000a317     libvcruntime:memcpy.obj
 0001:00009317       PalignTail8                1000a317     libvcruntime:memmove.obj
 0001:0000932e       PalignTailLE3              1000a32e     libvcruntime:memcpy.obj
 0001:0000932e       PalignTailLE3              1000a32e     libvcruntime:memmove.obj
 0001:00009337       Dword_align                1000a337     libvcruntime:memcpy.obj
 0001:00009337       Dword_align                1000a337     libvcruntime:memmove.obj
 0001:0000933f       Dword_up_align_loop        1000a33f     libvcruntime:memcpy.obj
 0001:0000933f       Dword_up_align_loop        1000a33f     libvcruntime:memmove.obj
 0001:00009352       Dword_align_Ok             1000a352     libvcruntime:memcpy.obj
 0001:00009352       Dword_align_Ok             1000a352     libvcruntime:memmove.obj
 0001:0000936c       ByteCopyUp                 1000a36c     libvcruntime:memcpy.obj
 0001:0000936c       ByteCopyUp                 1000a36c     libvcruntime:memmove.obj
 0001:00009374       TrailingUpVec              1000a374     libvcruntime:memcpy.obj
 0001:00009374       TrailingUpVec              1000a374     libvcruntime:memmove.obj
 0001:00009384       TrailingUp0                1000a384     libvcruntime:memcpy.obj
 0001:00009384       TrailingUp0                1000a384     libvcruntime:memmove.obj
 0001:0000938c       TrailingUp1                1000a38c     libvcruntime:memcpy.obj
 0001:0000938c       TrailingUp1                1000a38c     libvcruntime:memmove.obj
 0001:00009398       TrailingUp2                1000a398     libvcruntime:memcpy.obj
 0001:00009398       TrailingUp2                1000a398     libvcruntime:memmove.obj
 0001:000093ac       TrailingUp3                1000a3ac     libvcruntime:memcpy.obj
 0001:000093ac       TrailingUp3                1000a3ac     libvcruntime:memmove.obj
 0001:000093c4       CopyDown                   1000a3c4     libvcruntime:memcpy.obj
 0001:000093c4       CopyDown                   1000a3c4     libvcruntime:memmove.obj
 0001:000093e9       CopyDownNotAligned         1000a3e9     libvcruntime:memcpy.obj
 0001:000093e9       CopyDownNotAligned         1000a3e9     libvcruntime:memmove.obj
 0001:000093f0       CopyDownAlignLoop          1000a3f0     libvcruntime:memcpy.obj
 0001:000093f0       CopyDownAlignLoop          1000a3f0     libvcruntime:memmove.obj
 0001:000093fd       CopyDownAligned            1000a3fd     libvcruntime:memcpy.obj
 0001:000093fd       CopyDownAligned            1000a3fd     libvcruntime:memmove.obj
 0001:00009420       TrailingDownVec            1000a420     libvcruntime:memcpy.obj
 0001:00009420       TrailingDownVec            1000a420     libvcruntime:memmove.obj
 0001:00009430       TrailingDown0              1000a430     libvcruntime:memcpy.obj
 0001:00009430       TrailingDown0              1000a430     libvcruntime:memmove.obj
 0001:00009438       TrailingDown1              1000a438     libvcruntime:memcpy.obj
 0001:00009438       TrailingDown1              1000a438     libvcruntime:memmove.obj
 0001:00009448       TrailingDown2              1000a448     libvcruntime:memcpy.obj
 0001:00009448       TrailingDown2              1000a448     libvcruntime:memmove.obj
 0001:0000945c       TrailingDown3              1000a45c     libvcruntime:memcpy.obj
 0001:0000945c       TrailingDown3              1000a45c     libvcruntime:memmove.obj
 0001:00009475       XmmMovLargeAlignTest       1000a475     libvcruntime:memcpy.obj
 0001:00009475       XmmMovLargeAlignTest       1000a475     libvcruntime:memmove.obj
 0001:0000947d       XmmMovAlignLoop            1000a47d     libvcruntime:memcpy.obj
 0001:0000947d       XmmMovAlignLoop            1000a47d     libvcruntime:memmove.obj
 0001:0000948c       XmmMovLargeLoop            1000a48c     libvcruntime:memcpy.obj
 0001:0000948c       XmmMovLargeLoop            1000a48c     libvcruntime:memmove.obj
 0001:000094fc       XmmMovSmallTest            1000a4fc     libvcruntime:memcpy.obj
 0001:000094fc       XmmMovSmallTest            1000a4fc     libvcruntime:memmove.obj
 0001:00009501       XmmMovSmallLoop            1000a501     libvcruntime:memcpy.obj
 0001:00009501       XmmMovSmallLoop            1000a501     libvcruntime:memmove.obj
 0001:00009524       CopyDownSmall              1000a524     libvcruntime:memcpy.obj
 0001:00009524       CopyDownSmall              1000a524     libvcruntime:memmove.obj
 0001:0000952c       CopyDownDwordLoop          1000a52c     libvcruntime:memcpy.obj
 0001:0000952c       CopyDownDwordLoop          1000a52c     libvcruntime:memmove.obj
 0001:00009541       CopyDownByteTest           1000a541     libvcruntime:memcpy.obj
 0001:00009541       CopyDownByteTest           1000a541     libvcruntime:memmove.obj
 0001:00009545       CopyDownByteLoop           1000a545     libvcruntime:memcpy.obj
 0001:00009545       CopyDownByteLoop           1000a545     libvcruntime:memmove.obj
 0001:00009554       CopyDownReturn             1000a554     libvcruntime:memcpy.obj
 0001:00009554       CopyDownReturn             1000a554     libvcruntime:memmove.obj
 0001:00009560       XmmCopy                    1000a560     libvcruntime:memcpy.obj
 0001:00009560       XmmCopy                    1000a560     libvcruntime:memmove.obj
 0001:0000956d       XmmCopyAligned             1000a56d     libvcruntime:memcpy.obj
 0001:0000956d       XmmCopyAligned             1000a56d     libvcruntime:memmove.obj
 0001:00009580       XmmCopyLargeLoop           1000a580     libvcruntime:memcpy.obj
 0001:00009580       XmmCopyLargeLoop           1000a580     libvcruntime:memmove.obj
 0001:000095dd       XmmCopySmallTest           1000a5dd     libvcruntime:memcpy.obj
 0001:000095dd       XmmCopySmallTest           1000a5dd     libvcruntime:memmove.obj
 0001:000095f0       XmmCopySmallLoop           1000a5f0     libvcruntime:memcpy.obj
 0001:000095f0       XmmCopySmallLoop           1000a5f0     libvcruntime:memmove.obj
 0001:0000960b       CopyUpDwordMov             1000a60b     libvcruntime:memcpy.obj
 0001:0000960b       CopyUpDwordMov             1000a60b     libvcruntime:memmove.obj
 0001:00009610       CopyUpDwordTest            1000a610     libvcruntime:memcpy.obj
 0001:00009610       CopyUpDwordTest            1000a610     libvcruntime:memmove.obj
 0001:00009617       CopyUpDwordLoop            1000a617     libvcruntime:memcpy.obj
 0001:00009617       CopyUpDwordLoop            1000a617     libvcruntime:memmove.obj
 0001:00009626       CopyUpByteTest             1000a626     libvcruntime:memcpy.obj
 0001:00009626       CopyUpByteTest             1000a626     libvcruntime:memmove.obj
 0001:0000962d       CopyUpByteLoop             1000a62d     libvcruntime:memcpy.obj
 0001:0000962d       CopyUpByteLoop             1000a62d     libvcruntime:memmove.obj
 0001:00009640       CopyUpReturn               1000a640     libvcruntime:memcpy.obj
 0001:00009640       CopyUpReturn               1000a640     libvcruntime:memmove.obj
 0001:00009650       XmmCopyUnaligned           1000a650     libvcruntime:memcpy.obj
 0001:00009650       XmmCopyUnaligned           1000a650     libvcruntime:memmove.obj
 0001:00009663       XmmAlignByte               1000a663     libvcruntime:memcpy.obj
 0001:00009663       XmmAlignByte               1000a663     libvcruntime:memmove.obj
 0001:0000966c       XmmAlignDwordTest          1000a66c     libvcruntime:memcpy.obj
 0001:0000966c       XmmAlignDwordTest          1000a66c     libvcruntime:memmove.obj
 0001:00009671       XmmAlignDwordLoop          1000a671     libvcruntime:memcpy.obj
 0001:00009671       XmmAlignDwordLoop          1000a671     libvcruntime:memmove.obj
 0001:0000967e       XmmAlignAdjustCnt          1000a67e     libvcruntime:memcpy.obj
 0001:0000967e       XmmAlignAdjustCnt          1000a67e     libvcruntime:memmove.obj
 0001:00009690       $$000000                   1000a690     libvcruntime:memset.obj
 0001:000096d5       XMMMov                     1000a6d5     libvcruntime:memset.obj
 0001:00009710       LargeRangeBytes            1000a710     libvcruntime:memset.obj
 0001:0000974d       XmmMovSmall                1000a74d     libvcruntime:memset.obj
 0001:00009760       XmmSmallLoop               1000a760     libvcruntime:memset.obj
 0001:00009765       MidRangeBytes              1000a765     libvcruntime:memset.obj
 0001:00009781       XMMTrailingBytes           1000a781     libvcruntime:memset.obj
 0001:00009795       SmallMov                   1000a795     libvcruntime:memset.obj
 0001:0000979d       ByteLoop                   1000a79d     libvcruntime:memset.obj
 0001:000097ab       DwordTest                  1000a7ab     libvcruntime:memset.obj
 0001:000097bb       QwordTest                  1000a7bb     libvcruntime:memset.obj
 0001:000097d0       QwordLoop                  1000a7d0     libvcruntime:memset.obj
 0001:000097e3       toend                      1000a7e3     libvcruntime:memset.obj
 0001:000097f0       $$000000                   1000a7f0     libvcruntime:strchr.obj
 0001:00009823       strchr_sse_loop            1000a823     libvcruntime:strchr.obj
 0001:00009847       strchr_sse_break           1000a847     libvcruntime:strchr.obj
 0001:00009858       strchr_no_sse2             1000a858     libvcruntime:strchr.obj
 0001:00009870       str_misaligned             1000a870     libvcruntime:strchr.obj
 0001:00009885       main_loop_start            1000a885     libvcruntime:strchr.obj
 0001:00009890       main_loop                  1000a890     libvcruntime:strchr.obj
 0001:000098cc       retnull                    1000a8cc     libvcruntime:strchr.obj
 0001:000098ce       retnull_bx                 1000a8ce     libvcruntime:strchr.obj
 0001:000098d2       found_bx                   1000a8d2     libvcruntime:strchr.obj
 0001:000098d7       chr_is_found               1000a8d7     libvcruntime:strchr.obj
 0001:000098ff       byte_3                     1000a8ff     libvcruntime:strchr.obj
 0001:00009906       byte_2                     1000a906     libvcruntime:strchr.obj
 0001:0000990d       byte_1                     1000a90d     libvcruntime:strchr.obj
 0001:00009914       byte_0                     1000a914     libvcruntime:strchr.obj
 0001:00009920       $$000000                   1000a920     libvcruntime:strrchr.obj
 0001:0000995d       strrchr_sse_loop           1000a95d     libvcruntime:strrchr.obj
 0001:0000998d       strrchr_sse_break          1000a98d     libvcruntime:strrchr.obj
 0001:000099ad       strrchr_sttni              1000a9ad     libvcruntime:strrchr.obj
 0001:000099bf       strrchr_sttni_chars        1000a9bf     libvcruntime:strrchr.obj
 0001:000099d4       strrchr_sttni_aligned      1000a9d4     libvcruntime:strrchr.obj
 0001:000099d8       strrchr_sttni_xmm          1000a9d8     libvcruntime:strrchr.obj
 0001:000099eb       exit                       1000a9eb     libvcruntime:strrchr.obj
 0001:000099ee       strrchr_zero               1000a9ee     libvcruntime:strrchr.obj
 0001:00009a13       strchr_zero_loop           1000aa13     libvcruntime:strrchr.obj
 0001:00009a27       strchr_zero_result         1000aa27     libvcruntime:strrchr.obj
 0001:00009a2e       strrchr_no_sse             1000aa2e     libvcruntime:strrchr.obj
 0001:00009a51       returndi                   1000aa51     libvcruntime:strrchr.obj
 0001:00009a53       toend                      1000aa53     libvcruntime:strrchr.obj
 0001:0000b053       $LN1250                    1000c053     libvcruntime:memcmp.obj
 0001:0000b0e0       _ValidateLocalCookies      1000c0e0 f   libvcruntime:chandler4.obj
 0001:0000b3dc       ?_FilterSetCurrentException@@YAKPAU_EXCEPTION_POINTERS@@E@Z 1000c3dc f   libvcruntime:ehhelpers.obj
 0001:0000b4e0       $$000000                   1000c4e0     libvcruntime:exsup4.obj
 0001:0000b512       _lu_top                    1000c512     libvcruntime:exsup4.obj
 0001:0000b571       _lu_done                   1000c571     libvcruntime:exsup4.obj
 0001:0000b580       $$000000                   1000c580     libvcruntime:exsup4.obj
 0001:0000b580       __unwind_handler4          1000c580 f   libvcruntime:exsup4.obj
 0001:0000b5d0       $$000000                   1000c5d0     libvcruntime:exsup4.obj
 0001:0000b5f0       $$000000                   1000c5f0     libvcruntime:exsup4.obj
 0001:0000b610       $$000000                   1000c610     libvcruntime:exsup4.obj
 0001:0000b625       ReturnPoint                1000c625     libvcruntime:exsup4.obj
 0001:0000b630       $$000000                   1000c630     libvcruntime:exsup4.obj
 0001:0000b820       $$000000                   1000c820     libvcruntime:exsup.obj
 0001:0000b830       $$000000                   1000c830     libvcruntime:exsup.obj
 0001:0000b83b       __NLG_Go                   1000c83b     libvcruntime:exsup.obj
 0001:0000b850       $$000000                   1000c850     libvcruntime:exsup.obj
 0001:0000bc09       ?try_get_function@@YAPAXW4function_id@?A0x14174aea@@QBDQBW4module_id@2@2@Z 1000cc09 f   libvcruntime:winapi_downlevel.obj
 0001:0000bca9       ?try_load_library_from_system_directory@@YAPAUHINSTANCE__@@QB_W@Z 1000cca9 f   libvcruntime:winapi_downlevel.obj
 0001:0000be2a       ??$BuildCatchObjectHelperInternal@V__FrameHandler3@@@@YAHPAUEHExceptionRecord@@PAXPBU_s_HandlerType@@PBU_s_CatchableType@@@Z 1000ce2a f   libvcruntime:frame.obj
 0001:0000bf68       ??$BuildCatchObjectInternal@V__FrameHandler3@@@@YAXPAUEHExceptionRecord@@PAXPBU_s_HandlerType@@PBU_s_CatchableType@@@Z 1000cf68 f   libvcruntime:frame.obj
 0001:0000c001       ??$CatchIt@V__FrameHandler3@@@@YAXPAUEHExceptionRecord@@PAUEHRegistrationNode@@PAU_CONTEXT@@PAXPBU_s_FuncInfo@@PBU_s_HandlerType@@PBU_s_CatchableType@@PBU_s_TryBlockMapEntry@@H1EE@Z 1000d001 f   libvcruntime:frame.obj
 0001:0000c081       ??$FindHandler@V__FrameHandler3@@@@YAXPAUEHExceptionRecord@@PAUEHRegistrationNode@@PAU_CONTEXT@@PAXPBU_s_FuncInfo@@EH1@Z 1000d081 f   libvcruntime:frame.obj
 0001:0000c426       ??$FindHandlerForForeignException@V__FrameHandler3@@@@YAXPAUEHExceptionRecord@@PAUEHRegistrationNode@@PAU_CONTEXT@@PAXPBU_s_FuncInfo@@HH1@Z 1000d426 f   libvcruntime:frame.obj
 0001:0000c7b1       ?CallCatchBlock@@YAPAXPAUEHExceptionRecord@@PAUEHRegistrationNode@@PAU_CONTEXT@@PBU_s_FuncInfo@@PAXHK@Z 1000d7b1 f   libvcruntime:frame.obj
 0001:0000c980       ?CallUnexpected@@YAXPBU_s_ESTypeList@@@Z 1000d980 f   libvcruntime:frame.obj
 0001:0000c9a0       __catch$?CallUnexpected@@YAXPBU_s_ESTypeList@@@Z$0 1000d9a0 f   libvcruntime:frame.obj
 0001:0000c9bf       ?ExFilterRethrow@@YAHPAU_EXCEPTION_POINTERS@@@Z 1000d9bf f   libvcruntime:frame.obj
 0001:0000cb09       ?IsInExceptionSpec@@YAEPAUEHExceptionRecord@@PBU_s_ESTypeList@@@Z 1000db09 f   libvcruntime:frame.obj
 0001:0000cbe0       $$000000                   1000dbe0     libvcruntime:lowhelpr.obj
 0001:0000cc1f       _NLG_Continue              1000dc1f     libvcruntime:lowhelpr.obj
 0001:0000cf32       ?_fclose_internal@@YAHQAU_iobuf@@AAV__crt_cached_ptd_host@@@Z 1000df32 f   libucrt:fclose.obj
 0001:0000cfc9       ?_fclose_nolock_internal@@YAHQAU_iobuf@@AAV__crt_cached_ptd_host@@@Z 1000dfc9 f   libucrt:fclose.obj
 0001:0000d0ea       ??$common_fgets@D@@YAPADQADHV__crt_stdio_stream@@@Z 1000e0ea f   libucrt:fgets.obj
 0001:0000d24e       ??$common_fsopen@D@@YAPAU_iobuf@@QBD0H@Z 1000e24e f   libucrt:fopen.obj
 0001:0000d31c       ??$?RV<lambda_62491a2101a2aba6cc4a769149c84f1f>@@AAV<lambda_826c27fce7726908515bbc79a5266961>@@V<lambda_4e64bbd54b50a7b070e3ea8d795375b6>@@@?$__crt_seh_guarded_call@H@@QAEH$$QAV<lambda_62491a2101a2aba6cc4a769149c84f1f>@@AAV<lambda_826c27fce7726908515bbc79a5266961>@@$$QAV<lambda_4e64bbd54b50a7b070e3ea8d795375b6>@@@Z 1000e31c f   libucrt:output.obj
 0001:0000d377       ??$common_vsprintf@Vstandard_base@__crt_stdio_output@@D@@YAH_KQADIQBDAAV__crt_cached_ptd_host@@1@Z 1000e377 f   libucrt:output.obj
 0001:0000e08d       ??R<lambda_826c27fce7726908515bbc79a5266961>@@QBEHXZ 1000f08d f   libucrt:output.obj
 0001:0000e528       $LN121                     1000f528     libucrt:output.obj
 0001:0000e7fc       $LN130                     1000f7fc     libucrt:output.obj
 0001:0000f1a3       $LN18                      100101a3     libucrt:output.obj
 0001:0000f1b7       $LN17                      100101b7     libucrt:output.obj
 0001:0000f9b7       ??$common_vsscanf@D@@YAH_KQBDI1QAU__crt_locale_pointers@@QAD@Z 100109b7 f   libucrt:input.obj
 0001:00010443       $LN32                      10011443     libucrt:input.obj
 0001:00010567       $LN30                      10011567     libucrt:input.obj
 0001:00013980       $LN16                      10014980     libucrt:input.obj
 0001:0001398c       $LN15                      1001498c     libucrt:input.obj
 0001:00013a95       $LN15                      10014a95     libucrt:input.obj
 0001:0001421e       $LN17                      1001521e     libucrt:input.obj
 0001:00014232       $LN16                      10015232     libucrt:input.obj
 0001:00014459       _memcpy_s                  10015459 f   libucrt:cfout.obj
 0001:00014459       _memcpy_s                  10015459 f   libucrt:fullpath.obj
 0001:00014459       _memcpy_s                  10015459 f   libucrt:mbctype.obj
 0001:00014459       _memcpy_s                  10015459 f   libucrt:input.obj
 0001:000144f5       ??$?RV<lambda_03b1d95aef87969028cfba75ccab2455>@@AAV<lambda_6e4b09c48022b2350581041d5f6b0c4c>@@V<lambda_22bdf7517842c4b3e53723af5aa32b9e>@@@?$__crt_seh_guarded_call@X@@QAEX$$QAV<lambda_03b1d95aef87969028cfba75ccab2455>@@AAV<lambda_6e4b09c48022b2350581041d5f6b0c4c>@@$$QAV<lambda_22bdf7517842c4b3e53723af5aa32b9e>@@@Z 100154f5 f   libucrt:exit.obj
 0001:0001455d       ??R<lambda_6e4b09c48022b2350581041d5f6b0c4c>@@QBE@XZ 1001555d f   libucrt:exit.obj
 0001:00014645       ?common_exit@@YAXHW4_crt_exit_cleanup_mode@@W4_crt_exit_return_mode@@@Z 10015645 f   libucrt:exit.obj
 0001:000146dc       ?exit_or_terminate_process@@YAXI@Z 100156dc f   libucrt:exit.obj
 0001:0001470d       ?is_managed_app@@YA_NXZ    1001570d f   libucrt:exit.obj
 0001:0001474f       ?should_call_terminate_process@@YA_NXZ 1001574f f   libucrt:exit.obj
 0001:00014768       ?try_cor_exit_process@@YAXI@Z 10015768 f   libucrt:exit.obj
 0001:0001483b       ??$common_getenv@D@@YAPADQBD@Z 1001583b f   libucrt:getenv.obj
 0001:000148ba       ??$common_getenv_nolock@D@@YAPADQBD@Z 100158ba f   libucrt:getenv.obj
 0001:00014927       ??$common_getenv_nolock@_W@@YAPA_WQB_W@Z 10015927 f   libucrt:getenv.obj
 0001:000149ab       ??$common_getenv_s@_W@@YAHQAIQA_WIQB_W@Z 100159ab f   libucrt:getenv.obj
 0001:00014a0a       ??$common_getenv_s_nolock@_W@@YAHQAIQA_WIQB_W@Z 10015a0a f   libucrt:getenv.obj
 0001:00014ace       ??$common_putenv@D@@YAHQBD0@Z 10015ace f   libucrt:putenv.obj
 0001:00014b26       ??$common_putenv_nolock@D@@YAHQBD0@Z 10015b26 f   libucrt:putenv.obj
 0001:00014ba7       ??$create_environment_string@D@@YAPADQBD0@Z 10015ba7 f   libucrt:putenv.obj
 0001:00014ca1       ??$set_variable_in_other_environment@D@@YA_NQBD0@Z 10015ca1 f   libucrt:putenv.obj
 0001:00014d90       $$000000                   10015d90     libucrt:strcat.obj
 0001:00014e90       $$000000                   10015e90     libucrt:strcmp.obj
 0001:00014f20       $$000000                   10015f20     libucrt:strcspn.obj
 0001:00014f70       $$000000                   10015f70     libucrt:strlen.obj
 0001:00015000       $$000000                   10016000     libucrt:strspn.obj
 0001:000150fc       ??$common_strerror@D@@YAPADH@Z 100160fc f   libucrt:strerror.obj
 0001:000151e0       $$000000                   100161e0     libucrt:strncmp.obj
 0001:00015468       ??$thread_start@P6GIPAX@Z$00@@YGKQAX@Z 10016468 f   libucrt:thread.obj
 0001:000154e6       ??1?$__crt_unique_heap_ptr@U__acrt_thread_parameter@@Uthread_parameter_free_policy@?A0x4e93fcdd@@@@QAE@XZ 100164e6 f   libucrt:thread.obj
 0001:0001551d       ?common_end_thread@@YAXI@Z 1001651d f   libucrt:thread.obj
 0001:00015574       ?create_thread_parameter@@YAPAU__acrt_thread_parameter@@QAX0@Z 10016574 f   libucrt:thread.obj
 0001:00015655       ??$?RV<lambda_2866be3712abc81a800a822484c830d8>@@AAV<lambda_39ca0ed439415581b5b15c265174cece>@@V<lambda_2b24c74d71094a6cd0cb82e44167d71b>@@@?$__crt_seh_guarded_call@X@@QAEX$$QAV<lambda_2866be3712abc81a800a822484c830d8>@@AAV<lambda_39ca0ed439415581b5b15c265174cece>@@$$QAV<lambda_2b24c74d71094a6cd0cb82e44167d71b>@@@Z 10016655 f   libucrt:fflush.obj
 0001:000156e1       ??$?RV<lambda_2cc53f568c5a2bb6f192f930a45d44ea>@@AAV<lambda_ab61a845afdef5b7c387490eaf3616ee>@@V<lambda_c2ffc0b7726aa6be21d5f0026187e748>@@@?$__crt_seh_guarded_call@X@@QAEX$$QAV<lambda_2cc53f568c5a2bb6f192f930a45d44ea>@@AAV<lambda_ab61a845afdef5b7c387490eaf3616ee>@@$$QAV<lambda_c2ffc0b7726aa6be21d5f0026187e748>@@@Z 100166e1 f   libucrt:fflush.obj
 0001:0001578d       ??$?RV<lambda_6d20deecaf4856105ebacbad442d1079>@@AAV<lambda_9a32fed5bf61b6b509b2d3f6003082a1>@@V<lambda_63ea2239ed67c638ddbae41947fdf875>@@@?$__crt_seh_guarded_call@H@@QAEH$$QAV<lambda_6d20deecaf4856105ebacbad442d1079>@@AAV<lambda_9a32fed5bf61b6b509b2d3f6003082a1>@@$$QAV<lambda_63ea2239ed67c638ddbae41947fdf875>@@@Z 1001678d f   libucrt:fflush.obj
 0001:000157ed       ?common_flush_all@@YAH_N@Z 100167ed f   libucrt:fflush.obj
 0001:0001583a       ?common_flush_all_should_try_to_flush_stream@@YA_NV__crt_stdio_stream@@QAH@Z 1001683a f   libucrt:fflush.obj
 0001:0001586b       ?is_stream_flushable_or_commitable@@YA_NJ@Z 1001686b f   libucrt:fflush.obj
 0001:000159b8       ??$common_stat@U_stat64i32@@@@YAHQBDQAU_stat64i32@@@Z 100169b8 f   libucrt:stat.obj
 0001:00015a39       ??$common_stat@U_stat64i32@@@@YAHQB_WQAU_stat64i32@@@Z 10016a39 f   libucrt:stat.obj
 0001:00015b39       ??$common_stat_handle_file_not_opened@U_stat64i32@@@@YA_NQB_WAAU_stat64i32@@@Z 10016b39 f   libucrt:stat.obj
 0001:00015bc3       ??$common_stat_handle_file_opened@U_stat64i32@@@@YA_NQB_WHQAXAAU_stat64i32@@@Z 10016bc3 f   libucrt:stat.obj
 0001:00015d33       ??$convert_filetime_to_time_t@_J@@YA_JU_FILETIME@@_J@Z 10016d33 f   libucrt:stat.obj
 0001:00015df8       ?call_wfullpath@@YAPA_WQA_WQB_WIQAPA_W@Z 10016df8 f   libucrt:stat.obj
 0001:00015e58       ?compute_size@@YA_NABU_BY_HANDLE_FILE_INFORMATION@@AAJ@Z 10016e58 f   libucrt:stat.obj
 0001:00015e8b       ?convert_to_stat_mode@@YAGHQB_W@Z 10016e8b f   libucrt:stat.obj
 0001:00015f39       ?get_drive_number_from_path@@YA_NQB_WAAH@Z 10016f39 f   libucrt:stat.obj
 0001:00015f95       ?is_root_or_empty@@YA_NQB_W@Z 10016f95 f   libucrt:stat.obj
 0001:00015fee       ?is_root_unc_name@@YA_NQB_W@Z 10016fee f   libucrt:stat.obj
 0001:0001609c       ?is_slash@@YA_N_W@Z        1001709c f   libucrt:stat.obj
 0001:000160b7       ?is_usable_drive_or_unc_root@@YA_NQB_W@Z 100170b7 f   libucrt:stat.obj
 0001:0001617a       ?_perror_internal@@YAXQBDAAV__crt_cached_ptd_host@@@Z 1001717a f   libucrt:perror.obj
 0001:00016270       $$000000                   10017270     libucrt:strpbrk.obj
 0001:000162b0       ??$common_lseek@_J@@YA_JH_JHAAV__crt_cached_ptd_host@@@Z 100172b0 f   libucrt:lseek.obj
 0001:000163d5       ??$common_lseek_nolock@_J@@YA_JH_JHAAV__crt_cached_ptd_host@@@Z 100173d5 f   libucrt:lseek.obj
 0001:000167d3       ??$common_configure_argv@D@@YAHW4_crt_argv_mode@@@Z 100177d3 f   libucrt:argv_parsing.obj
 0001:00016910       ??$parse_command_line@D@@YAXPADPAPAD0PAI2@Z 10017910 f   libucrt:argv_parsing.obj
 0001:00016ade       ??$common_get_or_create_environment_nolock@D@@YAPAPADXZ 10017ade f   libucrt:environment_initialization.obj
 0001:00016b0a       ??$common_get_or_create_environment_nolock@_W@@YAPAPA_WXZ 10017b0a f   libucrt:environment_initialization.obj
 0001:00016b36       ??$common_initialize_environment_nolock@D@@YAHXZ 10017b36 f   libucrt:environment_initialization.obj
 0001:00016b90       ??$common_initialize_environment_nolock@_W@@YAHXZ 10017b90 f   libucrt:environment_initialization.obj
 0001:00016be5       ??$create_environment@D@@YAQAPADQAD@Z 10017be5 f   libucrt:environment_initialization.obj
 0001:00016cc7       ??$create_environment@_W@@YAQAPA_WQA_W@Z 10017cc7 f   libucrt:environment_initialization.obj
 0001:00016de5       ??$free_environment@D@@YAXQAPAD@Z 10017de5 f   libucrt:environment_initialization.obj
 0001:00016de5       ??$free_environment@_W@@YAXQAPA_W@Z 10017de5 f   libucrt:environment_initialization.obj
 0001:00016e14       ??$initialize_environment_by_cloning_nolock@D@@YAHXZ 10017e14 f   libucrt:environment_initialization.obj
 0001:00016e97       ??$initialize_environment_by_cloning_nolock@_W@@YAHXZ 10017e97 f   libucrt:environment_initialization.obj
 0001:00016f18       ??$uninitialize_environment_internal@D@@YAXAAPAPAD@Z 10017f18 f   libucrt:environment_initialization.obj
 0001:00016f33       ??$uninitialize_environment_internal@_W@@YAXAAPAPA_W@Z 10017f33 f   libucrt:environment_initialization.obj
 0001:00016fae       ??$?RV<lambda_69a2805e680e0e292e8ba93315fe43a8>@@AAV<lambda_f03950bc5685219e0bcd2087efbe011e>@@V<lambda_03fcd07e894ec930e3f35da366ca99d6>@@@?$__crt_seh_guarded_call@H@@QAEH$$QAV<lambda_69a2805e680e0e292e8ba93315fe43a8>@@AAV<lambda_f03950bc5685219e0bcd2087efbe011e>@@$$QAV<lambda_03fcd07e894ec930e3f35da366ca99d6>@@@Z 10017fae f   libucrt:onexit.obj
 0001:00017009       ??R<lambda_f03950bc5685219e0bcd2087efbe011e>@@QBE@XZ 10018009 f   libucrt:onexit.obj
 0001:0001714a       _initialize_global_variables 1001814a f   libucrt:initialization.obj
 0001:00017157       _initialize_c              10018157 f   libucrt:initialization.obj
 0001:00017171       _initialize_environment    10018171 f   libucrt:initialization.obj
 0001:00017171       _initialize_global_state_isolation 10018171 f   libucrt:initialization.obj
 0001:00017171       _report_memory_leaks       10018171 f   libucrt:initialization.obj
 0001:00017171       _uninitialize_c            10018171 f   libucrt:initialization.obj
 0001:00017171       _uninitialize_global_state_isolation 10018171 f   libucrt:initialization.obj
 0001:00017174       _uninitialize_environment  10018174 f   libucrt:initialization.obj
 0001:0001717c       _initialize_pointers       1001817c f   libucrt:initialization.obj
 0001:000171aa       _uninitialize_vcruntime    100181aa f   libucrt:initialization.obj
 0001:000171b3       _uninitialize_allocated_memory 100181b3 f   libucrt:initialization.obj
 0001:000171ca       _uninitialize_allocated_io_buffers 100181ca f   libucrt:initialization.obj
 0001:00017239       ??R<lambda_af42a3ee9806e9a7305d451646e05244>@@QBE@AAPAU__crt_multibyte_data@@@Z 10018239 f   libucrt:initialization.obj
 0001:000175a8       ??$?RV<lambda_d422a76eb4c3bf3ad751449ab71a6ea4>@@AAV<lambda_c9ba49e555ba839a7b07aa3fbecb7617>@@V<lambda_9476263c8ee91a25d21c55370bdb50de>@@@?$__crt_seh_guarded_call@H@@QAEH$$QAV<lambda_d422a76eb4c3bf3ad751449ab71a6ea4>@@AAV<lambda_c9ba49e555ba839a7b07aa3fbecb7617>@@$$QAV<lambda_9476263c8ee91a25d21c55370bdb50de>@@@Z 100185a8 f   libucrt:close.obj
 0001:000177dc       ??$common_open@D@@YAHQBDHH@Z 100187dc f   libucrt:open.obj
 0001:000178ad       ??$common_sopen_dispatch@D@@YAHQBDHHHQAHH@Z 100188ad f   libucrt:open.obj
 0001:00017988       ?configure_text_mode@@YAHHUfile_options@?A0xa9d50aae@@HAAW4__crt_lowio_text_mode@@@Z 10018988 f   libucrt:open.obj
 0001:00017bde       ?create_file@@YAPAXQB_WQAU_SECURITY_ATTRIBUTES@@Ufile_options@?A0xa9d50aae@@@Z 10018bde f   libucrt:open.obj
 0001:00017c03       ?decode_open_create_flags@@YAKH@Z 10018c03 f   libucrt:open.obj
 0001:00017c73       ?decode_options@@YA?AUfile_options@?A0xa9d50aae@@HHH@Z 10018c73 f   libucrt:open.obj
 0001:00017ded       ?truncate_ctrl_z_if_present@@YAHH@Z 10018ded f   libucrt:open.obj
 0001:00018267       ??$translate_text_mode_nolock@D@@YAHHQADI@Z 10019267 f   libucrt:read.obj
 0001:000183b4       ??$translate_text_mode_nolock@_W@@YAHHQA_WI@Z 100193b4 f   libucrt:read.obj
 0001:0001856e       ?translate_ansi_or_utf8_nolock@@YAHHQADIQA_WI@Z 1001956e f   libucrt:read.obj
 0001:000186c5       ?translate_utf16_from_console_nolock@@YAHHQA_WI@Z 100196c5 f   libucrt:read.obj
 0001:000198a0       ?try_get_AreFileApisANSI@@YAP6GHXZXZ 1001a8a0 f   libucrt:winapi_thunks.obj
 0001:000198ba       ?try_get_CompareStringEx@@YAP6GHPB_WK0H0HPAU_nlsversioninfo@@PAXJ@ZXZ 1001a8ba f   libucrt:winapi_thunks.obj
 0001:000198d4       ?try_get_LCMapStringEx@@YAP6GHPB_WK0HPA_WHPAU_nlsversioninfo@@PAXJ@ZXZ 1001a8d4 f   libucrt:winapi_thunks.obj
 0001:000198ee       ?try_get_LocaleNameToLCID@@YAP6GKPB_WK@ZXZ 1001a8ee f   libucrt:winapi_thunks.obj
 0001:00019908       ?try_get_first_available_module@@YAPAUHINSTANCE__@@QBW4module_id@?A0x391cf84c@@0@Z 1001a908 f   libucrt:winapi_thunks.obj
 0001:000199d3       ?try_get_function@@YAPAXW4function_id@?A0x391cf84c@@QBDQBW4module_id@2@2@Z 1001a9d3 f   libucrt:winapi_thunks.obj
 0001:00019eca       ?initialize_inherited_file_handles_nolock@@YAXXZ 1001aeca f   libucrt:ioinit.obj
 0001:00019f80       ?initialize_stdio_handles_nolock@@YAXXZ 1001af80 f   libucrt:ioinit.obj
 0001:0001a187       ?find_or_allocate_unused_stream_nolock@@YA?AV__crt_stdio_stream@@XZ 1001b187 f   libucrt:stream.obj
 0001:0001a249       ??$?RV<lambda_15ade71b0218206bbe3333a0c9b79046>@@AAV<lambda_da44e0f8b0f19ba52fefafb335991732>@@V<lambda_207f2d024fc103971653565357d6cd41>@@@?$__crt_seh_guarded_call@X@@QAEX$$QAV<lambda_15ade71b0218206bbe3333a0c9b79046>@@AAV<lambda_da44e0f8b0f19ba52fefafb335991732>@@$$QAV<lambda_207f2d024fc103971653565357d6cd41>@@@Z 1001b249 f   libucrt:per_thread_data.obj
 0001:0001a29b       ??$?RV<lambda_38edbb1296d33220d7e4dd0ed76b244a>@@AAV<lambda_5ce1d447e08cb34b2473517608e21441>@@V<lambda_fb385d3da700c9147fc39e65dd577a8c>@@@?$__crt_seh_guarded_call@X@@QAEX$$QAV<lambda_38edbb1296d33220d7e4dd0ed76b244a>@@AAV<lambda_5ce1d447e08cb34b2473517608e21441>@@$$QAV<lambda_fb385d3da700c9147fc39e65dd577a8c>@@@Z 1001b29b f   libucrt:per_thread_data.obj
 0001:0001a306       ??$?RV<lambda_6affb1475c98b40b75cdec977db92e3c>@@AAV<lambda_b8d4b9c228a6ecc3f80208dbb4b4a104>@@V<lambda_608742c3c92a14382c1684fc64f96c88>@@@?$__crt_seh_guarded_call@X@@QAEX$$QAV<lambda_6affb1475c98b40b75cdec977db92e3c>@@AAV<lambda_b8d4b9c228a6ecc3f80208dbb4b4a104>@@$$QAV<lambda_608742c3c92a14382c1684fc64f96c88>@@@Z 1001b306 f   libucrt:per_thread_data.obj
 0001:0001a35b       ??$?RV<lambda_a7e850c220f1c8d1e6efeecdedd162c6>@@AAV<lambda_46720907175c18b6c9d2717bc0d2d362>@@V<lambda_9048902d66e8d99359bc9897bbb930a8>@@@?$__crt_seh_guarded_call@X@@QAEX$$QAV<lambda_a7e850c220f1c8d1e6efeecdedd162c6>@@AAV<lambda_46720907175c18b6c9d2717bc0d2d362>@@$$QAV<lambda_9048902d66e8d99359bc9897bbb930a8>@@@Z 1001b35b f   libucrt:per_thread_data.obj
 0001:0001a3b5       ?construct_ptd@@YAXQAU__acrt_ptd@@QAPAU__crt_locale_data@@@Z 1001b3b5 f   libucrt:per_thread_data.obj
 0001:0001a44e       ?destroy_fls@@YGXPAX@Z     1001b44e f   libucrt:per_thread_data.obj
 0001:0001a46f       ?destroy_ptd@@YAXQAU__acrt_ptd@@@Z 1001b46f f   libucrt:per_thread_data.obj
 0001:0001a53c       ?replace_current_thread_locale_nolock@@YAXQAU__acrt_ptd@@QAU__crt_locale_data@@@Z 1001b53c f   libucrt:per_thread_data.obj
 0001:0001a89e       ??$?RV<lambda_e5124f882df8998aaf41531e079ba474>@@AAV<lambda_3e16ef9562a7dcce91392c22ab16ea36>@@V<lambda_e25ca0880e6ef98be67edffd8c599615>@@@?$__crt_seh_guarded_call@X@@QAEX$$QAV<lambda_e5124f882df8998aaf41531e079ba474>@@AAV<lambda_3e16ef9562a7dcce91392c22ab16ea36>@@$$QAV<lambda_e25ca0880e6ef98be67edffd8c599615>@@@Z 1001b89e f   libucrt:wsetlocale.obj
 0001:0001abaf       ??$common_openfile@D@@YAPAU_iobuf@@QBD0HV__crt_stdio_stream@@@Z 1001bbaf f   libucrt:openfile.obj
 0001:0001b18f       ?fe_to_nearest@@YA_NQBN_KF@Z 1001c18f f   libucrt:cvt.obj
 0001:0001b232       ?fp_format_a@@YAHQBNPADIQADIH_NIW4__acrt_rounding_mode@@AAV__crt_cached_ptd_host@@@Z 1001c232 f   libucrt:cvt.obj
 0001:0001b55f       ?fp_format_e@@YAHQBNQADI1IH_NIW4__acrt_rounding_mode@@AAV__crt_cached_ptd_host@@@Z 1001c55f f   libucrt:cvt.obj
 0001:0001b603       ?fp_format_e_internal@@YAHQADIH_NIQAU_strflt@@1AAV__crt_cached_ptd_host@@@Z 1001c603 f   libucrt:cvt.obj
 0001:0001b756       ?fp_format_f@@YAHQBNQADI1IHW4__acrt_rounding_mode@@AAV__crt_cached_ptd_host@@@Z 1001c756 f   libucrt:cvt.obj
 0001:0001b7ec       ?fp_format_f_internal@@YAHQADIHQAU_strflt@@_NAAV__crt_cached_ptd_host@@@Z 1001c7ec f   libucrt:cvt.obj
 0001:0001b8da       ?fp_format_g@@YAHQBNQADI1IH_NIW4__acrt_rounding_mode@@AAV__crt_cached_ptd_host@@@Z 1001c8da f   libucrt:cvt.obj
 0001:0001b9a9       ?fp_format_nan_or_infinity@@YAHW4__acrt_fp_class@@_NPADI1@Z 1001c9a9 f   libucrt:cvt.obj
 0001:0001ba3e       ?shift_bytes@@YAXQADI0H@Z  1001ca3e f   libucrt:cvt.obj
 0001:0001ba72       ?should_round_up@@YA_NQBN_KFW4__acrt_rounding_mode@@@Z 1001ca72 f   libucrt:cvt.obj
 0001:0001c663       ?filter_mbtowcs_flags@@YAKIK@Z 1001d663 f   libucrt:multibytetowidechar.obj
 0001:0001c725       ?filter_wcstomb_flags@@YAKIK@Z 1001d725 f   libucrt:widechartomultibyte.obj
 0001:0001c821       ??$common_set_variable_in_environment_nolock@D@@YAHQADH@Z 1001d821 f   libucrt:setenv.obj
 0001:0001ca81       ??$common_set_variable_in_environment_nolock@_W@@YAHQA_WH@Z 1001da81 f   libucrt:setenv.obj
 0001:0001cd0c       ??$copy_environment@D@@YAPAPADQAPAD@Z 1001dd0c f   libucrt:setenv.obj
 0001:0001cdbc       ??$copy_environment@_W@@YAPAPA_WQAPA_W@Z 1001ddbc f   libucrt:setenv.obj
 0001:0001ce7a       ??$ensure_current_environment_is_not_initial_environment_nolock@D@@YAXXZ 1001de7a f   libucrt:setenv.obj
 0001:0001ce94       ??$ensure_current_environment_is_not_initial_environment_nolock@_W@@YAXXZ 1001de94 f   libucrt:setenv.obj
 0001:0001ceae       ??$find_in_environment_nolock@D@@YAHQBDI@Z 1001deae f   libucrt:setenv.obj
 0001:0001cf03       ??$find_in_environment_nolock@_W@@YAHQB_WI@Z 1001df03 f   libucrt:setenv.obj
 0001:0001cf7d       ??$common_tcsncpy_s@D@@YAHQADIQBDI@Z 1001df7d f   libucrt:strncpy_s.obj
 0001:0001d0fd       ??$?RV<lambda_9e9de3de5fa147e2223d7db92bc10aa6>@@AAV<lambda_38ce7e780aa69e748d6df282ebc68efe>@@V<lambda_8ca6da459f0f6780f1cff60fdc3d00e5>@@@?$__crt_seh_guarded_call@H@@QAEH$$QAV<lambda_9e9de3de5fa147e2223d7db92bc10aa6>@@AAV<lambda_38ce7e780aa69e748d6df282ebc68efe>@@$$QAV<lambda_8ca6da459f0f6780f1cff60fdc3d00e5>@@@Z 1001e0fd f   libucrt:commit.obj
 0001:0001d21c       ?write_double_translated_ansi_nolock@@YA?AUwrite_result@?A0x17268360@@HQBDIAAV__crt_cached_ptd_host@@@Z 1001e21c f   libucrt:write.obj
 0001:0001d5e3       ?write_double_translated_unicode_nolock@@YA?AUwrite_result@?A0x17268360@@QBDI@Z 1001e5e3 f   libucrt:write.obj
 0001:0001d64b       ?write_requires_double_translation_nolock@@YA_NHAAV__crt_cached_ptd_host@@@Z 1001e64b f   libucrt:write.obj
 0001:0001d6c8       ?write_text_ansi_nolock@@YA?AUwrite_result@?A0x17268360@@HQBDI@Z 1001e6c8 f   libucrt:write.obj
 0001:0001d7a3       ?write_text_utf16le_nolock@@YA?AUwrite_result@?A0x17268360@@HQBDI@Z 1001e7a3 f   libucrt:write.obj
 0001:0001d88c       ?write_text_utf8_nolock@@YA?AUwrite_result@?A0x17268360@@HQBDI@Z 1001e88c f   libucrt:write.obj
 0001:0001dd22       ?get_drive_number_from_path@@YAHQB_W@Z 1001ed22 f   libucrt:drive.obj
 0001:0001dfb3       ??$common_fullpath@_W@@YAPA_WQA_WQB_WIHQBDH@Z 1001efb3 f   libucrt:fullpath.obj
 0001:0001e80a       ??$common_loctotime_t@_J@@YA_JHHHHHHH@Z 1001f80a f   libucrt:loctotime.obj
 0001:0001ea93       ?<lambda_invoker_cdecl>@<lambda_838c7f62c73c983481e27c09e84b0b5d>@@CAHPBX0@Z 1001fa93 f   libucrt:argv_wildcards.obj
 0001:0001eb71       ??$common_expand_argv_wildcards@D@@YAHQAPADQAPAPAD@Z 1001fb71 f   libucrt:argv_wildcards.obj
 0001:0001ecee       ??$copy_and_add_argument_to_buffer@D@@YAHQBD0IAAV?$argument_list@D@?A0x5f5c8891@@@Z 1001fcee f   libucrt:argv_wildcards.obj
 0001:0001ed9f       ??$expand_argument_wildcards@D@@YAHQAD0AAV?$argument_list@D@?A0x5f5c8891@@@Z 1001fd9f f   libucrt:argv_wildcards.obj
 0001:0001f024       ??1?$argument_list@D@?A0x5f5c8891@@QAE@XZ 10020024 f   libucrt:argv_wildcards.obj
 0001:0001f085       ?expand_if_necessary@?$argument_list@D@?A0x5f5c8891@@AAEHXZ 10020085 f   libucrt:argv_wildcards.obj
 0001:0001f1b8       ??$?RV<lambda_ceb1ee4838e85a9d631eb091e2fbe199>@@AAV<lambda_ae742caa10f662c28703da3d2ea5e57e>@@V<lambda_cd08b5d6af4937fe54fc07d0c9bf6b37>@@@?$__crt_seh_guarded_call@X@@QAEX$$QAV<lambda_ceb1ee4838e85a9d631eb091e2fbe199>@@AAV<lambda_ae742caa10f662c28703da3d2ea5e57e>@@$$QAV<lambda_cd08b5d6af4937fe54fc07d0c9bf6b37>@@@Z 100201b8 f   libucrt:mbctype.obj
 0001:0001f205       ??R<lambda_ae742caa10f662c28703da3d2ea5e57e>@@QBE@XZ 10020205 f   libucrt:mbctype.obj
 0001:0001f288       ?CPtoLocaleName@@YAPB_WH@Z 10020288 f   libucrt:mbctype.obj
 0001:0001f2c6       ?getSystemCP@@YAHH@Z       100202c6 f   libucrt:mbctype.obj
 0001:0001f337       ?setSBCS@@YAXPAU__crt_multibyte_data@@@Z 10020337 f   libucrt:mbctype.obj
 0001:0001f39a       ?setSBUpLow@@YAXPAU__crt_multibyte_data@@@Z 1002039a f   libucrt:mbctype.obj
 0001:0001f53f       ?setmbcp_internal@@YAHH_NQAU__acrt_ptd@@QAPAU__crt_multibyte_data@@@Z 1002053f f   libucrt:mbctype.obj
 0001:0001f694       ?update_thread_multibyte_data_internal@@YAPAU__crt_multibyte_data@@QAU__acrt_ptd@@QAPAU1@@Z 10020694 f   libucrt:mbctype.obj
 0001:0001f994       ?x_ismbbtype_l@@YAHPAU__crt_locale_pointers@@IHH@Z 10020994 f   libucrt:ismbbyte.obj
 0001:0001fa15       ?find_end_of_double_null_terminated_sequence@@YAPB_WQB_W@Z 10020a15 f   libucrt:get_environment_from_os.obj
 0001:0001fced       ??$?RV<lambda_cbab9ec6f41b0180b23cc171c22676b0>@@AAV<lambda_44731a7d0e6d81c3e6aa82d741081786>@@V<lambda_4b292cb8dd18144e164572427af410ab>@@@?$__crt_seh_guarded_call@P6AXH@Z@@QAEP6AXH@Z$$QAV<lambda_cbab9ec6f41b0180b23cc171c22676b0>@@AAV<lambda_44731a7d0e6d81c3e6aa82d741081786>@@$$QAV<lambda_4b292cb8dd18144e164572427af410ab>@@@Z 10020ced f   libucrt:signal.obj
 0001:0001fd55       ?get_global_action_nolock@@YAPAP6AXH@ZH@Z 10020d55 f   libucrt:signal.obj
 0001:0001fd97       ?siglookup@@YAPAU__crt_signal_action_t@@HQAU1@@Z 10020d97 f   libucrt:signal.obj
 0001:00020060       $$000000                   10021060     libucrt:_strnicm.obj
 0001:00020435       ?GetTableIndexFromLocaleName@@YAHPB_W@Z 10021435 f   libucrt:lcidtoname_downlevel.obj
 0001:000209d7       ?free_crt_array_internal@@YAXQAPBXI@Z 100219d7 f   libucrt:inittime.obj
 0001:00020ae0       ??$common_tcsncpy_s@_W@@YAHQA_WIQB_WI@Z 10021ae0 f   libucrt:wcsncpy_s.obj
 0001:00020cda       ??$common_refill_and_read_nolock@D@@YAHV__crt_stdio_stream@@@Z 10021cda f   libucrt:_filbuf.obj
 0001:00020ec3       ?check_trailing@@YA_NPBDW4__acrt_has_trailing_digits@@@Z 10021ec3 f   libucrt:_fptostr.obj
 0001:00020ee6       ?should_round_up@@YA_NQBD0HW4__acrt_has_trailing_digits@@W4__acrt_rounding_mode@@@Z 10021ee6 f   libucrt:_fptostr.obj
 0001:00022706       ??R<lambda_e96123212306c92459f955e8e4eac55d>@@QBEIPBD@Z 10023706 f   libucrt:mbrtowc.obj
 0001:0002287d       ??$common_flush_and_write_nolock@D@@YAHHV__crt_stdio_stream@@AAV__crt_cached_ptd_host@@@Z 1002387d f   libucrt:_flsbuf.obj
 0001:00022973       ??$write_buffer_nolock@D@@YA_NDV__crt_stdio_stream@@AAV__crt_cached_ptd_host@@@Z 10023973 f   libucrt:_flsbuf.obj
 0001:00022a45       ?stream_is_at_end_of_file_nolock@@YA_NV__crt_stdio_stream@@@Z 10023a45 f   libucrt:_flsbuf.obj
 0001:00022b4a       ?to_abstract_control@@YA?AW4__acrt_fenv_abstract_control@@W4__acrt_fenv_machine_sse_control@@@Z 10023b4a f   libucrt:_fenvutils.obj
 0001:00022bfa       ?to_abstract_control@@YA?AW4__acrt_fenv_abstract_control@@W4__acrt_fenv_machine_x87_control@@@Z 10023bfa f   libucrt:_fenvutils.obj
 0001:00022ca7       ?to_machine_sse_control@@YA?AW4__acrt_fenv_machine_sse_control@@W4__acrt_fenv_abstract_control@@@Z 10023ca7 f   libucrt:_fenvutils.obj
 0001:00022d5d       ?to_machine_x87_control@@YA?AW4__acrt_fenv_machine_x87_control@@W4__acrt_fenv_abstract_control@@@Z 10023d5d f   libucrt:_fenvutils.obj
 0001:0002313b       ?InternalCompareStringA@@YAHPAU__crt_locale_pointers@@PB_WKPBDH2HH@Z 1002413b f   libucrt:comparestringa.obj
 0001:000234e7       ??$common_getdcwd@_W@@YAPA_WHPA_WHHQBDH@Z 100244e7 f   libucrt:getcwd.obj
 0001:0002363b       ?is_valid_drive@@YAHI@Z    1002463b f   libucrt:getcwd.obj
 0001:00023887       ?_isindst_nolock@@YAHQAUtm@@@Z 10024887 f   libucrt:tzset.obj
 0001:00023aa1       ?cvtdate@@YAXW4transition_type@?A0x7639d0b4@@W4date_type@2@HHHHHHHHH@Z 10024aa1 f   libucrt:tzset.obj
 0001:00023be4       ?get_tz_environment_variable@@YAPA_WAAY0BAA@_W@Z 10024be4 f   libucrt:tzset.obj
 0001:00023c5b       ?tzset_env_copy_to_tzname@@YAXQB_WQA_WQADI@Z 10024c5b f   libucrt:tzset.obj
 0001:00023ca2       ?tzset_from_environment_nolock@@YAXPA_W@Z 10024ca2 f   libucrt:tzset.obj
 0001:00023f34       ?tzset_from_system_nolock@@YAXXZ 10024f34 f   libucrt:tzset.obj
 0001:0002408e       ?tzset_nolock@@YAXXZ       1002508e f   libucrt:tzset.obj
 0001:00024104       ?tzset_os_copy_to_tzname@@YAXQB_WQA_WQADI@Z 10025104 f   libucrt:tzset.obj
 0001:00024792       ?__acrt_LCMapStringA_stat@@YAHPAU__crt_locale_pointers@@PB_WKPBDHPADHHH@Z 10025792 f   libucrt:lcmapstringa.obj
 0001:000249ca       ?initialize_multibyte@@YAHXZ 100259ca f   libucrt:multibyte_initializer.obj
 0001:00024b40       $$000000                   10025b40     libucrt:log10_impl.obj
 0001:00024c50       $$000000                   10025c50     libucrt:ceil_pentium4.obj
 0001:00024f70       ?__dcrt_lowio_initialize_console_output@@YAXXZ 10025f70 f   libucrt:initcon.obj
 0001:00025058       ___hw_cw_sse2              10026058 f   libucrt:ieee87.obj
 0001:000254de       __hw_cw                    100264de f   libucrt:ieee87.obj
 0001:00025590       $$000000                   10026590     libucrt:log10_pentium4.obj
 0001:00025820       $$000000                   10026820     libucrt:87tran.obj
 0001:00025a30       $$000000                   10026a30     libucrt:87disp.obj
 0001:00025c90       $$000000                   10026c90     libucrt:common.obj
 0001:00025e20       $$000000                   10026e20     libucrt:genexcep.obj
 0001:00027070       $$000000                   10028070     LIBCMT:ulldiv.obj
 0001:00027092       L1                         10028092     LIBCMT:ulldiv.obj
 0001:000270a0       L3                         100280a0     LIBCMT:ulldiv.obj
 0001:000270ce       L4                         100280ce     LIBCMT:ulldiv.obj
 0001:000270cf       L5                         100280cf     LIBCMT:ulldiv.obj
 0001:000270d3       L2                         100280d3     LIBCMT:ulldiv.obj
 0001:000270e0       $$000000                   100280e0     LIBCMT:ullrem.obj
 0001:00027101       L1                         10028101     LIBCMT:ullrem.obj
 0001:0002710f       L3                         1002810f     LIBCMT:ullrem.obj
 0001:0002713a       L4                         1002813a     LIBCMT:ullrem.obj
 0001:00027142       L5                         10028142     LIBCMT:ullrem.obj
 0001:00027151       L2                         10028151     LIBCMT:ullrem.obj
 0001:00027160       $$000000                   10028160     LIBCMT:llshl.obj
 0001:00027170       MORE32                     10028170     LIBCMT:llshl.obj
 0001:0002717a       RETZERO                    1002817a     LIBCMT:llshl.obj
 0001:00027180       $$000000                   10028180     LIBCMT:ullshr.obj
 0001:00027190       MORE32                     10028190     LIBCMT:ullshr.obj
 0001:0002719a       RETZERO                    1002819a     LIBCMT:ullshr.obj
 0001:000271a0       $$000000                   100281a0     LIBCMT:chkstk.obj
 0001:000271b4       cs10                       100281b4     LIBCMT:chkstk.obj
 0001:000271c2       cs20                       100281c2     LIBCMT:chkstk.obj
 0001:000271d0       $$000000                   100281d0     LIBCMT:alloca16.obj
 0001:000271e6       alloca_8                   100281e6     LIBCMT:alloca16.obj
 0001:00027200       $$000000                   10028200     LIBCMT:ftol2.obj
 0001:00027210       $$000000                   10028210     LIBCMT:ftol2.obj
 0001:00027221       L3B                        10028221     LIBCMT:ftol2.obj
 0001:00027264       L3F                        10028264     LIBCMT:ftol2.obj
 0001:0002726c       L40                        1002826c     LIBCMT:ftol2.obj
 0001:0002727f       L41                        1002827f     LIBCMT:ftol2.obj
 0001:00027455       __ehhandler$?CallUnexpected@@YAXPBU_s_ESTypeList@@@Z 10028455 f   libvcruntime:frame.obj
 0001:00027472       __ehhandler$?common_exit@@YAXHW4_crt_exit_cleanup_mode@@W4_crt_exit_return_mode@@@Z 10028472 f   libucrt:exit.obj
 0001:0002748f       __ehhandler$?try_cor_exit_process@@YAXI@Z 1002848f f   libucrt:exit.obj
 0001:000274ac       __ehhandler$___dcrt_uninitialize_environments_nolock 100284ac f   libucrt:environment_initialization.obj
 0001:000274c9       __ehhandler$__execute_onexit_table 100284c9 f   libucrt:onexit.obj
 0001:000274e6       __ehhandler$?write_double_translated_ansi_nolock@@YA?AUwrite_result@?A0x17268360@@HQBDIAAV__crt_cached_ptd_host@@@Z 100284e6 f   libucrt:write.obj
 0002:00000268       ?lenfix@?1??fixedtables@@9@9 10029268     inflate.obj
 0002:00000a68       ?distfix@?1??fixedtables@@9@9 10029a68     inflate.obj
 0002:00000ae8       ?order@?1??inflate@@9@9    10029ae8     inflate.obj
 0002:00000cd8       ?lbase@?1??inflate_table@@9@9 10029cd8     inftrees.obj
 0002:00000d18       ?lext@?1??inflate_table@@9@9 10029d18     inftrees.obj
 0002:00000d58       ?dbase@?1??inflate_table@@9@9 10029d58     inftrees.obj
 0002:00000d98       ?dext@?1??inflate_table@@9@9 10029d98     inftrees.obj
 0002:00000de4       ?format@?1??SetClassPath@@9@9 10029de4     java.obj
 0002:000026a0       _crc_table                 1002b6a0     zcrc32.obj
 0002:00002aa0       _crc_big_table             1002baa0     zcrc32.obj
 0002:00002ea0       _crc_braid_table           1002bea0     zcrc32.obj
 0002:00003ea0       _crc_braid_big_table       1002cea0     zcrc32.obj
 0002:00004ea0       _x2n_table                 1002dea0     zcrc32.obj
 0002:00004fc8       _GS_ExceptionPointers      1002dfc8     LIBCMT:gs_report.obj
 0002:00004fd8       ?tokenTable@@3QBUStringLiteral@@B 1002dfd8     libvcruntime:undname.obj
 0002:00005060       ?nameTable@@3QBUStringLiteral@@B 1002e060     libvcruntime:undname.obj
 0002:000052f8       ?rttiTable@@3QBUStringLiteral@@B 1002e2f8     libvcruntime:undname.obj
 0002:00005320       ?IndirectionName@@3QBUStringLiteral@@B 1002e320     libvcruntime:undname.obj
 0002:00005350       ?PrefixName@@3QBUStringLiteral@@B 1002e350     libvcruntime:undname.obj
 0002:00005988       ?module_names@?A0x14174aea@@3QBQB_WB 1002e988     libvcruntime:winapi_downlevel.obj
 0002:00005a30       ?candidate_modules@?1??try_get_FlsAlloc@@YAP6GKP6GXPAX@Z@ZXZ@4QBW4module_id@?A0x14174aea@@B 1002ea30     libvcruntime:winapi_downlevel.obj
 0002:00005a44       ?candidate_modules@?1??try_get_FlsFree@@YAP6GHK@ZXZ@4QBW4module_id@?A0x14174aea@@B 1002ea44     libvcruntime:winapi_downlevel.obj
 0002:00005a54       ?candidate_modules@?1??try_get_FlsGetValue@@YAP6GPAXK@ZXZ@4QBW4module_id@?A0x14174aea@@B 1002ea54     libvcruntime:winapi_downlevel.obj
 0002:00005a68       ?candidate_modules@?1??try_get_FlsSetValue@@YAP6GHKPAX@ZXZ@4QBW4module_id@?A0x14174aea@@B 1002ea68     libvcruntime:winapi_downlevel.obj
 0002:00005a7c       ?candidate_modules@?1??try_get_InitializeCriticalSectionEx@@YAP6GHPAU_RTL_CRITICAL_SECTION@@KK@ZXZ@4QBW4module_id@?A0x14174aea@@B 1002ea7c     libvcruntime:winapi_downlevel.obj
 0002:000067f0       ?errtable@@3QBUerrentry@?A0x31fdb9ec@@B 1002f7f0     libucrt:errno.obj
 0002:00006a78       ___acrt_initializers       1002fa78     libucrt:initialization.obj
 0002:00006af8       ?module_names@?A0x391cf84c@@3QBQB_WB 1002faf8     libucrt:winapi_thunks.obj
 0002:00007004       ?candidate_modules@?1??try_get_AreFileApisANSI@@YAP6GHXZXZ@4QBW4module_id@?A0x391cf84c@@B 10030004     libucrt:winapi_thunks.obj
 0002:00007018       ?candidate_modules@?1??try_get_CompareStringEx@@YAP6GHPB_WK0H0HPAU_nlsversioninfo@@PAXJ@ZXZ@4QBW4module_id@?A0x391cf84c@@B 10030018     libucrt:winapi_thunks.obj
 0002:00007030       ?candidate_modules@?1??try_get_InitializeCriticalSectionEx@@YAP6GHPAU_RTL_CRITICAL_SECTION@@KK@ZXZ@4QBW4module_id@?A0x391cf84c@@B 10030030     libucrt:winapi_thunks.obj
 0002:00007038       ?candidate_modules@?1??try_get_LCMapStringEx@@YAP6GHPB_WK0HPA_WHPAU_nlsversioninfo@@PAXJ@ZXZ@4QBW4module_id@?A0x391cf84c@@B 10030038     libucrt:winapi_thunks.obj
 0002:00007050       ?candidate_modules@?1??try_get_LocaleNameToLCID@@YAP6GKPB_WK@ZXZ@4QBW4module_id@?A0x391cf84c@@B 10030050     libucrt:winapi_thunks.obj
 0002:0000706c       ?candidate_modules@?1??try_get_RoInitialize@@YAP6GJW4RO_INIT_TYPE@@@ZXZ@4QBW4module_id@?A0x391cf84c@@B 1003006c     libucrt:winapi_thunks.obj
 0002:00007080       ?candidate_modules@?1??try_get_RoUninitialize@@YAP6GXXZXZ@4QBW4module_id@?A0x391cf84c@@B 10030080     libucrt:winapi_thunks.obj
 0002:00007094       ?candidate_modules@?1??try_get_AppPolicyGetProcessTerminationMethod@@YAP6GJPAXPAW4AppPolicyProcessTerminationMethod@@@ZXZ@4QBW4module_id@?A0x391cf84c@@B 10030094     libucrt:winapi_thunks.obj
 0002:000070c0       ?candidate_modules@?1??try_get_AppPolicyGetThreadInitializationType@@YAP6GJPAXPAW4AppPolicyThreadInitializationType@@@ZXZ@4QBW4module_id@?A0x391cf84c@@B 100300c0     libucrt:winapi_thunks.obj
 0002:000070ec       ?candidate_modules@?1??try_get_FlsAlloc@@YAP6GKP6GXPAX@Z@ZXZ@4QBW4module_id@?A0x391cf84c@@B 100300ec     libucrt:winapi_thunks.obj
 0002:000070f4       ?candidate_modules@?1??try_get_FlsFree@@YAP6GHK@ZXZ@4QBW4module_id@?A0x391cf84c@@B 100300f4     libucrt:winapi_thunks.obj
 0002:000070fc       ?candidate_modules@?1??try_get_FlsGetValue@@YAP6GPAXK@ZXZ@4QBW4module_id@?A0x391cf84c@@B 100300fc     libucrt:winapi_thunks.obj
 0002:00007104       ?candidate_modules@?1??try_get_FlsSetValue@@YAP6GHKPAX@ZXZ@4QBW4module_id@?A0x391cf84c@@B 10030104     libucrt:winapi_thunks.obj
 0002:000075f0       ?strings@?1??fp_format_nan_or_infinity@@YAHW4__acrt_fp_class@@_NPADI1@Z@4QAY03QBDA 100305f0     libucrt:cvt.obj
 0002:00008628       ?_mb_locale_names@@3QBQB_WB 10031628     libucrt:mbctype.obj
 0002:00008668       ?LcidToLocaleNameTable@?A0x881e4c05@@3QBULcidToLocaleName@1@B 10031668     libucrt:lcidtoname_downlevel.obj
 0002:00009790       ?LocaleNameToIndexTable@?A0x881e4c05@@3QBULocaleNameIndex@1@B 10032790     libucrt:lcidtoname_downlevel.obj
 0002:0000a770       LOG_name                   10033770     libucrt:log10_impl.obj
 0002:0000a780       _One                       10033780     libucrt:ceil_pentium4.obj
 0002:0000a790       _Bns                       10033790     libucrt:ceil_pentium4.obj
 0002:0000a7a0       _Zero                      100337a0     libucrt:ceil_pentium4.obj
 0002:0000a7b0       _S                         100337b0     libucrt:ceil_pentium4.obj
 0002:0000a7c0       _NegZero                   100337c0     libucrt:ceil_pentium4.obj
 0002:0000a7e0       emask                      100337e0     libucrt:log10_pentium4.obj
 0002:0000a7f0       CC                         100337f0     libucrt:log10_pentium4.obj
 0002:0000a800       Magic                      10033800     libucrt:log10_pentium4.obj
 0002:0000a810       hi_mask                    10033810     libucrt:log10_pentium4.obj
 0002:0000a820       LOG10_2                    10033820     libucrt:log10_pentium4.obj
 0002:0000a830       place_L                    10033830     libucrt:log10_pentium4.obj
 0002:0000a850       One                        10033850     libucrt:log10_pentium4.obj
 0002:0000a860       Zero                       10033860     libucrt:log10_pentium4.obj
 0002:0000a870       Two52                      10033870     libucrt:log10_pentium4.obj
 0002:0000a880       Infs                       10033880     libucrt:log10_pentium4.obj
 0002:0000a890       NaN                        10033890     libucrt:log10_pentium4.obj
 0002:0000a8a0       coeff                      100338a0     libucrt:log10_pentium4.obj
 0002:0000a8fe       _log2max                   100338fe     libucrt:87tran.obj
 0002:0000a908       _smallarg                  10033908     libucrt:87tran.obj
 0002:0000a912       _half                      10033912     libucrt:87tran.obj
 0002:0000a95e       One                        1003395e     libucrt:87disp.obj
 0002:0000a966       Three                      10033966     libucrt:87disp.obj
 0002:0000a96e       XAMtoTagTab                1003396e     libucrt:87disp.obj
 0002:0000a980       One                        10033980     libucrt:common.obj
 0002:0000a994       DblMax                     10033994     libucrt:common.obj
 0002:0000a99c       DblMin                     1003399c     libucrt:common.obj
 0002:0000a9a4       IeeeAdjO                   100339a4     libucrt:common.obj
 0002:0000a9ac       IeeeAdjU                   100339ac     libucrt:common.obj
 0002:0000a9b4       _infinity                  100339b4     libucrt:common.obj
 0002:0000a9bc       _zero                      100339bc     libucrt:common.obj
 0002:0000a9f8       _over                      100339f8     libucrt:fpctrl.obj
 0002:0000aa04       _under                     10033a04     libucrt:fpctrl.obj
 0002:0000b238       ?_names@?1??_get_fname@@9@4QBU<unnamed-type-_names>@?1??1@YAPADI@Z@B 10034238     libucrt:fpexcept.obj
 0002:0000b3e0       two32                      100343e0     LIBCMT:ftol2.obj
 0002:0000b3e4       two63                      100343e4     LIBCMT:ftol2.obj
 0002:0000b3e8       _NaN                       100343e8     LIBCMT:ftol2.obj
 0002:0000bbe8       __sehtable$?dllmain_crt_process_attach@@YAHQAUHINSTANCE__@@QAX@Z 10034be8     LIBCMT:dll_dllmain.obj
 0002:0000bc08       __sehtable$?dllmain_crt_process_detach@@YAH_N@Z 10034c08     LIBCMT:dll_dllmain.obj
 0002:0000bc30       __sehtable$?dllmain_dispatch@@YAHQAUHINSTANCE__@@KQAX@Z 10034c30     LIBCMT:dll_dllmain.obj
 0002:0000bc50       __sehtable$___scrt_is_nonwritable_in_current_image 10034c50     LIBCMT:utility.obj
 0002:0000bc70       __sehtable$___DestructExceptionObject 10034c70     libvcruntime:ehhelpers.obj
 0002:0000bc90       __sehtable$?FrameUnwindToState@__FrameHandler3@@SAXPAUEHRegistrationNode@@PAXPBU_s_FuncInfo@@H@Z 10034c90     libvcruntime:frame.obj
 0002:0000bcb8       __sehtable$?CallCatchBlock@@YAPAXPAUEHExceptionRecord@@PAUEHRegistrationNode@@PAU_CONTEXT@@PBU_s_FuncInfo@@PAXHK@Z 10034cb8     libvcruntime:frame.obj
 0002:0000bce0       __catchsym$?CallUnexpected@@YAXPBU_s_ESTypeList@@@Z$2 10034ce0     libvcruntime:frame.obj
 0002:0000bcf0       __unwindtable$?CallUnexpected@@YAXPBU_s_ESTypeList@@@Z 10034cf0     libvcruntime:frame.obj
 0002:0000bd00       __tryblocktable$?CallUnexpected@@YAXPBU_s_ESTypeList@@@Z 10034d00     libvcruntime:frame.obj
 0002:0000bd14       __ehfuncinfo$?CallUnexpected@@YAXPBU_s_ESTypeList@@@Z 10034d14     libvcruntime:frame.obj
 0002:0000bd38       __sehtable$??$BuildCatchObjectHelperInternal@V__FrameHandler3@@@@YAHPAUEHExceptionRecord@@PAXPBU_s_HandlerType@@PBU_s_CatchableType@@@Z 10034d38     libvcruntime:frame.obj
 0002:0000bd58       __sehtable$??$BuildCatchObjectInternal@V__FrameHandler3@@@@YAXPAUEHExceptionRecord@@PAXPBU_s_HandlerType@@PBU_s_CatchableType@@@Z 10034d58     libvcruntime:frame.obj
 0002:0000bdc8       __sehtable$?_fclose_internal@@YAHQAU_iobuf@@AAV__crt_cached_ptd_host@@@Z 10034dc8     libucrt:fclose.obj
 0002:0000bde8       __sehtable$??$common_fgets@D@@YAPADQADHV__crt_stdio_stream@@@Z 10034de8     libucrt:fgets.obj
 0002:0000be08       __sehtable$??$common_fsopen@D@@YAPAU_iobuf@@QBD0H@Z 10034e08     libucrt:fopen.obj
 0002:0000be28       __sehtable$??$?RV<lambda_62491a2101a2aba6cc4a769149c84f1f>@@AAV<lambda_826c27fce7726908515bbc79a5266961>@@V<lambda_4e64bbd54b50a7b070e3ea8d795375b6>@@@?$__crt_seh_guarded_call@H@@QAEH$$QAV<lambda_62491a2101a2aba6cc4a769149c84f1f>@@AAV<lambda_826c27fce7726908515bbc79a5266961>@@$$QAV<lambda_4e64bbd54b50a7b070e3ea8d795375b6>@@@Z 10034e28     libucrt:output.obj
 0002:0000be44       __ehfuncinfo$?write_double_translated_ansi_nolock@@YA?AUwrite_result@?A0x17268360@@HQBDIAAV__crt_cached_ptd_host@@@Z 10034e44     libucrt:write.obj
 0002:0000be44       __ehfuncinfo$?try_cor_exit_process@@YAXI@Z 10034e44     libucrt:exit.obj
 0002:0000be68       __unwindtable$?common_exit@@YAXHW4_crt_exit_cleanup_mode@@W4_crt_exit_return_mode@@@Z 10034e68     libucrt:exit.obj
 0002:0000be70       __ehfuncinfo$?common_exit@@YAXHW4_crt_exit_cleanup_mode@@W4_crt_exit_return_mode@@@Z 10034e70     libucrt:exit.obj
 0002:0000be98       __sehtable$??R<lambda_6e4b09c48022b2350581041d5f6b0c4c>@@QBE@XZ 10034e98     libucrt:exit.obj
 0002:0000beb8       __sehtable$??$?RV<lambda_03b1d95aef87969028cfba75ccab2455>@@AAV<lambda_6e4b09c48022b2350581041d5f6b0c4c>@@V<lambda_22bdf7517842c4b3e53723af5aa32b9e>@@@?$__crt_seh_guarded_call@X@@QAEX$$QAV<lambda_03b1d95aef87969028cfba75ccab2455>@@AAV<lambda_6e4b09c48022b2350581041d5f6b0c4c>@@$$QAV<lambda_22bdf7517842c4b3e53723af5aa32b9e>@@@Z 10034eb8     libucrt:exit.obj
 0002:0000bed8       __sehtable$??$common_getenv@D@@YAPADQBD@Z 10034ed8     libucrt:getenv.obj
 0002:0000bef8       __sehtable$??$common_getenv_s@_W@@YAHQAIQA_WIQB_W@Z 10034ef8     libucrt:getenv.obj
 0002:0000bf18       __sehtable$??$common_putenv@D@@YAHQBD0@Z 10034f18     libucrt:putenv.obj
 0002:0000bf38       __sehtable$??$thread_start@P6GIPAX@Z$00@@YGKQAX@Z 10034f38     libucrt:thread.obj
 0002:0000bf58       __sehtable$??$?RV<lambda_2866be3712abc81a800a822484c830d8>@@AAV<lambda_39ca0ed439415581b5b15c265174cece>@@V<lambda_2b24c74d71094a6cd0cb82e44167d71b>@@@?$__crt_seh_guarded_call@X@@QAEX$$QAV<lambda_2866be3712abc81a800a822484c830d8>@@AAV<lambda_39ca0ed439415581b5b15c265174cece>@@$$QAV<lambda_2b24c74d71094a6cd0cb82e44167d71b>@@@Z 10034f58     libucrt:fflush.obj
 0002:0000bf78       __sehtable$??$?RV<lambda_2cc53f568c5a2bb6f192f930a45d44ea>@@AAV<lambda_ab61a845afdef5b7c387490eaf3616ee>@@V<lambda_c2ffc0b7726aa6be21d5f0026187e748>@@@?$__crt_seh_guarded_call@X@@QAEX$$QAV<lambda_2cc53f568c5a2bb6f192f930a45d44ea>@@AAV<lambda_ab61a845afdef5b7c387490eaf3616ee>@@$$QAV<lambda_c2ffc0b7726aa6be21d5f0026187e748>@@@Z 10034f78     libucrt:fflush.obj
 0002:0000bf98       __sehtable$??$?RV<lambda_6d20deecaf4856105ebacbad442d1079>@@AAV<lambda_9a32fed5bf61b6b509b2d3f6003082a1>@@V<lambda_63ea2239ed67c638ddbae41947fdf875>@@@?$__crt_seh_guarded_call@H@@QAEH$$QAV<lambda_6d20deecaf4856105ebacbad442d1079>@@AAV<lambda_9a32fed5bf61b6b509b2d3f6003082a1>@@$$QAV<lambda_63ea2239ed67c638ddbae41947fdf875>@@@Z 10034f98     libucrt:fflush.obj
 0002:0000bfb8       __sehtable$?_perror_internal@@YAXQBDAAV__crt_cached_ptd_host@@@Z 10034fb8     libucrt:perror.obj
 0002:0000bfd8       __sehtable$??$common_lseek@_J@@YA_JH_JHAAV__crt_cached_ptd_host@@@Z 10034fd8     libucrt:lseek.obj
 0002:0000bff4       __unwindtable$___dcrt_uninitialize_environments_nolock 10034ff4     libucrt:environment_initialization.obj
 0002:0000c004       __ehfuncinfo$___dcrt_uninitialize_environments_nolock 10035004     libucrt:environment_initialization.obj
 0002:0000c028       __unwindtable$__execute_onexit_table 10035028     libucrt:onexit.obj
 0002:0000c030       __ehfuncinfo$__execute_onexit_table 10035030     libucrt:onexit.obj
 0002:0000c058       __sehtable$??$?RV<lambda_69a2805e680e0e292e8ba93315fe43a8>@@AAV<lambda_f03950bc5685219e0bcd2087efbe011e>@@V<lambda_03fcd07e894ec930e3f35da366ca99d6>@@@?$__crt_seh_guarded_call@H@@QAEH$$QAV<lambda_69a2805e680e0e292e8ba93315fe43a8>@@AAV<lambda_f03950bc5685219e0bcd2087efbe011e>@@$$QAV<lambda_03fcd07e894ec930e3f35da366ca99d6>@@@Z 10035058     libucrt:onexit.obj
 0002:0000c078       __sehtable$_terminate      10035078     libucrt:terminate.obj
 0002:0000c098       __sehtable$??$?RV<lambda_d422a76eb4c3bf3ad751449ab71a6ea4>@@AAV<lambda_c9ba49e555ba839a7b07aa3fbecb7617>@@V<lambda_9476263c8ee91a25d21c55370bdb50de>@@@?$__crt_seh_guarded_call@H@@QAEH$$QAV<lambda_d422a76eb4c3bf3ad751449ab71a6ea4>@@AAV<lambda_c9ba49e555ba839a7b07aa3fbecb7617>@@$$QAV<lambda_9476263c8ee91a25d21c55370bdb50de>@@@Z 10035098     libucrt:close.obj
 0002:0000c0b8       __sehtable$??$common_open@D@@YAHQBDHH@Z 100350b8     libucrt:open.obj
 0002:0000c0d8       __sehtable$??$common_sopen_dispatch@D@@YAHQBDHHHQAHH@Z 100350d8     libucrt:open.obj
 0002:0000c0f8       __sehtable$__read          100350f8     libucrt:read.obj
 0002:0000c118       __sehtable$__fcloseall     10035118     libucrt:closeall.obj
 0002:0000c138       __sehtable$___acrt_initialize_lowio 10035138     libucrt:ioinit.obj
 0002:0000c158       __sehtable$?__acrt_stdio_allocate_stream@@YA?AV__crt_stdio_stream@@XZ 10035158     libucrt:stream.obj
 0002:0000c178       __sehtable$??$?RV<lambda_15ade71b0218206bbe3333a0c9b79046>@@AAV<lambda_da44e0f8b0f19ba52fefafb335991732>@@V<lambda_207f2d024fc103971653565357d6cd41>@@@?$__crt_seh_guarded_call@X@@QAEX$$QAV<lambda_15ade71b0218206bbe3333a0c9b79046>@@AAV<lambda_da44e0f8b0f19ba52fefafb335991732>@@$$QAV<lambda_207f2d024fc103971653565357d6cd41>@@@Z 10035178     libucrt:per_thread_data.obj
 0002:0000c198       __sehtable$??$?RV<lambda_a7e850c220f1c8d1e6efeecdedd162c6>@@AAV<lambda_46720907175c18b6c9d2717bc0d2d362>@@V<lambda_9048902d66e8d99359bc9897bbb930a8>@@@?$__crt_seh_guarded_call@X@@QAEX$$QAV<lambda_a7e850c220f1c8d1e6efeecdedd162c6>@@AAV<lambda_46720907175c18b6c9d2717bc0d2d362>@@$$QAV<lambda_9048902d66e8d99359bc9897bbb930a8>@@@Z 10035198     libucrt:per_thread_data.obj
 0002:0000c1b8       __sehtable$??$?RV<lambda_38edbb1296d33220d7e4dd0ed76b244a>@@AAV<lambda_5ce1d447e08cb34b2473517608e21441>@@V<lambda_fb385d3da700c9147fc39e65dd577a8c>@@@?$__crt_seh_guarded_call@X@@QAEX$$QAV<lambda_38edbb1296d33220d7e4dd0ed76b244a>@@AAV<lambda_5ce1d447e08cb34b2473517608e21441>@@$$QAV<lambda_fb385d3da700c9147fc39e65dd577a8c>@@@Z 100351b8     libucrt:per_thread_data.obj
 0002:0000c1d8       __sehtable$??$?RV<lambda_6affb1475c98b40b75cdec977db92e3c>@@AAV<lambda_b8d4b9c228a6ecc3f80208dbb4b4a104>@@V<lambda_608742c3c92a14382c1684fc64f96c88>@@@?$__crt_seh_guarded_call@X@@QAEX$$QAV<lambda_6affb1475c98b40b75cdec977db92e3c>@@AAV<lambda_b8d4b9c228a6ecc3f80208dbb4b4a104>@@$$QAV<lambda_608742c3c92a14382c1684fc64f96c88>@@@Z 100351d8     libucrt:per_thread_data.obj
 0002:0000c1f8       __sehtable$??$?RV<lambda_e5124f882df8998aaf41531e079ba474>@@AAV<lambda_3e16ef9562a7dcce91392c22ab16ea36>@@V<lambda_e25ca0880e6ef98be67edffd8c599615>@@@?$__crt_seh_guarded_call@X@@QAEX$$QAV<lambda_e5124f882df8998aaf41531e079ba474>@@AAV<lambda_3e16ef9562a7dcce91392c22ab16ea36>@@$$QAV<lambda_e25ca0880e6ef98be67edffd8c599615>@@@Z 100351f8     libucrt:wsetlocale.obj
 0002:0000c218       __sehtable$??$?RV<lambda_9e9de3de5fa147e2223d7db92bc10aa6>@@AAV<lambda_38ce7e780aa69e748d6df282ebc68efe>@@V<lambda_8ca6da459f0f6780f1cff60fdc3d00e5>@@@?$__crt_seh_guarded_call@H@@QAEH$$QAV<lambda_9e9de3de5fa147e2223d7db92bc10aa6>@@AAV<lambda_38ce7e780aa69e748d6df282ebc68efe>@@$$QAV<lambda_8ca6da459f0f6780f1cff60fdc3d00e5>@@@Z 10035218     libucrt:commit.obj
 0002:0000c238       __sehtable$__write_internal 10035238     libucrt:write.obj
 0002:0000c258       __sehtable$__alloc_osfhnd  10035258     libucrt:osfinfo.obj
 0002:0000c278       __sehtable$___acrt_lowio_ensure_fh_exists 10035278     libucrt:osfinfo.obj
 0002:0000c298       __sehtable$?update_thread_multibyte_data_internal@@YAPAU__crt_multibyte_data@@QAU__acrt_ptd@@QAPAU1@@Z 10035298     libucrt:mbctype.obj
 0002:0000c2b8       __sehtable$??$?RV<lambda_ceb1ee4838e85a9d631eb091e2fbe199>@@AAV<lambda_ae742caa10f662c28703da3d2ea5e57e>@@V<lambda_cd08b5d6af4937fe54fc07d0c9bf6b37>@@@?$__crt_seh_guarded_call@X@@QAEX$$QAV<lambda_ceb1ee4838e85a9d631eb091e2fbe199>@@AAV<lambda_ae742caa10f662c28703da3d2ea5e57e>@@$$QAV<lambda_cd08b5d6af4937fe54fc07d0c9bf6b37>@@@Z 100352b8     libucrt:mbctype.obj
 0002:0000c2d8       __sehtable$__query_new_handler 100352d8     libucrt:new_handler.obj
 0002:0000c2f8       __sehtable$_raise          100352f8     libucrt:signal.obj
 0002:0000c318       __sehtable$??$?RV<lambda_cbab9ec6f41b0180b23cc171c22676b0>@@AAV<lambda_44731a7d0e6d81c3e6aa82d741081786>@@V<lambda_4b292cb8dd18144e164572427af410ab>@@@?$__crt_seh_guarded_call@P6AXH@Z@@QAEP6AXH@Z$$QAV<lambda_cbab9ec6f41b0180b23cc171c22676b0>@@AAV<lambda_44731a7d0e6d81c3e6aa82d741081786>@@$$QAV<lambda_4b292cb8dd18144e164572427af410ab>@@@Z 10035318     libucrt:signal.obj
 0002:0000c338       __sehtable$___acrt_update_thread_locale_data 10035338     libucrt:locale_refcounting.obj
 0002:0000c358       __sehtable$__isindst       10035358     libucrt:tzset.obj
 0002:0000c378       __sehtable$___tzset        10035378     libucrt:tzset.obj
 0002:0000c398       __sehtable$___set_fpsr_sse2 10035398     libucrt:fpctrl.obj
 0002:0000c3b8       __sehtable$__IsNonwritableInCurrentImage 100353b8     LIBCMT:pesect.obj
 0002:0000c3e0       .edata                     100353e0     jli.exp
 0002:0000c408       rgpv                       10035408     jli.exp
 0002:0000c434       rgszName                   10035434     jli.exp
 0002:0000c460       rgwOrd                     10035460     jli.exp
 0002:0000c476       szName                     10035476     jli.exp
 0002:0000c47e       $N00001                    1003547e     jli.exp
 0002:0000c48c       $N00002                    1003548c     jli.exp
 0002:0000c49b       $N00003                    1003549b     jli.exp
 0002:0000c4aa       $N00004                    100354aa     jli.exp
 0002:0000c4b5       $N00005                    100354b5     jli.exp
 0002:0000c4c9       $N00006                    100354c9     jli.exp
 0002:0000c4d6       $N00007                    100354d6     jli.exp
 0002:0000c4ed       $N00008                    100354ed     jli.exp
 0002:0000c507       $N00009                    10035507     jli.exp
 0002:0000c526       $N00010                    10035526     jli.exp
 0002:0000c538       $N00011                    10035538     jli.exp
 0002:0000c79c       .idata$6                   1003579c     advapi32:ADVAPI32.dll
 0002:0000c7c2       .idata$6                   100357c2     comctl32:COMCTL32.dll
 0002:0000c7ec       .idata$6                   100357ec     user32:USER32.dll
 0002:0000ca6a       .idata$6                   10035a6a     kernel32:KERNEL32.dll
 0003:00000000       _launchModeNames           10036000     java.obj
 0003:0000000c       ?NMT_Env_Name@?1??SetJvmEnvironment@@9@9 1003600c     java.obj
 0003:00000010       ?whiteSpace@?1??ReadKnownVMs@@9@9 10036010     java.obj
 0003:00000018       _SPLASHSCREEN_SO           10036018     java_md.obj
 0003:0000001c       _manifest_name             1003601c     parse_manifest.obj
 0003:00000020       _separators                10036020     version_comp.obj
 0003:00000024       _zero_string               10036024     version_comp.obj
 0003:00000060       ?__vcrt_flsindex@@3KA      10036060     libvcruntime:per_thread_data.obj
 0003:00000130       ?errno_no_memory@@3HA      10036130     libucrt:errno.obj
 0003:00000134       ?doserrno_no_memory@@3KA   10036134     libucrt:errno.obj
 0003:00000280       ?__acrt_flsindex@@3KA      10036280     libucrt:per_thread_data.obj
 0003:00000570       __mbctypes                 10036570     libucrt:mbctype.obj
 0003:00000678       __mbcasemaps               10036678     libucrt:mbctype.obj
 0003:00000778       ?__rgctypeflag@@3PADA      10036778     libucrt:mbctype.obj
 0003:00000780       ?__rgcode_page_info@@3PAUcode_page_info@@A 10036780     libucrt:mbctype.obj
 0003:000008d0       ?tzstd_program@@3PADA      100368d0     libucrt:timeset.obj
 0003:00000910       ?tzdst_program@@3PADA      10036910     libucrt:timeset.obj
 0003:00000950       ?w_tzstd_program@@3PA_WA   10036950     libucrt:timeset.obj
 0003:000009d0       ?w_tzdst_program@@3PA_WA   100369d0     libucrt:timeset.obj
 0003:00000a50       ?tzname_states@@3PAY01PADA 10036a50     libucrt:timeset.obj
 0003:00000a58       ?w_tzname_states@@3PAY01PA_WA 10036a58     libucrt:timeset.obj
 0003:00000a60       ?dststart@@3Utransitiondate@?A0x7639d0b4@@A 10036a60     libucrt:tzset.obj
 0003:00000a6c       ?dstend@@3Utransitiondate@?A0x7639d0b4@@A 10036a6c     libucrt:tzset.obj
 0003:00000a80       ?__dcrt_lowio_console_output_handle@@3PAXA 10036a80     libucrt:initcon.obj
 0003:00000a90       ?__DAZ_ENABLED@?1??__set_fpsr_sse2@@9@9 10036a90     libucrt:fpctrl.obj
 0003:00000af8       _stdargs                   10036af8     cmdtoargs.obj
 0003:00000afc       _stdargc                   10036afc     cmdtoargs.obj
 0003:00000b00       _printVersion              10036b00     java.obj
 0003:00000b01       _showVersion               10036b01     java.obj
 0003:00000b02       _printUsage                10036b02     java.obj
 0003:00000b03       _printXUsage               10036b03     java.obj
 0003:00000b04       _showSettings              10036b04     java.obj
 0003:00000b08       __program_name             10036b08     java.obj
 0003:00000b0c       __launcher_name            10036b0c     java.obj
 0003:00000b10       __is_java_args             10036b10     java.obj
 0003:00000b11       __wc_enabled               10036b11     java.obj
 0003:00000b14       __fVersion                 10036b14     java.obj
 0003:00000b18       __dVersion                 10036b18     java.obj
 0003:00000b1c       __ergo_policy              10036b1c     java.obj
 0003:00000b20       _splash_file_entry         10036b20     java.obj
 0003:00000b24       _splash_jar_entry          10036b24     java.obj
 0003:00000b28       _options                   10036b28     java.obj
 0003:00000b2c       _numOptions                10036b2c     java.obj
 0003:00000b30       _maxOptions                10036b30     java.obj
 0003:00000b34       _knownVMs                  10036b34     java.obj
 0003:00000b38       _knownVMsCount             10036b38     java.obj
 0003:00000b3c       _knownVMsLimit             10036b3c     java.obj
 0003:00000b40       _threadStackSize           10036b40     java.obj
 0003:00000b48       _maxHeapSize               10036b48     java.obj
 0003:00000b50       _initialHeapSize           10036b50     java.obj
 0003:00000b58       _helperClass               10036b58     java.obj
 0003:00000b5c       _makePlatformStringMID     10036b5c     java.obj
 0003:00000b64       __isjavaw                  10036b64     java_md.obj
 0003:00000b65       _counterAvailable          10036b65     java_md.obj
 0003:00000b66       _counterInitialized        10036b66     java_md.obj
 0003:00000b68       ?loaded@?1??LoadMSVCRT@@9@9 10036b68     java_md.obj
 0003:00000b6c       _hSplashLib                10036b6c     java_md.obj
 0003:00000b70       _counterFrequency          10036b70     java_md.obj
 0003:00000b78       _findBootClass             10036b78     java_md.obj
 0003:00000b7c       _fnPreloadStop             10036b7c     java_md.obj
 0003:00000b80       _hPreloadAwt               10036b80     java_md.obj
 0003:00000b84       __launcher_debug           10036b84     jli_util.obj
 0003:00000b88       _manifest                  10036b88     parse_manifest.obj
 0003:00000b8c       _zip64_present             10036b8c     parse_manifest.obj
 0003:00000b90       ?proc@?1??DoSplashLoadMemory@@9@9 10036b90     splashscreen_stubs.obj
 0003:00000b94       ?proc@?1??DoSplashLoadFile@@9@9 10036b94     splashscreen_stubs.obj
 0003:00000b98       ?proc@?1??DoSplashInit@@9@9 10036b98     splashscreen_stubs.obj
 0003:00000b9c       ?proc@?1??DoSplashClose@@9@9 10036b9c     splashscreen_stubs.obj
 0003:00000ba0       ?proc@?1??DoSplashSetFileJarName@@9@9 10036ba0     splashscreen_stubs.obj
 0003:00000ba4       ?proc@?1??DoSplashSetScaleFactor@@9@9 10036ba4     splashscreen_stubs.obj
 0003:00000ba8       ?proc@?1??DoSplashGetScaledImageName@@9@9 10036ba8     splashscreen_stubs.obj
 0003:00000bb0       _find_data                 10036bb0     wildcard.obj
 0003:00000cf0       _GS_ExceptionRecord        10036cf0     LIBCMT:gs_report.obj
 0003:00000d40       _GS_ContextRecord          10036d40     LIBCMT:gs_report.obj
 0003:0000100c       ?__proc_attached@@3HA      1003700c     LIBCMT:dll_dllmain.obj
 0003:00001020       ?is_initialized_as_dll@@3_NA 10037020     LIBCMT:utility.obj
 0003:00001021       ?module_local_atexit_table_initialized@@3_NA 10037021     LIBCMT:utility.obj
 0003:00001024       ?module_local_atexit_table@@3U_onexit_table_t@@A 10037024     LIBCMT:utility.obj
 0003:00001030       ?module_local_at_quick_exit_table@@3U_onexit_table_t@@A 10037030     LIBCMT:utility.obj
 0003:00001074       ?heap@@3V_HeapManager@@A   10037074     libvcruntime:undname.obj
 0003:00001088       ?__vcrt_startup_thread_ptd@@3U__vcrt_ptd@@A 10037088     libvcruntime:per_thread_data.obj
 0003:000010b0       ___vcrt_lock_table         100370b0     libvcruntime:locks.obj
 0003:000010c8       ___vcrt_locks_initialized  100370c8     libvcruntime:locks.obj
 0003:000010cc       ?module_handles@@3PAPAUHINSTANCE__@@A 100370cc     libvcruntime:winapi_downlevel.obj
 0003:000010d8       ?function_pointers@@3PAPAXA 100370d8     libvcruntime:winapi_downlevel.obj
 0003:000010fc       ?c_termination_complete@@3JA 100370fc     libucrt:exit.obj
 0003:00001100       ?thread_local_exit_callback_func@@3P6GXPAXK0@ZA 10037100     libucrt:exit.obj
 0003:00001104       ?c_exit_complete@?1???R<lambda_6e4b09c48022b2350581041d5f6b0c4c>@@QBE@XZ@4_NA 10037104     libucrt:exit.obj
 0003:00001108       ?program_name@?1???$common_configure_argv@D@@YAHW4_crt_argv_mode@@@Z@4PADA 10037108     libucrt:argv_parsing.obj
 0003:00001238       ?__acrt_invalid_parameter_handler@@3V?$dual_state_global@P6AXPB_W00II@Z@__crt_state_management@@A 10037238     libucrt:invalid_parameter.obj
 0003:00001240       ?module_handles@@3PAPAUHINSTANCE__@@A 10037240     libucrt:winapi_thunks.obj
 0003:00001298       ?encoded_function_pointers@@3PAPAXA 10037298     libucrt:winapi_thunks.obj
 0003:00001534       ?internal_state@?1??_mbtowc_internal@@9@4U_Mbstatet@@A 10037534     libucrt:mbtowc.obj
 0003:0000153c       ?enable_percent_n@@3IA     1003753c     libucrt:printf_count_output.obj
 0003:00001548       ?__acrt_lock_table@@3PAU_RTL_CRITICAL_SECTION@@A 10037548     libucrt:locks.obj
 0003:00001698       ?__acrt_locks_initialized@@3IA 10037698     libucrt:locks.obj
 0003:0000169c       ?state_cache@?1???$get_cached_win_policy@Ubegin_thread_init_policy_properties@?1??__acrt_get_begin_thread_init_policy@@YA?AW4begin_thread_init_policy@@XZ@@@YA?AW4begin_thread_init_policy@@W4AppPolicyThreadInitializationType@@@Z@4JA 1003769c     libucrt:win_policies.obj
 0003:000016ac       ?fSystemSet@@3HA           100376ac     libucrt:mbctype.obj
 0003:000016b0       ?initialized@?1??__acrt_initialize_multibyte@@9@4_NA 100376b0     libucrt:mbctype.obj
 0003:000016d0       ?__acrt_new_handler@@3V?$dual_state_global@P6AHI@Z@__crt_state_management@@A 100376d0     libucrt:new_handler.obj
 0003:000016d4       ?ctrlc_action@@3V?$dual_state_global@P6AXH@Z@__crt_state_management@@A 100376d4     libucrt:signal.obj
 0003:000016d8       ?ctrlbreak_action@@3V?$dual_state_global@P6AXH@Z@__crt_state_management@@A 100376d8     libucrt:signal.obj
 0003:000016dc       ?abort_action@@3V?$dual_state_global@P6AXH@Z@__crt_state_management@@A 100376dc     libucrt:signal.obj
 0003:000016e0       ?term_action@@3V?$dual_state_global@P6AXH@Z@__crt_state_management@@A 100376e0     libucrt:signal.obj
 0003:000016e4       ?user_matherr@@3V?$dual_state_global@P6AHPAU_exception@@@Z@__crt_state_management@@A 100376e4     libucrt:matherr.obj
 0003:000016ec       ?__acrt_global_new_mode@@3V?$dual_state_global@J@__crt_state_management@@A 100376ec     libucrt:new_mode.obj
 0003:000016fc       ?__acrt_app_type@@3W4_crt_app_type@@A 100376fc     libucrt:report_runtime_error.obj
 0003:0000170c       ?_tzname@@3V?$dual_state_global@PAPAD@__crt_state_management@@A 1003770c     libucrt:timeset.obj
 0003:00001710       ?w_tzname@@3V?$dual_state_global@PAPA_W@__crt_state_management@@A 10037710     libucrt:timeset.obj
 0003:00001714       ?last_wide_tz@@3PA_WA      10037714     libucrt:tzset.obj
 0003:00001718       ?tz_api_used@@3HA          10037718     libucrt:tzset.obj
 0003:0000171c       ?tzset_init_state@@3V?$dual_state_global@J@__crt_state_management@@A 1003771c     libucrt:tzset.obj
 0003:00001720       ?tz_info@@3U_TIME_ZONE_INFORMATION@@A 10037720     libucrt:tzset.obj
 0003:000017d0       ?internal_pst@?1??__mbrtoc32_utf8@__crt_mbstring@@YAIPA_UPBDIPAU_Mbstatet@@AAV__crt_cached_ptd_host@@@Z@4U3@A 100377d0     libucrt:mbrtoc32.obj
 0003:000017dc       __pmatherr_set             100377dc     libucrt:libm_error.obj
 0004:00000060       $R000000                   10038060     jli.dll.res
